 ServerApp_x64

 Timestamp is 61019155 (Thu Jul 29 02:18:13 2021)

 Preferred load address is 0000000140000000

 Start         Length     Name                   Class
 0001:00000000 000007a0H .text$di                CODE
 0001:000007a0 00016a00H .text$mn                CODE
 0001:000171a0 00000020H .text$mn$00             CODE
 0001:000171c0 00000ae0H .text$x                 CODE
 0001:00017ca0 000006c8H .text$yd                CODE
 0002:00000000 00000d18H .idata$5                DATA
 0002:00000d18 00000010H .00cfg                  DATA
 0002:00000d28 00000008H .CRT$XCA                DATA
 0002:00000d30 00000008H .CRT$XCAA               DATA
 0002:00000d38 00000010H .CRT$XCL                DATA
 0002:00000d48 00000180H .CRT$XCU                DATA
 0002:00000ec8 00000008H .CRT$XCZ                DATA
 0002:00000ed0 00000008H .CRT$XIA                DATA
 0002:00000ed8 00000008H .CRT$XIAA               DATA
 0002:00000ee0 00000008H .CRT$XIAC               DATA
 0002:00000ee8 00000008H .CRT$XIC                DATA
 0002:00000ef0 00000008H .CRT$XIZ                DATA
 0002:00000ef8 00000008H .CRT$XLA                DATA
 0002:00000f00 00000008H .CRT$XLZ                DATA
 0002:00000f08 00000008H .CRT$XPA                DATA
 0002:00000f10 00000008H .CRT$XPZ                DATA
 0002:00000f18 00000008H .CRT$XTA                DATA
 0002:00000f20 00000010H .CRT$XTZ                DATA
 0002:00000f28 00000000H .gfids$y                DATA
 0002:00000f30 00007d80H .rdata                  DATA
 0002:00008cb0 00000030H .rdata$T                DATA
 0002:00008ce0 0000100cH .rdata$r                DATA
 0002:00009cec 000003ecH .rdata$zzzdbg           DATA
 0002:0000a0d8 00000008H .rtc$IAA                DATA
 0002:0000a0e0 00000008H .rtc$IZZ                DATA
 0002:0000a0e8 00000008H .rtc$TAA                DATA
 0002:0000a0f0 00000010H .rtc$TZZ                DATA
 0002:0000a100 00000010H .tls                    DATA
 0002:0000a110 00000004H .tls$                   DATA
 0002:0000a114 0000000cH .tls$ZZZ                DATA
 0002:0000a120 00002448H .xdata                  DATA
 0002:0000c568 00000058H .xdata$x                DATA
 0002:0000c5c0 00000000H ATL$__a                 DATA
 0002:0000c5c0 00000000H ATL$__z                 DATA
 0002:0000c5c0 0000006cH .edata                  DATA
 0002:0000c62c 000001ccH .idata$2                DATA
 0002:0000c7f8 00000018H .idata$3                DATA
 0002:0000c810 00000d18H .idata$4                DATA
 0002:0000d528 000014feH .idata$6                DATA
 0003:00000000 000005d0H .data                   DATA
 0003:000005d0 00000690H .data$r                 DATA
 0003:00000c60 002353f8H .bss                    DATA
 0004:00000000 000011acH .pdata                  DATA
 0005:00000000 000001b0H .rsrc$01                DATA
 0005:000001b0 00000a38H .rsrc$02                DATA

  Address         Publics by Value              Rva+Base               Lib:Object

 0000:00000000       __hybrid_code_map          0000000000000000     <absolute>
 0000:00000000       __hybrid_code_map_count    0000000000000000     <absolute>
 0000:00000000       __guard_fids_count         0000000000000000     <absolute>
 0000:00000000       __volatile_metadata        0000000000000000     <absolute>
 0000:00000000       __guard_longjmp_count      0000000000000000     <absolute>
 0000:00000000       __guard_longjmp_table      0000000000000000     <absolute>
 0000:00000000       __guard_iat_count          0000000000000000     <absolute>
 0000:00000000       __guard_iat_table          0000000000000000     <absolute>
 0000:00000000       ___safe_se_handler_count   0000000000000000     <absolute>
 0000:00000000       __enclave_config           0000000000000000     <absolute>
 0000:00000000       ___safe_se_handler_table   0000000000000000     <absolute>
 0000:00000000       __guard_fids_table         0000000000000000     <absolute>
 0000:00000000       __hybrid_auxiliary_iat     0000000000000000     <absolute>
 0000:00000000       __dynamic_value_reloc_table 0000000000000000     <absolute>
 0000:00000100       __guard_flags              0000000000000100     <absolute>
 0000:00000000       __ImageBase                0000000140000000     <linker-defined>
 0001:00000910       ?threadCreateDumpFile@@YAKPEAX@Z 0000000140001910 f   BugReporter.obj
 0001:00000cf0       ?CrashExceptionDump@@YAJPEAU_EXCEPTION_POINTERS@@@Z 0000000140001cf0 f   BugReporter.obj
 0001:00000d60       ?InvalidParameterHandler@@YAXPEB_W00I_K@Z 0000000140001d60 f   BugReporter.obj
 0001:00000d80       ?InitBugReporter@@YAXPEAD0000@Z 0000000140001d80 f   BugReporter.obj
 0001:000010d0       ?InitInstance@CServerAppApp@@UEAAHXZ 00000001400020d0 f   ServerApp.obj
 0001:000010d0       ?CrashExceptionNoneDump@@YAJPEAU_EXCEPTION_POINTERS@@@Z 00000001400020d0 f   BugReporter.obj
 0001:000010d0       _get_startup_argv_mode     00000001400020d0 f   msvcrt:argv_mode.obj
 0001:000010e0       ?Dump@CObject@@UEBAXAEAVCDumpContext@@@Z 00000001400020e0 f i ServerApp.obj
 0001:000010e0       _guard_check_icall_nop     00000001400020e0 f i msvcrt:guard_support.obj
 0001:000010e0       ?__global_delete@@YAXPEAX_K@Z 00000001400020e0 f i * CIL library *:* CIL module *
 0001:000010e0       ?Serialize@CObject@@UEAAXAEAVCArchive@@@Z 00000001400020e0 f i ServerApp.obj
 0001:000010e0       _initialize_denormal_control 00000001400020e0 f i msvcrt:denormal_control.obj
 0001:000010e0       ?AssertValid@CObject@@UEBAXXZ 00000001400020e0 f i ServerApp.obj
 0001:000010e0       _initialize_invalid_parameter_handler 00000001400020e0 f i msvcrt:invalid_parameter_handler.obj
 0001:000010e0       ?__empty_global_delete@@YAXPEAX_K@Z 00000001400020e0 f i BugReporter.obj
 0001:000010e0       ?DoDataExchange@CWnd@@MEAAXPEAVCDataExchange@@@Z 00000001400020e0 f i ServerAppDlg.obj
 0001:000010f0       ??$sprintf_s@$0BAA@@cf@@YAHAEAY0BAA@DPEBDZZ 00000001400020f0 f i BugReporter.obj
 0001:00001130       ??$sprintf_s@$0BJB@@cf@@YAHAEAY0BJB@DPEBDZZ 0000000140002130 f i BugReporter.obj
 0001:00001170       ??$sprintf_s@$0BE@@cf@@YAHAEAY0BE@DPEBDZZ 0000000140002170 f i BugReporter.obj
 0001:000011b0       ??$sprintf_s@$0DOJ@@cf@@YAHAEAY0DOJ@DPEBDZZ 00000001400021b0 f i BugReporter.obj
 0001:000011f0       ??$sprintf_s@$0BAE@@cf@@YAHAEAY0BAE@DPEBDZZ 00000001400021f0 f i BugReporter.obj
 0001:00001230       ??1?$basic_string@DU?$char_traits@D@std@@V?$allocator@D@2@@std@@QEAA@XZ 0000000140002230 f i BugReporter.obj
 0001:00001290       ?_Xlen@?$basic_string@DU?$char_traits@D@std@@V?$allocator@D@2@@std@@SAXXZ 0000000140002290 f i BugReporter.obj
 0001:00001290       ?_Xlen@?$basic_string@_WU?$char_traits@_W@std@@V?$allocator@_W@2@@std@@SAXXZ 0000000140002290 f i crs_uploader.obj
 0001:000012b0       ?assign@?$basic_string@DU?$char_traits@D@std@@V?$allocator@D@2@@std@@QEAAAEAV12@QEBD_K@Z 00000001400022b0 f i BugReporter.obj
 0001:00001410       _snprintf_s                0000000140002410 f i BugReporter.obj
 0001:00001480       __local_stdio_printf_options 0000000140002480 f i BugReporter.obj
 0001:00001490       ?recordExceptionLog@Uploader@crs@@QEAAXAEAVLogBuffer@2@PEBDZZ 0000000140002490 f i crs_uploader.obj
 0001:000015a0       ?readURL@Uploader@crs@@AEAAXAEAV?$basic_string@_WU?$char_traits@_W@std@@V?$allocator@_W@2@@std@@@Z 00000001400025a0 f i crs_uploader.obj
 0001:000017b0       ?iniPath@Uploader@crs@@AEAA?AV?$basic_string@_WU?$char_traits@_W@std@@V?$allocator@_W@2@@std@@AEBV34@@Z 00000001400027b0 f i crs_uploader.obj
 0001:000019d0       ?makeBaseInfo@Uploader@crs@@AEAAXPEAD0@Z 00000001400029d0 f i crs_uploader.obj
 0001:00001c20       ?error@Uploader@crs@@AEAA_NPEBDZZ 0000000140002c20 f i crs_uploader.obj
 0001:00001c80       ??1Uploader@crs@@QEAA@XZ   0000000140002c80 f   crs_uploader.obj
 0001:00001e70       ?init@Uploader@crs@@QEAA_N_NPEAD1@Z 0000000140002e70 f   crs_uploader.obj
 0001:000022c0       ?upload@Uploader@crs@@QEAA_N_NAEBV?$basic_string@DU?$char_traits@D@std@@V?$allocator@D@2@@std@@AEAVLogBuffer@2@@Z 00000001400032c0 f   crs_uploader.obj
 0001:00002550       ?makeExceptionLog@Uploader@crs@@QEAAXPEAU_EXCEPTION_POINTERS@@AEAVLogBuffer@2@@Z 0000000140003550 f   crs_uploader.obj
 0001:00002910       ?prepare@Uploader@crs@@AEAA_NAEAVHttpHandles@2@@Z 0000000140003910 f   crs_uploader.obj
 0001:00002a10       ?uploadHTTP@Uploader@crs@@AEAA_NAEAVHttpHandle@2@PEBDPEB_W2@Z 0000000140003a10 f   crs_uploader.obj
 0001:00002d70       ?uploadLOG@Uploader@crs@@AEAA_NAEAVHttpHandle@2@AEAU_SYSTEMTIME@@AEAVLogBuffer@2@@Z 0000000140003d70 f   crs_uploader.obj
 0001:00003060       ?success@Uploader@crs@@AEAA_NPEBDAEAVHttpHandle@2@@Z 0000000140004060 f   crs_uploader.obj
 0001:000031a0       ??1?$auto_ptr@VUrl@crs@@@std@@QEAA@XZ 00000001400041a0 f i crs_uploader.obj
 0001:000032c0       ??$_snprintf_s@$0IA@@@YAHAEAY0IA@D_KPEBDZZ 00000001400042c0 f i crs_uploader.obj
 0001:00003330       ??$_Reallocate_grow_by@V<lambda_1dfe18491bcca09701d8ccb01d0b0af4>@@PEB_W_K@?$basic_string@_WU?$char_traits@_W@std@@V?$allocator@_W@2@@std@@QEAAAEAV01@_KV<lambda_1dfe18491bcca09701d8ccb01d0b0af4>@@PEB_W_K@Z 0000000140004330 f i crs_uploader.obj
 0001:000034e0       ?append@?$basic_string@_WU?$char_traits@_W@std@@V?$allocator@_W@2@@std@@QEAAAEAV12@QEB_W_K@Z 00000001400044e0 f i crs_uploader.obj
 0001:00003560       _snwprintf_s               0000000140004560 f i crs_uploader.obj
 0001:000035d0       ??1?$basic_string@_WU?$char_traits@_W@std@@V?$allocator@_W@2@@std@@QEAA@XZ 00000001400045d0 f i crs_uploader.obj
 0001:000035d0       ?_Tidy_deallocate@?$basic_string@_WU?$char_traits@_W@std@@V?$allocator@_W@2@@std@@QEAAXXZ 00000001400045d0 f i crs_uploader.obj
 0001:00003640       ?assign@?$basic_string@_WU?$char_traits@_W@std@@V?$allocator@_W@2@@std@@QEAAAEAV12@QEB_W_K@Z 0000000140004640 f i crs_uploader.obj
 0001:000037d0       ??_GCServerLog@@UEAAPEAXI@Z 00000001400047d0 f i LogMgmt.obj
 0001:000037d0       ??_ECServerLog@@UEAAPEAXI@Z 00000001400047d0 f i * CIL library *:* CIL module *
 0001:00003810       ??1CServerLog@@UEAA@XZ     0000000140004810 f   LogMgmt.obj
 0001:00003940       ?Log@rwpmlog@@YAXPEBDFPEBUPROTO_START_HOST_tag@@@Z 0000000140004940 f   RWPMLog.obj
 0001:00003e70       ?Log@rwpmlog@@YAXPEBDFPEBUPROTO_GAME_USER_INFO_tag@@@Z 0000000140004e70 f   RWPMLog.obj
 0001:000044d0       ?Log@rwpmlog@@YAXPEBDFPEBUPROTO_GAMEGT_INGAME_AIGACHA_ITEM_INSERT_RESULT@@@Z 00000001400054d0 f   RWPMLog.obj
 0001:00004790       ?Log@rwpmlog@@YAXPEBDFPEBUPROTO_GAMEGT_INGAME_AIGACHA_GROUP_RATE_RESULT@@@Z 0000000140005790 f   RWPMLog.obj
 0001:00004a50       ??$sprintf_s@$0EA@@cf@@YAHAEAY0EA@DPEBDZZ 0000000140005a50 f i RWPMLog.obj
 0001:00004c10       ??0CInterfaceDatabase@@QEAA@XZ 0000000140005c10 f   ltmodule.obj
 0001:00004ca0       ?AddHolder@CInterfaceDatabase@@SAXPEAVCAPIHolderBase@@@Z 0000000140005ca0 f   ltmodule.obj
 0001:00004d20       ?Add@CInterfaceDatabase@@EEAAXPEAVIBase@@PEBDH@Z 0000000140005d20 f   ltmodule.obj
 0001:00004df0       ?Remove@CInterfaceDatabase@@EEAAXPEAVIBase@@PEBD@Z 0000000140005df0 f   ltmodule.obj
 0001:00004f60       ?Add@CInterfaceDatabase@@EEAAXPEAVCAPIHolderBase@@@Z 0000000140005f60 f   ltmodule.obj
 0001:000050c0       ?Remove@CInterfaceDatabase@@EEAAXPEAVCAPIHolderBase@@@Z 00000001400060c0 f   ltmodule.obj
 0001:00005170       ?Add@CInterfaceDatabase@@EEAAXPEAVCInterfaceChooser@@@Z 0000000140006170 f   ltmodule.obj
 0001:000052d0       ?Remove@CInterfaceDatabase@@EEAAXPEAVCInterfaceChooser@@@Z 00000001400062d0 f   ltmodule.obj
 0001:000053b0       ?Run@CInterfaceDatabase@@EEAA?AW4EChooserRun@@PEAVCInterfaceChooser@@@Z 00000001400063b0 f   ltmodule.obj
 0001:00005440       ?TransferFrom@CInterfaceDatabase@@UEAAXPEAV1@@Z 0000000140006440 f   ltmodule.obj
 0001:00005560       ?IsEmpty@CInterfaceDatabase@@EEAA_NXZ 0000000140006560 f   ltmodule.obj
 0001:00005570       ?Destroy@CInterfaceDatabase@@UEAAXXZ 0000000140006570 f   ltmodule.obj
 0001:000056a0       ?SortedArrayFindNameMgr@@YA?AW4RELATION@@PEBDPEAVCInterfaceNameMgr@@@Z 00000001400066a0 f   ltmodule.obj
 0001:000056e0       ??0CInterfaceNameMgr@@QEAA@PEBDH@Z 00000001400066e0 f   ltmodule.obj
 0001:000057e0       ??_ECInterfaceNameMgr@@UEAAPEAXI@Z 00000001400067e0 f i * CIL library *:* CIL module *
 0001:000057e0       ??_GCInterfaceNameMgr@@UEAAPEAXI@Z 00000001400067e0 f i ltmodule.obj
 0001:00005920       ?Add@CInterfaceNameMgr@@QEAAXPEAVIBase@@@Z 0000000140006920 f   ltmodule.obj
 0001:00005af0       ?ConnectHolders@CInterfaceNameMgr@@IEAAXPEAVIBase@@@Z 0000000140006af0 f   ltmodule.obj
 0001:00005b60       ?TransferFrom@CInterfaceNameMgr@@QEAAXPEAV1@@Z 0000000140006b60 f   ltmodule.obj
 0001:00005dc0       ??_GCAPIHolderBase@@UEAAPEAXI@Z 0000000140006dc0 f i ltmodule.obj
 0001:00005dc0       ??_ECAPIHolderBase@@UEAAPEAXI@Z 0000000140006dc0 f i * CIL library *:* CIL module *
 0001:00005e10       ??1CAPIHolderBase@@UEAA@XZ 0000000140006e10 f   ltmodule.obj
 0001:00005e30       SetMasterDatabase          0000000140006e30 f   ltmodule.obj
 0001:00005f20       ??1?$CPointerTrackedTarget@VCInterfaceDatabase@@@@QEAA@XZ 0000000140006f20 f i ltmodule.obj
 0001:00005f80       ??4?$CPointerTracked@VCInterfaceDatabase@@@@QEAAAEAV0@AEAV0@@Z 0000000140006f80 f i ltmodule.obj
 0001:00006010       ??4?$CPointerTracked@VCInterfaceDatabase@@@@QEAAAEAV0@PEAVCInterfaceDatabase@@@Z 0000000140007010 f i ltmodule.obj
 0001:000060a0       ?add@?$database_array@VCInterfaceNameMgr@@PEBD@@QEAAXPEAVCInterfaceNameMgr@@P6A?AW4RELATION@@00@Z@Z 00000001400070a0 f i ltmodule.obj
 0001:000061c0       ?get@?$database_array@VCInterfaceNameMgr@@PEBD@@QEAAPEAVCInterfaceNameMgr@@PEBDP6A?AW4RELATION@@0PEAV2@@Z@Z 00000001400071c0 f i ltmodule.obj
 0001:00006290       ?remove@?$database_array@VCInterfaceNameMgr@@PEBD@@QEAA_NPEAVCInterfaceNameMgr@@@Z 0000000140007290 f i ltmodule.obj
 0001:000062f0       ?insert@?$database_array@VIBase@@PEBD@@IEAAXPEAVIBase@@I@Z 00000001400072f0 f i ltmodule.obj
 0001:000062f0       ?insert@?$database_array@VCInterfaceNameMgr@@PEBD@@IEAAXPEAVCInterfaceNameMgr@@I@Z 00000001400072f0 f i ltmodule.obj
 0001:000063f0       ?_InitPathNameInfo@CHLogger@@CAXPEBD000@Z 00000001400073f0 f   HostLogger.obj
 0001:000068d0       ?Log@CHLogger@@SAXW4ELOG_LEVEL@1@PEBDZZ 00000001400078d0 f   HostLogger.obj
 0001:00006920       ?LogKernel@CHLogger@@SAXW4ELOG_LEVEL@1@PEBDZZ 0000000140007920 f   HostLogger.obj
 0001:00006970       ?LogTimeOut@CHLogger@@SAXPEBDZZ 0000000140007970 f   HostLogger.obj
 0001:00006b80       ?LogEtc@CHLogger@@SAXPEBDZZ 0000000140007b80 f   HostLogger.obj
 0001:00006da0       ?LogPacket@CHLogger@@SAXPEBDZZ 0000000140007da0 f   HostLogger.obj
 0001:00006fc0       ?LogRWProcessMemory@CHLogger@@SAXPEBDZZ 0000000140007fc0 f   HostLogger.obj
 0001:00007190       ?LogIPCMessage@CHLogger@@SAXPEBDZZ 0000000140008190 f   HostLogger.obj
 0001:00007360       ?_BuildDirectory@CHLogger@@CAXAEBU_SYSTEMTIME@@@Z 0000000140008360 f   HostLogger.obj
 0001:000077a0       ?_DoLogWithLevel@CHLogger@@CAXPEBDW4ELOG_LEVEL@1@0PEAD@Z 00000001400087a0 f   HostLogger.obj
 0001:000079a0       ??$_Traits_find@U?$char_traits@D@std@@@std@@YA_KQEBD_K101@Z 00000001400089a0 f i HostLogger.obj
 0001:00007a60       ?_Xran@?$_String_val@U?$_Simple_types@D@std@@@std@@SAXXZ 0000000140008a60 f i HostLogger.obj
 0001:00007a80       ??$_Reallocate_grow_by@V<lambda_65e615be2a453ca0576c979606f46740>@@PEBD_K@?$basic_string@DU?$char_traits@D@std@@V?$allocator@D@2@@std@@QEAAAEAV01@_KV<lambda_65e615be2a453ca0576c979606f46740>@@PEBD_K@Z 0000000140008a80 f i HostLogger.obj
 0001:00007c00       ?append@?$basic_string@DU?$char_traits@D@std@@V?$allocator@D@2@@std@@QEAAAEAV12@QEBD_K@Z 0000000140008c00 f i HostLogger.obj
 0001:00007c80       ??1CSynchronizedLog@@QEAA@XZ 0000000140008c80 f i HostLogger.obj
 0001:00007ca0       ??_ECMustSyncObjectLog@@UEAAPEAXI@Z 0000000140008ca0 f i * CIL library *:* CIL module *
 0001:00007ca0       ??_GCMustSyncObjectLog@@UEAAPEAXI@Z 0000000140008ca0 f i HostLogger.obj
 0001:00007cf0       ?Init@CLogMsgManager@@SA_NW4ESHARED_MEM_USAGE_TYPE@1@@Z 0000000140008cf0 f   LogMsgManager.obj
 0001:00008000       ?GetString@CLogMsgManager@@SA?BV?$basic_string@DU?$char_traits@D@std@@V?$allocator@D@2@@std@@I@Z 0000000140009000 f   LogMsgManager.obj
 0001:000081b0       ?_WriteXlsDataToSharedMemory@CLogMsgManager@@CA_NXZ 00000001400091b0 f   LogMsgManager.obj
 0001:00008490       ??$sprintf_s@$0CA@@cf@@YAHAEAY0CA@DPEBDZZ 0000000140009490 f i LogMsgManager.obj
 0001:000084d0       ??$_Emplace_reallocate@AEBQEAX@?$vector@PEAXV?$allocator@PEAX@std@@@std@@QEAAPEAPEAXQEAPEAXAEBQEAX@Z 00000001400094d0 f i LogMsgManager.obj
 0001:00008680       ?_Xlength@?$vector@PEAXV?$allocator@PEAX@std@@@std@@CAXXZ 0000000140009680 f i LogMsgManager.obj
 0001:000086a0       ??0FindXlsMsg@@QEAA@XZ     00000001400096a0 f   LoadXlsMsg.obj
 0001:00008700       ??_EFindXlsMsg@@UEAAPEAXI@Z 0000000140009700 f i * CIL library *:* CIL module *
 0001:00008700       ??_GFindXlsMsg@@UEAAPEAXI@Z 0000000140009700 f i LoadXlsMsg.obj
 0001:00008800       ?GetMessageByIndex@FindXlsMsg@@QEAAPEBD_JPEAD@Z 0000000140009800 f   LoadXlsMsg.obj
 0001:000088b0       ?LoadWMszFile@FindXlsMsg@@QEAA_NPEAD@Z 00000001400098b0 f   LoadXlsMsg.obj
 0001:00008be0       ??A?$map@_JV?$basic_string@DU?$char_traits@D@std@@V?$allocator@D@2@@std@@U?$less@_J@2@V?$allocator@U?$pair@$$CB_JV?$basic_string@DU?$char_traits@D@std@@V?$allocator@D@2@@std@@@std@@@2@@std@@QEAAAEAV?$basic_string@DU?$char_traits@D@std@@V?$allocator@D@2@@1@AEB_J@Z 0000000140009be0 f i LoadXlsMsg.obj
 0001:00008c70       ?_Erase@?$_Tree@V?$_Tmap_traits@_JV?$basic_string@DU?$char_traits@D@std@@V?$allocator@D@2@@std@@U?$less@_J@2@V?$allocator@U?$pair@$$CB_JV?$basic_string@DU?$char_traits@D@std@@V?$allocator@D@2@@std@@@std@@@2@$0A@@std@@@std@@IEAAXPEAU?$_Tree_node@U?$pair@$$CB_JV?$basic_string@DU?$char_traits@D@std@@V?$allocator@D@2@@std@@@std@@PEAX@2@@Z 0000000140009c70 f i LoadXlsMsg.obj
 0001:00008d30       ?erase@?$_Tree@V?$_Tmap_traits@_JV?$basic_string@DU?$char_traits@D@std@@V?$allocator@D@2@@std@@U?$less@_J@2@V?$allocator@U?$pair@$$CB_JV?$basic_string@DU?$char_traits@D@std@@V?$allocator@D@2@@std@@@std@@@2@$0A@@std@@@std@@QEAA?AV?$_Tree_iterator@V?$_Tree_val@U?$_Tree_simple_types@U?$pair@$$CB_JV?$basic_string@DU?$char_traits@D@std@@V?$allocator@D@2@@std@@@std@@@std@@@std@@@2@V?$_Tree_const_iterator@V?$_Tree_val@U?$_Tree_simple_types@U?$pair@$$CB_JV?$basic_string@DU?$char_traits@D@std@@V?$allocator@D@2@@std@@@std@@@std@@@std@@@2@0@Z 0000000140009d30 f i LoadXlsMsg.obj
 0001:00008ee0       ?_Extract@?$_Tree_val@U?$_Tree_simple_types@U?$pair@$$CB_JV?$basic_string@DU?$char_traits@D@std@@V?$allocator@D@2@@std@@@std@@@std@@@std@@QEAAPEAU?$_Tree_node@U?$pair@$$CB_JV?$basic_string@DU?$char_traits@D@std@@V?$allocator@D@2@@std@@@std@@PEAX@2@V?$_Tree_const_iterator@V?$_Tree_val@U?$_Tree_simple_types@U?$pair@$$CB_JV?$basic_string@DU?$char_traits@D@std@@V?$allocator@D@2@@std@@@std@@@std@@@std@@@2@@Z 0000000140009ee0 f i LoadXlsMsg.obj
 0001:00009370       ?_Buyheadnode@?$_Tree_comp_alloc@V?$_Tmap_traits@_JV?$basic_string@DU?$char_traits@D@std@@V?$allocator@D@2@@std@@U?$less@_J@2@V?$allocator@U?$pair@$$CB_JV?$basic_string@DU?$char_traits@D@std@@V?$allocator@D@2@@std@@@std@@@2@$0A@@std@@@std@@QEAAPEAU?$_Tree_node@U?$pair@$$CB_JV?$basic_string@DU?$char_traits@D@std@@V?$allocator@D@2@@std@@@std@@PEAX@2@XZ 000000014000a370 f i LoadXlsMsg.obj
 0001:000093a0       ??$_Buynode@AEBUpiecewise_construct_t@std@@V?$tuple@AEB_J@2@V?$tuple@$$V@2@@?$_Tree_comp_alloc@V?$_Tmap_traits@_JV?$basic_string@DU?$char_traits@D@std@@V?$allocator@D@2@@std@@U?$less@_J@2@V?$allocator@U?$pair@$$CB_JV?$basic_string@DU?$char_traits@D@std@@V?$allocator@D@2@@std@@@std@@@2@$0A@@std@@@std@@QEAAPEAU?$_Tree_node@U?$pair@$$CB_JV?$basic_string@DU?$char_traits@D@std@@V?$allocator@D@2@@std@@@std@@PEAX@1@AEBUpiecewise_construct_t@1@$$QEAV?$tuple@AEB_J@1@$$QEAV?$tuple@$$V@1@@Z 000000014000a3a0 f i LoadXlsMsg.obj
 0001:000093e0       ??$_Insert_hint@AEAU?$pair@$$CB_JV?$basic_string@DU?$char_traits@D@std@@V?$allocator@D@2@@std@@@std@@PEAU?$_Tree_node@U?$pair@$$CB_JV?$basic_string@DU?$char_traits@D@std@@V?$allocator@D@2@@std@@@std@@PEAX@2@@?$_Tree@V?$_Tmap_traits@_JV?$basic_string@DU?$char_traits@D@std@@V?$allocator@D@2@@std@@U?$less@_J@2@V?$allocator@U?$pair@$$CB_JV?$basic_string@DU?$char_traits@D@std@@V?$allocator@D@2@@std@@@std@@@2@$0A@@std@@@std@@IEAA?AV?$_Tree_iterator@V?$_Tree_val@U?$_Tree_simple_types@U?$pair@$$CB_JV?$basic_string@DU?$char_traits@D@std@@V?$allocator@D@2@@std@@@std@@@std@@@std@@@1@V?$_Tree_const_iterator@V?$_Tree_val@U?$_Tree_simple_types@U?$pair@$$CB_JV?$basic_string@DU?$char_traits@D@std@@V?$allocator@D@2@@std@@@std@@@std@@@std@@@1@AEAU?$pair@$$CB_JV?$basic_string@DU?$char_traits@D@std@@V?$allocator@D@2@@std@@@1@PEAU?$_Tree_node@U?$pair@$$CB_JV?$basic_string@DU?$char_traits@D@std@@V?$allocator@D@2@@std@@@std@@PEAX@1@@Z 000000014000a3e0 f i LoadXlsMsg.obj
 0001:00009630       ?_Buynode0@?$_Tree_comp_alloc@V?$_Tmap_traits@_JV?$basic_string@DU?$char_traits@D@std@@V?$allocator@D@2@@std@@U?$less@_J@2@V?$allocator@U?$pair@$$CB_JV?$basic_string@DU?$char_traits@D@std@@V?$allocator@D@2@@std@@@std@@@2@$0A@@std@@@std@@QEAAPEAU?$_Tree_node@U?$pair@$$CB_JV?$basic_string@DU?$char_traits@D@std@@V?$allocator@D@2@@std@@@std@@PEAX@2@XZ 000000014000a630 f i LoadXlsMsg.obj
 0001:00009660       ?_Destroy_if_node@?$_Tree@V?$_Tmap_traits@_JV?$basic_string@DU?$char_traits@D@std@@V?$allocator@D@2@@std@@U?$less@_J@2@V?$allocator@U?$pair@$$CB_JV?$basic_string@DU?$char_traits@D@std@@V?$allocator@D@2@@std@@@std@@@2@$0A@@std@@@std@@IEAAXPEAU?$_Tree_node@U?$pair@$$CB_JV?$basic_string@DU?$char_traits@D@std@@V?$allocator@D@2@@std@@@std@@PEAX@2@@Z 000000014000a660 f i LoadXlsMsg.obj
 0001:000096d0       ??$_Insert_at@AEAU?$pair@$$CB_JV?$basic_string@DU?$char_traits@D@std@@V?$allocator@D@2@@std@@@std@@PEAU?$_Tree_node@U?$pair@$$CB_JV?$basic_string@DU?$char_traits@D@std@@V?$allocator@D@2@@std@@@std@@PEAX@2@@?$_Tree@V?$_Tmap_traits@_JV?$basic_string@DU?$char_traits@D@std@@V?$allocator@D@2@@std@@U?$less@_J@2@V?$allocator@U?$pair@$$CB_JV?$basic_string@DU?$char_traits@D@std@@V?$allocator@D@2@@std@@@std@@@2@$0A@@std@@@std@@IEAA?AV?$_Tree_iterator@V?$_Tree_val@U?$_Tree_simple_types@U?$pair@$$CB_JV?$basic_string@DU?$char_traits@D@std@@V?$allocator@D@2@@std@@@std@@@std@@@std@@@1@_NPEAU?$_Tree_node@U?$pair@$$CB_JV?$basic_string@DU?$char_traits@D@std@@V?$allocator@D@2@@std@@@std@@PEAX@1@AEAU?$pair@$$CB_JV?$basic_string@DU?$char_traits@D@std@@V?$allocator@D@2@@std@@@1@1@Z 000000014000a6d0 f i LoadXlsMsg.obj
 0001:00009980       ??$_Insert_nohint@AEAU?$pair@$$CB_JV?$basic_string@DU?$char_traits@D@std@@V?$allocator@D@2@@std@@@std@@PEAU?$_Tree_node@U?$pair@$$CB_JV?$basic_string@DU?$char_traits@D@std@@V?$allocator@D@2@@std@@@std@@PEAX@2@@?$_Tree@V?$_Tmap_traits@_JV?$basic_string@DU?$char_traits@D@std@@V?$allocator@D@2@@std@@U?$less@_J@2@V?$allocator@U?$pair@$$CB_JV?$basic_string@DU?$char_traits@D@std@@V?$allocator@D@2@@std@@@std@@@2@$0A@@std@@@std@@IEAA?AU?$pair@V?$_Tree_iterator@V?$_Tree_val@U?$_Tree_simple_types@U?$pair@$$CB_JV?$basic_string@DU?$char_traits@D@std@@V?$allocator@D@2@@std@@@std@@@std@@@std@@@std@@_N@1@_NAEAU?$pair@$$CB_JV?$basic_string@DU?$char_traits@D@std@@V?$allocator@D@2@@std@@@1@PEAU?$_Tree_node@U?$pair@$$CB_JV?$basic_string@DU?$char_traits@D@std@@V?$allocator@D@2@@std@@@std@@PEAX@1@@Z 000000014000a980 f i LoadXlsMsg.obj
 0001:00009ae0       ??4?$basic_string@DU?$char_traits@D@std@@V?$allocator@D@2@@std@@QEAAAEAV01@$$QEAV01@@Z 000000014000aae0 f i LoadXlsMsg.obj
 0001:00009b70       ?GetMessageMap@CServerAppApp@@MEBAPEBUAFX_MSGMAP@@XZ 000000014000ab70 f   ServerApp.obj
 0001:00009b80       ?GetLogFileDir@ServerAppHandler@@UEAA_NPEADH@Z 000000014000ab80 f   ServerAppDlg.obj
 0001:00009b80       IsDebugMode                000000014000ab80 f   ServerApp.obj
 0001:00009b90       ??_GCServerAppApp@@UEAAPEAXI@Z 000000014000ab90 f i ServerApp.obj
 0001:00009b90       ??_ECServerAppApp@@UEAAPEAXI@Z 000000014000ab90 f i * CIL library *:* CIL module *
 0001:00009bf0       ?Run@CServerAppApp@@UEAAHXZ 000000014000abf0 f   ServerApp.obj
 0001:00009c70       ?GetApplicationRecoveryPingInterval@CWinApp@@UEAAKXZ 000000014000ac70 f i ServerApp.obj
 0001:00009c80       __scrt_initialize_winrt    000000014000ac80 f i msvcrt:utility_desktop.obj
 0001:00009c80       _matherr                   000000014000ac80 f i msvcrt:matherr.obj
 0001:00009c80       __scrt_stub_for_initialize_mta 000000014000ac80 f i msvcrt:utility_desktop.obj
 0001:00009c80       _get_startup_commit_mode   000000014000ac80 f i msvcrt:commit_mode.obj
 0001:00009c80       ?GetApplicationRestartFlags@CWinApp@@UEAAKXZ 000000014000ac80 f i ServerApp.obj
 0001:00009c80       _get_startup_new_mode      000000014000ac80 f i msvcrt:new_mode.obj
 0001:00009c80       __scrt_exe_initialize_mta  000000014000ac80 f i msvcrt:utility_desktop.obj
 0001:00009c80       ?GetApplicationRecoveryParameter@CWinApp@@UEAAPEAXXZ 000000014000ac80 f i ServerApp.obj
 0001:00009c80       ?ProcessPacket@ServerAppHandler@@UEAAIAEAVILTMessage_Read@@QEAEG@Z 000000014000ac80 f i ServerAppDlg.obj
 0001:00009c80       _get_startup_thread_locale_mode 000000014000ac80 f i msvcrt:thread_locale.obj
 0001:00009c90       ?RestoreAutosavedFilesAtRestart@CWinApp@@UEBAHXZ 000000014000ac90 f i ServerApp.obj
 0001:00009ca0       ?ReopenPreviousFilesAtRestart@CWinApp@@UEBAHXZ 000000014000aca0 f i ServerApp.obj
 0001:00009cb0       ?SupportsAutosaveAtInterval@CWinApp@@UEBAHXZ 000000014000acb0 f i ServerApp.obj
 0001:00009cc0       ?SupportsAutosaveAtRestart@CWinApp@@UEBAHXZ 000000014000acc0 f i ServerApp.obj
 0001:00009cd0       ?SupportsApplicationRecovery@CWinApp@@UEBAHXZ 000000014000acd0 f i ServerApp.obj
 0001:00009ce0       ?SupportsRestartManager@CWinApp@@UEBAHXZ 000000014000ace0 f i ServerApp.obj
 0001:00009cf0       ?GetCPUUtilization@ServerAppHandler@@UEAAMXZ 000000014000acf0 f i ServerAppDlg.obj
 0001:00009d00       ?IsGameEnded@CGameServerAppHandler@@UEAA_NXZ 000000014000ad00 f i ServerAppDlg.obj
 0001:00009d10       ??0PROTO_GAME_USER_INFO_tag@@QEAA@XZ 000000014000ad10 f i ServerAppDlg.obj
 0001:0000a2c0       ??0PROTO_AI_BOSS_TOWER_REWARD_REQ@@QEAA@XZ 000000014000b2c0 f i ServerAppDlg.obj
 0001:0000a3e0       ?ShellMessageFn@CGameServerAppHandler@@UEAAIAEAVILTMessage_Read@@@Z 000000014000b3e0 f   ServerAppDlg.obj
 0001:0000a400       ?ConsoleOutputFn@CGameServerAppHandler@@UEAAIPEBD@Z 000000014000b400 f   ServerAppDlg.obj
 0001:0000a410       ?ConsoleOutputFn@CGameServerAppHandler@@UEAAIHHPEBD@Z 000000014000b410 f   ServerAppDlg.obj
 0001:0000a6b0       ?OutOfMemory@CGameServerAppHandler@@UEAAIXZ 000000014000b6b0 f   ServerAppDlg.obj
 0001:0000a750       ?NetworkDelayCount@CGameServerAppHandler@@UEAAIXZ 000000014000b750 f   ServerAppDlg.obj
 0001:0000a790       ?GetProcessMemoryUsage@CGameServerAppHandler@@UEAAKXZ 000000014000b790 f   ServerAppDlg.obj
 0001:0000a8b0       ??0PROTO_START_HOST_tag@@QEAA@XZ 000000014000b8b0 f i ServerAppDlg.obj
 0001:0000a930       ??0CServerAppDlg@@QEAA@PEAVCWnd@@@Z 000000014000b930 f   ServerAppDlg.obj
 0001:0000ab20       ??_ECServerAppDlg@@UEAAPEAXI@Z 000000014000bb20 f i * CIL library *:* CIL module *
 0001:0000ab20       ??_GCServerAppDlg@@UEAAPEAXI@Z 000000014000bb20 f i ServerAppDlg.obj
 0001:0000ab70       ??1tUCCGamePlayInfo@CServerAppDlg@@QEAA@XZ 000000014000bb70 f i ServerAppDlg.obj
 0001:0000abe0       ??1CServerAppDlg@@UEAA@XZ  000000014000bbe0 f   ServerAppDlg.obj
 0001:0000ade0       ?DoDataExchange@CServerAppDlg@@MEAAXPEAVCDataExchange@@@Z 000000014000bde0 f   ServerAppDlg.obj
 0001:0000ae30       ?GetMessageMap@CServerAppDlg@@MEBAPEBUAFX_MSGMAP@@XZ 000000014000be30 f   ServerAppDlg.obj
 0001:0000ae40       ?OnInitDialog@CServerAppDlg@@MEAAHXZ 000000014000be40 f   ServerAppDlg.obj
 0001:0000b8f0       ?OnPaint@CServerAppDlg@@IEAAXXZ 000000014000c8f0 f   ServerAppDlg.obj
 0001:0000b900       ?OnQueryDragIcon@CServerAppDlg@@IEAAPEAUHICON__@@XZ 000000014000c900 f   ServerAppDlg.obj
 0001:0000b910       ?OnShellMessage@CServerAppDlg@@QEAAXAEAVILTMessage_Read@@@Z 000000014000c910 f   ServerAppDlg.obj
 0001:0000d950       ?AddServerMsg@CServerAppDlg@@QEAAXPEBDH@Z 000000014000e950 f   ServerAppDlg.obj
 0001:0000db00       ?LoadServer@CServerAppDlg@@QEAA_NXZ 000000014000eb00 f   ServerAppDlg.obj
 0001:0000de20       ?RunServer@CServerAppDlg@@QEAA_NXZ 000000014000ee20 f   ServerAppDlg.obj
 0001:0000e1f0       ?StopServer@CServerAppDlg@@QEAA_NXZ 000000014000f1f0 f   ServerAppDlg.obj
 0001:0000e3a0       ?Thread_SendGameInfo@@YAXPEAVCServerAppDlg@@AEAUPROTO_START_HOST_tag@@@Z 000000014000f3a0 f   ServerAppDlg.obj
 0001:0000ea50       ?Thread_SendUserInfo@@YAXPEAVCServerAppDlg@@AEAUPROTO_GAME_USER_INFO_tag@@@Z 000000014000fa50 f   ServerAppDlg.obj
 0001:0000ec90       ?ThreadUpdate@CServerAppDlg@@SAXPEAX@Z 000000014000fc90 f   ServerAppDlg.obj
 0001:0000f230       ?ServerUpdate@CServerAppDlg@@QEAAXXZ 0000000140010230 f   ServerAppDlg.obj
 0001:0000f460       ?AddResources@CServerAppDlg@@QEAA_NXZ 0000000140010460 f   ServerAppDlg.obj
 0001:0000f700       ?OnGameServerMsg@CServerAppDlg@@IEAA_J_K_J@Z 0000000140010700 f   ServerAppDlg.obj
 0001:00010040       ?OnCopyData@CServerAppDlg@@IEAAHPEAVCWnd@@PEAUtagCOPYDATASTRUCT@@@Z 0000000140011040 f   ServerAppDlg.obj
 0001:00011050       ?OnTimer@CServerAppDlg@@QEAAX_K@Z 0000000140012050 f   ServerAppDlg.obj
 0001:000111c0       ?OnBnClickedButtonGo@CServerAppDlg@@QEAAXXZ 00000001400121c0 f   ServerAppDlg.obj
 0001:00011290       ?SaveHostGameInfo@CServerAppDlg@@IEAAXXZ 0000000140012290 f   ServerAppDlg.obj
 0001:00011570       ?LoadHostGameInfo@CServerAppDlg@@IEAAXXZ 0000000140012570 f   ServerAppDlg.obj
 0001:00011a60       ?GetOptionValueString@CServerAppDlg@@IEAA?AV?$basic_string@DU?$char_traits@D@std@@V?$allocator@D@2@@std@@V23@00@Z 0000000140012a60 f   ServerAppDlg.obj
 0001:00011f00       ?ReadGSMMemory@CServerAppDlg@@QEAA_NPEAX0_K@Z 0000000140012f00 f   ServerAppDlg.obj
 0001:00012020       ?RECV_MSG_INSERTCHARACTER@CServerAppDlg@@AEAAX_J@Z 0000000140013020 f   ServerAppDlg.obj
 0001:00012250       ?RECV_MSG_AIITEM_DEC@CServerAppDlg@@AEAAX_J@Z 0000000140013250 f   ServerAppDlg.obj
 0001:000124c0       ?RECV_MSG_AIITEM_GROUP_RATE_RESULT@CServerAppDlg@@AEAAX_J@Z 00000001400134c0 f   ServerAppDlg.obj
 0001:00012750       ?RECV_MSG_USER_DISCONNECTED@CServerAppDlg@@AEAAX_J@Z 0000000140013750 f   ServerAppDlg.obj
 0001:000129e0       ?SendServerAppInit@CServerAppDlg@@AEAAXXZ 00000001400139e0 f   ServerAppDlg.obj
 0001:00012ba0       ?DownloadUCCMapFile_HTTP@CServerAppDlg@@AEAA?AW4UCCMAPDOWNLOADREAULT@@V?$basic_string@DU?$char_traits@D@std@@V?$allocator@D@2@@std@@@Z 0000000140013ba0 f   ServerAppDlg.obj
 0001:00013900       ?SendServerAppInitFail@CServerAppDlg@@AEAAXHH@Z 0000000140014900 f   ServerAppDlg.obj
 0001:00013a20       ?GetDownloadPath@CServerAppDlg@@AEAA?AV?$basic_string@DU?$char_traits@D@std@@V?$allocator@D@2@@std@@XZ 0000000140014a20 f   ServerAppDlg.obj
 0001:00013b10       ?SendToServerShellAutoMatchStartingUserInfo@CServerAppDlg@@AEAAXPEAUtagCOPYDATASTRUCT@@@Z 0000000140014b10 f   ServerAppDlg.obj
 0001:00013d50       ??1?$CAPIHolder@VILTCommon@@@@UEAA@XZ 0000000140014d50 f i ServerAppDlg.obj
 0001:00013e40       ?APIRemoved@?$CAPIHolder@VILTCommon@@@@UEAAXXZ 0000000140014e40 f i ServerAppDlg.obj
 0001:00013e50       ?APIFound@?$CAPIHolder@VILTCommon@@@@UEAAXPEAVIBase@@@Z 0000000140014e50 f i ServerAppDlg.obj
 0001:00013e60       ?Interface@?$CAPIHolder@VILTCommon@@@@UEAAPEAVIBase@@XZ 0000000140014e60 f i ServerAppDlg.obj
 0001:00013e70       ??$sprintf_s@$0IA@@cf@@YAHAEAY0IA@DPEBDZZ 0000000140014e70 f i ServerAppDlg.obj
 0001:00013eb0       ??$?HDU?$char_traits@D@std@@V?$allocator@D@1@@std@@YA?AV?$basic_string@DU?$char_traits@D@std@@V?$allocator@D@2@@0@AEBV10@0@Z 0000000140014eb0 f i ServerAppDlg.obj
 0001:00013f60       ??_G?$CAPIHolder@VILTCommon@@@@UEAAPEAXI@Z 0000000140014f60 f i ServerAppDlg.obj
 0001:00013f60       ??_E?$CAPIHolder@VILTCommon@@@@UEAAPEAXI@Z 0000000140014f60 f i * CIL library *:* CIL module *
 0001:00013fa0       ?reserve@?$basic_string@DU?$char_traits@D@std@@V?$allocator@D@2@@std@@QEAAX_K@Z 0000000140014fa0 f i ServerAppDlg.obj
 0001:00014160       ?Create@CDialog@@UEAAHIPEAVCWnd@@@Z 0000000140015160 f i ServerAppDlg.obj
 0001:00014170       __local_stdio_scanf_options 0000000140015170 f i ServerAppDlg.obj
 0001:00014180       fscanf_s                   0000000140015180 f i ServerAppDlg.obj
 0001:000141d0       ??1CWaitCursor@@QEAA@XZ    00000001400151d0 f i ServerAppDlg.obj
 0001:00014220       ?Readint32@ILTMessage_Read@@QEAAHXZ 0000000140015220 f i ServerAppDlg.obj
 0001:00014220       ?Readuint32@ILTMessage_Read@@QEAAIXZ 0000000140015220 f i ServerAppDlg.obj
 0001:00014260       ??0exception@std@@QEAA@QEBD@Z 0000000140015260 f i ServerAppDlg.obj
 0001:000142b0       ??1exception@std@@UEAA@XZ  00000001400152b0 f i ServerAppDlg.obj
 0001:000142d0       ??_Eexception@std@@UEAAPEAXI@Z 00000001400152d0 f i * CIL library *:* CIL module *
 0001:000142d0       ??_Gexception@std@@UEAAPEAXI@Z 00000001400152d0 f i ServerAppDlg.obj
 0001:00014320       ?what@exception@std@@UEBAPEBDXZ 0000000140015320 f i ServerAppDlg.obj
 0001:00014340       ??0exception@std@@QEAA@AEBV01@@Z 0000000140015340 f i ServerAppDlg.obj
 0001:00014430       ?PreWriteData@GAMEPROTO_SC_COMMON@@UEAA_NPEAVILTMessage_Write@@@Z 0000000140015430 f i ServerAppDlg.obj
 0001:00014430       ?PreReadData@GAMEPROTO_SC_COMMON@@UEAA_NPEAVILTMessage_Read@@@Z 0000000140015430 f i ServerAppDlg.obj
 0001:00014430       __scrt_stub_for_acrt_initialize 0000000140015430 f i msvcrt:ucrt_stubs.obj
 0001:00014430       __vcrt_initialize          0000000140015430 f i msvcrt:ucrt_stubs.obj
 0001:00014430       _should_initialize_environment 0000000140015430 f i msvcrt:env_mode.obj
 0001:00014430       __vcrt_uninitialize        0000000140015430 f i msvcrt:ucrt_stubs.obj
 0001:00014430       __acrt_initialize          0000000140015430 f i msvcrt:ucrt_stubs.obj
 0001:00014430       __acrt_uninitialize        0000000140015430 f i msvcrt:ucrt_stubs.obj
 0001:00014430       __scrt_stub_for_acrt_uninitialize 0000000140015430 f i msvcrt:ucrt_stubs.obj
 0001:00014440       ?PostReadData@GAMEPROTO_SC_COMMON@@UEAA_NPEAVILTMessage_Read@@@Z 0000000140015440 f i ServerAppDlg.obj
 0001:000144d0       ?ReadData@PROTO_SERVERAPPMSG_INIT@@UEAA_NPEAVILTMessage_Read@@@Z 00000001400154d0 f i ServerAppDlg.obj
 0001:000145d0       ?PostWriteData@GAMEPROTO_SC_COMMON@@UEAA_NPEAVILTMessage_Write@@@Z 00000001400155d0 f i ServerAppDlg.obj
 0001:00014630       ?WriteData@PROTO_SERVERAPPMSG_INIT@@UEAA_NPEAVILTMessage_Write@@@Z 0000000140015630 f i ServerAppDlg.obj
 0001:00014710       ??_GCListBox@@UEAAPEAXI@Z  0000000140015710 f i ServerAppDlg.obj
 0001:00014710       ??_ECListBox@@UEAAPEAXI@Z  0000000140015710 f i * CIL library *:* CIL module *
 0001:00014760       ??_GCEdit@@UEAAPEAXI@Z     0000000140015760 f i ServerAppDlg.obj
 0001:00014760       ??_ECEdit@@UEAAPEAXI@Z     0000000140015760 f i * CIL library *:* CIL module *
 0001:000147b0       ?BeginModalState@CWnd@@UEAAXXZ 00000001400157b0 f i ServerAppDlg.obj
 0001:000147c0       ?EndModalState@CWnd@@UEAAXXZ 00000001400157c0 f i ServerAppDlg.obj
 0001:000147d0       ?_AtlInitializeCriticalSectionEx@ATL@@YAHPEAU_RTL_CRITICAL_SECTION@@KK@Z 00000001400157d0 f i StdAfx.obj
 0001:000147e0       ?sprintf_s@internal@cf@@YAHPEAD_KPEBDAEAPEAD@Z 00000001400157e0 f   safe_string_x64:safe_string.obj
 0001:00014ac0       ??_D?$basic_stringstream@DU?$char_traits@D@std@@V?$allocator@D@2@@std@@QEAAXXZ 0000000140015ac0 f i safe_string_x64:safe_string.obj
 0001:00014b20       ?strcpy_s@cf@@YAHPEAD_KPEBD@Z 0000000140015b20 f   safe_string_x64:safe_string.obj
 0001:00014dd0       ?strncpy_s@cf@@YAHPEAD_KPEBD1@Z 0000000140015dd0 f   safe_string_x64:safe_string.obj
 0001:000150a0       ?sprintf_s@cf@@YAHPEAD_KPEBDZZ 00000001400160a0 f   safe_string_x64:safe_string.obj
 0001:000150d0       ??0?$basic_stringstream@DU?$char_traits@D@std@@V?$allocator@D@2@@std@@QEAA@H@Z 00000001400160d0 f i safe_string_x64:safe_string.obj
 0001:00015190       ?seekpos@?$basic_stringbuf@DU?$char_traits@D@std@@V?$allocator@D@2@@std@@MEAA?AV?$fpos@U_Mbstatet@@@2@V32@H@Z 0000000140016190 f i safe_string_x64:safe_string.obj
 0001:00015280       ?seekoff@?$basic_stringbuf@DU?$char_traits@D@std@@V?$allocator@D@2@@std@@MEAA?AV?$fpos@U_Mbstatet@@@2@_JHH@Z 0000000140016280 f i safe_string_x64:safe_string.obj
 0001:000153d0       ?underflow@?$basic_stringbuf@DU?$char_traits@D@std@@V?$allocator@D@2@@std@@MEAAHXZ 00000001400163d0 f i safe_string_x64:safe_string.obj
 0001:00015440       ?pbackfail@?$basic_stringbuf@DU?$char_traits@D@std@@V?$allocator@D@2@@std@@MEAAHH@Z 0000000140016440 f i safe_string_x64:safe_string.obj
 0001:000154a0       ?overflow@?$basic_stringbuf@DU?$char_traits@D@std@@V?$allocator@D@2@@std@@MEAAHH@Z 00000001400164a0 f i safe_string_x64:safe_string.obj
 0001:000156a0       ??1?$basic_stringbuf@DU?$char_traits@D@std@@V?$allocator@D@2@@std@@UEAA@XZ 00000001400166a0 f i safe_string_x64:safe_string.obj
 0001:00015760       ??_G?$basic_stringstream@DU?$char_traits@D@std@@V?$allocator@D@2@@std@@UEAAPEAXI@Z 0000000140016760 f i safe_string_x64:safe_string.obj
 0001:00015760       ??_E?$basic_stringstream@DU?$char_traits@D@std@@V?$allocator@D@2@@std@@UEAAPEAXI@Z 0000000140016760 f i * CIL library *:* CIL module *
 0001:00015800       ??_E?$basic_stringbuf@DU?$char_traits@D@std@@V?$allocator@D@2@@std@@UEAAPEAXI@Z 0000000140016800 f i * CIL library *:* CIL module *
 0001:00015800       ??_G?$basic_stringbuf@DU?$char_traits@D@std@@V?$allocator@D@2@@std@@UEAAPEAXI@Z 0000000140016800 f i safe_string_x64:safe_string.obj
 0001:00015840       ??1sentry@?$basic_ostream@DU?$char_traits@D@std@@@std@@QEAA@XZ 0000000140016840 f i safe_string_x64:safe_string.obj
 0001:00015890       ??1_Sentry_base@?$basic_ostream@DU?$char_traits@D@std@@@std@@QEAA@XZ 0000000140016890 f i safe_string_x64:safe_string.obj
 0001:000158c0       ??$?6U?$char_traits@D@std@@@std@@YAAEAV?$basic_ostream@DU?$char_traits@D@std@@@0@AEAV10@PEBD@Z 00000001400168c0 f i safe_string_x64:safe_string.obj
 0001:00015a90       ??$endl@DU?$char_traits@D@std@@@std@@YAAEAV?$basic_ostream@DU?$char_traits@D@std@@@0@AEAV10@@Z 0000000140016a90 f i safe_string_x64:safe_string.obj
 0001:00015acc       ??_E?$basic_stringstream@DU?$char_traits@D@std@@V?$allocator@D@2@@std@@$4PPPPPPPM@A@EAAPEAXI@Z 0000000140016acc f i safe_string_x64:safe_string.obj
 0001:00015ad8       ??3@YAXPEAX@Z              0000000140016ad8 f   mfc140:mfc140.dll
 0001:00015ade       ?OnHelp@CWinApp@@IEAAXXZ   0000000140016ade f   mfc140:mfc140.dll
 0001:00015ae4       ?GetThisMessageMap@CWinApp@@KAPEBUAFX_MSGMAP@@XZ 0000000140016ae4 f   mfc140:mfc140.dll
 0001:00015aea       ?DoModal@CDialog@@UEAA_JXZ 0000000140016aea f   mfc140:mfc140.dll
 0001:00015af0       ?GetRuntimeClass@CWinApp@@UEBAPEAUCRuntimeClass@@XZ 0000000140016af0 f   mfc140:mfc140.dll
 0001:00015af6       ?OnCmdMsg@CCmdTarget@@UEAAHIHPEAXPEAUAFX_CMDHANDLERINFO@@@Z 0000000140016af6 f   mfc140:mfc140.dll
 0001:00015afc       ?OnFinalRelease@CCmdTarget@@UEAAXXZ 0000000140016afc f   mfc140:mfc140.dll
 0001:00015b02       ?IsInvokeAllowed@CCmdTarget@@UEAAHJ@Z 0000000140016b02 f   mfc140:mfc140.dll
 0001:00015b08       ?GetDispatchIID@CCmdTarget@@UEAAHPEAU_GUID@@@Z 0000000140016b08 f   mfc140:mfc140.dll
 0001:00015b0e       ?GetTypeInfoCount@CCmdTarget@@UEAAIXZ 0000000140016b0e f   mfc140:mfc140.dll
 0001:00015b14       ?GetTypeLibCache@CCmdTarget@@UEAAPEAVCTypeLibCache@@XZ 0000000140016b14 f   mfc140:mfc140.dll
 0001:00015b1a       ?GetTypeLib@CCmdTarget@@UEAAJKPEAPEAUITypeLib@@@Z 0000000140016b1a f   mfc140:mfc140.dll
 0001:00015b20       ?GetCommandMap@CCmdTarget@@MEBAPEBUAFX_OLECMDMAP@@XZ 0000000140016b20 f   mfc140:mfc140.dll
 0001:00015b26       ?GetDispatchMap@CCmdTarget@@MEBAPEBUAFX_DISPMAP@@XZ 0000000140016b26 f   mfc140:mfc140.dll
 0001:00015b2c       ?GetConnectionMap@CCmdTarget@@MEBAPEBUAFX_CONNECTIONMAP@@XZ 0000000140016b2c f   mfc140:mfc140.dll
 0001:00015b32       ?GetInterfaceMap@CCmdTarget@@MEBAPEBUAFX_INTERFACEMAP@@XZ 0000000140016b32 f   mfc140:mfc140.dll
 0001:00015b38       ?GetEventSinkMap@CCmdTarget@@MEBAPEBUAFX_EVENTSINKMAP@@XZ 0000000140016b38 f   mfc140:mfc140.dll
 0001:00015b3e       ?OnCreateAggregates@CCmdTarget@@UEAAHXZ 0000000140016b3e f   mfc140:mfc140.dll
 0001:00015b44       ?GetInterfaceHook@CCmdTarget@@UEAAPEAUIUnknown@@PEBX@Z 0000000140016b44 f   mfc140:mfc140.dll
 0001:00015b4a       ?GetExtraConnectionPoints@CCmdTarget@@MEAAHPEAVCPtrArray@@@Z 0000000140016b4a f   mfc140:mfc140.dll
 0001:00015b50       ?GetConnectionHook@CCmdTarget@@MEAAPEAUIConnectionPoint@@AEBU_GUID@@@Z 0000000140016b50 f   mfc140:mfc140.dll
 0001:00015b56       ?PreTranslateMessage@CWinThread@@UEAAHPEAUtagMSG@@@Z 0000000140016b56 f   mfc140:mfc140.dll
 0001:00015b5c       ?PumpMessage@CWinThread@@UEAAHXZ 0000000140016b5c f   mfc140:mfc140.dll
 0001:00015b62       ?OnIdle@CWinApp@@UEAAHJ@Z  0000000140016b62 f   mfc140:mfc140.dll
 0001:00015b68       ?IsIdleMessage@CWinThread@@UEAAHPEAUtagMSG@@@Z 0000000140016b68 f   mfc140:mfc140.dll
 0001:00015b6e       ?ExitInstance@CWinApp@@UEAAHXZ 0000000140016b6e f   mfc140:mfc140.dll
 0001:00015b74       ?ProcessWndProcException@CWinApp@@UEAA_JPEAVCException@@PEBUtagMSG@@@Z 0000000140016b74 f   mfc140:mfc140.dll
 0001:00015b7a       ?ProcessMessageFilter@CWinThread@@UEAAHHPEAUtagMSG@@@Z 0000000140016b7a f   mfc140:mfc140.dll
 0001:00015b80       ?GetMainWnd@CWinThread@@UEAAPEAVCWnd@@XZ 0000000140016b80 f   mfc140:mfc140.dll
 0001:00015b86       ?Delete@CWinThread@@UEAAXXZ 0000000140016b86 f   mfc140:mfc140.dll
 0001:00015b8c       ?GetProfileIntA@CWinApp@@UEAAIPEBD0H@Z 0000000140016b8c f   mfc140:mfc140.dll
 0001:00015b92       ?WriteProfileInt@CWinApp@@UEAAHPEBD0H@Z 0000000140016b92 f   mfc140:mfc140.dll
 0001:00015b98       ?GetProfileStringA@CWinApp@@UEAA?AV?$CStringT@DV?$StrTraitMFC_DLL@DV?$ChTraitsCRT@D@ATL@@@@@ATL@@PEBD00@Z 0000000140016b98 f   mfc140:mfc140.dll
 0001:00015b9e       ?WriteProfileStringA@CWinApp@@UEAAHPEBD00@Z 0000000140016b9e f   mfc140:mfc140.dll
 0001:00015ba4       ?GetProfileBinary@CWinApp@@UEAAHPEBD0PEAPEAEPEAI@Z 0000000140016ba4 f   mfc140:mfc140.dll
 0001:00015baa       ?WriteProfileBinary@CWinApp@@UEAAHPEBD0PEAEI@Z 0000000140016baa f   mfc140:mfc140.dll
 0001:00015bb0       ?InitLibId@CWinApp@@UEAAXXZ 0000000140016bb0 f   mfc140:mfc140.dll
 0001:00015bb6       ?Register@CWinApp@@UEAAHXZ 0000000140016bb6 f   mfc140:mfc140.dll
 0001:00015bbc       ?Unregister@CWinApp@@UEAAHXZ 0000000140016bbc f   mfc140:mfc140.dll
 0001:00015bc2       ?OpenDocumentFile@CWinApp@@UEAAPEAVCDocument@@PEBDH@Z 0000000140016bc2 f   mfc140:mfc140.dll
 0001:00015bc8       ?OpenDocumentFile@CWinApp@@UEAAPEAVCDocument@@PEBD@Z 0000000140016bc8 f   mfc140:mfc140.dll
 0001:00015bce       ?AddToRecentFileList@CWinApp@@UEAAXPEBD@Z 0000000140016bce f   mfc140:mfc140.dll
 0001:00015bd4       ?InitApplication@CWinApp@@UEAAHXZ 0000000140016bd4 f   mfc140:mfc140.dll
 0001:00015bda       ?SaveAllModified@CWinApp@@UEAAHXZ 0000000140016bda f   mfc140:mfc140.dll
 0001:00015be0       ?DoMessageBox@CWinApp@@UEAAHPEBDII@Z 0000000140016be0 f   mfc140:mfc140.dll
 0001:00015be6       ?DoWaitCursor@CWinApp@@UEAAXH@Z 0000000140016be6 f   mfc140:mfc140.dll
 0001:00015bec       ?OnDDECommand@CWinApp@@UEAAHPEAD@Z 0000000140016bec f   mfc140:mfc140.dll
 0001:00015bf2       ?WinHelpA@CWinApp@@UEAAX_KI@Z 0000000140016bf2 f   mfc140:mfc140.dll
 0001:00015bf8       ?HtmlHelpA@CWinApp@@UEAAX_KI@Z 0000000140016bf8 f   mfc140:mfc140.dll
 0001:00015bfe       ?WinHelpInternal@CWinApp@@UEAAX_KI@Z 0000000140016bfe f   mfc140:mfc140.dll
 0001:00015c04       ?RegisterWithRestartManager@CWinApp@@UEAAJPEB_WKP6AKPEAX@Z1KK@Z 0000000140016c04 f   mfc140:mfc140.dll
 0001:00015c0a       ?RegisterWithRestartManager@CWinApp@@UEAAJHAEBV?$CStringT@DV?$StrTraitMFC_DLL@DV?$ChTraitsCRT@D@ATL@@@@@ATL@@@Z 0000000140016c0a f   mfc140:mfc140.dll
 0001:00015c10       ?ApplicationRecoveryCallback@CWinApp@@UEAAKPEAX@Z 0000000140016c10 f   mfc140:mfc140.dll
 0001:00015c16       ?GetDataRecoveryHandler@CWinApp@@UEAAPEAVCDataRecoveryHandler@@XZ 0000000140016c16 f   mfc140:mfc140.dll
 0001:00015c1c       ?IsTaskbarInteractionEnabled@CWinApp@@UEAAHXZ 0000000140016c1c f   mfc140:mfc140.dll
 0001:00015c22       ?RestartInstance@CWinApp@@UEAAHXZ 0000000140016c22 f   mfc140:mfc140.dll
 0001:00015c28       ?LoadAppLangResourceDLL@CWinApp@@UEAAPEAUHINSTANCE__@@XZ 0000000140016c28 f   mfc140:mfc140.dll
 0001:00015c2e       ?LoadSysPolicies@CWinApp@@UEAAHXZ 0000000140016c2e f   mfc140:mfc140.dll
 0001:00015c34       ?GetOccDialogInfo@CWnd@@MEAAPEAU_AFX_OCC_DIALOG_INFO@@XZ 0000000140016c34 f   mfc140:mfc140.dll
 0001:00015c3a       ?SetOccDialogInfo@CWnd@@MEAAHPEAU_AFX_OCC_DIALOG_INFO@@@Z 0000000140016c3a f   mfc140:mfc140.dll
 0001:00015c40       ?CreateControlSite@CWnd@@MEAAHPEAVCOleControlContainer@@PEAPEAVCOleControlSite@@IAEBU_GUID@@@Z 0000000140016c40 f   mfc140:mfc140.dll
 0001:00015c46       ?CreateControlContainer@CWnd@@MEAAHPEAPEAVCOleControlContainer@@@Z 0000000140016c46 f   mfc140:mfc140.dll
 0001:00015c4c       ?IsFrameWnd@CWnd@@UEBAHXZ  0000000140016c4c f   mfc140:mfc140.dll
 0001:00015c52       ?CheckAutoCenter@CWnd@@UEAAHXZ 0000000140016c52 f   mfc140:mfc140.dll
 0001:00015c58       ?ResizeDynamicLayout@CWnd@@MEAAXXZ 0000000140016c58 f   mfc140:mfc140.dll
 0001:00015c5e       ?OnGesturePressAndTap@CWnd@@MEAAHVCPoint@@J@Z 0000000140016c5e f   mfc140:mfc140.dll
 0001:00015c64       ?OnGestureTwoFingerTap@CWnd@@MEAAHVCPoint@@@Z 0000000140016c64 f   mfc140:mfc140.dll
 0001:00015c6a       ?OnGestureRotate@CWnd@@MEAAHVCPoint@@N@Z 0000000140016c6a f   mfc140:mfc140.dll
 0001:00015c70       ?OnGesturePan@CWnd@@MEAAHVCPoint@@0@Z 0000000140016c70 f   mfc140:mfc140.dll
 0001:00015c76       ?OnGestureZoom@CWnd@@MEAAHVCPoint@@J@Z 0000000140016c76 f   mfc140:mfc140.dll
 0001:00015c7c       ?GetGestureStatus@CWnd@@MEAAKVCPoint@@@Z 0000000140016c7c f   mfc140:mfc140.dll
 0001:00015c82       ?OnTouchInput@CWnd@@MEAAHVCPoint@@HHPEAUtagTOUCHINPUT@@@Z 0000000140016c82 f   mfc140:mfc140.dll
 0001:00015c88       ?OnTouchInputs@CWnd@@MEAAHIPEAUtagTOUCHINPUT@@@Z 0000000140016c88 f   mfc140:mfc140.dll
 0001:00015c8e       ?OnChildNotify@CWnd@@MEAAHI_K_JPEA_J@Z 0000000140016c8e f   mfc140:mfc140.dll
 0001:00015c94       ?PostNcDestroy@CWnd@@MEAAXXZ 0000000140016c94 f   mfc140:mfc140.dll
 0001:00015c9a       ?DefWindowProcA@CWnd@@MEAA_JI_K_J@Z 0000000140016c9a f   mfc140:mfc140.dll
 0001:00015ca0       ?OnWndMsg@CWnd@@MEAAHI_K_JPEA_J@Z 0000000140016ca0 f   mfc140:mfc140.dll
 0001:00015ca6       ?WindowProc@CWnd@@MEAA_JI_K_J@Z 0000000140016ca6 f   mfc140:mfc140.dll
 0001:00015cac       ?OnAmbientProperty@CWnd@@UEAAHPEAVCOleControlSite@@JPEAUtagVARIANT@@@Z 0000000140016cac f   mfc140:mfc140.dll
 0001:00015cb2       ?PreTranslateMessage@CWnd@@UEAAHPEAUtagMSG@@@Z 0000000140016cb2 f   mfc140:mfc140.dll
 0001:00015cb8       ?GetSuperWndProcAddr@CWnd@@MEAAPEAP6A_JPEAUHWND__@@I_K_J@ZXZ 0000000140016cb8 f   mfc140:mfc140.dll
 0001:00015cbe       ?OnNotify@CWnd@@MEAAH_K_JPEA_J@Z 0000000140016cbe f   mfc140:mfc140.dll
 0001:00015cc4       ?OnCommand@CWnd@@MEAAH_K_J@Z 0000000140016cc4 f   mfc140:mfc140.dll
 0001:00015cca       ?CreateAccessibleProxy@CWnd@@UEAAJ_K_JPEA_J@Z 0000000140016cca f   mfc140:mfc140.dll
 0001:00015cd0       ?SetProxy@CWnd@@UEAAJPEAUIAccessibleProxy@@@Z 0000000140016cd0 f   mfc140:mfc140.dll
 0001:00015cd6       ?put_accValue@CWnd@@UEAAJUtagVARIANT@@PEA_W@Z 0000000140016cd6 f   mfc140:mfc140.dll
 0001:00015cdc       ?put_accName@CWnd@@UEAAJUtagVARIANT@@PEA_W@Z 0000000140016cdc f   mfc140:mfc140.dll
 0001:00015ce2       ?accDoDefaultAction@CWnd@@UEAAJUtagVARIANT@@@Z 0000000140016ce2 f   mfc140:mfc140.dll
 0001:00015ce8       ?accHitTest@CWnd@@UEAAJJJPEAUtagVARIANT@@@Z 0000000140016ce8 f   mfc140:mfc140.dll
 0001:00015cee       ?accNavigate@CWnd@@UEAAJJUtagVARIANT@@PEAU2@@Z 0000000140016cee f   mfc140:mfc140.dll
 0001:00015cf4       ?accLocation@CWnd@@UEAAJPEAJ000UtagVARIANT@@@Z 0000000140016cf4 f   mfc140:mfc140.dll
 0001:00015cfa       ?accSelect@CWnd@@UEAAJJUtagVARIANT@@@Z 0000000140016cfa f   mfc140:mfc140.dll
 0001:00015d00       ?get_accDefaultAction@CWnd@@UEAAJUtagVARIANT@@PEAPEA_W@Z 0000000140016d00 f   mfc140:mfc140.dll
 0001:00015d06       ?get_accSelection@CWnd@@UEAAJPEAUtagVARIANT@@@Z 0000000140016d06 f   mfc140:mfc140.dll
 0001:00015d0c       ?get_accFocus@CWnd@@UEAAJPEAUtagVARIANT@@@Z 0000000140016d0c f   mfc140:mfc140.dll
 0001:00015d12       ?get_accKeyboardShortcut@CWnd@@UEAAJUtagVARIANT@@PEAPEA_W@Z 0000000140016d12 f   mfc140:mfc140.dll
 0001:00015d18       ?get_accHelpTopic@CWnd@@UEAAJPEAPEA_WUtagVARIANT@@PEAJ@Z 0000000140016d18 f   mfc140:mfc140.dll
 0001:00015d1e       ?get_accHelp@CWnd@@UEAAJUtagVARIANT@@PEAPEA_W@Z 0000000140016d1e f   mfc140:mfc140.dll
 0001:00015d24       ?get_accState@CWnd@@UEAAJUtagVARIANT@@PEAU2@@Z 0000000140016d24 f   mfc140:mfc140.dll
 0001:00015d2a       ?get_accRole@CWnd@@UEAAJUtagVARIANT@@PEAU2@@Z 0000000140016d2a f   mfc140:mfc140.dll
 0001:00015d30       ?get_accDescription@CWnd@@UEAAJUtagVARIANT@@PEAPEA_W@Z 0000000140016d30 f   mfc140:mfc140.dll
 0001:00015d36       ?get_accValue@CWnd@@UEAAJUtagVARIANT@@PEAPEA_W@Z 0000000140016d36 f   mfc140:mfc140.dll
 0001:00015d3c       ?get_accName@CWnd@@UEAAJUtagVARIANT@@PEAPEA_W@Z 0000000140016d3c f   mfc140:mfc140.dll
 0001:00015d42       ?get_accChild@CWnd@@UEAAJUtagVARIANT@@PEAPEAUIDispatch@@@Z 0000000140016d42 f   mfc140:mfc140.dll
 0001:00015d48       ?get_accChildCount@CWnd@@UEAAJPEAJ@Z 0000000140016d48 f   mfc140:mfc140.dll
 0001:00015d4e       ?get_accParent@CWnd@@UEAAJPEAPEAUIDispatch@@@Z 0000000140016d4e f   mfc140:mfc140.dll
 0001:00015d54       ?EnsureStdObj@CWnd@@UEAAJXZ 0000000140016d54 f   mfc140:mfc140.dll
 0001:00015d5a       ?OnDrawIconicThumbnailOrLivePreview@CWnd@@UEAAXAEAVCDC@@VCRect@@VCSize@@HAEAH@Z 0000000140016d5a f   mfc140:mfc140.dll
 0001:00015d60       ?EndModalLoop@CWnd@@UEAAXH@Z 0000000140016d60 f   mfc140:mfc140.dll
 0001:00015d66       ?ContinueModal@CWnd@@UEAAHXZ 0000000140016d66 f   mfc140:mfc140.dll
 0001:00015d6c       ?WinHelpInternal@CWnd@@UEAAX_KI@Z 0000000140016d6c f   mfc140:mfc140.dll
 0001:00015d72       ?HtmlHelpA@CWnd@@UEAAX_KI@Z 0000000140016d72 f   mfc140:mfc140.dll
 0001:00015d78       ?WinHelpA@CWnd@@UEAAX_KI@Z 0000000140016d78 f   mfc140:mfc140.dll
 0001:00015d7e       ?GetScrollBarCtrl@CWnd@@UEBAPEAVCScrollBar@@H@Z 0000000140016d7e f   mfc140:mfc140.dll
 0001:00015d84       ?OnToolHitTest@CWnd@@UEBA_JVCPoint@@PEAUtagTOOLINFOA@@@Z 0000000140016d84 f   mfc140:mfc140.dll
 0001:00015d8a       ?SetMenu@CWnd@@UEAAHPEAVCMenu@@@Z 0000000140016d8a f   mfc140:mfc140.dll
 0001:00015d90       ?GetMenu@CWnd@@UEBAPEAVCMenu@@XZ 0000000140016d90 f   mfc140:mfc140.dll
 0001:00015d96       ?CalcWindowRect@CWnd@@UEAAXPEAUtagRECT@@I@Z 0000000140016d96 f   mfc140:mfc140.dll
 0001:00015d9c       ?PreCreateWindow@CWnd@@UEAAHAEAUtagCREATESTRUCTA@@@Z 0000000140016d9c f   mfc140:mfc140.dll
 0001:00015da2       ?DestroyWindow@CWnd@@UEAAHXZ 0000000140016da2 f   mfc140:mfc140.dll
 0001:00015da8       ?CreateEx@CWnd@@UEAAHKPEBD0KHHHHPEAUHWND__@@PEAUHMENU__@@PEAX@Z 0000000140016da8 f   mfc140:mfc140.dll
 0001:00015dae       ?CreateEx@CWnd@@UEAAHKPEBD0KAEBUtagRECT@@PEAV1@IPEAX@Z 0000000140016dae f   mfc140:mfc140.dll
 0001:00015db4       ?Create@CWnd@@UEAAHPEBD0KAEBUtagRECT@@PEAV1@IPEAUCCreateContext@@@Z 0000000140016db4 f   mfc140:mfc140.dll
 0001:00015dba       ?PreSubclassWindow@CWnd@@UEAAXXZ 0000000140016dba f   mfc140:mfc140.dll
 0001:00015dc0       ?GetInterfaceMap@CWnd@@MEBAPEBUAFX_INTERFACEMAP@@XZ 0000000140016dc0 f   mfc140:mfc140.dll
 0001:00015dc6       ?GetMessageMap@CWnd@@MEBAPEBUAFX_MSGMAP@@XZ 0000000140016dc6 f   mfc140:mfc140.dll
 0001:00015dcc       ?OnFinalRelease@CWnd@@UEAAXXZ 0000000140016dcc f   mfc140:mfc140.dll
 0001:00015dd2       ?GetRuntimeClass@CEdit@@UEBAPEAUCRuntimeClass@@XZ 0000000140016dd2 f   mfc140:mfc140.dll
 0001:00015dd8       ?CharToItem@CListBox@@UEAAHII@Z 0000000140016dd8 f   mfc140:mfc140.dll
 0001:00015dde       ?VKeyToItem@CListBox@@UEAAHII@Z 0000000140016dde f   mfc140:mfc140.dll
 0001:00015de4       ?DeleteItem@CListBox@@UEAAXPEAUtagDELETEITEMSTRUCT@@@Z 0000000140016de4 f   mfc140:mfc140.dll
 0001:00015dea       ?CompareItem@CListBox@@UEAAHPEAUtagCOMPAREITEMSTRUCT@@@Z 0000000140016dea f   mfc140:mfc140.dll
 0001:00015df0       ?MeasureItem@CListBox@@UEAAXPEAUtagMEASUREITEMSTRUCT@@@Z 0000000140016df0 f   mfc140:mfc140.dll
 0001:00015df6       ?DrawItem@CListBox@@UEAAXPEAUtagDRAWITEMSTRUCT@@@Z 0000000140016df6 f   mfc140:mfc140.dll
 0001:00015dfc       ?Create@CListBox@@UEAAHKAEBUtagRECT@@PEAVCWnd@@I@Z 0000000140016dfc f   mfc140:mfc140.dll
 0001:00015e02       ?OnChildNotify@CListBox@@MEAAHI_K_JPEA_J@Z 0000000140016e02 f   mfc140:mfc140.dll
 0001:00015e08       ?GetRuntimeClass@CListBox@@UEBAPEAUCRuntimeClass@@XZ 0000000140016e08 f   mfc140:mfc140.dll
 0001:00015e0e       ?AfxGetModuleState@@YAPEAVAFX_MODULE_STATE@@XZ 0000000140016e0e f   mfc140:mfc140.dll
 0001:00015e14       ?GetThisMessageMap@CDialog@@KAPEBUAFX_MSGMAP@@XZ 0000000140016e14 f   mfc140:mfc140.dll
 0001:00015e1a       ?OnOK@CDialog@@MEAAXXZ     0000000140016e1a f   mfc140:mfc140.dll
 0001:00015e20       ?GetRuntimeClass@CDialog@@UEBAPEAUCRuntimeClass@@XZ 0000000140016e20 f   mfc140:mfc140.dll
 0001:00015e26       ?OnCmdMsg@CDialog@@UEAAHIHPEAXPEAUAFX_CMDHANDLERINFO@@@Z 0000000140016e26 f   mfc140:mfc140.dll
 0001:00015e2c       ?PreTranslateMessage@CDialog@@UEAAHPEAUtagMSG@@@Z 0000000140016e2c f   mfc140:mfc140.dll
 0001:00015e32       ?CheckAutoCenter@CDialog@@UEAAHXZ 0000000140016e32 f   mfc140:mfc140.dll
 0001:00015e38       ?SetOccDialogInfo@CDialog@@MEAAHPEAU_AFX_OCC_DIALOG_INFO@@@Z 0000000140016e38 f   mfc140:mfc140.dll
 0001:00015e3e       ?GetOccDialogInfo@CDialog@@MEAAPEAU_AFX_OCC_DIALOG_INFO@@XZ 0000000140016e3e f   mfc140:mfc140.dll
 0001:00015e44       ?Create@CDialog@@UEAAHPEBDPEAVCWnd@@@Z 0000000140016e44 f   mfc140:mfc140.dll
 0001:00015e4a       ?CreateIndirect@CDialog@@UEAAHPEAXPEAVCWnd@@@Z 0000000140016e4a f   mfc140:mfc140.dll
 0001:00015e50       ?CreateIndirect@CDialog@@UEAAHPEBUDLGTEMPLATE@@PEAVCWnd@@PEAX@Z 0000000140016e50 f   mfc140:mfc140.dll
 0001:00015e56       ?OnSetFont@CDialog@@UEAAXPEAVCFont@@@Z 0000000140016e56 f   mfc140:mfc140.dll
 0001:00015e5c       ?OnCancel@CDialog@@MEAAXXZ 0000000140016e5c f   mfc140:mfc140.dll
 0001:00015e62       ?PreInitDialog@CDialog@@MEAAXXZ 0000000140016e62 f   mfc140:mfc140.dll
 0001:00015e80       __security_check_cookie    0000000140016e80 f   msvcrt:amdsecgs.obj
 0001:00015ea4       ??3@YAXPEAX_K@Z            0000000140016ea4 f   msvcrt:delete_scalar_size.obj
 0001:00016034       _Init_thread_abort         0000000140017034 f   msvcrt:thread_safe_statics.obj
 0001:00016064       _Init_thread_footer        0000000140017064 f   msvcrt:thread_safe_statics.obj
 0001:000160c4       _Init_thread_header        00000001400170c4 f   msvcrt:thread_safe_statics.obj
 0001:0001612c       _Init_thread_notify        000000014001712c f   msvcrt:thread_safe_statics.obj
 0001:0001617c       _Init_thread_wait          000000014001717c f   msvcrt:thread_safe_statics.obj
 0001:000161f4       __scrt_acquire_startup_lock 00000001400171f4 f   msvcrt:utility.obj
 0001:00016230       __scrt_initialize_crt      0000000140017230 f   msvcrt:utility.obj
 0001:0001627c       __scrt_initialize_onexit_tables 000000014001727c f   msvcrt:utility.obj
 0001:00016354       __scrt_is_nonwritable_in_current_image 0000000140017354 f   msvcrt:utility.obj
 0001:000163f0       __scrt_release_startup_lock 00000001400173f0 f   msvcrt:utility.obj
 0001:00016414       __scrt_uninitialize_crt    0000000140017414 f   msvcrt:utility.obj
 0001:00016440       _onexit                    0000000140017440 f   msvcrt:utility.obj
 0001:00016490       atexit                     0000000140017490 f   msvcrt:utility.obj
 0001:000164a8       ??_Etype_info@@UEAAPEAXI@Z 00000001400174a8 f i msvcrt:std_type_info_static.obj
 0001:000164a8       ??_Gtype_info@@UEAAPEAXI@Z 00000001400174a8 f i msvcrt:std_type_info_static.obj
 0001:000164d4       __raise_securityfailure    00000001400174d4 f   msvcrt:gs_report.obj
 0001:00016508       __report_gsfailure         0000000140017508 f   msvcrt:gs_report.obj
 0001:000168a8       WinMainCRTStartup          00000001400178a8 f   msvcrt:exe_winmain.obj
 0001:000168bc       __crt_debugger_hook        00000001400178bc f   msvcrt:utility_desktop.obj
 0001:000168c4       __scrt_fastfail            00000001400178c4 f   msvcrt:utility_desktop.obj
 0001:00016a10       __scrt_get_show_window_mode 0000000140017a10 f   msvcrt:utility_desktop.obj
 0001:00016a4c       __scrt_initialize_mta      0000000140017a4c f   msvcrt:utility_desktop.obj
 0001:00016a54       __scrt_is_managed_app      0000000140017a54 f   msvcrt:utility_desktop.obj
 0001:00016aa8       __scrt_set_unhandled_exception_filter 0000000140017aa8 f   msvcrt:utility_desktop.obj
 0001:00016ab8       __scrt_unhandled_exception_filter 0000000140017ab8 f   msvcrt:utility_desktop.obj
 0001:00016af0       __isa_available_init       0000000140017af0 f   msvcrt:cpu_disp.obj
 0001:00016c6c       __scrt_is_ucrt_dll_in_use  0000000140017c6c f   msvcrt:ucrt_detection.obj
 0001:00016c78       __security_init_cookie     0000000140017c78 f   msvcrt:gs_support.obj
 0001:00016d24       _get_startup_file_mode     0000000140017d24 f   msvcrt:file_mode.obj
 0001:00016d2c       ?__scrt_initialize_type_info@@YAXXZ 0000000140017d2c f   msvcrt:tncleanup.obj
 0001:00016d3c       __scrt_initialize_default_local_stdio_options 0000000140017d3c f   msvcrt:default_local_stdio_options.obj
 0001:00016d58       __scrt_is_user_matherr_present 0000000140017d58 f   msvcrt:matherr_detection.obj
 0001:00016d64       __scrt_get_dyn_tls_init_callback 0000000140017d64 f   msvcrt:dyn_tls_init.obj
 0001:00016d6c       __scrt_get_dyn_tls_dtor_callback 0000000140017d6c f   msvcrt:dyn_tls_dtor.obj
 0001:00016d74       _RTC_Initialize            0000000140017d74 f   msvcrt:initsect.obj
 0001:00016db0       _RTC_Terminate             0000000140017db0 f   msvcrt:initsect.obj
 0001:00016dec       __GSHandlerCheck           0000000140017dec f   msvcrt:gshandler.obj
 0001:00016e0c       __GSHandlerCheckCommon     0000000140017e0c f   msvcrt:gshandler.obj
 0001:00016e70       IsProcessorFeaturePresent  0000000140017e70 f   kernel32:KERNEL32.dll
 0001:00016e78       ??0CAtlBaseModule@ATL@@QEAA@XZ 0000000140017e78 f   atls:atlbase.obj
 0001:00016f20       ??1CAtlBaseModule@ATL@@QEAA@XZ 0000000140017f20 f   atls:atlbase.obj
 0001:00016f54       __CxxFrameHandler3         0000000140017f54 f   vcruntime:VCRUNTIME140.dll
 0001:00016f5a       __std_terminate            0000000140017f5a f   vcruntime:VCRUNTIME140.dll
 0001:00016f60       _purecall                  0000000140017f60 f   vcruntime:VCRUNTIME140.dll
 0001:00016f66       memset                     0000000140017f66 f   vcruntime:VCRUNTIME140.dll
 0001:00016f6c       __C_specific_handler       0000000140017f6c f   vcruntime:VCRUNTIME140.dll
 0001:00016f72       memmove                    0000000140017f72 f   vcruntime:VCRUNTIME140.dll
 0001:00016f78       free                       0000000140017f78 f   ucrt:api-ms-win-crt-heap-l1-1-0.dll
 0001:00016f7e       _configure_narrow_argv     0000000140017f7e f   ucrt:api-ms-win-crt-runtime-l1-1-0.dll
 0001:00016f84       _initialize_narrow_environment 0000000140017f84 f   ucrt:api-ms-win-crt-runtime-l1-1-0.dll
 0001:00016f8a       _initialize_onexit_table   0000000140017f8a f   ucrt:api-ms-win-crt-runtime-l1-1-0.dll
 0001:00016f90       _register_onexit_function  0000000140017f90 f   ucrt:api-ms-win-crt-runtime-l1-1-0.dll
 0001:00016f96       _crt_atexit                0000000140017f96 f   ucrt:api-ms-win-crt-runtime-l1-1-0.dll
 0001:00016f9c       _cexit                     0000000140017f9c f   ucrt:api-ms-win-crt-runtime-l1-1-0.dll
 0001:00016fa2       _seh_filter_exe            0000000140017fa2 f   ucrt:api-ms-win-crt-runtime-l1-1-0.dll
 0001:00016fa8       _set_app_type              0000000140017fa8 f   ucrt:api-ms-win-crt-runtime-l1-1-0.dll
 0001:00016fae       __setusermatherr           0000000140017fae f   ucrt:api-ms-win-crt-math-l1-1-0.dll
 0001:00016fb4       _get_narrow_winmain_command_line 0000000140017fb4 f   ucrt:api-ms-win-crt-runtime-l1-1-0.dll
 0001:00016fba       _initterm                  0000000140017fba f   ucrt:api-ms-win-crt-runtime-l1-1-0.dll
 0001:00016fc0       _initterm_e                0000000140017fc0 f   ucrt:api-ms-win-crt-runtime-l1-1-0.dll
 0001:00016fc6       exit                       0000000140017fc6 f   ucrt:api-ms-win-crt-runtime-l1-1-0.dll
 0001:00016fcc       _exit                      0000000140017fcc f   ucrt:api-ms-win-crt-runtime-l1-1-0.dll
 0001:00016fd2       _set_fmode                 0000000140017fd2 f   ucrt:api-ms-win-crt-stdio-l1-1-0.dll
 0001:00016fd8       _c_exit                    0000000140017fd8 f   ucrt:api-ms-win-crt-runtime-l1-1-0.dll
 0001:00016fde       _register_thread_local_exe_atexit_callback 0000000140017fde f   ucrt:api-ms-win-crt-runtime-l1-1-0.dll
 0001:00016fe4       _configthreadlocale        0000000140017fe4 f   ucrt:api-ms-win-crt-locale-l1-1-0.dll
 0001:00016fea       _set_new_mode              0000000140017fea f   ucrt:api-ms-win-crt-heap-l1-1-0.dll
 0001:00016ff0       __p__commode               0000000140017ff0 f   ucrt:api-ms-win-crt-stdio-l1-1-0.dll
 0001:00016ff6       terminate                  0000000140017ff6 f   ucrt:api-ms-win-crt-runtime-l1-1-0.dll
 0001:00016ffc       ?AfxInitialize@@YAHHK@Z    0000000140017ffc f   mfcs140:appmodul.obj
 0001:00017034       WinMain                    0000000140018034 f   mfcs140:appmodul.obj
 0001:00017039       ?_Lock@?$basic_streambuf@DU?$char_traits@D@std@@@std@@UEAAXXZ 0000000140018039 f   msvcprt:MSVCP140.dll
 0001:0001703f       ?_Unlock@?$basic_streambuf@DU?$char_traits@D@std@@@std@@UEAAXXZ 000000014001803f f   msvcprt:MSVCP140.dll
 0001:00017045       ?showmanyc@?$basic_streambuf@DU?$char_traits@D@std@@@std@@MEAA_JXZ 0000000140018045 f   msvcprt:MSVCP140.dll
 0001:0001704b       ?uflow@?$basic_streambuf@DU?$char_traits@D@std@@@std@@MEAAHXZ 000000014001804b f   msvcprt:MSVCP140.dll
 0001:00017051       ?xsgetn@?$basic_streambuf@DU?$char_traits@D@std@@@std@@MEAA_JPEAD_J@Z 0000000140018051 f   msvcprt:MSVCP140.dll
 0001:00017057       ?xsputn@?$basic_streambuf@DU?$char_traits@D@std@@@std@@MEAA_JPEBD_J@Z 0000000140018057 f   msvcprt:MSVCP140.dll
 0001:0001705d       ?setbuf@?$basic_streambuf@DU?$char_traits@D@std@@@std@@MEAAPEAV12@PEAD_J@Z 000000014001805d f   msvcprt:MSVCP140.dll
 0001:00017063       ?sync@?$basic_streambuf@DU?$char_traits@D@std@@@std@@MEAAHXZ 0000000140018063 f   msvcprt:MSVCP140.dll
 0001:00017069       ?imbue@?$basic_streambuf@DU?$char_traits@D@std@@@std@@MEAAXAEBVlocale@2@@Z 0000000140018069 f   msvcprt:MSVCP140.dll
 0001:0001706f       ?AfxWinMain@@YAHPEAUHINSTANCE__@@0PEADH@Z 000000014001806f f   mfc140:mfc140.dll
 0001:00017078       __GSHandlerCheck_EH        0000000140018078 f   msvcrt:gshandlereh.obj
 0001:00017110       __chkstk                   0000000140018110 f   msvcrt:chkstk.obj
 0001:00017110       _alloca_probe              0000000140018110 f   msvcrt:chkstk.obj
 0001:00017161       _CxxThrowException         0000000140018161 f   vcruntime:VCRUNTIME140.dll
 0001:00017167       __RTDynamicCast            0000000140018167 f   vcruntime:VCRUNTIME140.dll
 0001:0001716d       memchr                     000000014001816d f   vcruntime:VCRUNTIME140.dll
 0001:00017173       memcmp                     0000000140018173 f   vcruntime:VCRUNTIME140.dll
 0001:00017179       memcpy                     0000000140018179 f   vcruntime:VCRUNTIME140.dll
 0001:0001717f       atan                       000000014001817f f   ucrt:api-ms-win-crt-math-l1-1-0.dll
 0001:00017185       sqrt                       0000000140018185 f   ucrt:api-ms-win-crt-math-l1-1-0.dll
 0001:0001718b       sqrtf                      000000014001818b f   ucrt:api-ms-win-crt-math-l1-1-0.dll
 0001:000171b0       _guard_dispatch_icall_nop  00000001400181b0 f   msvcrt:guard_dispatch.obj
 0002:00000000       __imp_OpenFileMappingA     000000014001a000     kernel32:KERNEL32.dll
 0002:00000008       __imp_ReadFile             000000014001a008     kernel32:KERNEL32.dll
 0002:00000010       __imp_CloseHandle          000000014001a010     kernel32:KERNEL32.dll
 0002:00000018       __imp_GetCurrentDirectoryA 000000014001a018     kernel32:KERNEL32.dll
 0002:00000020       __imp_SetCurrentDirectoryA 000000014001a020     kernel32:KERNEL32.dll
 0002:00000028       __imp_GetLocalTime         000000014001a028     kernel32:KERNEL32.dll
 0002:00000030       __imp_GetCurrentThreadId   000000014001a030     kernel32:KERNEL32.dll
 0002:00000038       __imp_GetPrivateProfileIntA 000000014001a038     kernel32:KERNEL32.dll
 0002:00000040       __imp_GetCurrentProcessId  000000014001a040     kernel32:KERNEL32.dll
 0002:00000048       __imp_GetCurrentProcess    000000014001a048     kernel32:KERNEL32.dll
 0002:00000050       __imp_CreateThread         000000014001a050     kernel32:KERNEL32.dll
 0002:00000058       __imp_WaitForSingleObject  000000014001a058     kernel32:KERNEL32.dll
 0002:00000060       __imp_RaiseException       000000014001a060     kernel32:KERNEL32.dll
 0002:00000068       __imp_SetUnhandledExceptionFilter 000000014001a068     kernel32:KERNEL32.dll
 0002:00000070       __imp_GetPrivateProfileStringW 000000014001a070     kernel32:KERNEL32.dll
 0002:00000078       __imp_GetModuleFileNameW   000000014001a078     kernel32:KERNEL32.dll
 0002:00000080       __imp_MultiByteToWideChar  000000014001a080     kernel32:KERNEL32.dll
 0002:00000088       __imp_GetComputerNameW     000000014001a088     kernel32:KERNEL32.dll
 0002:00000090       __imp_WideCharToMultiByte  000000014001a090     kernel32:KERNEL32.dll
 0002:00000098       __imp_GetLastError         000000014001a098     kernel32:KERNEL32.dll
 0002:000000a0       __imp_GetCurrentThread     000000014001a0a0     kernel32:KERNEL32.dll
 0002:000000a8       __imp_CreateFileW          000000014001a0a8     kernel32:KERNEL32.dll
 0002:000000b0       __imp_GetFileSize          000000014001a0b0     kernel32:KERNEL32.dll
 0002:000000b8       __imp_InitializeCriticalSection 000000014001a0b8     kernel32:KERNEL32.dll
 0002:000000c0       __imp_DeleteCriticalSection 000000014001a0c0     kernel32:KERNEL32.dll
 0002:000000c8       __imp_EnterCriticalSection 000000014001a0c8     kernel32:KERNEL32.dll
 0002:000000d0       __imp_LeaveCriticalSection 000000014001a0d0     kernel32:KERNEL32.dll
 0002:000000d8       __imp_MapViewOfFile        000000014001a0d8     kernel32:KERNEL32.dll
 0002:000000e0       __imp_UnmapViewOfFile      000000014001a0e0     kernel32:KERNEL32.dll
 0002:000000e8       __imp_CreateFileMappingA   000000014001a0e8     kernel32:KERNEL32.dll
 0002:000000f0       __imp_GetTickCount         000000014001a0f0     kernel32:KERNEL32.dll
 0002:000000f8       __imp_Sleep                000000014001a0f8     kernel32:KERNEL32.dll
 0002:00000100       __imp_OpenProcess          000000014001a100     kernel32:KERNEL32.dll
 0002:00000108       __imp_CreateEventA         000000014001a108     kernel32:KERNEL32.dll
 0002:00000110       __imp_GetProcAddress       000000014001a110     kernel32:KERNEL32.dll
 0002:00000118       __imp_GetModuleHandleA     000000014001a118     kernel32:KERNEL32.dll
 0002:00000120       __imp_ResetEvent           000000014001a120     kernel32:KERNEL32.dll
 0002:00000128       __imp_SetEvent             000000014001a128     kernel32:KERNEL32.dll
 0002:00000130       __imp_OutputDebugStringW   000000014001a130     kernel32:KERNEL32.dll
 0002:00000138       __imp_TerminateThread      000000014001a138     kernel32:KERNEL32.dll
 0002:00000140       __imp_FindFirstFileA       000000014001a140     kernel32:KERNEL32.dll
 0002:00000148       __imp_ReadProcessMemory    000000014001a148     kernel32:KERNEL32.dll
 0002:00000150       __imp_GetPrivateProfileStringA 000000014001a150     kernel32:KERNEL32.dll
 0002:00000158       __imp_InitializeSListHead  000000014001a158     kernel32:KERNEL32.dll
 0002:00000160       __imp_GetSystemTimeAsFileTime 000000014001a160     kernel32:KERNEL32.dll
 0002:00000168       __imp_QueryPerformanceCounter 000000014001a168     kernel32:KERNEL32.dll
 0002:00000170       __imp_GetStartupInfoW      000000014001a170     kernel32:KERNEL32.dll
 0002:00000178       __imp_IsDebuggerPresent    000000014001a178     kernel32:KERNEL32.dll
 0002:00000180       __imp_IsProcessorFeaturePresent 000000014001a180     kernel32:KERNEL32.dll
 0002:00000188       __imp_TerminateProcess     000000014001a188     kernel32:KERNEL32.dll
 0002:00000190       __imp_UnhandledExceptionFilter 000000014001a190     kernel32:KERNEL32.dll
 0002:00000198       __imp_RtlVirtualUnwind     000000014001a198     kernel32:KERNEL32.dll
 0002:000001a0       __imp_RtlLookupFunctionEntry 000000014001a1a0     kernel32:KERNEL32.dll
 0002:000001a8       __imp_RtlCaptureContext    000000014001a1a8     kernel32:KERNEL32.dll
 0002:000001b0       __imp_GetModuleHandleW     000000014001a1b0     kernel32:KERNEL32.dll
 0002:000001b8       __imp_CreateEventW         000000014001a1b8     kernel32:KERNEL32.dll
 0002:000001c0       __imp_WaitForSingleObjectEx 000000014001a1c0     kernel32:KERNEL32.dll
 0002:000001c8       __imp_InitializeCriticalSectionAndSpinCount 000000014001a1c8     kernel32:KERNEL32.dll
 0002:000001d0       __imp_CreateFileA          000000014001a1d0     kernel32:KERNEL32.dll
 0002:000001d8       \177KERNEL32_NULL_THUNK_DATA 000000014001a1d8     kernel32:KERNEL32.dll
 0002:000001e0       __imp_?_Xlength_error@std@@YAXPEBD@Z 000000014001a1e0     msvcprt:MSVCP140.dll
 0002:000001e8       __imp_?_Xout_of_range@std@@YAXPEBD@Z 000000014001a1e8     msvcprt:MSVCP140.dll
 0002:000001f0       __imp_?uncaught_exception@std@@YA_NXZ 000000014001a1f0     msvcprt:MSVCP140.dll
 0002:000001f8       __imp_?sputn@?$basic_streambuf@DU?$char_traits@D@std@@@std@@QEAA_JPEBD_J@Z 000000014001a1f8     msvcprt:MSVCP140.dll
 0002:00000200       __imp_?put@?$basic_ostream@DU?$char_traits@D@std@@@std@@QEAAAEAV12@D@Z 000000014001a200     msvcprt:MSVCP140.dll
 0002:00000208       __imp_?widen@?$basic_ios@DU?$char_traits@D@std@@@std@@QEBADD@Z 000000014001a208     msvcprt:MSVCP140.dll
 0002:00000210       __imp_?sputc@?$basic_streambuf@DU?$char_traits@D@std@@@std@@QEAAHD@Z 000000014001a210     msvcprt:MSVCP140.dll
 0002:00000218       __imp_??0?$basic_streambuf@DU?$char_traits@D@std@@@std@@IEAA@XZ 000000014001a218     msvcprt:MSVCP140.dll
 0002:00000220       __imp_?_Osfx@?$basic_ostream@DU?$char_traits@D@std@@@std@@QEAAXXZ 000000014001a220     msvcprt:MSVCP140.dll
 0002:00000228       __imp_?flush@?$basic_ostream@DU?$char_traits@D@std@@@std@@QEAAAEAV12@XZ 000000014001a228     msvcprt:MSVCP140.dll
 0002:00000230       __imp_?setstate@?$basic_ios@DU?$char_traits@D@std@@@std@@QEAAXH_N@Z 000000014001a230     msvcprt:MSVCP140.dll
 0002:00000238       __imp_??0?$basic_ios@DU?$char_traits@D@std@@@std@@IEAA@XZ 000000014001a238     msvcprt:MSVCP140.dll
 0002:00000240       __imp_?_Pninc@?$basic_streambuf@DU?$char_traits@D@std@@@std@@IEAAPEADXZ 000000014001a240     msvcprt:MSVCP140.dll
 0002:00000248       __imp_??0?$basic_iostream@DU?$char_traits@D@std@@@std@@QEAA@PEAV?$basic_streambuf@DU?$char_traits@D@std@@@1@@Z 000000014001a248     msvcprt:MSVCP140.dll
 0002:00000250       __imp_??1?$basic_ios@DU?$char_traits@D@std@@@std@@UEAA@XZ 000000014001a250     msvcprt:MSVCP140.dll
 0002:00000258       __imp_??1?$basic_streambuf@DU?$char_traits@D@std@@@std@@UEAA@XZ 000000014001a258     msvcprt:MSVCP140.dll
 0002:00000260       __imp_?_Lock@?$basic_streambuf@DU?$char_traits@D@std@@@std@@UEAAXXZ 000000014001a260     msvcprt:MSVCP140.dll
 0002:00000268       __imp_?_Unlock@?$basic_streambuf@DU?$char_traits@D@std@@@std@@UEAAXXZ 000000014001a268     msvcprt:MSVCP140.dll
 0002:00000270       __imp_?showmanyc@?$basic_streambuf@DU?$char_traits@D@std@@@std@@MEAA_JXZ 000000014001a270     msvcprt:MSVCP140.dll
 0002:00000278       __imp_?uflow@?$basic_streambuf@DU?$char_traits@D@std@@@std@@MEAAHXZ 000000014001a278     msvcprt:MSVCP140.dll
 0002:00000280       __imp_?xsgetn@?$basic_streambuf@DU?$char_traits@D@std@@@std@@MEAA_JPEAD_J@Z 000000014001a280     msvcprt:MSVCP140.dll
 0002:00000288       __imp_?xsputn@?$basic_streambuf@DU?$char_traits@D@std@@@std@@MEAA_JPEBD_J@Z 000000014001a288     msvcprt:MSVCP140.dll
 0002:00000290       __imp_?setbuf@?$basic_streambuf@DU?$char_traits@D@std@@@std@@MEAAPEAV12@PEAD_J@Z 000000014001a290     msvcprt:MSVCP140.dll
 0002:00000298       __imp_?sync@?$basic_streambuf@DU?$char_traits@D@std@@@std@@MEAAHXZ 000000014001a298     msvcprt:MSVCP140.dll
 0002:000002a0       __imp_?imbue@?$basic_streambuf@DU?$char_traits@D@std@@@std@@MEAAXAEBVlocale@2@@Z 000000014001a2a0     msvcprt:MSVCP140.dll
 0002:000002a8       __imp_??6?$basic_ostream@DU?$char_traits@D@std@@@std@@QEAAAEAV01@P6AAEAV01@AEAV01@@Z@Z 000000014001a2a8     msvcprt:MSVCP140.dll
 0002:000002b0       __imp_??6?$basic_ostream@DU?$char_traits@D@std@@@std@@QEAAAEAV01@_K@Z 000000014001a2b0     msvcprt:MSVCP140.dll
 0002:000002b8       __imp_??1?$basic_iostream@DU?$char_traits@D@std@@@std@@UEAA@XZ 000000014001a2b8     msvcprt:MSVCP140.dll
 0002:000002c0       \177MSVCP140_NULL_THUNK_DATA 000000014001a2c0     msvcprt:MSVCP140.dll
 0002:000002c8       __imp_GetProcessMemoryInfo 000000014001a2c8     Psapi:PSAPI.DLL
 0002:000002d0       \177PSAPI_NULL_THUNK_DATA  000000014001a2d0     Psapi:PSAPI.DLL
 0002:000002d8       __imp_SHCreateDirectoryExA 000000014001a2d8     shell32:SHELL32.dll
 0002:000002e0       \177SHELL32_NULL_THUNK_DATA 000000014001a2e0     shell32:SHELL32.dll
 0002:000002e8       __imp_PathFileExistsW      000000014001a2e8     shlwapi:SHLWAPI.dll
 0002:000002f0       \177SHLWAPI_NULL_THUNK_DATA 000000014001a2f0     shlwapi:SHLWAPI.dll
 0002:000002f8       __imp_SendMessageA         000000014001a2f8     user32:USER32.dll
 0002:00000300       __imp_LoadIconW            000000014001a300     user32:USER32.dll
 0002:00000308       __imp_EnableWindow         000000014001a308     user32:USER32.dll
 0002:00000310       __imp_wsprintfA            000000014001a310     user32:USER32.dll
 0002:00000318       __imp_IsWindow             000000014001a318     user32:USER32.dll
 0002:00000320       __imp_PostMessageA         000000014001a320     user32:USER32.dll
 0002:00000328       __imp_KillTimer            000000014001a328     user32:USER32.dll
 0002:00000330       __imp_GetWindowThreadProcessId 000000014001a330     user32:USER32.dll
 0002:00000338       \177USER32_NULL_THUNK_DATA 000000014001a338     user32:USER32.dll
 0002:00000340       __imp__CxxThrowException   000000014001a340     vcruntime:VCRUNTIME140.dll
 0002:00000348       __imp___RTDynamicCast      000000014001a348     vcruntime:VCRUNTIME140.dll
 0002:00000350       __imp_memchr               000000014001a350     vcruntime:VCRUNTIME140.dll
 0002:00000358       __imp_memcmp               000000014001a358     vcruntime:VCRUNTIME140.dll
 0002:00000360       __imp_memcpy               000000014001a360     vcruntime:VCRUNTIME140.dll
 0002:00000368       __imp___std_terminate      000000014001a368     vcruntime:VCRUNTIME140.dll
 0002:00000370       __imp_wcsrchr              000000014001a370     vcruntime:VCRUNTIME140.dll
 0002:00000378       __imp__purecall            000000014001a378     vcruntime:VCRUNTIME140.dll
 0002:00000380       __imp_strstr               000000014001a380     vcruntime:VCRUNTIME140.dll
 0002:00000388       __imp___std_exception_copy 000000014001a388     vcruntime:VCRUNTIME140.dll
 0002:00000390       __imp___std_exception_destroy 000000014001a390     vcruntime:VCRUNTIME140.dll
 0002:00000398       __imp___CxxFrameHandler3   000000014001a398     vcruntime:VCRUNTIME140.dll
 0002:000003a0       __imp_memset               000000014001a3a0     vcruntime:VCRUNTIME140.dll
 0002:000003a8       __imp_memmove              000000014001a3a8     vcruntime:VCRUNTIME140.dll
 0002:000003b0       __imp___C_specific_handler 000000014001a3b0     vcruntime:VCRUNTIME140.dll
 0002:000003b8       \177VCRUNTIME140_NULL_THUNK_DATA 000000014001a3b8     vcruntime:VCRUNTIME140.dll
 0002:000003c0       __imp_WinHttpQueryHeaders  000000014001a3c0     winhttp:WINHTTP.dll
 0002:000003c8       __imp_WinHttpReceiveResponse 000000014001a3c8     winhttp:WINHTTP.dll
 0002:000003d0       __imp_WinHttpWriteData     000000014001a3d0     winhttp:WINHTTP.dll
 0002:000003d8       __imp_WinHttpConnect       000000014001a3d8     winhttp:WINHTTP.dll
 0002:000003e0       __imp_WinHttpOpen          000000014001a3e0     winhttp:WINHTTP.dll
 0002:000003e8       __imp_WinHttpOpenRequest   000000014001a3e8     winhttp:WINHTTP.dll
 0002:000003f0       __imp_WinHttpSendRequest   000000014001a3f0     winhttp:WINHTTP.dll
 0002:000003f8       __imp_WinHttpCrackUrl      000000014001a3f8     winhttp:WINHTTP.dll
 0002:00000400       __imp_WinHttpCloseHandle   000000014001a400     winhttp:WINHTTP.dll
 0002:00000408       \177WINHTTP_NULL_THUNK_DATA 000000014001a408     winhttp:WINHTTP.dll
 0002:00000410       __imp_InternetReadFile     000000014001a410     Wininet:WININET.dll
 0002:00000418       __imp_InternetCloseHandle  000000014001a418     Wininet:WININET.dll
 0002:00000420       __imp_InternetOpenA        000000014001a420     Wininet:WININET.dll
 0002:00000428       __imp_InternetOpenUrlA     000000014001a428     Wininet:WININET.dll
 0002:00000430       \177WININET_NULL_THUNK_DATA 000000014001a430     Wininet:WININET.dll
 0002:00000438       __imp_timeGetTime          000000014001a438     winmm:WINMM.dll
 0002:00000440       \177WINMM_NULL_THUNK_DATA  000000014001a440     winmm:WINMM.dll
 0002:00000448       __imp_WSACleanup           000000014001a448     ws2_32:WS2_32.dll
 0002:00000450       __imp_gethostname          000000014001a450     ws2_32:WS2_32.dll
 0002:00000458       __imp_WSAStartup           000000014001a458     ws2_32:WS2_32.dll
 0002:00000460       \177WS2_32_NULL_THUNK_DATA 000000014001a460     ws2_32:WS2_32.dll
 0002:00000468       __imp_mbstowcs             000000014001a468     ucrt:api-ms-win-crt-convert-l1-1-0.dll
 0002:00000470       __imp_atoll                000000014001a470     ucrt:api-ms-win-crt-convert-l1-1-0.dll
 0002:00000478       __imp_atol                 000000014001a478     ucrt:api-ms-win-crt-convert-l1-1-0.dll
 0002:00000480       __imp_atoi                 000000014001a480     ucrt:api-ms-win-crt-convert-l1-1-0.dll
 0002:00000488       \177api-ms-win-crt-convert-l1-1-0_NULL_THUNK_DATA 000000014001a488     ucrt:api-ms-win-crt-convert-l1-1-0.dll
 0002:00000490       __imp__mkdir               000000014001a490     ucrt:api-ms-win-crt-filesystem-l1-1-0.dll
 0002:00000498       __imp_rename               000000014001a498     ucrt:api-ms-win-crt-filesystem-l1-1-0.dll
 0002:000004a0       __imp__splitpath_s         000000014001a4a0     ucrt:api-ms-win-crt-filesystem-l1-1-0.dll
 0002:000004a8       __imp_remove               000000014001a4a8     ucrt:api-ms-win-crt-filesystem-l1-1-0.dll
 0002:000004b0       \177api-ms-win-crt-filesystem-l1-1-0_NULL_THUNK_DATA 000000014001a4b0     ucrt:api-ms-win-crt-filesystem-l1-1-0.dll
 0002:000004b8       __imp__set_new_mode        000000014001a4b8     ucrt:api-ms-win-crt-heap-l1-1-0.dll
 0002:000004c0       __imp_free                 000000014001a4c0     ucrt:api-ms-win-crt-heap-l1-1-0.dll
 0002:000004c8       \177api-ms-win-crt-heap-l1-1-0_NULL_THUNK_DATA 000000014001a4c8     ucrt:api-ms-win-crt-heap-l1-1-0.dll
 0002:000004d0       __imp__setmbcp             000000014001a4d0     ucrt:api-ms-win-crt-locale-l1-1-0.dll
 0002:000004d8       __imp__configthreadlocale  000000014001a4d8     ucrt:api-ms-win-crt-locale-l1-1-0.dll
 0002:000004e0       \177api-ms-win-crt-locale-l1-1-0_NULL_THUNK_DATA 000000014001a4e0     ucrt:api-ms-win-crt-locale-l1-1-0.dll
 0002:000004e8       __imp_atan                 000000014001a4e8     ucrt:api-ms-win-crt-math-l1-1-0.dll
 0002:000004f0       __imp_sqrt                 000000014001a4f0     ucrt:api-ms-win-crt-math-l1-1-0.dll
 0002:000004f8       __imp___setusermatherr     000000014001a4f8     ucrt:api-ms-win-crt-math-l1-1-0.dll
 0002:00000500       __imp_sqrtf                000000014001a500     ucrt:api-ms-win-crt-math-l1-1-0.dll
 0002:00000508       \177api-ms-win-crt-math-l1-1-0_NULL_THUNK_DATA 000000014001a508     ucrt:api-ms-win-crt-math-l1-1-0.dll
 0002:00000510       __imp__invalid_parameter_noinfo_noreturn 000000014001a510     ucrt:api-ms-win-crt-runtime-l1-1-0.dll
 0002:00000518       __imp__set_invalid_parameter_handler 000000014001a518     ucrt:api-ms-win-crt-runtime-l1-1-0.dll
 0002:00000520       __imp__invalid_parameter_noinfo 000000014001a520     ucrt:api-ms-win-crt-runtime-l1-1-0.dll
 0002:00000528       __imp__errno               000000014001a528     ucrt:api-ms-win-crt-runtime-l1-1-0.dll
 0002:00000530       __imp___p___argc           000000014001a530     ucrt:api-ms-win-crt-runtime-l1-1-0.dll
 0002:00000538       __imp___p___argv           000000014001a538     ucrt:api-ms-win-crt-runtime-l1-1-0.dll
 0002:00000540       __imp__beginthread         000000014001a540     ucrt:api-ms-win-crt-runtime-l1-1-0.dll
 0002:00000548       __imp__endthread           000000014001a548     ucrt:api-ms-win-crt-runtime-l1-1-0.dll
 0002:00000550       __imp_terminate            000000014001a550     ucrt:api-ms-win-crt-runtime-l1-1-0.dll
 0002:00000558       __imp__register_thread_local_exe_atexit_callback 000000014001a558     ucrt:api-ms-win-crt-runtime-l1-1-0.dll
 0002:00000560       __imp__c_exit              000000014001a560     ucrt:api-ms-win-crt-runtime-l1-1-0.dll
 0002:00000568       __imp__configure_narrow_argv 000000014001a568     ucrt:api-ms-win-crt-runtime-l1-1-0.dll
 0002:00000570       __imp__exit                000000014001a570     ucrt:api-ms-win-crt-runtime-l1-1-0.dll
 0002:00000578       __imp_exit                 000000014001a578     ucrt:api-ms-win-crt-runtime-l1-1-0.dll
 0002:00000580       __imp__initterm_e          000000014001a580     ucrt:api-ms-win-crt-runtime-l1-1-0.dll
 0002:00000588       __imp__initterm            000000014001a588     ucrt:api-ms-win-crt-runtime-l1-1-0.dll
 0002:00000590       __imp__get_narrow_winmain_command_line 000000014001a590     ucrt:api-ms-win-crt-runtime-l1-1-0.dll
 0002:00000598       __imp__set_app_type        000000014001a598     ucrt:api-ms-win-crt-runtime-l1-1-0.dll
 0002:000005a0       __imp__seh_filter_exe      000000014001a5a0     ucrt:api-ms-win-crt-runtime-l1-1-0.dll
 0002:000005a8       __imp__cexit               000000014001a5a8     ucrt:api-ms-win-crt-runtime-l1-1-0.dll
 0002:000005b0       __imp__crt_atexit          000000014001a5b0     ucrt:api-ms-win-crt-runtime-l1-1-0.dll
 0002:000005b8       __imp__register_onexit_function 000000014001a5b8     ucrt:api-ms-win-crt-runtime-l1-1-0.dll
 0002:000005c0       __imp__initialize_onexit_table 000000014001a5c0     ucrt:api-ms-win-crt-runtime-l1-1-0.dll
 0002:000005c8       __imp__initialize_narrow_environment 000000014001a5c8     ucrt:api-ms-win-crt-runtime-l1-1-0.dll
 0002:000005d0       \177api-ms-win-crt-runtime-l1-1-0_NULL_THUNK_DATA 000000014001a5d0     ucrt:api-ms-win-crt-runtime-l1-1-0.dll
 0002:000005d8       __imp___p__commode         000000014001a5d8     ucrt:api-ms-win-crt-stdio-l1-1-0.dll
 0002:000005e0       __imp___stdio_common_vfscanf 000000014001a5e0     ucrt:api-ms-win-crt-stdio-l1-1-0.dll
 0002:000005e8       __imp___stdio_common_vsnwprintf_s 000000014001a5e8     ucrt:api-ms-win-crt-stdio-l1-1-0.dll
 0002:000005f0       __imp___stdio_common_vsprintf_s 000000014001a5f0     ucrt:api-ms-win-crt-stdio-l1-1-0.dll
 0002:000005f8       __imp___stdio_common_vsprintf 000000014001a5f8     ucrt:api-ms-win-crt-stdio-l1-1-0.dll
 0002:00000600       __imp___stdio_common_vfprintf 000000014001a600     ucrt:api-ms-win-crt-stdio-l1-1-0.dll
 0002:00000608       __imp_fclose               000000014001a608     ucrt:api-ms-win-crt-stdio-l1-1-0.dll
 0002:00000610       __imp__set_fmode           000000014001a610     ucrt:api-ms-win-crt-stdio-l1-1-0.dll
 0002:00000618       __imp__setmaxstdio         000000014001a618     ucrt:api-ms-win-crt-stdio-l1-1-0.dll
 0002:00000620       __imp_fwrite               000000014001a620     ucrt:api-ms-win-crt-stdio-l1-1-0.dll
 0002:00000628       __imp___stdio_common_vsnprintf_s 000000014001a628     ucrt:api-ms-win-crt-stdio-l1-1-0.dll
 0002:00000630       __imp_fopen_s              000000014001a630     ucrt:api-ms-win-crt-stdio-l1-1-0.dll
 0002:00000638       \177api-ms-win-crt-stdio-l1-1-0_NULL_THUNK_DATA 000000014001a638     ucrt:api-ms-win-crt-stdio-l1-1-0.dll
 0002:00000640       __imp__wcsicmp             000000014001a640     ucrt:api-ms-win-crt-string-l1-1-0.dll
 0002:00000648       __imp_strcat_s             000000014001a648     ucrt:api-ms-win-crt-string-l1-1-0.dll
 0002:00000650       __imp_strncpy_s            000000014001a650     ucrt:api-ms-win-crt-string-l1-1-0.dll
 0002:00000658       __imp_strcpy_s             000000014001a658     ucrt:api-ms-win-crt-string-l1-1-0.dll
 0002:00000660       __imp_wcscpy_s             000000014001a660     ucrt:api-ms-win-crt-string-l1-1-0.dll
 0002:00000668       __imp_tolower              000000014001a668     ucrt:api-ms-win-crt-string-l1-1-0.dll
 0002:00000670       \177api-ms-win-crt-string-l1-1-0_NULL_THUNK_DATA 000000014001a670     ucrt:api-ms-win-crt-string-l1-1-0.dll
 0002:00000678       __imp__time32              000000014001a678     ucrt:api-ms-win-crt-time-l1-1-0.dll
 0002:00000680       \177api-ms-win-crt-time-l1-1-0_NULL_THUNK_DATA 000000014001a680     ucrt:api-ms-win-crt-time-l1-1-0.dll
 0002:00000688       __imp_srand                000000014001a688     ucrt:api-ms-win-crt-utility-l1-1-0.dll
 0002:00000690       \177api-ms-win-crt-utility-l1-1-0_NULL_THUNK_DATA 000000014001a690     ucrt:api-ms-win-crt-utility-l1-1-0.dll
 0002:00000698       __imp_SymCleanup           000000014001a698     DbgHelp:dbghelp.dll
 0002:000006a0       __imp_EnumerateLoadedModules64 000000014001a6a0     DbgHelp:dbghelp.dll
 0002:000006a8       __imp_SymFunctionTableAccess64 000000014001a6a8     DbgHelp:dbghelp.dll
 0002:000006b0       __imp_SymGetModuleBase64   000000014001a6b0     DbgHelp:dbghelp.dll
 0002:000006b8       __imp_StackWalk64          000000014001a6b8     DbgHelp:dbghelp.dll
 0002:000006c0       __imp_SymInitialize        000000014001a6c0     DbgHelp:dbghelp.dll
 0002:000006c8       __imp_SymSetOptions        000000014001a6c8     DbgHelp:dbghelp.dll
 0002:000006d0       __imp_MiniDumpWriteDump    000000014001a6d0     DbgHelp:dbghelp.dll
 0002:000006d8       \177dbghelp_NULL_THUNK_DATA 000000014001a6d8     DbgHelp:dbghelp.dll
 0002:000006e0       __imp_?GetDataRecoveryHandler@CWinApp@@UEAAPEAVCDataRecoveryHandler@@XZ 000000014001a6e0     mfc140:mfc140.dll
 0002:000006e8       __imp_?ApplicationRecoveryCallback@CWinApp@@UEAAKPEAX@Z 000000014001a6e8     mfc140:mfc140.dll
 0002:000006f0       __imp_?RegisterWithRestartManager@CWinApp@@UEAAJHAEBV?$CStringT@DV?$StrTraitMFC_DLL@DV?$ChTraitsCRT@D@ATL@@@@@ATL@@@Z 000000014001a6f0     mfc140:mfc140.dll
 0002:000006f8       __imp_?RegisterWithRestartManager@CWinApp@@UEAAJPEB_WKP6AKPEAX@Z1KK@Z 000000014001a6f8     mfc140:mfc140.dll
 0002:00000700       __imp_?WinHelpInternal@CWinApp@@UEAAX_KI@Z 000000014001a700     mfc140:mfc140.dll
 0002:00000708       __imp_?HtmlHelpA@CWinApp@@UEAAX_KI@Z 000000014001a708     mfc140:mfc140.dll
 0002:00000710       __imp_?WinHelpA@CWinApp@@UEAAX_KI@Z 000000014001a710     mfc140:mfc140.dll
 0002:00000718       __imp_?OnDDECommand@CWinApp@@UEAAHPEAD@Z 000000014001a718     mfc140:mfc140.dll
 0002:00000720       __imp_?DoWaitCursor@CWinApp@@UEAAXH@Z 000000014001a720     mfc140:mfc140.dll
 0002:00000728       __imp_?DoMessageBox@CWinApp@@UEAAHPEBDII@Z 000000014001a728     mfc140:mfc140.dll
 0002:00000730       __imp_?OnToolHitTest@CWnd@@UEBA_JVCPoint@@PEAUtagTOOLINFOA@@@Z 000000014001a730     mfc140:mfc140.dll
 0002:00000738       __imp_?SetMenu@CWnd@@UEAAHPEAVCMenu@@@Z 000000014001a738     mfc140:mfc140.dll
 0002:00000740       __imp_?GetMenu@CWnd@@UEBAPEAVCMenu@@XZ 000000014001a740     mfc140:mfc140.dll
 0002:00000748       __imp_?CalcWindowRect@CWnd@@UEAAXPEAUtagRECT@@I@Z 000000014001a748     mfc140:mfc140.dll
 0002:00000750       __imp_?PreCreateWindow@CWnd@@UEAAHAEAUtagCREATESTRUCTA@@@Z 000000014001a750     mfc140:mfc140.dll
 0002:00000758       __imp_?DestroyWindow@CWnd@@UEAAHXZ 000000014001a758     mfc140:mfc140.dll
 0002:00000760       __imp_?CreateEx@CWnd@@UEAAHKPEBD0KHHHHPEAUHWND__@@PEAUHMENU__@@PEAX@Z 000000014001a760     mfc140:mfc140.dll
 0002:00000768       __imp_?CreateEx@CWnd@@UEAAHKPEBD0KAEBUtagRECT@@PEAV1@IPEAX@Z 000000014001a768     mfc140:mfc140.dll
 0002:00000770       __imp_?PreSubclassWindow@CWnd@@UEAAXXZ 000000014001a770     mfc140:mfc140.dll
 0002:00000778       __imp_?FindOneOf@?$CStringT@DV?$StrTraitMFC_DLL@DV?$ChTraitsCRT@D@ATL@@@@@ATL@@QEBAHPEBD@Z 000000014001a778     mfc140:mfc140.dll
 0002:00000780       __imp_??Y?$CStringT@DV?$StrTraitMFC_DLL@DV?$ChTraitsCRT@D@ATL@@@@@ATL@@QEAAAEAV01@PEBD@Z 000000014001a780     mfc140:mfc140.dll
 0002:00000788       __imp_??Y?$CStringT@DV?$StrTraitMFC_DLL@DV?$ChTraitsCRT@D@ATL@@@@@ATL@@QEAAAEAV01@AEBV?$CSimpleStringT@D$00@1@@Z 000000014001a788     mfc140:mfc140.dll
 0002:00000790       __imp_?Compare@?$CStringT@DV?$StrTraitMFC_DLL@DV?$ChTraitsCRT@D@ATL@@@@@ATL@@QEBAHPEBD@Z 000000014001a790     mfc140:mfc140.dll
 0002:00000798       __imp_?PreInitDialog@CDialog@@MEAAXXZ 000000014001a798     mfc140:mfc140.dll
 0002:000007a0       __imp_?SaveAllModified@CWinApp@@UEAAHXZ 000000014001a7a0     mfc140:mfc140.dll
 0002:000007a8       __imp_?InitApplication@CWinApp@@UEAAHXZ 000000014001a7a8     mfc140:mfc140.dll
 0002:000007b0       __imp_?AddToRecentFileList@CWinApp@@UEAAXPEBD@Z 000000014001a7b0     mfc140:mfc140.dll
 0002:000007b8       __imp_?OpenDocumentFile@CWinApp@@UEAAPEAVCDocument@@PEBD@Z 000000014001a7b8     mfc140:mfc140.dll
 0002:000007c0       __imp_?OpenDocumentFile@CWinApp@@UEAAPEAVCDocument@@PEBDH@Z 000000014001a7c0     mfc140:mfc140.dll
 0002:000007c8       __imp_?OnCancel@CDialog@@MEAAXXZ 000000014001a7c8     mfc140:mfc140.dll
 0002:000007d0       __imp_?OnSetFont@CDialog@@UEAAXPEAVCFont@@@Z 000000014001a7d0     mfc140:mfc140.dll
 0002:000007d8       __imp_?CreateIndirect@CDialog@@UEAAHPEBUDLGTEMPLATE@@PEAVCWnd@@PEAX@Z 000000014001a7d8     mfc140:mfc140.dll
 0002:000007e0       __imp_?CreateIndirect@CDialog@@UEAAHPEAXPEAVCWnd@@@Z 000000014001a7e0     mfc140:mfc140.dll
 0002:000007e8       __imp_?Create@CDialog@@UEAAHPEBDPEAVCWnd@@@Z 000000014001a7e8     mfc140:mfc140.dll
 0002:000007f0       __imp_?GetOccDialogInfo@CDialog@@MEAAPEAU_AFX_OCC_DIALOG_INFO@@XZ 000000014001a7f0     mfc140:mfc140.dll
 0002:000007f8       __imp_?SetOccDialogInfo@CDialog@@MEAAHPEAU_AFX_OCC_DIALOG_INFO@@@Z 000000014001a7f8     mfc140:mfc140.dll
 0002:00000800       __imp_?CheckAutoCenter@CDialog@@UEAAHXZ 000000014001a800     mfc140:mfc140.dll
 0002:00000808       __imp_?PreTranslateMessage@CDialog@@UEAAHPEAUtagMSG@@@Z 000000014001a808     mfc140:mfc140.dll
 0002:00000810       __imp_?RestartInstance@CWinApp@@UEAAHXZ 000000014001a810     mfc140:mfc140.dll
 0002:00000818       __imp_?LoadAppLangResourceDLL@CWinApp@@UEAAPEAUHINSTANCE__@@XZ 000000014001a818     mfc140:mfc140.dll
 0002:00000820       __imp_?LoadSysPolicies@CWinApp@@UEAAHXZ 000000014001a820     mfc140:mfc140.dll
 0002:00000828       __imp_??0CDialog@@QEAA@IPEAVCWnd@@@Z 000000014001a828     mfc140:mfc140.dll
 0002:00000830       __imp_??1CDialog@@UEAA@XZ  000000014001a830     mfc140:mfc140.dll
 0002:00000838       __imp_??0?$CStringT@DV?$StrTraitMFC_DLL@DV?$ChTraitsCRT@D@ATL@@@@@ATL@@QEAA@XZ 000000014001a838     mfc140:mfc140.dll
 0002:00000840       __imp_??1?$CStringT@DV?$StrTraitMFC_DLL@DV?$ChTraitsCRT@D@ATL@@@@@ATL@@QEAA@XZ 000000014001a840     mfc140:mfc140.dll
 0002:00000848       __imp_?GetOccDialogInfo@CWnd@@MEAAPEAU_AFX_OCC_DIALOG_INFO@@XZ 000000014001a848     mfc140:mfc140.dll
 0002:00000850       __imp_?IsTaskbarInteractionEnabled@CWinApp@@UEAAHXZ 000000014001a850     mfc140:mfc140.dll
 0002:00000858       __imp_?OnCmdMsg@CDialog@@UEAAHIHPEAXPEAUAFX_CMDHANDLERINFO@@@Z 000000014001a858     mfc140:mfc140.dll
 0002:00000860       __imp_?GetRuntimeClass@CDialog@@UEBAPEAUCRuntimeClass@@XZ 000000014001a860     mfc140:mfc140.dll
 0002:00000868       __imp_?Default@CWnd@@IEAA_JXZ 000000014001a868     mfc140:mfc140.dll
 0002:00000870       __imp_?OnOK@CDialog@@MEAAXXZ 000000014001a870     mfc140:mfc140.dll
 0002:00000878       __imp_?AfxThrowInvalidArgException@@YAXXZ 000000014001a878     mfc140:mfc140.dll
 0002:00000880       __imp_?Close@CFileFind@@QEAAXXZ 000000014001a880     mfc140:mfc140.dll
 0002:00000888       __imp_?AddTail@CStringList@@QEAAPEAU__POSITION@@AEBV?$CStringT@DV?$StrTraitMFC_DLL@DV?$ChTraitsCRT@D@ATL@@@@@ATL@@@Z 000000014001a888     mfc140:mfc140.dll
 0002:00000890       __imp_?GetFileName@CFileFind@@UEBA?AV?$CStringT@DV?$StrTraitMFC_DLL@DV?$ChTraitsCRT@D@ATL@@@@@ATL@@XZ 000000014001a890     mfc140:mfc140.dll
 0002:00000898       __imp_?IsDots@CFileFind@@UEBAHXZ 000000014001a898     mfc140:mfc140.dll
 0002:000008a0       __imp_?FindNextFileA@CFileFind@@UEAAHXZ 000000014001a8a0     mfc140:mfc140.dll
 0002:000008a8       __imp_?FindFile@CFileFind@@UEAAHPEBDK@Z 000000014001a8a8     mfc140:mfc140.dll
 0002:000008b0       __imp_??1CFileFind@@UEAA@XZ 000000014001a8b0     mfc140:mfc140.dll
 0002:000008b8       __imp_??0CFileFind@@QEAA@XZ 000000014001a8b8     mfc140:mfc140.dll
 0002:000008c0       __imp_??1CStringList@@UEAA@XZ 000000014001a8c0     mfc140:mfc140.dll
 0002:000008c8       __imp_??0CStringList@@QEAA@_J@Z 000000014001a8c8     mfc140:mfc140.dll
 0002:000008d0       __imp_?AfxFreeLibrary@@YAHPEAUHINSTANCE__@@@Z 000000014001a8d0     mfc140:mfc140.dll
 0002:000008d8       __imp_?MessageBoxA@CWnd@@QEAAHPEBD0I@Z 000000014001a8d8     mfc140:mfc140.dll
 0002:000008e0       __imp_?AfxLoadLibrary@@YAPEAUHINSTANCE__@@PEBD@Z 000000014001a8e0     mfc140:mfc140.dll
 0002:000008e8       __imp_?EndWaitCursor@CCmdTarget@@QEAAXXZ 000000014001a8e8     mfc140:mfc140.dll
 0002:000008f0       __imp_?BeginWaitCursor@CCmdTarget@@QEAAXXZ 000000014001a8f0     mfc140:mfc140.dll
 0002:000008f8       __imp_?OnPaint@CDialog@@IEAAXXZ 000000014001a8f8     mfc140:mfc140.dll
 0002:00000900       __imp_?SetFocus@CWnd@@QEAAPEAV1@XZ 000000014001a900     mfc140:mfc140.dll
 0002:00000908       __imp_?GetDlgItem@CWnd@@QEBAPEAV1@H@Z 000000014001a908     mfc140:mfc140.dll
 0002:00000910       __imp_?Format@?$CStringT@DV?$StrTraitMFC_DLL@DV?$ChTraitsCRT@D@ATL@@@@@ATL@@QEAAXPEBDZZ 000000014001a910     mfc140:mfc140.dll
 0002:00000918       __imp_?AfxMessageBox@@YAHPEBDII@Z 000000014001a918     mfc140:mfc140.dll
 0002:00000920       __imp_?SetWindowTextA@CWnd@@QEAAXPEBD@Z 000000014001a920     mfc140:mfc140.dll
 0002:00000928       __imp_?GetWindowTextA@CWnd@@QEBAHPEADH@Z 000000014001a928     mfc140:mfc140.dll
 0002:00000930       __imp_?SetOccDialogInfo@CWnd@@MEAAHPEAU_AFX_OCC_DIALOG_INFO@@@Z 000000014001a930     mfc140:mfc140.dll
 0002:00000938       __imp_?CreateControlSite@CWnd@@MEAAHPEAVCOleControlContainer@@PEAPEAVCOleControlSite@@IAEBU_GUID@@@Z 000000014001a938     mfc140:mfc140.dll
 0002:00000940       __imp_?Empty@?$CSimpleStringT@D$00@ATL@@QEAAXXZ 000000014001a940     mfc140:mfc140.dll
 0002:00000948       __imp_?CreateControlContainer@CWnd@@MEAAHPEAPEAVCOleControlContainer@@@Z 000000014001a948     mfc140:mfc140.dll
 0002:00000950       __imp_?IsFrameWnd@CWnd@@UEBAHXZ 000000014001a950     mfc140:mfc140.dll
 0002:00000958       __imp_?CheckAutoCenter@CWnd@@UEAAHXZ 000000014001a958     mfc140:mfc140.dll
 0002:00000960       __imp_?ResizeDynamicLayout@CWnd@@MEAAXXZ 000000014001a960     mfc140:mfc140.dll
 0002:00000968       __imp_??4?$CStringT@DV?$StrTraitMFC_DLL@DV?$ChTraitsCRT@D@ATL@@@@@ATL@@QEAAAEAV01@PEBD@Z 000000014001a968     mfc140:mfc140.dll
 0002:00000970       __imp_?OnGesturePressAndTap@CWnd@@MEAAHVCPoint@@J@Z 000000014001a970     mfc140:mfc140.dll
 0002:00000978       __imp_?OnGestureTwoFingerTap@CWnd@@MEAAHVCPoint@@@Z 000000014001a978     mfc140:mfc140.dll
 0002:00000980       __imp_?OnGestureRotate@CWnd@@MEAAHVCPoint@@N@Z 000000014001a980     mfc140:mfc140.dll
 0002:00000988       __imp_?OnGesturePan@CWnd@@MEAAHVCPoint@@0@Z 000000014001a988     mfc140:mfc140.dll
 0002:00000990       __imp_?OnGestureZoom@CWnd@@MEAAHVCPoint@@J@Z 000000014001a990     mfc140:mfc140.dll
 0002:00000998       __imp_?GetGestureStatus@CWnd@@MEAAKVCPoint@@@Z 000000014001a998     mfc140:mfc140.dll
 0002:000009a0       __imp_?OnTouchInput@CWnd@@MEAAHVCPoint@@HHPEAUtagTOUCHINPUT@@@Z 000000014001a9a0     mfc140:mfc140.dll
 0002:000009a8       __imp_?OnTouchInputs@CWnd@@MEAAHIPEAUtagTOUCHINPUT@@@Z 000000014001a9a8     mfc140:mfc140.dll
 0002:000009b0       __imp_?OnChildNotify@CWnd@@MEAAHI_K_JPEA_J@Z 000000014001a9b0     mfc140:mfc140.dll
 0002:000009b8       __imp_?PostNcDestroy@CWnd@@MEAAXXZ 000000014001a9b8     mfc140:mfc140.dll
 0002:000009c0       __imp_?DefWindowProcA@CWnd@@MEAA_JI_K_J@Z 000000014001a9c0     mfc140:mfc140.dll
 0002:000009c8       __imp_?OnWndMsg@CWnd@@MEAAHI_K_JPEA_J@Z 000000014001a9c8     mfc140:mfc140.dll
 0002:000009d0       __imp_?WindowProc@CWnd@@MEAA_JI_K_J@Z 000000014001a9d0     mfc140:mfc140.dll
 0002:000009d8       __imp_?OnAmbientProperty@CWnd@@UEAAHPEAVCOleControlSite@@JPEAUtagVARIANT@@@Z 000000014001a9d8     mfc140:mfc140.dll
 0002:000009e0       __imp_?PreTranslateMessage@CWnd@@UEAAHPEAUtagMSG@@@Z 000000014001a9e0     mfc140:mfc140.dll
 0002:000009e8       __imp_?OnInitDialog@CDialog@@UEAAHXZ 000000014001a9e8     mfc140:mfc140.dll
 0002:000009f0       __imp_?GetSuperWndProcAddr@CWnd@@MEAAPEAP6A_JPEAUHWND__@@I_K_J@ZXZ 000000014001a9f0     mfc140:mfc140.dll
 0002:000009f8       __imp_?GetThisMessageMap@CDialog@@KAPEBUAFX_MSGMAP@@XZ 000000014001a9f8     mfc140:mfc140.dll
 0002:00000a00       __imp_?DDX_Control@@YAXPEAVCDataExchange@@HAEAVCWnd@@@Z 000000014001aa00     mfc140:mfc140.dll
 0002:00000a08       __imp_?OnNotify@CWnd@@MEAAH_K_JPEA_J@Z 000000014001aa08     mfc140:mfc140.dll
 0002:00000a10       __imp_?OnCommand@CWnd@@MEAAH_K_J@Z 000000014001aa10     mfc140:mfc140.dll
 0002:00000a18       __imp_?CreateAccessibleProxy@CWnd@@UEAAJ_K_JPEA_J@Z 000000014001aa18     mfc140:mfc140.dll
 0002:00000a20       __imp_?AfxGetModuleState@@YAPEAVAFX_MODULE_STATE@@XZ 000000014001aa20     mfc140:mfc140.dll
 0002:00000a28       __imp_?AfxFindResourceHandle@@YAPEAUHINSTANCE__@@PEBD0@Z 000000014001aa28     mfc140:mfc140.dll
 0002:00000a30       __imp_??1CListBox@@UEAA@XZ 000000014001aa30     mfc140:mfc140.dll
 0002:00000a38       __imp_?SetProxy@CWnd@@UEAAJPEAUIAccessibleProxy@@@Z 000000014001aa38     mfc140:mfc140.dll
 0002:00000a40       __imp_?put_accValue@CWnd@@UEAAJUtagVARIANT@@PEA_W@Z 000000014001aa40     mfc140:mfc140.dll
 0002:00000a48       __imp_?put_accName@CWnd@@UEAAJUtagVARIANT@@PEA_W@Z 000000014001aa48     mfc140:mfc140.dll
 0002:00000a50       __imp_?accDoDefaultAction@CWnd@@UEAAJUtagVARIANT@@@Z 000000014001aa50     mfc140:mfc140.dll
 0002:00000a58       __imp_?accHitTest@CWnd@@UEAAJJJPEAUtagVARIANT@@@Z 000000014001aa58     mfc140:mfc140.dll
 0002:00000a60       __imp_?accNavigate@CWnd@@UEAAJJUtagVARIANT@@PEAU2@@Z 000000014001aa60     mfc140:mfc140.dll
 0002:00000a68       __imp_?accLocation@CWnd@@UEAAJPEAJ000UtagVARIANT@@@Z 000000014001aa68     mfc140:mfc140.dll
 0002:00000a70       __imp_?accSelect@CWnd@@UEAAJJUtagVARIANT@@@Z 000000014001aa70     mfc140:mfc140.dll
 0002:00000a78       __imp_?get_accDefaultAction@CWnd@@UEAAJUtagVARIANT@@PEAPEA_W@Z 000000014001aa78     mfc140:mfc140.dll
 0002:00000a80       __imp_?get_accSelection@CWnd@@UEAAJPEAUtagVARIANT@@@Z 000000014001aa80     mfc140:mfc140.dll
 0002:00000a88       __imp_?get_accFocus@CWnd@@UEAAJPEAUtagVARIANT@@@Z 000000014001aa88     mfc140:mfc140.dll
 0002:00000a90       __imp_?GetRuntimeClass@CListBox@@UEBAPEAUCRuntimeClass@@XZ 000000014001aa90     mfc140:mfc140.dll
 0002:00000a98       __imp_?get_accKeyboardShortcut@CWnd@@UEAAJUtagVARIANT@@PEAPEA_W@Z 000000014001aa98     mfc140:mfc140.dll
 0002:00000aa0       __imp_?get_accHelpTopic@CWnd@@UEAAJPEAPEA_WUtagVARIANT@@PEAJ@Z 000000014001aaa0     mfc140:mfc140.dll
 0002:00000aa8       __imp_?get_accHelp@CWnd@@UEAAJUtagVARIANT@@PEAPEA_W@Z 000000014001aaa8     mfc140:mfc140.dll
 0002:00000ab0       __imp_?get_accState@CWnd@@UEAAJUtagVARIANT@@PEAU2@@Z 000000014001aab0     mfc140:mfc140.dll
 0002:00000ab8       __imp_?get_accRole@CWnd@@UEAAJUtagVARIANT@@PEAU2@@Z 000000014001aab8     mfc140:mfc140.dll
 0002:00000ac0       __imp_?get_accDescription@CWnd@@UEAAJUtagVARIANT@@PEAPEA_W@Z 000000014001aac0     mfc140:mfc140.dll
 0002:00000ac8       __imp_?get_accValue@CWnd@@UEAAJUtagVARIANT@@PEAPEA_W@Z 000000014001aac8     mfc140:mfc140.dll
 0002:00000ad0       __imp_?get_accName@CWnd@@UEAAJUtagVARIANT@@PEAPEA_W@Z 000000014001aad0     mfc140:mfc140.dll
 0002:00000ad8       __imp_?OnChildNotify@CListBox@@MEAAHI_K_JPEA_J@Z 000000014001aad8     mfc140:mfc140.dll
 0002:00000ae0       __imp_?Create@CListBox@@UEAAHKAEBUtagRECT@@PEAVCWnd@@I@Z 000000014001aae0     mfc140:mfc140.dll
 0002:00000ae8       __imp_?get_accChild@CWnd@@UEAAJUtagVARIANT@@PEAPEAUIDispatch@@@Z 000000014001aae8     mfc140:mfc140.dll
 0002:00000af0       __imp_?get_accChildCount@CWnd@@UEAAJPEAJ@Z 000000014001aaf0     mfc140:mfc140.dll
 0002:00000af8       __imp_?DrawItem@CListBox@@UEAAXPEAUtagDRAWITEMSTRUCT@@@Z 000000014001aaf8     mfc140:mfc140.dll
 0002:00000b00       __imp_?get_accParent@CWnd@@UEAAJPEAPEAUIDispatch@@@Z 000000014001ab00     mfc140:mfc140.dll
 0002:00000b08       __imp_?EnsureStdObj@CWnd@@UEAAJXZ 000000014001ab08     mfc140:mfc140.dll
 0002:00000b10       __imp_?OnDrawIconicThumbnailOrLivePreview@CWnd@@UEAAXAEAVCDC@@VCRect@@VCSize@@HAEAH@Z 000000014001ab10     mfc140:mfc140.dll
 0002:00000b18       __imp_?EndModalLoop@CWnd@@UEAAXH@Z 000000014001ab18     mfc140:mfc140.dll
 0002:00000b20       __imp_?ContinueModal@CWnd@@UEAAHXZ 000000014001ab20     mfc140:mfc140.dll
 0002:00000b28       __imp_?MeasureItem@CListBox@@UEAAXPEAUtagMEASUREITEMSTRUCT@@@Z 000000014001ab28     mfc140:mfc140.dll
 0002:00000b30       __imp_?WinHelpInternal@CWnd@@UEAAX_KI@Z 000000014001ab30     mfc140:mfc140.dll
 0002:00000b38       __imp_?CompareItem@CListBox@@UEAAHPEAUtagCOMPAREITEMSTRUCT@@@Z 000000014001ab38     mfc140:mfc140.dll
 0002:00000b40       __imp_?HtmlHelpA@CWnd@@UEAAX_KI@Z 000000014001ab40     mfc140:mfc140.dll
 0002:00000b48       __imp_?WinHelpA@CWnd@@UEAAX_KI@Z 000000014001ab48     mfc140:mfc140.dll
 0002:00000b50       __imp_?DeleteItem@CListBox@@UEAAXPEAUtagDELETEITEMSTRUCT@@@Z 000000014001ab50     mfc140:mfc140.dll
 0002:00000b58       __imp_?GetScrollBarCtrl@CWnd@@UEBAPEAVCScrollBar@@H@Z 000000014001ab58     mfc140:mfc140.dll
 0002:00000b60       __imp_?VKeyToItem@CListBox@@UEAAHII@Z 000000014001ab60     mfc140:mfc140.dll
 0002:00000b68       __imp_?Unregister@CWinApp@@UEAAHXZ 000000014001ab68     mfc140:mfc140.dll
 0002:00000b70       __imp_?Register@CWinApp@@UEAAHXZ 000000014001ab70     mfc140:mfc140.dll
 0002:00000b78       __imp_?InitLibId@CWinApp@@UEAAXXZ 000000014001ab78     mfc140:mfc140.dll
 0002:00000b80       __imp_?WriteProfileBinary@CWinApp@@UEAAHPEBD0PEAEI@Z 000000014001ab80     mfc140:mfc140.dll
 0002:00000b88       __imp_?GetProfileBinary@CWinApp@@UEAAHPEBD0PEAPEAEPEAI@Z 000000014001ab88     mfc140:mfc140.dll
 0002:00000b90       __imp_?WriteProfileStringA@CWinApp@@UEAAHPEBD00@Z 000000014001ab90     mfc140:mfc140.dll
 0002:00000b98       __imp_?GetProfileStringA@CWinApp@@UEAA?AV?$CStringT@DV?$StrTraitMFC_DLL@DV?$ChTraitsCRT@D@ATL@@@@@ATL@@PEBD00@Z 000000014001ab98     mfc140:mfc140.dll
 0002:00000ba0       __imp_?WriteProfileInt@CWinApp@@UEAAHPEBD0H@Z 000000014001aba0     mfc140:mfc140.dll
 0002:00000ba8       __imp_?GetProfileIntA@CWinApp@@UEAAIPEBD0H@Z 000000014001aba8     mfc140:mfc140.dll
 0002:00000bb0       __imp_?Delete@CWinThread@@UEAAXXZ 000000014001abb0     mfc140:mfc140.dll
 0002:00000bb8       __imp_?GetMainWnd@CWinThread@@UEAAPEAVCWnd@@XZ 000000014001abb8     mfc140:mfc140.dll
 0002:00000bc0       __imp_?ProcessMessageFilter@CWinThread@@UEAAHHPEAUtagMSG@@@Z 000000014001abc0     mfc140:mfc140.dll
 0002:00000bc8       __imp_?ProcessWndProcException@CWinApp@@UEAA_JPEAVCException@@PEBUtagMSG@@@Z 000000014001abc8     mfc140:mfc140.dll
 0002:00000bd0       __imp_?ExitInstance@CWinApp@@UEAAHXZ 000000014001abd0     mfc140:mfc140.dll
 0002:00000bd8       __imp_?IsIdleMessage@CWinThread@@UEAAHPEAUtagMSG@@@Z 000000014001abd8     mfc140:mfc140.dll
 0002:00000be0       __imp_?OnIdle@CWinApp@@UEAAHJ@Z 000000014001abe0     mfc140:mfc140.dll
 0002:00000be8       __imp_?PumpMessage@CWinThread@@UEAAHXZ 000000014001abe8     mfc140:mfc140.dll
 0002:00000bf0       __imp_?PreTranslateMessage@CWinThread@@UEAAHPEAUtagMSG@@@Z 000000014001abf0     mfc140:mfc140.dll
 0002:00000bf8       __imp_?GetConnectionHook@CCmdTarget@@MEAAPEAUIConnectionPoint@@AEBU_GUID@@@Z 000000014001abf8     mfc140:mfc140.dll
 0002:00000c00       __imp_?GetExtraConnectionPoints@CCmdTarget@@MEAAHPEAVCPtrArray@@@Z 000000014001ac00     mfc140:mfc140.dll
 0002:00000c08       __imp_?GetInterfaceHook@CCmdTarget@@UEAAPEAUIUnknown@@PEBX@Z 000000014001ac08     mfc140:mfc140.dll
 0002:00000c10       __imp_?OnCreateAggregates@CCmdTarget@@UEAAHXZ 000000014001ac10     mfc140:mfc140.dll
 0002:00000c18       __imp_?GetEventSinkMap@CCmdTarget@@MEBAPEBUAFX_EVENTSINKMAP@@XZ 000000014001ac18     mfc140:mfc140.dll
 0002:00000c20       __imp_?GetInterfaceMap@CCmdTarget@@MEBAPEBUAFX_INTERFACEMAP@@XZ 000000014001ac20     mfc140:mfc140.dll
 0002:00000c28       __imp_?GetConnectionMap@CCmdTarget@@MEBAPEBUAFX_CONNECTIONMAP@@XZ 000000014001ac28     mfc140:mfc140.dll
 0002:00000c30       __imp_?GetDispatchMap@CCmdTarget@@MEBAPEBUAFX_DISPMAP@@XZ 000000014001ac30     mfc140:mfc140.dll
 0002:00000c38       __imp_?GetCommandMap@CCmdTarget@@MEBAPEBUAFX_OLECMDMAP@@XZ 000000014001ac38     mfc140:mfc140.dll
 0002:00000c40       __imp_?GetTypeLib@CCmdTarget@@UEAAJKPEAPEAUITypeLib@@@Z 000000014001ac40     mfc140:mfc140.dll
 0002:00000c48       __imp_?GetTypeLibCache@CCmdTarget@@UEAAPEAVCTypeLibCache@@XZ 000000014001ac48     mfc140:mfc140.dll
 0002:00000c50       __imp_?GetTypeInfoCount@CCmdTarget@@UEAAIXZ 000000014001ac50     mfc140:mfc140.dll
 0002:00000c58       __imp_?GetDispatchIID@CCmdTarget@@UEAAHPEAU_GUID@@@Z 000000014001ac58     mfc140:mfc140.dll
 0002:00000c60       __imp_?IsInvokeAllowed@CCmdTarget@@UEAAHJ@Z 000000014001ac60     mfc140:mfc140.dll
 0002:00000c68       __imp_?OnFinalRelease@CCmdTarget@@UEAAXXZ 000000014001ac68     mfc140:mfc140.dll
 0002:00000c70       __imp_?OnCmdMsg@CCmdTarget@@UEAAHIHPEAXPEAUAFX_CMDHANDLERINFO@@@Z 000000014001ac70     mfc140:mfc140.dll
 0002:00000c78       __imp_?GetRuntimeClass@CWinApp@@UEBAPEAUCRuntimeClass@@XZ 000000014001ac78     mfc140:mfc140.dll
 0002:00000c80       __imp_?DoModal@CDialog@@UEAA_JXZ 000000014001ac80     mfc140:mfc140.dll
 0002:00000c88       __imp_??1CWinApp@@UEAA@XZ  000000014001ac88     mfc140:mfc140.dll
 0002:00000c90       __imp_??0CWinApp@@QEAA@PEBD@Z 000000014001ac90     mfc140:mfc140.dll
 0002:00000c98       __imp_?GetThisMessageMap@CWinApp@@KAPEBUAFX_MSGMAP@@XZ 000000014001ac98     mfc140:mfc140.dll
 0002:00000ca0       __imp_?OnHelp@CWinApp@@IEAAXXZ 000000014001aca0     mfc140:mfc140.dll
 0002:00000ca8       __imp_??_U@YAPEAX_K@Z      000000014001aca8     mfc140:mfc140.dll
 0002:00000cb0       __imp_??_V@YAXPEAX@Z       000000014001acb0     mfc140:mfc140.dll
 0002:00000cb8       __imp_??2@YAPEAX_K@Z       000000014001acb8     mfc140:mfc140.dll
 0002:00000cc0       __imp_??3@YAXPEAX@Z        000000014001acc0     mfc140:mfc140.dll
 0002:00000cc8       __imp_?CharToItem@CListBox@@UEAAHII@Z 000000014001acc8     mfc140:mfc140.dll
 0002:00000cd0       __imp_??1CEdit@@UEAA@XZ    000000014001acd0     mfc140:mfc140.dll
 0002:00000cd8       __imp_?AfxWinMain@@YAHPEAUHINSTANCE__@@0PEADH@Z 000000014001acd8     mfc140:mfc140.dll
 0002:00000ce0       __imp_??0CWnd@@QEAA@XZ     000000014001ace0     mfc140:mfc140.dll
 0002:00000ce8       __imp_?GetRuntimeClass@CEdit@@UEBAPEAUCRuntimeClass@@XZ 000000014001ace8     mfc140:mfc140.dll
 0002:00000cf0       __imp_?OnFinalRelease@CWnd@@UEAAXXZ 000000014001acf0     mfc140:mfc140.dll
 0002:00000cf8       __imp_?GetMessageMap@CWnd@@MEBAPEBUAFX_MSGMAP@@XZ 000000014001acf8     mfc140:mfc140.dll
 0002:00000d00       __imp_?GetInterfaceMap@CWnd@@MEBAPEBUAFX_INTERFACEMAP@@XZ 000000014001ad00     mfc140:mfc140.dll
 0002:00000d08       __imp_?Create@CWnd@@UEAAHPEBD0KAEBUtagRECT@@PEAV1@IPEAUCCreateContext@@@Z 000000014001ad08     mfc140:mfc140.dll
 0002:00000d10       \177mfc140_NULL_THUNK_DATA 000000014001ad10     mfc140:mfc140.dll
 0002:00000d18       __guard_check_icall_fptr   000000014001ad18     msvcrt:guard_support.obj
 0002:00000d20       __guard_dispatch_icall_fptr 000000014001ad20     msvcrt:guard_support.obj
 0002:00000d28       __xc_a                     000000014001ad28     msvcrt:initializers.obj
 0002:00000ec8       __xc_z                     000000014001aec8     msvcrt:initializers.obj
 0002:00000ed0       __xi_a                     000000014001aed0     msvcrt:initializers.obj
 0002:00000ef0       __xi_z                     000000014001aef0     msvcrt:initializers.obj
 0002:00000ef8       __xl_a                     000000014001aef8     msvcrt:tlssup.obj
 0002:00000f00       __xl_z                     000000014001af00     msvcrt:tlssup.obj
 0002:00000f08       __xp_a                     000000014001af08     msvcrt:initializers.obj
 0002:00000f10       __xp_z                     000000014001af10     msvcrt:initializers.obj
 0002:00000f18       __xt_a                     000000014001af18     msvcrt:initializers.obj
 0002:00000f20       __xt_z                     000000014001af20     msvcrt:initializers.obj
 0002:00000f60       ??_C@_1EC@JIJBPKFM@?$AAa?$AAp?$AAi?$AA?9?$AAm?$AAs?$AA?9?$AAw?$AAi?$AAn?$AA?9?$AAc?$AAo?$AAr?$AAe@ 000000014001af60     msvcrt:thread_safe_statics.obj
 0002:00000fa8       ??_C@_1BK@MGMFAEKH@?$AAk?$AAe?$AAr?$AAn?$AAe?$AAl?$AA3?$AA2?$AA?4?$AAd?$AAl?$AAl@ 000000014001afa8     msvcrt:thread_safe_statics.obj
 0002:00000fc8       ??_C@_0BM@HLJJNPAH@InitializeConditionVariable@ 000000014001afc8     msvcrt:thread_safe_statics.obj
 0002:00000fe8       ??_C@_0BJ@JEBJOJFJ@SleepConditionVariableCS@ 000000014001afe8     msvcrt:thread_safe_statics.obj
 0002:00001008       ??_C@_0BJ@PGPPEPCC@WakeAllConditionVariable@ 000000014001b008     msvcrt:thread_safe_statics.obj
 0002:00001030       ??_7type_info@@6B@         000000014001b030     msvcrt:std_type_info_static.obj
 0002:00001048       GUID_ATLVer110             000000014001b048     atls:atlbase.obj
 0002:00001060       ??_C@_1IC@ONKHOIDK@?$AAE?$AAR?$AAR?$AAO?$AAR?$AA?5?$AA?3?$AA?5?$AAU?$AAn?$AAa?$AAb?$AAl?$AAe?$AA?5@ 000000014001b060     atls:atlbase.obj
 0002:000010e8       ??_C@_0BE@OHABKPEK@C?3?2log?2crossfire?2?$CFs@ 000000014001b0e8     BugReporter.obj
 0002:00001100       ??_C@_0BC@OFAGFEDM@?$CFs?2?$CFsdmp_?$CFs_?$CFs_?$CFs@ 000000014001b100     BugReporter.obj
 0002:00001118       ??_C@_0CC@FCEOPKOK@?$CF04d?$CF02d?$CF02d?9?$CF02d?$CF02d?$CF02d?$CF03d?4d@ 000000014001b118     BugReporter.obj
 0002:0000113c       ??_C@_02DKCKIIND@?$CFs@    000000014001b13c     BugReporter.obj
 0002:00001140       ??_C@_0BF@IAOALLHJ@C?3?2log?2crossfire?2?$CFs?2@ 000000014001b140     BugReporter.obj
 0002:00001158       ??_C@_01KICIPPFI@?2@       000000014001b158     BugReporter.obj
 0002:0000115c       ??_C@_04KBDJOJNB@?$FL?$CFd?$FN@ 000000014001b15c     BugReporter.obj
 0002:00001168       ??_C@_0L@IFPJGDKC@?$CFd?$CF02d?$CF02d@ 000000014001b168     BugReporter.obj
 0002:00001178       ??_C@_0O@EMHFIMLF@?4?2Setting?4ini@ 000000014001b178     BugReporter.obj
 0002:00001188       ??_C@_08PNEMGIDK@FullDump@ 000000014001b188     BugReporter.obj
 0002:00001198       ??_C@_08NCCBLF@GameMgmt@   000000014001b198     BugReporter.obj
 0002:000011a8       ??_C@_0BJ@DAFBOCMI@CRS?5Upload?5Succeeded?3?5?$CFs@ 000000014001b1a8     BugReporter.obj
 0002:000011c8       ??_C@_0BG@LEKOEBGH@CRS?5Upload?5Failed?3?5?$CFs@ 000000014001b1c8     BugReporter.obj
 0002:000011e0       ??_C@_03GIOIKFCO@C?3?2@    000000014001b1e0     BugReporter.obj
 0002:000011e4       ??_C@_03MGHMBJCF@log@      000000014001b1e4     BugReporter.obj
 0002:000011e8       ??_C@_04FNMMLKAG@log?2@    000000014001b1e8     BugReporter.obj
 0002:000011f0       ??_C@_09LOKONNNP@crossfire@ 000000014001b1f0     BugReporter.obj
 0002:000011fc       ??_C@_05BMGBEOOC@?$CFs?2?$CFs@ 000000014001b1fc     BugReporter.obj
 0002:00001208       ??_C@_0BA@JFNIOLAK@string?5too?5long@ 000000014001b208     BugReporter.obj
 0002:000052b0       ??_C@_1BA@HDJCCPDO@?$AAC?$AAR?$AAS?$AA?4?$AAi?$AAn?$AAi@ 000000014001f2b0     crs_uploader.obj
 0002:000052c0       ??_C@_17BHJPJDEN@?$AAU?$AAR?$AAL@ 000000014001f2c0     crs_uploader.obj
 0002:000052c8       ??_C@_17KFDBOMCI@?$AAC?$AAR?$AAS@ 000000014001f2c8     crs_uploader.obj
 0002:000052d0       ??_C@_1CG@KLCLFNNP@?$AAD?$AAe?$AAl?$AAe?$AAt?$AAe?$AAM?$AAi?$AAn?$AAi?$AAd?$AAu?$AAm?$AAp?$AAF@ 000000014001f2d0     crs_uploader.obj
 0002:000052f8       ??_C@_19FKLFLPMF@?$AAt?$AAr?$AAu?$AAe@ 000000014001f2f8     crs_uploader.obj
 0002:00005308       ??_C@_1BG@BMKKPDAI@?$AA?$CF?$AAs?$AA?2?$AAC?$AAR?$AAS?$AA?4?$AAi?$AAn?$AAi@ 000000014001f308     crs_uploader.obj
 0002:00005320       ??_C@_1BA@ODBNFJPP@?$AAu?$AAn?$AAk?$AAn?$AAw?$AAo?$AAn@ 000000014001f320     crs_uploader.obj
 0002:00005330       ??_C@_1M@LLCLNBHO@?$AA?$CF?$AAs?$AA_?$AA?$CF?$AAs@ 000000014001f330     crs_uploader.obj
 0002:00005340       ??_C@_0L@CIKECLEP@version?3?$CFd@ 000000014001f340     crs_uploader.obj
 0002:00005350       ??_C@_09BNNAOANA@empty?5url@ 000000014001f350     crs_uploader.obj
 0002:00005360       ??_C@_1O@NBDODAKG@?$AAu?$AAp?$AAl?$AAo?$AAa?$AAd@ 000000014001f360     crs_uploader.obj
 0002:00005370       ??_C@_0BL@ININHFIP@output_dir?5is?5empty?5URL?$DN?$CFs@ 000000014001f370     crs_uploader.obj
 0002:00005390       ??_C@_0BI@LFPNAEAK@invalid?5url?$FL?$CFlu?$FN?5URL?$DN?$CFs@ 000000014001f390     crs_uploader.obj
 0002:000053a8       ??_C@_0BA@ELPOGNCH@disabled?5URL?$DN?$CFs@ 000000014001f3a8     crs_uploader.obj
 0002:000053b8       ??_C@_0BA@GOHDMMKI@unknown?5path?$DN?$CFs@ 000000014001f3b8     crs_uploader.obj
 0002:000053c8       ??_C@_0BD@BMMMPMLP@exists?5not?5path?$DN?$CFs@ 000000014001f3c8     crs_uploader.obj
 0002:000053e0       ??_C@_0CC@NKABMACB@?$CFs?5WinHttpOpenRequest?$FL?$CFlu?$FN?5URL?$DN@ 000000014001f3e0     crs_uploader.obj
 0002:00005408       ??_C@_0CC@MFDBFDLN@?$CFs?5WinHttpSendRequest?$FL?$CFlu?$FN?5URL?$DN@ 000000014001f408     crs_uploader.obj
 0002:00005430       ??_C@_07CIFAGBMG@unknown@  000000014001f430     crs_uploader.obj
 0002:00005438       ??_C@_0L@KCOBBBIC@?$CFs?$CL0x?$CFI64X@ 000000014001f438     crs_uploader.obj
 0002:00005448       ??_C@_0DE@FBPBPEDJ@?$CD?5Exception?5Infomation?5?3?5EXCEPT@ 000000014001f448     crs_uploader.obj
 0002:00005480       ??_C@_0BH@GDOLEHPB@?$CD?5Exception?5Infomation@ 000000014001f480     crs_uploader.obj
 0002:00005498       ??_C@_08LLIHJNDD@02?318?305@ 000000014001f498     crs_uploader.obj
 0002:000054a8       ??_C@_0M@KPOGGKFB@Jul?529?52021@ 000000014001f4a8     crs_uploader.obj
 0002:000054b8       ??_C@_0BC@CEMNINJG@?$CD?5DATESTAMP?$DN?$CFs?5?$CFs@ 000000014001f4b8     crs_uploader.obj
 0002:000054d0       ??_C@_0BC@KFCCOPHA@?$CD?5Address?$DN0x?$CF016X@ 000000014001f4d0     crs_uploader.obj
 0002:000054e8       ??_C@_0BF@CCECPKIO@?$CD?5ExceptionCode?$DN0x?$CFX@ 000000014001f4e8     crs_uploader.obj
 0002:00005500       ??_C@_0BO@HFLEEEGJ@?$CF2d?50x?$CF08X?50x?$CF08X?50x?$CF08X?5?$CI?$CFs?$CJ@ 000000014001f500     crs_uploader.obj
 0002:00005520       ??_C@_0BK@ENPPOBB@?$CD?5SymInitialize?5FAIL?$FL?$CFlu?$FN@ 000000014001f520     crs_uploader.obj
 0002:00005540       ??_C@_1BM@PEICEKM@?$AAS?$AAm?$AAi?$AAl?$AAe?$AAG?$AAa?$AAt?$AAe?$AA?5?$AAC?$AAR?$AAS@ 000000014001f540     crs_uploader.obj
 0002:00005560       ??_C@_0BI@JANBAAPF@WinHttpOpen?$FL?$CFlu?$FN?5URL?$DN?$CFs@ 000000014001f560     crs_uploader.obj
 0002:00005578       ??_C@_0BL@EFGBFCEJ@WinHttpConnect?$FL?$CFlu?$FN?5URL?$DN?$CFs@ 000000014001f578     crs_uploader.obj
 0002:00005598       ??_C@_17NHNHNCOB@?$AAP?$AAU?$AAT@ 000000014001f598     crs_uploader.obj
 0002:000055a0       ??_C@_0BP@IIOECOIJ@?$CFs?5CreateFile?5READ?$FL?$CFlu?$FN?5URL?$DN?$CFs@ 000000014001f5a0     crs_uploader.obj
 0002:000055c0       ??_C@_0BL@MLCFLFFE@?$CFs?5GetFileSize?$FL?$CFlu?$FN?5URL?$DN?$CFs@ 000000014001f5c0     crs_uploader.obj
 0002:000055e0       ??_C@_0BI@GHDKNBPJ@?$CFs?5ReadFile?$FL?$CFlu?$FN?5URL?$DN?$CFs@ 000000014001f5e0     crs_uploader.obj
 0002:000055f8       ??_C@_0CA@OMIDHMOL@?$CFs?5WinHttpWriteData?$FL?$CFlu?$FN?5URL?$DN?$CFs@ 000000014001f5f8     crs_uploader.obj
 0002:00005618       ??_C@_1BA@NCJLFNJB@?$AAc?$AAr?$AAs?$AA?4?$AAl?$AAo?$AAg@ 000000014001f618     crs_uploader.obj
 0002:00005628       ??_C@_0CG@LLGLPKJE@?$CFs?5WinHttpReceiveResponse?$FL?$CFlu?$FN?5@ 000000014001f628     crs_uploader.obj
 0002:00005650       ??_C@_0CD@ODMPMKPE@?$CFs?5WinHttpQueryHeaders?$FL?$CFlu?$FN?5URL@ 000000014001f650     crs_uploader.obj
 0002:00005678       ??_C@_0BE@IDLGBAE@?$CFs?5HTTP?$FL?$CFlu?$FN?5URL?$DN?$CFs@ 000000014001f678     crs_uploader.obj
 0002:00005690       ??_C@_1FA@CNNLBJGF@?$AA?$CF?$AAs?$AA_?$AA?$CF?$AA0?$AA4?$AAd?$AA?$CF?$AA0?$AA2?$AAd?$AA?$CF?$AA0?$AA2?$AAd@ 000000014001f690     crs_uploader.obj
 0002:000056e0       ??_C@_1M@BHHLEAOO@?$AA?$CF?$AAs?$AA?1?$AA?$CF?$AAs@ 000000014001f6e0     crs_uploader.obj
 0002:000056f0       ??_C@_19LJDFFCJJ@?$AA?$CF?$AAs?$AA?$CF?$AAs@ 000000014001f6f0     crs_uploader.obj
 0002:00005700       ??_C@_0BI@CFPLBAOH@invalid?5string?5position@ 000000014001f700     crs_uploader.obj
 0002:00005718       ??_C@_11LOCGONAA@@         000000014001f718     crs_uploader.obj
 0002:00005720       ??_C@_0BE@DLJIFIGP@?$CFs?2timeout_?$CFs_?$CFs_?$CFs@ 000000014001f720     LogMgmt.obj
 0002:00005738       ??_C@_0BC@BCEHJAGO@?$CFs?2error_?$CFs_?$CFs_?$CFs@ 000000014001f738     LogMgmt.obj
 0002:00005750       ??_C@_0BE@KIEDFKMI@?$CFs?2etcinfo_?$CFs_?$CFs_?$CFs@ 000000014001f750     LogMgmt.obj
 0002:00005768       ??_C@_0BG@NJNBAHKK@?$CF04d?$CF02d?$CF02d_?$CF02d?4log@ 000000014001f768     LogMgmt.obj
 0002:00005780       ??_C@_0BB@FLNJAMGH@?$CF04d?$CF02d?$CF02d?4log@ 000000014001f780     LogMgmt.obj
 0002:00005794       ??_C@_02DPNLHKJD@a?$CL@    000000014001f794     LogMgmt.obj
 0002:00005798       ??_C@_0BE@MNIJIMLO@?$CF02d?3?$CF02d?3?$CF02d?4?$CF03d@ 000000014001f798     LogMgmt.obj
 0002:000057b8       ??_7CServerLog@@6B@        000000014001f7b8     LogMgmt.obj
 0002:000057c0       ??_C@_00CNPNBAHC@@         000000014001f7c0     LogMgmt.obj
 0002:000057c4       ??_C@_04LIFAFMCE@?$FL?$CFs?$FN@ 000000014001f7c4     RWPMLog.obj
 0002:000057cc       ??_C@_06HJNJJLFL@?$FL?$CFlld?$FN@ 000000014001f7cc     RWPMLog.obj
 0002:000057d8       ??_C@_0BP@BMCLPMN@?$CFs?0?5?$CFd?0?5MEMORY_ADDRESS?$FL?$CFd?$FN?0?5?$CFs@ 000000014001f7d8     RWPMLog.obj
 0002:000057f8       ??_C@_0BN@OCKGOCDF@?$CFs?0?5?$CFd?0?5PROTO_START_HOST?0?5?$CFs@ 000000014001f7f8     RWPMLog.obj
 0002:00005818       ??_C@_0CB@GNMPLMEI@?$CFs?0?5?$CFd?0?5PROTO_GAME_USER_INFO?0?5?$CF@ 000000014001f818     RWPMLog.obj
 0002:00005840       ??_C@_0DK@MGKONJKE@?$CFs?0?5?$CFd?0?5PROTO_GAMEGT_INGAME_AIG@ 000000014001f840     RWPMLog.obj
 0002:00005880       ??_C@_0P@IEFPNEK@?$CFs?0?5?$CFd?0?5?$CFs?0?5?$CFs@ 000000014001f880     RWPMLog.obj
 0002:00005898       ??_7CInterfaceDatabase@@6B@ 000000014001f898     ltmodule.obj
 0002:000058f0       ??_7CInterfaceNameMgr@@6B@ 000000014001f8f0     ltmodule.obj
 0002:00005900       ??_7CAPIHolderBase@@6B@    000000014001f900     ltmodule.obj
 0002:00005920       ??_C@_08IGMCDLDE@LogLevel@ 000000014001f920     HostLogger.obj
 0002:00005930       ??_C@_07KMMFIOCI@LogInfo@  000000014001f930     HostLogger.obj
 0002:00005938       ??_C@_06LFKIJBMM@IPCMsg@   000000014001f938     HostLogger.obj
 0002:00005940       ??_C@_09HNBAJPOD@IPCMemory@ 000000014001f940     HostLogger.obj
 0002:00005950       ??_C@_0N@MJMCCHJI@?2?$CFd?$CF02d?$CF02d?2@ 000000014001f950     HostLogger.obj
 0002:00005960       ??_C@_0BI@PDBNHNN@?$CFs?2BattleRoyal_?$CFs_?$CFs_?$CFs@ 000000014001f960     HostLogger.obj
 0002:00005978       ??_C@_0BD@PBMCFJCL@?$CFs?2kernel_?$CFs_?$CFs_?$CFs@ 000000014001f978     HostLogger.obj
 0002:00005990       ??_C@_0BD@DFOFGCOM@?$CFs?2packet_?$CFs_?$CFs_?$CFs@ 000000014001f990     HostLogger.obj
 0002:000059a8       ??_C@_0BM@EPJGHEGG@?$CFs?2mode_user_count_?$CFs_?$CFs_?$CFs@ 000000014001f9a8     HostLogger.obj
 0002:000059c8       ??_C@_0CA@HLCLJLLN@?$CFs?2serverapp_use_count_?$CFs_?$CFs_?$CFs@ 000000014001f9c8     HostLogger.obj
 0002:000059e8       ??_C@_0BB@HFDGAAKA@?$CFs?2RWPM_?$CFs_?$CFs_?$CFs@ 000000014001f9e8     HostLogger.obj
 0002:00005a00       ??_C@_0BD@PILJABOB@?$CFs?2IPCMSG_?$CFs_?$CFs_?$CFs@ 000000014001fa00     HostLogger.obj
 0002:00005a18       ??_C@_0DE@LGCHENKA@?$CFs?0?$CFs?0?$CF04d?4?$CF02d?4?$CF02d?5?$CF02d?3?$CF02d?3@ 000000014001fa18     HostLogger.obj
 0002:00005a50       ??_C@_0CJ@NOHHCMFI@?$CF04d?9?$CF02d?9?$CF02d?9?$CF02d?3?$CF02d?3?$CF02d?4?$CF@ 000000014001fa50     HostLogger.obj
 0002:00005a7c       ??_C@_01JLIPDDHJ@?3@       000000014001fa7c     HostLogger.obj
 0002:00005a80       ??_C@_0L@PIHNNPCB@?$CFs?5?$FLLOW__?$FN@ 000000014001fa80     HostLogger.obj
 0002:00005a90       ??_C@_0L@GMIAMKIO@?$CFs?5?$FLINFO_?$FN@ 000000014001fa90     HostLogger.obj
 0002:00005aa0       ??_C@_0L@IHOLMJOP@?$CFs?5?$FLWARN_?$FN@ 000000014001faa0     HostLogger.obj
 0002:00005ab0       ??_C@_0L@ECIMMAAL@?$CFs?5?$FLERROR?$FN@ 000000014001fab0     HostLogger.obj
 0002:00005ac0       ??_C@_0L@IPABKGEK@?$CFs?5?$FLFATAL?$FN@ 000000014001fac0     HostLogger.obj
 0002:00005ad0       ??_C@_08IHOEFJCP@?$CFs?5?$CFs?5?$AN?6@ 000000014001fad0     HostLogger.obj
 0002:00005ae8       ??_7CMustSyncObjectLog@@6B@ 000000014001fae8     HostLogger.obj
 0002:00005af0       ??_C@_0CN@PIILFGPG@?4?1rez?1NationMsz?1MSG_DEFINE_Serv@ 000000014001faf0     LogMsgManager.obj
 0002:00005b20       ??_C@_0BA@KICEHKPF@App_LogDataSize@ 000000014001fb20     LogMsgManager.obj
 0002:00005b30       ??_C@_0BA@CGBPPCJP@App_LogData?9?$CFzd@ 000000014001fb30     LogMsgManager.obj
 0002:00005b40       ??_C@_0BD@OLBABOEK@vector?$DMT?$DO?5too?5long@ 000000014001fb40     LogMsgManager.obj
 0002:00005b58       ??_C@_0BE@JONHPENG@map?1set?$DMT?$DO?5too?5long@ 000000014001fb58     LoadXlsMsg.obj
 0002:00005b78       ??_7FindXlsMsg@@6B@        000000014001fb78     LoadXlsMsg.obj
 0002:00005b88       ??_7CServerAppApp@@6B@     000000014001fb88     ServerApp.obj
 0002:00005e10       ??_C@_0BB@DCFJGGKM@ILTCommon?4Server@ 000000014001fe10     ServerAppDlg.obj
 0002:00005e28       ??_C@_0BO@KPHFACMM@ServerappIndex?$CI?$CFd?$CJ?0?5Port?$CI?$CFd?$CJ?5@ 000000014001fe28     ServerAppDlg.obj
 0002:00005e50       ??_C@_0EM@HPPCGKPO@GetProcessMemoryUsage?$CI?$CJ?5Get?5pid@ 000000014001fe50     ServerAppDlg.obj
 0002:00005ea0       ??_C@_0FB@MCFDPFPL@GetProcessMemoryUsage?$CI?$CJ?5Open?5pr@ 000000014001fea0     ServerAppDlg.obj
 0002:00005f00       ??_C@_0FJ@NOKGHOF@GetProcessMemoryUsage?$CI?$CJ?5GetProc@ 000000014001ff00     ServerAppDlg.obj
 0002:00005f60       ??_C@_09BJIIPNM@LocalHost@ 000000014001ff60     ServerAppDlg.obj
 0002:00005f70       ??_C@_0DB@MCLBLGGG@Number?5of?5parameters?5is?5invalid@ 000000014001ff70     ServerAppDlg.obj
 0002:00005fa8       ??_C@_0DP@PDKDOPFG@ServerApp?5Init?5GSM_WND_HANDLE?5?3@ 000000014001ffa8     ServerAppDlg.obj
 0002:00005fe8       ??_C@_0DF@FJFGJCKG@Invalid?5manager?5window?5handle?5f@ 000000014001ffe8     ServerAppDlg.obj
 0002:00006020       ??_C@_0CM@IIIDOGJI@Invalid?5server?5index?5found?4?5Ter@ 0000000140020020     ServerAppDlg.obj
 0002:0000604c       ??_C@_06EAOLBNEK@?$CFld_?$CFd@ 000000014002004c     ServerAppDlg.obj
 0002:00006058       ??_C@_09LKCCBOGN@ServerApp@ 0000000140020058     ServerAppDlg.obj
 0002:00006068       ??_C@_0BC@LFNIPHGA@ReadProcessMemory@ 0000000140020068     ServerAppDlg.obj
 0002:00006080       ??_C@_0BD@PBGEEFCK@WriteProcessMemory@ 0000000140020080     ServerAppDlg.obj
 0002:00006098       ??_C@_0CM@GMMNNKDE@ReadProcessMemory?$DN?$CFd?0?5WriteProc@ 0000000140020098     ServerAppDlg.obj
 0002:000060d0       ??_C@_0HI@HCIAJJJC@GAMESERVERMSG_REPORT_HWND?5PostM@ 00000001400200d0     ServerAppDlg.obj
 0002:00006148       ??_C@_0CO@GKLAPNMD@GAMESERVERMSG_LOADING_COMPLETE?5@ 0000000140020148     ServerAppDlg.obj
 0002:00006178       ??_C@_0CF@FEDDMDMI@Recv?5SERVERAPPMSG_ADDCLIENT?5?9?5U@ 0000000140020178     ServerAppDlg.obj
 0002:000061a0       ??_C@_0EG@BLGLGGEG@CServerAppDlg?3?3OnShellMessage?3?3@ 00000001400201a0     ServerAppDlg.obj
 0002:000061e8       ??_C@_0CF@INADFEIB@?7usn?5?$DN?5?$CFs?0?5Index?5?$DN?5?$CFd?0?5IsReward@ 00000001400201e8     ServerAppDlg.obj
 0002:00006210       ??_C@_0DP@HJDGIELG@CServerAppDlg?9OnShellMessage?3?3S@ 0000000140020210     ServerAppDlg.obj
 0002:00006250       ??_C@_0DJ@LJHNNKOC@?7usn?5?$DN?5?$CFs?0?5loop?5?$DN?5?$CFd?0?5IsReward?5@ 0000000140020250     ServerAppDlg.obj
 0002:00006290       ??_C@_0EG@LLNDFMKB@CServerAppDlg?3?3OnShellMessage?3?3@ 0000000140020290     ServerAppDlg.obj
 0002:000062e0       ??_C@_0EA@FGCLOCKG@CServerAppDlg?3?3OnShellMessage?3?3@ 00000001400202e0     ServerAppDlg.obj
 0002:00006320       ??_C@_0EJ@KIIACGNL@CServerAppDlg?3?3OnShellMessage?3?3@ 0000000140020320     ServerAppDlg.obj
 0002:00006370       ??_C@_0BC@JEAOIFOC@?7usn?5?$DN?5?$CFs?0?5i?5?$DN?5?$CFd@ 0000000140020370     ServerAppDlg.obj
 0002:00006388       ??_C@_0DA@LFNOFNFI@GAMESERVERMSG_AUTO_MATCH_STARTI@ 0000000140020388     ServerAppDlg.obj
 0002:000063b8       ??_C@_05GAPFHKKC@?$CBerr?3@ 00000001400203b8     ServerAppDlg.obj
 0002:000063c0       ??_C@_06DBEGDDG@?$CBhack?3@ 00000001400203c0     ServerAppDlg.obj
 0002:000063c8       ??_C@_0P@DBKFBJAC@server_x64?4dll@ 00000001400203c8     ServerAppDlg.obj
 0002:000063d8       ??_C@_0N@MGAIABNC@CreateServer@ 00000001400203d8     ServerAppDlg.obj
 0002:000063f0       ??_C@_0FP@EDNMACCM@CServerAppDlg?3?3LoadServer?$CI?$CJ?0?5Fa@ 00000001400203f0     ServerAppDlg.obj
 0002:00006450       ??_C@_0BC@NENPAAMN@SetMasterDatabase@ 0000000140020450     ServerAppDlg.obj
 0002:00006468       ??_C@_0BF@HFLCBNHD@Resource?5Load?5Failed@ 0000000140020468     ServerAppDlg.obj
 0002:00006480       ??_C@_0N@LBFNJNAG@DeleteServer@ 0000000140020480     ServerAppDlg.obj
 0002:00006490       ??_C@_06NLDEMLK@HAHAHA@    0000000140020490     ServerAppDlg.obj
 0002:000064a0       ??_C@_0ED@GKCGBJAB@GAMESERVERMSG_INSERTCHARACTER_A@ 00000001400204a0     ServerAppDlg.obj
 0002:000064f0       ??_C@_0FJ@IGOJOCLB@CServerAppDlg?3?3ThreadUpdate?5Sen@ 00000001400204f0     ServerAppDlg.obj
 0002:00006550       ??_C@_0FJ@BOALIPHF@CServerAppDlg?3?3ThreadUpdate?5Sen@ 0000000140020550     ServerAppDlg.obj
 0002:000065b0       ??_C@_0FJ@HNGKKIND@CServerAppDlg?3?3ThreadUpdate?5Sen@ 00000001400205b0     ServerAppDlg.obj
 0002:00006610       ??_C@_0GN@EKGJFLNH@CServerAppDlg?3?3ThreadUpdate?5Sen@ 0000000140020610     ServerAppDlg.obj
 0002:00006680       ??_C@_0EA@GOMMNBJL@CServerAppDlg?3?3ThreadUpdate?5?9?5C@ 0000000140020680     ServerAppDlg.obj
 0002:000066c0       ??_C@_0DO@DOJLKLON@CServerAppDlg?3?3ThreadUpdate?5?9?5C@ 00000001400206c0     ServerAppDlg.obj
 0002:00006700       ??_C@_0CO@ENFPBBBP@CServerAppDlg?3?3ThreadUpdate?5?9?5S@ 0000000140020700     ServerAppDlg.obj
 0002:00006730       ??_C@_0CM@EGAFBNIJ@CServerAppDlg?3?3ThreadUpdate?5?9?5S@ 0000000140020730     ServerAppDlg.obj
 0002:00006760       ??_C@_0DC@GMIOFBC@?$FLUCCLog?$FN?5rez?5file?5download?5succ@ 0000000140020760     ServerAppDlg.obj
 0002:00006798       ??_C@_0DJ@PNMLFLAA@?$FLUCCLog?$FN?5rez?5file?5download?5fail@ 0000000140020798     ServerAppDlg.obj
 0002:000067d4       ??_C@_03IEEBNAED@rez@      00000001400207d4     ServerAppDlg.obj
 0002:000067d8       ??_C@_08JFAGHOJI@?$CFs?2?$CK?4rez@ 00000001400207d8     ServerAppDlg.obj
 0002:000067e4       ??_C@_01IDAFKMJL@_@        00000001400207e4     ServerAppDlg.obj
 0002:000067e8       ??_C@_0BL@IJJEJKPA@S_P_F?3?5HOST_HEARTBEAT?5?3?5?$CFd@ 00000001400207e8     ServerAppDlg.obj
 0002:00006810       ??_C@_0EP@CPNDGEAA@GAMESERVERMSG_LOAD_MAP?5?9?5tMapIn@ 0000000140020810     ServerAppDlg.obj
 0002:00006860       ??_C@_0GB@BLONMNPP@Error?5while?5processing?5SendToSe@ 0000000140020860     ServerAppDlg.obj
 0002:000068d0       ??_C@_0FC@CBEKAGGK@Error?5while?5processing?5SendToSe@ 00000001400208d0     ServerAppDlg.obj
 0002:00006928       ??_C@_0CP@ODPBIJII@?$FLRECV?$FN?5tIndex?$FL?$CF02d?$FN?0?5msgID?$FL?$CF02d@ 0000000140020928     ServerAppDlg.obj
 0002:00006958       ??_C@_0DC@LELNLDON@Not?5Supported?5Message?$CB?$CB?$CB?$CB?$CB?5tInd@ 0000000140020958     ServerAppDlg.obj
 0002:00006990       ??_C@_0GC@FCJGOKJC@g_sGameInfos?5?9?5Push?5GameInfo?5Su@ 0000000140020990     ServerAppDlg.obj
 0002:00006a00       ??_C@_0FP@EONMPNCI@g_sGameInfos?5?9?5Push?5GameInfo?5Fa@ 0000000140020a00     ServerAppDlg.obj
 0002:00006a60       ??_C@_0GG@NEAGNFAL@g_sUserInfos?5?9?5Push?5UserInfo?5Su@ 0000000140020a60     ServerAppDlg.obj
 0002:00006ad0       ??_C@_0GD@KPPLLAEO@g_sUserInfos?5?9?5Push?5UserInfo?5Fa@ 0000000140020ad0     ServerAppDlg.obj
 0002:00006b38       ??_C@_0DB@BBOAIBIB@?$FLUCCLog?$FN?5Already?5Has?5the?5rez?5fi@ 0000000140020b38     ServerAppDlg.obj
 0002:00006b70       ??_C@_0DA@IPOEBJEM@?$FLUCCLog?$FN?5start?5rez?5file?5downloa@ 0000000140020b70     ServerAppDlg.obj
 0002:00006ba0       ??_C@_0FK@CANCCIAA@?$FLUCCLog?$FN?5rez?5file?5download?5fail@ 0000000140020ba0     ServerAppDlg.obj
 0002:00006c00       ??_C@_0BI@HNLBPJDH@RunConsoleString?5error?4@ 0000000140020c00     ServerAppDlg.obj
 0002:00006c18       ??_C@_0CB@EMGJKHPD@Logger?5Init?5Failed?5?3?5ErrCode?$FL?$CFd@ 0000000140020c18     ServerAppDlg.obj
 0002:00006c40       ??_C@_0CC@ILNGBDNH@Log?5Msz?5File?5Load?5Failed?4?5Level@ 0000000140020c40     ServerAppDlg.obj
 0002:00006c68       ??_C@_0BO@PFCCNDDI@Log?5Msz?5Entering?5Read?5Mode?4?4?4@ 0000000140020c68     ServerAppDlg.obj
 0002:00006c88       ??_C@_0CC@OKBOBAOJ@Log?5Msz?5Read?9Mode?5Failed?4?5Level@ 0000000140020c88     ServerAppDlg.obj
 0002:00006cb0       ??_C@_0BK@MPHOBHIK@Logger?5USAGE_READ?5Setted?4@ 0000000140020cb0     ServerAppDlg.obj
 0002:00006cd0       ??_C@_0CC@KAPLEABE@Log?5Msz?5File?5Load?5Failed?4?5Level@ 0000000140020cd0     ServerAppDlg.obj
 0002:00006cf8       ??_C@_0BL@BMLEPNEM@Logger?5USAGE_NOUSE?5Setted?4@ 0000000140020cf8     ServerAppDlg.obj
 0002:00006d18       ??_C@_0P@KCHJOCJL@?9SaveGameInfo?$DN@ 0000000140020d18     ServerAppDlg.obj
 0002:00006d28       ??_C@_02GMLFBBN@wb@        0000000140020d28     ServerAppDlg.obj
 0002:00006d30       ??_C@_0P@NBLHLNAC@?9LoadGameInfo?$DN@ 0000000140020d30     ServerAppDlg.obj
 0002:00006d40       ??_C@_01KDCPPGHE@r@        0000000140020d40     ServerAppDlg.obj
 0002:00006d44       ??_C@_06GDNIANOG@?$CFs?5?$CFhd@ 0000000140020d44     ServerAppDlg.obj
 0002:00006d4c       ??_C@_05DIALNFFA@?$CFs?5?$CFd@ 0000000140020d4c     ServerAppDlg.obj
 0002:00006d54       ??_C@_05KDNLHNC@?$CFs?5?$CFf@ 0000000140020d54     ServerAppDlg.obj
 0002:00006d5c       ??_C@_01CLKCMJKC@?5@       0000000140020d5c     ServerAppDlg.obj
 0002:00006d60       ??_C@_0FN@CMEINILJ@?$FLRWPM?$FNReadGSMMemory?5Failed?$CB?$CB?5m_@ 0000000140020d60     ServerAppDlg.obj
 0002:00006dc0       ??_C@_0FE@NEFIKGOD@?$FLRWPM?$FNReadGSMMemory?5Failed?$CB?$CB?5Ad@ 0000000140020dc0     ServerAppDlg.obj
 0002:00006e20       ??_C@_0FG@OFPAPHCO@?$FLRWPM?$FNReadGSMMemory?5Failed?$CB?$CB?5bu@ 0000000140020e20     ServerAppDlg.obj
 0002:00006e80       ??_C@_0FJ@FBMAGNKE@?$FLRWPM?$FNReadGSMMemory?5Failed?$CB?$CB?5Pr@ 0000000140020e80     ServerAppDlg.obj
 0002:00006ee0       ??_C@_0FI@LNJBBJAM@?$FLRWPM?$FNReadGSMMemory?5Failed?$CB?$CB?5Op@ 0000000140020ee0     ServerAppDlg.obj
 0002:00006f40       ??_C@_0FO@GEJFEOLN@?$FLRWPM?$FNReadGSMMemory?5Failed?$CB?$CB?5Re@ 0000000140020f40     ServerAppDlg.obj
 0002:00006fa0       ??_C@_0FB@HONOMPA@?$FLRWPM?$FN?$FLERROR?5?3?5New?5Memory?5Error@ 0000000140020fa0     ServerAppDlg.obj
 0002:00006ff4       ??_C@_06HMJBGFMB@?$FLRECV?$FN@ 0000000140020ff4     ServerAppDlg.obj
 0002:00007000       ??_C@_0DE@PGLLLGDD@?$FLRWPM?$FN?$FLERROR?5?3?5New?5Memory?5Error@ 0000000140021000     ServerAppDlg.obj
 0002:00007038       ??_C@_0DI@NEKPHLAC@?$FLRWPM?$FN?$FLERROR?5?3?5New?5Memory?5Error@ 0000000140021038     ServerAppDlg.obj
 0002:00007070       ??_C@_0DL@INGPPNNG@Recv?5GAMESERVERMSG_INSERTCHARAC@ 0000000140021070     ServerAppDlg.obj
 0002:000070b0       ??_C@_0FC@HOLPKAAP@?$FLRWPM?$FN?$FLERROR?5?3?5New?5Memory?5Error@ 00000001400210b0     ServerAppDlg.obj
 0002:00007110       ??_C@_0FB@GHOBMMIA@?$FLRWPM?$FN?$FLERROR?5?3?5New?5Memory?5Error@ 0000000140021110     ServerAppDlg.obj
 0002:00007170       ??_C@_0ED@JFDONNGO@?$FLRWPM?$FN?$FLERROR?5?3?5New?5Memory?5Error@ 0000000140021170     ServerAppDlg.obj
 0002:000071b8       ??_C@_0CA@FMNGHFIB@GAMESERVERMSG_USER_DISCONNECTED@ 00000001400211b8     ServerAppDlg.obj
 0002:000071d8       ??_C@_0BB@EBJDADCL@?4?2UCCSetting?4ini@ 00000001400211d8     ServerAppDlg.obj
 0002:000071f0       ??_C@_09CNGDDFNE@ServerURL@ 00000001400211f0     ServerAppDlg.obj
 0002:00007200       ??_C@_0O@KMFGOFBD@fileserverurl@ 0000000140021200     ServerAppDlg.obj
 0002:00007210       ??_C@_04MEDPFIKH@HTTP@     0000000140021210     ServerAppDlg.obj
 0002:00007218       ??_C@_0M@FHOHKDM@?$CFd?$CF02d?$CF02d_@ 0000000140021218     ServerAppDlg.obj
 0002:00007224       ??_C@_04FPOLKAEB@?4log@    0000000140021224     ServerAppDlg.obj
 0002:0000722c       ??_C@_03BFHAFKOB@wb?$CL@   000000014002122c     ServerAppDlg.obj
 0002:00007230       ??_C@_0CL@FMBHHKIH@?$FLucclog?$FN?5UCC?5file?5Write?5Error?5N@ 0000000140021230     ServerAppDlg.obj
 0002:00007260       ??_C@_0EF@JPAKIDCC@?$FLUCCLog?$FN?5rez?5temp?5file?5delete?5f@ 0000000140021260     ServerAppDlg.obj
 0002:000072a8       ??_C@_0DF@KLJPIDKF@?$FLUCCLog?$FN?5rez?5temp?5file?5delete?5s@ 00000001400212a8     ServerAppDlg.obj
 0002:000072e0       ??_C@_0M@KHNENFMD@RezFilePath@ 00000001400212e0     ServerAppDlg.obj
 0002:000072f0       ??_C@_0BC@OGNIILDB@rezrepositoryinfo@ 00000001400212f0     ServerAppDlg.obj
 0002:00007308       ??_C@_0DE@DGDLGEL@SERVERAPPMSG_AUTO_MATCH_STARTIN@ 0000000140021308     ServerAppDlg.obj
 0002:00007340       ??_C@_0CL@LPBDBFEP@SERVERAPPMSG_AUTO_MATCH_STARTIN@ 0000000140021340     ServerAppDlg.obj
 0002:00007378       ??_7?$CAPIHolder@VILTCommon@@@@6B@ 0000000140021378     ServerAppDlg.obj
 0002:00007398       ??_C@_0BB@HBOOMJBF@?$CFTs?5?$CI?$CFTs?3?$CFd?$CJ?6?$CFTs@ 0000000140021398     ServerAppDlg.obj
 0002:000073b0       ??_C@_0HG@IFNAKGBH@c?3?2program?5files?5?$CIx86?$CJ?2microsof@ 00000001400213b0     ServerAppDlg.obj
 0002:00007428       ??_C@_0BP@OIEOKIDM@Exception?5thrown?5in?5destructor@ 0000000140021428     ServerAppDlg.obj
 0002:00007448       ??_C@_0N@OMEMOKLE@?$CFTs?5?$CI?$CFTs?3?$CFd?$CJ@ 0000000140021448     ServerAppDlg.obj
 0002:00007458       ??_C@_0L@JODCLDGE@RTID?3?$CFs?3?$CFd@ 0000000140021458     ServerAppDlg.obj
 0002:00007468       ??_C@_0L@JBGDLKBH@read?5error@ 0000000140021468     ServerAppDlg.obj
 0002:00007478       ??_C@_0BC@EOODALEL@Unknown?5exception@ 0000000140021478     ServerAppDlg.obj
 0002:00007498       ??_7exception@std@@6B@     0000000140021498     ServerAppDlg.obj
 0002:000074a8       ??_C@_04BFAHMMK@?$CFlld@   00000001400214a8     ServerAppDlg.obj
 0002:000074b8       ??_7PROTO_SERVERAPPMSG_INIT@@6B@ 00000001400214b8     ServerAppDlg.obj
 0002:000075e8       ??_7CListBox@@6B@          00000001400215e8     ServerAppDlg.obj
 0002:00007900       ??_7CEdit@@6B@             0000000140021900     ServerAppDlg.obj
 0002:00007be0       ??_7CServerAppDlg@@6B@     0000000140021be0     ServerAppDlg.obj
 0002:00007f10       ??_7CGameServerAppHandler@@6B@ 0000000140021f10     ServerAppDlg.obj
 0002:00007f60       ??_C@_01BJJEKLCA@?$CC@     0000000140021f60     safe_string_x64:safe_string.obj
 0002:00007f64       ??_C@_03JMHOMAJH@?$CJ?5?$CC@ 0000000140021f64     safe_string_x64:safe_string.obj
 0002:00007f68       ??_C@_03MFPIGDOF@?5?$DO?5@ 0000000140021f68     safe_string_x64:safe_string.obj
 0002:00007f70       ??_C@_0BE@EGPJCBFC@?5warning?5sprintf?3?5?$CI@ 0000000140021f70     safe_string_x64:safe_string.obj
 0002:00007f88       ??_C@_07DNAEFDKF@sprintf@  0000000140021f88     safe_string_x64:safe_string.obj
 0002:00007f90       ??_C@_0BD@MFEJDGPJ@?5warning?5strcpy?3?5?$CI@ 0000000140021f90     safe_string_x64:safe_string.obj
 0002:00007fa8       ??_C@_08IBECHLLM@strcpy_s@ 0000000140021fa8     safe_string_x64:safe_string.obj
 0002:00007fb8       ??_C@_0BD@JCAAKJFN@warning?5strncpy?3?5?$CI@ 0000000140021fb8     safe_string_x64:safe_string.obj
 0002:00007fd0       ??_C@_07EDFCNFDJ@strncpy@  0000000140021fd0     safe_string_x64:safe_string.obj
 0002:00007fd8       ??_8?$basic_stringstream@DU?$char_traits@D@std@@V?$allocator@D@2@@std@@7B?$basic_ostream@DU?$char_traits@D@std@@@1@@ 0000000140021fd8     safe_string_x64:safe_string.obj
 0002:00007fe8       ??_7?$basic_stringbuf@DU?$char_traits@D@std@@V?$allocator@D@2@@std@@6B@ 0000000140021fe8     safe_string_x64:safe_string.obj
 0002:00008068       ??_7?$basic_stringstream@DU?$char_traits@D@std@@V?$allocator@D@2@@std@@6B@ 0000000140022068     safe_string_x64:safe_string.obj
 0002:00008070       ??_8?$basic_stringstream@DU?$char_traits@D@std@@V?$allocator@D@2@@std@@7B?$basic_istream@DU?$char_traits@D@std@@@1@@ 0000000140022070     safe_string_x64:safe_string.obj
 0002:000080c8       __real@3e666666            00000001400220c8     StdAfx.obj
 0002:000080cc       __real@3f466666            00000001400220cc     StdAfx.obj
 0002:000080d0       __real@3fccccccc0000000    00000001400220d0     ltmodule.obj
 0002:000080d8       __real@3fe8ccccc0000000    00000001400220d8     ltmodule.obj
 0002:000080e0       __real@3ff0000000000000    00000001400220e0     ltmodule.obj
 0002:000080e8       __real@4010000000000000    00000001400220e8     ltmodule.obj
 0002:000080f0       __real@4030000000000000    00000001400220f0     ltmodule.obj
 0002:000080f8       __real@41800000            00000001400220f8     StdAfx.obj
 0002:00008100       __xmm@00000000000000070000000000000000 0000000140022100     crs_uploader.obj
 0002:00008110       __xmm@000000000000000f0000000000000000 0000000140022110     ServerAppDlg.obj
 0002:00008120       __xmm@00000000ffffffffffffffffffffffff 0000000140022120     ltmodule.obj
 0002:00008130       __xmm@3e22f9833e22f9833e22f9833e22f983 0000000140022130     ltmodule.obj
 0002:00008140       __xmm@3f0000003f0000003f0000003f000000 0000000140022140     ltmodule.obj
 0002:00008150       __xmm@3f8000003f8000003f8000003f800000 0000000140022150     ltmodule.obj
 0002:00008160       __xmm@3fc90fdb3fc90fdb3fc90fdb3fc90fdb 0000000140022160     ltmodule.obj
 0002:00008170       __xmm@40c90fdb40c90fdb40c90fdb40c90fdb 0000000140022170     ltmodule.obj
 0002:00008180       __xmm@bf800000bf800000bf800000bf800000 0000000140022180     ltmodule.obj
 0002:00008bb0       _load_config_used          0000000140022bb0     msvcrt:loadcfg.obj
 0002:00008cb0       _tls_used                  0000000140022cb0     msvcrt:tlssup.obj
 0002:00008ce0       ??_R4type_info@@6B@        0000000140022ce0     msvcrt:std_type_info_static.obj
 0002:00008d08       ??_R3type_info@@8          0000000140022d08     msvcrt:std_type_info_static.obj
 0002:00008d20       ??_R2type_info@@8          0000000140022d20     msvcrt:std_type_info_static.obj
 0002:00008d30       ??_R1A@?0A@EA@type_info@@8 0000000140022d30     msvcrt:std_type_info_static.obj
 0002:00008d58       ??_R2CServerLog@@8         0000000140022d58     LogMgmt.obj
 0002:00008d68       ??_R1A@?0A@EA@CServerLog@@8 0000000140022d68     LogMgmt.obj
 0002:00008d90       ??_R3CServerLog@@8         0000000140022d90     LogMgmt.obj
 0002:00008da8       ??_R4CServerLog@@6B@       0000000140022da8     LogMgmt.obj
 0002:00008dd0       ??_R4CInterfaceDatabase@@6B@ 0000000140022dd0     ltmodule.obj
 0002:00008df8       ??_R3CInterfaceDatabase@@8 0000000140022df8     ltmodule.obj
 0002:00008e10       ??_R4CInterfaceNameMgr@@6B@ 0000000140022e10     ltmodule.obj
 0002:00008e38       ??_R3CInterfaceNameMgr@@8  0000000140022e38     ltmodule.obj
 0002:00008e50       ??_R1A@?0A@EA@CInterfaceNameMgr@@8 0000000140022e50     ltmodule.obj
 0002:00008e78       ??_R4CAPIHolderBase@@6B@   0000000140022e78     ltmodule.obj
 0002:00008ea0       ??_R3CAPIHolderBase@@8     0000000140022ea0     ltmodule.obj
 0002:00008eb8       ??_R2CInterfaceDatabase@@8 0000000140022eb8     ltmodule.obj
 0002:00008ec8       ??_R2CAPIHolderBase@@8     0000000140022ec8     ltmodule.obj
 0002:00008ed8       ??_R1A@?0A@EA@CInterfaceDatabase@@8 0000000140022ed8     ltmodule.obj
 0002:00008f00       ??_R2CInterfaceNameMgr@@8  0000000140022f00     ltmodule.obj
 0002:00008f10       ??_R1A@?0A@EA@CAPIHolderBase@@8 0000000140022f10     ltmodule.obj
 0002:00008f38       ??_R1A@?0A@EA@CMustSyncObjectLog@@8 0000000140022f38     HostLogger.obj
 0002:00008f60       ??_R1A@?0A@EA@_RTL_CRITICAL_SECTION@@8 0000000140022f60     HostLogger.obj
 0002:00008f88       ??_R2_RTL_CRITICAL_SECTION@@8 0000000140022f88     HostLogger.obj
 0002:00008f98       ??_R3_RTL_CRITICAL_SECTION@@8 0000000140022f98     HostLogger.obj
 0002:00008fb0       ??_R17?0A@EA@_RTL_CRITICAL_SECTION@@8 0000000140022fb0     HostLogger.obj
 0002:00008fd8       ??_R2CMustSyncObjectLog@@8 0000000140022fd8     HostLogger.obj
 0002:00008ff0       ??_R3CMustSyncObjectLog@@8 0000000140022ff0     HostLogger.obj
 0002:00009008       ??_R4CMustSyncObjectLog@@6B@ 0000000140023008     HostLogger.obj
 0002:00009030       ??_R2FindXlsMsg@@8         0000000140023030     LoadXlsMsg.obj
 0002:00009040       ??_R1A@?0A@EA@FindXlsMsg@@8 0000000140023040     LoadXlsMsg.obj
 0002:00009068       ??_R3FindXlsMsg@@8         0000000140023068     LoadXlsMsg.obj
 0002:00009080       ??_R4FindXlsMsg@@6B@       0000000140023080     LoadXlsMsg.obj
 0002:000090a8       ??_R2CServerAppApp@@8      00000001400230a8     ServerApp.obj
 0002:000090d8       ??_R2CWinApp@@8            00000001400230d8     ServerApp.obj
 0002:00009100       ??_R2CWinThread@@8         0000000140023100     ServerApp.obj
 0002:00009120       ??_R1A@?0A@EA@CServerAppApp@@8 0000000140023120     ServerApp.obj
 0002:00009148       ??_R1A@?0A@EA@CWinApp@@8   0000000140023148     ServerApp.obj
 0002:00009170       ??_R2CObject@@8            0000000140023170     ServerApp.obj
 0002:00009180       ??_R3CObject@@8            0000000140023180     ServerApp.obj
 0002:00009198       ??_R1A@?0A@EA@CObject@@8   0000000140023198     ServerApp.obj
 0002:000091c0       ??_R2CCmdTarget@@8         00000001400231c0     ServerApp.obj
 0002:000091d8       ??_R3CCmdTarget@@8         00000001400231d8     ServerApp.obj
 0002:000091f0       ??_R1A@?0A@EA@CCmdTarget@@8 00000001400231f0     ServerApp.obj
 0002:00009218       ??_R1A@?0A@EA@CWinThread@@8 0000000140023218     ServerApp.obj
 0002:00009240       ??_R3CWinApp@@8            0000000140023240     ServerApp.obj
 0002:00009258       ??_R3CWinThread@@8         0000000140023258     ServerApp.obj
 0002:00009270       ??_R3CServerAppApp@@8      0000000140023270     ServerApp.obj
 0002:00009288       ??_R4CServerAppApp@@6B@    0000000140023288     ServerApp.obj
 0002:000092b0       ??_R2?$CAPIHolder@VILTCommon@@@@8 00000001400232b0     ServerAppDlg.obj
 0002:000092c8       ??_R2CGameServerAppHandler@@8 00000001400232c8     ServerAppDlg.obj
 0002:000092e0       ??_R2CServerAppDlg@@8      00000001400232e0     ServerAppDlg.obj
 0002:00009310       ??_R2ServerAppHandler@@8   0000000140023310     ServerAppDlg.obj
 0002:00009320       ??_R1A@?0A@EA@?$CAPIHolder@VILTCommon@@@@8 0000000140023320     ServerAppDlg.obj
 0002:00009348       ??_R1A@?0A@EA@CGameServerAppHandler@@8 0000000140023348     ServerAppDlg.obj
 0002:00009370       ??_R2CDialog@@8            0000000140023370     ServerAppDlg.obj
 0002:00009398       ??_R3CDialog@@8            0000000140023398     ServerAppDlg.obj
 0002:000093b0       ??_R1A@?0A@EA@CDialog@@8   00000001400233b0     ServerAppDlg.obj
 0002:000093d8       ??_R1A@?0A@EA@CServerAppDlg@@8 00000001400233d8     ServerAppDlg.obj
 0002:00009400       ??_R1A@?0A@EA@ServerAppHandler@@8 0000000140023400     ServerAppDlg.obj
 0002:00009428       ??_R3?$CAPIHolder@VILTCommon@@@@8 0000000140023428     ServerAppDlg.obj
 0002:00009440       ??_R3CGameServerAppHandler@@8 0000000140023440     ServerAppDlg.obj
 0002:00009458       ??_R3CServerAppDlg@@8      0000000140023458     ServerAppDlg.obj
 0002:00009470       ??_R3ServerAppHandler@@8   0000000140023470     ServerAppDlg.obj
 0002:00009488       ??_R4?$CAPIHolder@VILTCommon@@@@6B@ 0000000140023488     ServerAppDlg.obj
 0002:000094b0       ??_R4CGameServerAppHandler@@6B@ 00000001400234b0     ServerAppDlg.obj
 0002:000094d8       ??_R4CServerAppDlg@@6B@    00000001400234d8     ServerAppDlg.obj
 0002:00009500       ??_R1A@?0A@EA@exception@std@@8 0000000140023500     ServerAppDlg.obj
 0002:00009528       ??_R2exception@std@@8      0000000140023528     ServerAppDlg.obj
 0002:00009538       ??_R3exception@std@@8      0000000140023538     ServerAppDlg.obj
 0002:00009550       ??_R4exception@std@@6B@    0000000140023550     ServerAppDlg.obj
 0002:00009578       ??_R1A@?0A@EA@PROTO_SERVERAPPMSG_INIT@@8 0000000140023578     ServerAppDlg.obj
 0002:000095a0       ??_R2GAMEPROTO_SC_COMMON@@8 00000001400235a0     ServerAppDlg.obj
 0002:000095b8       ??_R3GAMEPROTO_SC_COMMON@@8 00000001400235b8     ServerAppDlg.obj
 0002:000095d0       ??_R1A@?0A@EA@GAMEPROTO_SC_COMMON@@8 00000001400235d0     ServerAppDlg.obj
 0002:000095f8       ??_R2GAMEPROTO_COMMON@@8   00000001400235f8     ServerAppDlg.obj
 0002:00009608       ??_R3GAMEPROTO_COMMON@@8   0000000140023608     ServerAppDlg.obj
 0002:00009620       ??_R1A@?0A@EA@GAMEPROTO_COMMON@@8 0000000140023620     ServerAppDlg.obj
 0002:00009648       ??_R2PROTO_SERVERAPPMSG_INIT@@8 0000000140023648     ServerAppDlg.obj
 0002:00009668       ??_R3PROTO_SERVERAPPMSG_INIT@@8 0000000140023668     ServerAppDlg.obj
 0002:00009680       ??_R4PROTO_SERVERAPPMSG_INIT@@6B@ 0000000140023680     ServerAppDlg.obj
 0002:000096a8       ??_R1A@?0A@EA@CListBox@@8  00000001400236a8     ServerAppDlg.obj
 0002:000096d0       ??_R2CListBox@@8           00000001400236d0     ServerAppDlg.obj
 0002:000096f8       ??_R3CListBox@@8           00000001400236f8     ServerAppDlg.obj
 0002:00009710       ??_R4CListBox@@6B@         0000000140023710     ServerAppDlg.obj
 0002:00009738       ??_R1A@?0A@EA@CEdit@@8     0000000140023738     ServerAppDlg.obj
 0002:00009760       ??_R2CWnd@@8               0000000140023760     ServerAppDlg.obj
 0002:00009780       ??_R3CWnd@@8               0000000140023780     ServerAppDlg.obj
 0002:00009798       ??_R1A@?0A@EA@CWnd@@8      0000000140023798     ServerAppDlg.obj
 0002:000097c0       ??_R2CEdit@@8              00000001400237c0     ServerAppDlg.obj
 0002:000097e8       ??_R3CEdit@@8              00000001400237e8     ServerAppDlg.obj
 0002:00009800       ??_R4CEdit@@6B@            0000000140023800     ServerAppDlg.obj
 0002:00009828       ??_R3?$basic_istream@DU?$char_traits@D@std@@@std@@8 0000000140023828     safe_string_x64:safe_string.obj
 0002:00009840       ??_R3?$basic_iostream@DU?$char_traits@D@std@@@std@@8 0000000140023840     safe_string_x64:safe_string.obj
 0002:00009858       ??_R1A@?0A@EA@?$basic_istream@DU?$char_traits@D@std@@@std@@8 0000000140023858     safe_string_x64:safe_string.obj
 0002:00009880       ??_R2?$basic_stringbuf@DU?$char_traits@D@std@@V?$allocator@D@2@@std@@8 0000000140023880     safe_string_x64:safe_string.obj
 0002:00009898       ??_R17A@3EA@?$_Iosb@H@std@@8 0000000140023898     safe_string_x64:safe_string.obj
 0002:000098c0       ??_R1A@?0A@EA@?$basic_stringstream@DU?$char_traits@D@std@@V?$allocator@D@2@@std@@8 00000001400238c0     safe_string_x64:safe_string.obj
 0002:000098e8       ??_R1A@?0A@EA@?$basic_streambuf@DU?$char_traits@D@std@@@std@@8 00000001400238e8     safe_string_x64:safe_string.obj
 0002:00009910       ??_R2?$basic_istream@DU?$char_traits@D@std@@@std@@8 0000000140023910     safe_string_x64:safe_string.obj
 0002:00009938       ??_R3?$basic_stringbuf@DU?$char_traits@D@std@@V?$allocator@D@2@@std@@8 0000000140023938     safe_string_x64:safe_string.obj
 0002:00009950       ??_R2?$basic_ostream@DU?$char_traits@D@std@@@std@@8 0000000140023950     safe_string_x64:safe_string.obj
 0002:00009978       ??_R3?$basic_ios@DU?$char_traits@D@std@@@std@@8 0000000140023978     safe_string_x64:safe_string.obj
 0002:00009990       ??_R1BA@?0A@EA@?$basic_ostream@DU?$char_traits@D@std@@@std@@8 0000000140023990     safe_string_x64:safe_string.obj
 0002:000099b8       ??_R1A@?0A@EA@ios_base@std@@8 00000001400239b8     safe_string_x64:safe_string.obj
 0002:000099e0       ??_R1A@?0A@EA@?$basic_ostream@DU?$char_traits@D@std@@@std@@8 00000001400239e0     safe_string_x64:safe_string.obj
 0002:00009a08       ??_R2?$basic_streambuf@DU?$char_traits@D@std@@@std@@8 0000000140023a08     safe_string_x64:safe_string.obj
 0002:00009a18       ??_R1A@?0A@EA@?$_Iosb@H@std@@8 0000000140023a18     safe_string_x64:safe_string.obj
 0002:00009a40       ??_R1A@?0A@EA@?$basic_stringbuf@DU?$char_traits@D@std@@V?$allocator@D@2@@std@@8 0000000140023a40     safe_string_x64:safe_string.obj
 0002:00009a70       ??_R2?$basic_iostream@DU?$char_traits@D@std@@@std@@8 0000000140023a70     safe_string_x64:safe_string.obj
 0002:00009ac0       ??_R2?$basic_stringstream@DU?$char_traits@D@std@@V?$allocator@D@2@@std@@8 0000000140023ac0     safe_string_x64:safe_string.obj
 0002:00009b18       ??_R4?$basic_stringbuf@DU?$char_traits@D@std@@V?$allocator@D@2@@std@@6B@ 0000000140023b18     safe_string_x64:safe_string.obj
 0002:00009b40       ??_R4?$basic_stringstream@DU?$char_traits@D@std@@V?$allocator@D@2@@std@@6B@ 0000000140023b40     safe_string_x64:safe_string.obj
 0002:00009b68       ??_R1A@A@3FA@?$basic_ios@DU?$char_traits@D@std@@@std@@8 0000000140023b68     safe_string_x64:safe_string.obj
 0002:00009b90       ??_R2ios_base@std@@8       0000000140023b90     safe_string_x64:safe_string.obj
 0002:00009ba8       ??_R3?$basic_ostream@DU?$char_traits@D@std@@@std@@8 0000000140023ba8     safe_string_x64:safe_string.obj
 0002:00009bc0       ??_R1A@?0A@EA@?$basic_iostream@DU?$char_traits@D@std@@@std@@8 0000000140023bc0     safe_string_x64:safe_string.obj
 0002:00009be8       ??_R3ios_base@std@@8       0000000140023be8     safe_string_x64:safe_string.obj
 0002:00009c00       ??_R3?$basic_streambuf@DU?$char_traits@D@std@@@std@@8 0000000140023c00     safe_string_x64:safe_string.obj
 0002:00009c18       ??_R3?$basic_stringstream@DU?$char_traits@D@std@@V?$allocator@D@2@@std@@8 0000000140023c18     safe_string_x64:safe_string.obj
 0002:00009c30       ??_R2?$_Iosb@H@std@@8      0000000140023c30     safe_string_x64:safe_string.obj
 0002:00009c40       ??_R1A@A@3EA@ios_base@std@@8 0000000140023c40     safe_string_x64:safe_string.obj
 0002:00009c68       ??_R1A@?0A@EA@?$basic_ios@DU?$char_traits@D@std@@@std@@8 0000000140023c68     safe_string_x64:safe_string.obj
 0002:00009c90       ??_R3?$_Iosb@H@std@@8      0000000140023c90     safe_string_x64:safe_string.obj
 0002:00009ca8       ??_R17?0A@EA@?$_Iosb@H@std@@8 0000000140023ca8     safe_string_x64:safe_string.obj
 0002:00009cd0       ??_R2?$basic_ios@DU?$char_traits@D@std@@@std@@8 0000000140023cd0     safe_string_x64:safe_string.obj
 0002:0000a0d8       __rtc_iaa                  00000001400240d8     msvcrt:initsect.obj
 0002:0000a0e0       __rtc_izz                  00000001400240e0     msvcrt:initsect.obj
 0002:0000a0e8       __rtc_taa                  00000001400240e8     msvcrt:initsect.obj
 0002:0000a0f0       __rtc_tzz                  00000001400240f0     msvcrt:initsect.obj
 0002:0000a100       _tls_start                 0000000140024100     msvcrt:tlssup.obj
 0002:0000a110       _Init_thread_epoch         0000000140024110     msvcrt:thread_safe_statics.obj
 0002:0000a114       _tls_end                   0000000140024114     msvcrt:tlssup.obj
 0002:0000c568       _CT??_R0?AVexception@std@@@8??0exception@std@@QEAA@AEBV01@@Z24 0000000140026568     ServerAppDlg.obj
 0002:0000c590       _CTA1?AVexception@std@@    0000000140026590     ServerAppDlg.obj
 0002:0000c5a0       _TI1?AVexception@std@@     00000001400265a0     ServerAppDlg.obj
 0002:0000c62c       __IMPORT_DESCRIPTOR_PSAPI  000000014002662c     Psapi:PSAPI.DLL
 0002:0000c640       __IMPORT_DESCRIPTOR_mfc140 0000000140026640     mfc140:mfc140.dll
 0002:0000c654       __IMPORT_DESCRIPTOR_KERNEL32 0000000140026654     kernel32:KERNEL32.dll
 0002:0000c668       __IMPORT_DESCRIPTOR_USER32 0000000140026668     user32:USER32.dll
 0002:0000c67c       __IMPORT_DESCRIPTOR_SHELL32 000000014002667c     shell32:SHELL32.dll
 0002:0000c690       __IMPORT_DESCRIPTOR_SHLWAPI 0000000140026690     shlwapi:SHLWAPI.dll
 0002:0000c6a4       __IMPORT_DESCRIPTOR_MSVCP140 00000001400266a4     msvcprt:MSVCP140.dll
 0002:0000c6b8       __IMPORT_DESCRIPTOR_WININET 00000001400266b8     Wininet:WININET.dll
 0002:0000c6cc       __IMPORT_DESCRIPTOR_dbghelp 00000001400266cc     DbgHelp:dbghelp.dll
 0002:0000c6e0       __IMPORT_DESCRIPTOR_WINMM  00000001400266e0     winmm:WINMM.dll
 0002:0000c6f4       __IMPORT_DESCRIPTOR_WINHTTP 00000001400266f4     winhttp:WINHTTP.dll
 0002:0000c708       __IMPORT_DESCRIPTOR_WS2_32 0000000140026708     ws2_32:WS2_32.dll
 0002:0000c71c       __IMPORT_DESCRIPTOR_VCRUNTIME140 000000014002671c     vcruntime:VCRUNTIME140.dll
 0002:0000c730       __IMPORT_DESCRIPTOR_api-ms-win-crt-stdio-l1-1-0 0000000140026730     ucrt:api-ms-win-crt-stdio-l1-1-0.dll
 0002:0000c744       __IMPORT_DESCRIPTOR_api-ms-win-crt-runtime-l1-1-0 0000000140026744     ucrt:api-ms-win-crt-runtime-l1-1-0.dll
 0002:0000c758       __IMPORT_DESCRIPTOR_api-ms-win-crt-filesystem-l1-1-0 0000000140026758     ucrt:api-ms-win-crt-filesystem-l1-1-0.dll
 0002:0000c76c       __IMPORT_DESCRIPTOR_api-ms-win-crt-string-l1-1-0 000000014002676c     ucrt:api-ms-win-crt-string-l1-1-0.dll
 0002:0000c780       __IMPORT_DESCRIPTOR_api-ms-win-crt-convert-l1-1-0 0000000140026780     ucrt:api-ms-win-crt-convert-l1-1-0.dll
 0002:0000c794       __IMPORT_DESCRIPTOR_api-ms-win-crt-utility-l1-1-0 0000000140026794     ucrt:api-ms-win-crt-utility-l1-1-0.dll
 0002:0000c7a8       __IMPORT_DESCRIPTOR_api-ms-win-crt-time-l1-1-0 00000001400267a8     ucrt:api-ms-win-crt-time-l1-1-0.dll
 0002:0000c7bc       __IMPORT_DESCRIPTOR_api-ms-win-crt-heap-l1-1-0 00000001400267bc     ucrt:api-ms-win-crt-heap-l1-1-0.dll
 0002:0000c7d0       __IMPORT_DESCRIPTOR_api-ms-win-crt-math-l1-1-0 00000001400267d0     ucrt:api-ms-win-crt-math-l1-1-0.dll
 0002:0000c7e4       __IMPORT_DESCRIPTOR_api-ms-win-crt-locale-l1-1-0 00000001400267e4     ucrt:api-ms-win-crt-locale-l1-1-0.dll
 0002:0000c7f8       __NULL_IMPORT_DESCRIPTOR   00000001400267f8     Psapi:PSAPI.DLL
 0003:00000000       _Init_global_epoch         0000000140029000     msvcrt:thread_safe_statics.obj
 0003:00000004       __scrt_native_dllmain_reason 0000000140029004     msvcrt:utility.obj
 0003:00000008       __security_cookie_complement 0000000140029008     msvcrt:gs_cookie.obj
 0003:00000010       __security_cookie          0000000140029010     msvcrt:gs_cookie.obj
 0003:00000018       __isa_available            0000000140029018     msvcrt:cpu_disp.obj
 0003:0000001c       __isa_enabled              000000014002901c     msvcrt:cpu_disp.obj
 0003:00000020       __memcpy_nt_iters          0000000140029020     msvcrt:cpu_disp.obj
 0003:00000028       __scrt_default_matherr     0000000140029028     msvcrt:matherr.obj
 0003:00000030       __scrt_ucrt_dll_is_in_use  0000000140029030     msvcrt:ucrt_stubs.obj
 0003:00000040       ?m_LogLevel@CHLogger@@0IA  0000000140029040     HostLogger.obj
 0003:00000044       ?m_eSharedMemUsage@CLogMsgManager@@0W4ESHARED_MEM_USAGE_TYPE@1@A 0000000140029044     LogMsgManager.obj
 0003:00000048       ?g_lMinInterval@@3JA       0000000140029048     ServerAppDlg.obj
 0003:00000050       ?m_strFileFormat@CHLogger@@0V?$basic_string@DU?$char_traits@D@std@@V?$allocator@D@2@@std@@A 0000000140029050     HostLogger.obj
 0003:00000070       ?m_strBRFileFormat@CHLogger@@0V?$basic_string@DU?$char_traits@D@std@@V?$allocator@D@2@@std@@A 0000000140029070     HostLogger.obj
 0003:00000090       ?m_strKernelFileFormat@CHLogger@@0V?$basic_string@DU?$char_traits@D@std@@V?$allocator@D@2@@std@@A 0000000140029090     HostLogger.obj
 0003:000000b0       ?m_strEtcFileFormat@CHLogger@@0V?$basic_string@DU?$char_traits@D@std@@V?$allocator@D@2@@std@@A 00000001400290b0     HostLogger.obj
 0003:000000d0       ?m_strRWProcessMemoryFileFormat@CHLogger@@0V?$basic_string@DU?$char_traits@D@std@@V?$allocator@D@2@@std@@A 00000001400290d0     HostLogger.obj
 0003:000000f0       ?m_strIPCMessageFileFormat@CHLogger@@0V?$basic_string@DU?$char_traits@D@std@@V?$allocator@D@2@@std@@A 00000001400290f0     HostLogger.obj
 0003:00000110       ?m_strTimeOutFileFormat@CHLogger@@0V?$basic_string@DU?$char_traits@D@std@@V?$allocator@D@2@@std@@A 0000000140029110     HostLogger.obj
 0003:00000130       ?m_strPacketFileFormat@CHLogger@@0V?$basic_string@DU?$char_traits@D@std@@V?$allocator@D@2@@std@@A 0000000140029130     HostLogger.obj
 0003:00000150       ?m_strHostName@CHLogger@@0V?$basic_string@DU?$char_traits@D@std@@V?$allocator@D@2@@std@@A 0000000140029150     HostLogger.obj
 0003:00000170       ?m_strServerName@CHLogger@@0V?$basic_string@DU?$char_traits@D@std@@V?$allocator@D@2@@std@@A 0000000140029170     HostLogger.obj
 0003:00000190       ?m_strLogFolder@CHLogger@@0V?$basic_string@DU?$char_traits@D@std@@V?$allocator@D@2@@std@@A 0000000140029190     HostLogger.obj
 0003:000001b0       ?m_strModeUserCountFormat@CHLogger@@0V?$basic_string@DU?$char_traits@D@std@@V?$allocator@D@2@@std@@A 00000001400291b0     HostLogger.obj
 0003:000001d0       ?m_strServerAppUseCountFormat@CHLogger@@0V?$basic_string@DU?$char_traits@D@std@@V?$allocator@D@2@@std@@A 00000001400291d0     HostLogger.obj
 0003:000001f0       ?m_LogLock@CHLogger@@0VCMustSyncObjectLog@@A 00000001400291f0     HostLogger.obj
 0003:00000220       ?m_LogPacketLock@CHLogger@@0VCMustSyncObjectLog@@A 0000000140029220     HostLogger.obj
 0003:00000250       ?g_cServerLog@@3VCServerLog@@A 0000000140029250     ServerAppDlg.obj
 0003:000005c0       _fltused                   00000001400295c0     msvcrt:fltused.obj
 0003:000005d0       ??_R0?AVtype_info@@@8      00000001400295d0     msvcrt:std_type_info_static.obj
 0003:000005f0       ??_R0?AVCServerLog@@@8     00000001400295f0     LogMgmt.obj
 0003:00000618       ??_R0?AVCInterfaceNameMgr@@@8 0000000140029618     ltmodule.obj
 0003:00000640       ??_R0?AVCAPIHolderBase@@@8 0000000140029640     ltmodule.obj
 0003:00000668       ??_R0?AVCInterfaceDatabase@@@8 0000000140029668     ltmodule.obj
 0003:00000698       ??_R0?AVCMustSyncObjectLog@@@8 0000000140029698     HostLogger.obj
 0003:000006c8       ??_R0?AU_RTL_CRITICAL_SECTION@@@8 00000001400296c8     HostLogger.obj
 0003:000006f8       ??_R0?AVFindXlsMsg@@@8     00000001400296f8     LoadXlsMsg.obj
 0003:00000720       ??_R0?AVCCmdTarget@@@8     0000000140029720     ServerApp.obj
 0003:00000748       ??_R0?AVCObject@@@8        0000000140029748     ServerApp.obj
 0003:00000768       ??_R0?AVCWinApp@@@8        0000000140029768     ServerApp.obj
 0003:00000788       ??_R0?AVCWinThread@@@8     0000000140029788     ServerApp.obj
 0003:000007b0       ??_R0?AVCServerAppApp@@@8  00000001400297b0     ServerApp.obj
 0003:000007d8       ??_R0?AVCDialog@@@8        00000001400297d8     ServerAppDlg.obj
 0003:000007f8       ??_R0?AV?$CAPIHolder@VILTCommon@@@@@8 00000001400297f8     ServerAppDlg.obj
 0003:00000828       ??_R0?AVCGameServerAppHandler@@@8 0000000140029828     ServerAppDlg.obj
 0003:00000858       ??_R0?AVCServerAppDlg@@@8  0000000140029858     ServerAppDlg.obj
 0003:00000880       ??_R0?AVServerAppHandler@@@8 0000000140029880     ServerAppDlg.obj
 0003:000008a8       ??_R0PEAVCException@@@8    00000001400298a8     ServerAppDlg.obj
 0003:000008d0       ??_R0?AVexception@std@@@8  00000001400298d0     ServerAppDlg.obj
 0003:000008f8       ??_R0?AUPROTO_SERVERAPPMSG_INIT@@@8 00000001400298f8     ServerAppDlg.obj
 0003:00000928       ??_R0?AUGAMEPROTO_SC_COMMON@@@8 0000000140029928     ServerAppDlg.obj
 0003:00000958       ??_R0?AUGAMEPROTO_COMMON@@@8 0000000140029958     ServerAppDlg.obj
 0003:00000980       ??_R0?AVCListBox@@@8       0000000140029980     ServerAppDlg.obj
 0003:000009a0       ??_R0?AVCEdit@@@8          00000001400299a0     ServerAppDlg.obj
 0003:000009c0       ??_R0?AVCWnd@@@8           00000001400299c0     ServerAppDlg.obj
 0003:000009e0       ??_R0?AV?$basic_stringstream@DU?$char_traits@D@std@@V?$allocator@D@2@@std@@@8 00000001400299e0     safe_string_x64:safe_string.obj
 0003:00000a40       ??_R0?AV?$basic_stringbuf@DU?$char_traits@D@std@@V?$allocator@D@2@@std@@@8 0000000140029a40     safe_string_x64:safe_string.obj
 0003:00000a98       ??_R0?AVios_base@std@@@8   0000000140029a98     safe_string_x64:safe_string.obj
 0003:00000ac0       ??_R0?AV?$basic_iostream@DU?$char_traits@D@std@@@std@@@8 0000000140029ac0     safe_string_x64:safe_string.obj
 0003:00000b08       ??_R0?AV?$_Iosb@H@std@@@8  0000000140029b08     safe_string_x64:safe_string.obj
 0003:00000b30       ??_R0?AV?$basic_streambuf@DU?$char_traits@D@std@@@std@@@8 0000000140029b30     safe_string_x64:safe_string.obj
 0003:00000b80       ??_R0?AV?$basic_istream@DU?$char_traits@D@std@@@std@@@8 0000000140029b80     safe_string_x64:safe_string.obj
 0003:00000bc8       ??_R0?AV?$basic_ios@DU?$char_traits@D@std@@@std@@@8 0000000140029bc8     safe_string_x64:safe_string.obj
 0003:00000c10       ??_R0?AV?$basic_ostream@DU?$char_traits@D@std@@@std@@@8 0000000140029c10     safe_string_x64:safe_string.obj
 0003:00000c60       __afxForceEXCLUDE          0000000140029c60     mfcs140:nolib.obj
 0003:00000c64       __afxForceSTDAFX           0000000140029c64     mfcs140:stdafx.obj
 0003:00000cb0       __scrt_current_native_startup_state 0000000140029cb0     msvcrt:utility.obj
 0003:00000cb8       __scrt_native_startup_lock 0000000140029cb8     msvcrt:utility.obj
 0003:00001270       __scrt_debugger_hook_flag  000000014002a270     msvcrt:utility_desktop.obj
 0003:00001274       _tls_index                 000000014002a274     msvcrt:tlssup.obj
 0003:00001278       __favor                    000000014002a278     msvcrt:cpu_disp.obj
 0003:00001280       ?__type_info_root_node@@3U__type_info_node@@A 000000014002a280     msvcrt:tncleanup.obj
 0003:00001290       ?_AtlBaseModule@ATL@@3VCAtlBaseModule@1@A 000000014002a290     atls:atlbase.obj
 0003:000012f0       __@@_PchSym_@00@UztvmgUPdlipUCUhUrmgvinvwrzgvUexgllohUzgohOmzgrevkilqPBACIAJCBDBUlyqiUznwGEUhgwzucOlyq@4B2008FD98C1DD4 000000014002a2f0     atls:stdafx.obj
 0003:000012f4       ?_afxInitAppState@@3DA     000000014002a2f4     mfcs140:appmodul.obj
 0003:000012f8       ?_OptionsStorage@?1??__local_stdio_printf_options@@9@4_KA 000000014002a2f8     BugReporter.obj
 0003:00001300       ?m_szLogMailerFileName@CServerLog@@1PADA 000000014002a300     LogMgmt.obj
 0003:000016e9       ?m_isWriteLog_IPCMemory@CHLogger@@0_NA 000000014002a6e9     HostLogger.obj
 0003:000016ea       ?m_isWriteLog_IPCMsg@CHLogger@@0_NA 000000014002a6ea     HostLogger.obj
 0003:000016eb       ?g_useDialogConsoleOutput@@3_NA 000000014002a6eb     ServerAppDlg.obj
 0003:000016ec       ?m_eLastError@CLogMsgManager@@0W4EERROR_TYPE@1@A 000000014002a6ec     LogMsgManager.obj
 0003:000016f0       ?m_szLogTryWeaponItemFileName@CServerLog@@1PADA 000000014002a6f0     LogMgmt.obj
 0003:00001ae0       ?m_szLogMgrDataFileName@CServerLog@@1PADA 000000014002aae0     LogMgmt.obj
 0003:00001ed0       ?m_szLogKickUserFileName@CServerLog@@1PADA 000000014002aed0     LogMgmt.obj
 0003:000022c0       ?m_szLogServerSettingCheckFileName@CServerLog@@1PADA 000000014002b2c0     LogMgmt.obj
 0003:000026b0       ?m_szLogCriticalErrorPath@CServerLog@@1PADA 000000014002b6b0     LogMgmt.obj
 0003:00002aa0       ?m_szLogInGameClanFileName@CServerLog@@1PADA 000000014002baa0     LogMgmt.obj
 0003:00002e90       ?m_szLogHackingFileName@CServerLog@@1PADA 000000014002be90     LogMgmt.obj
 0003:00003280       ?m_szLogEmergencyStateFileName@CServerLog@@1PADA 000000014002c280     LogMgmt.obj
 0003:00003670       ?m_szLogMonitoringFileName@CServerLog@@1PADA 000000014002c670     LogMgmt.obj
 0003:00003a60       ?m_szLogMegaPhoneFileName@CServerLog@@1PADA 000000014002ca60     LogMgmt.obj
 0003:00003e50       ?m_szLogCountFileName@CServerLog@@1PADA 000000014002ce50     LogMgmt.obj
 0003:00004240       ?m_szLogHackFileName@CServerLog@@1PADA 000000014002d240     LogMgmt.obj
 0003:00004630       ?m_szLogTimeOutFileName@CServerLog@@1PADA 000000014002d630     LogMgmt.obj
 0003:00004a20       ?m_szLogTimeFileName@CServerLog@@1PADA 000000014002da20     LogMgmt.obj
 0003:00004e10       ?m_szLogEtcFileName@CServerLog@@1PADA 000000014002de10     LogMgmt.obj
 0003:00005200       ?m_szLogConnectCheckFileName@CServerLog@@1PADA 000000014002e200     LogMgmt.obj
 0003:000055f0       ?m_szLogGachaFileName@CServerLog@@1PADA 000000014002e5f0     LogMgmt.obj
 0003:000059e0       ?m_szLogUnknownDataFileName@CServerLog@@1PADA 000000014002e9e0     LogMgmt.obj
 0003:00005dd0       ?m_szLogCashFileName@CServerLog@@1PADA 000000014002edd0     LogMgmt.obj
 0003:000061c0       ?m_szLogErrorFileName@CServerLog@@1PADA 000000014002f1c0     LogMgmt.obj
 0003:000065b0       ?m_szLogFolder@CServerLog@@1PADA 000000014002f5b0     LogMgmt.obj
 0003:00006748       ?m_hSizeHandle@CLogMsgManager@@0PEAXEA 000000014002f748     LogMsgManager.obj
 0003:00006750       ?m_szServerName@CServerLog@@1PADA 000000014002f750     LogMgmt.obj
 0003:000067b8       ?m_pXlsLoader@CLogMsgManager@@0PEAVFindXlsMsg@@EA 000000014002f7b8     LogMsgManager.obj
 0003:000067c0       ?m_szHostName@CServerLog@@1PADA 000000014002f7c0     LogMgmt.obj
 0003:00006828       ?g_iQueuedUserInfosNum@@3HC 000000014002f828     ServerAppDlg.obj
 0003:0000682c       ?g_iQueuedGameInfosNum@@3HC 000000014002f82c     ServerAppDlg.obj
 0003:00006830       ?g_csUserInfoQueue@@3U_RTL_CRITICAL_SECTION@@A 000000014002f830     ServerAppDlg.obj
 0003:00006858       ?g_csGameInfoQueue@@3U_RTL_CRITICAL_SECTION@@A 000000014002f858     ServerAppDlg.obj
 0003:00006880       ?g_cs@@3U_RTL_CRITICAL_SECTION@@A 000000014002f880     ServerAppDlg.obj
 0003:000068a8       ?g_pLTSCommon@@3PEAVILTCommon@@EA 000000014002f8a8     ServerAppDlg.obj
 0003:000068b0       ?GAMEGUID@@3TLTGUID@@A     000000014002f8b0     ServerAppDlg.obj
 0003:000068c0       ?g_hServerDll@@3PEAUHINSTANCE__@@EA 000000014002f8c0     ServerAppDlg.obj
 0003:000068c8       ?handler@vars@cf@@2P6AXAEBV?$basic_string@DU?$char_traits@D@std@@V?$allocator@D@2@@std@@0@ZEA 000000014002f8c8     safe_string_x64:safe_string.obj
 0003:00006b70       ?_FILE_SHUTDOWN_var_ltmod_database_@@3V_FILE_SHUTDOWN_class_ltmod_database_@@A 000000014002fb70     ltmodule.obj
 0003:00006be8       ?m_vectSharedMapHandles@CLogMsgManager@@0V?$vector@PEAXV?$allocator@PEAX@std@@@std@@A 000000014002fbe8     LogMsgManager.obj
 0003:00006c10       ?theApp@@3VCServerAppApp@@A 000000014002fc10     ServerApp.obj
 0003:00006d90       ?g_sGameInfos@@3PAUPROTO_START_HOST_tag@@A 000000014002fd90     ServerAppDlg.obj
 0003:00202e90       ?g_sUserInfos@@3PAUPROTO_GAME_USER_INFO_tag@@A 000000014022be90     ServerAppDlg.obj
 0003:00235ef8       ?_OptionsStorage@?1??__local_stdio_scanf_options@@9@4_KA 000000014025eef8     ServerAppDlg.obj
 0003:00235f00       __@@_PchSym_@00@UdlipUhzPeCBAIUxorvmgUlyqUcGEUurmzoUhvievizkkUhgwzucOlyq@4B2008FD98C1DD4 000000014025ef00     StdAfx.obj
 0003:00235f04       ?m_bInitFailed@CAtlBaseModule@ATL@@2_NA 000000014025ef04     StdAfx.obj
 0003:00236048       __dyn_tls_dtor_callback    000000014025f048     <common>
 0003:00236050       __dyn_tls_init_callback    000000014025f050     <common>

 entry point at        0001:000168a8

 Static symbols

 0000:ffd9b000       .debug$S                   0000000140000000     Psapi:PSAPI.DLL
 0000:ffd9b000       .debug$S                   0000000140000000     mfc140:mfc140.dll
 0000:ffd9b000       .debug$S                   0000000140000000     mfc140:mfc140.dll
 0000:ffd9b000       .debug$S                   0000000140000000     mfc140:mfc140.dll
 0000:ffd9b000       .debug$S                   0000000140000000     mfc140:mfc140.dll
 0000:ffd9b000       .debug$S                   0000000140000000     mfc140:mfc140.dll
 0000:ffd9b000       .debug$S                   0000000140000000     ucrt:api-ms-win-crt-math-l1-1-0.dll
 0000:ffd9b000       .debug$S                   0000000140000000     ucrt:api-ms-win-crt-math-l1-1-0.dll
 0000:ffd9b000       .debug$S                   0000000140000000     ucrt:api-ms-win-crt-math-l1-1-0.dll
 0000:ffd9b000       .debug$S                   0000000140000000     vcruntime:VCRUNTIME140.dll
 0000:ffd9b000       .debug$S                   0000000140000000     vcruntime:VCRUNTIME140.dll
 0000:ffd9b000       .debug$S                   0000000140000000     vcruntime:VCRUNTIME140.dll
 0000:ffd9b000       .debug$S                   0000000140000000     vcruntime:VCRUNTIME140.dll
 0000:ffd9b000       .debug$S                   0000000140000000     vcruntime:VCRUNTIME140.dll
 0000:ffd9b000       .debug$S                   0000000140000000     ServerApp_x64.exp
 0000:ffd9b000       .debug$S                   0000000140000000     mfc140:mfc140.dll
 0000:ffd9b000       .debug$S                   0000000140000000     mfc140:mfc140.dll
 0000:ffd9b000       .debug$S                   0000000140000000     mfc140:mfc140.dll
 0000:ffd9b000       .debug$S                   0000000140000000     mfc140:mfc140.dll
 0000:ffd9b000       .debug$S                   0000000140000000     ucrt:api-ms-win-crt-locale-l1-1-0.dll
 0000:ffd9b000       .debug$S                   0000000140000000     msvcprt:MSVCP140.dll
 0000:ffd9b000       .debug$S                   0000000140000000     msvcprt:MSVCP140.dll
 0000:ffd9b000       .debug$S                   0000000140000000     msvcprt:MSVCP140.dll
 0000:ffd9b000       .debug$S                   0000000140000000     msvcprt:MSVCP140.dll
 0000:ffd9b000       .debug$S                   0000000140000000     msvcprt:MSVCP140.dll
 0000:ffd9b000       .debug$S                   0000000140000000     msvcprt:MSVCP140.dll
 0000:ffd9b000       .debug$S                   0000000140000000     msvcprt:MSVCP140.dll
 0000:ffd9b000       .debug$S                   0000000140000000     msvcprt:MSVCP140.dll
 0000:ffd9b000       .debug$S                   0000000140000000     msvcprt:MSVCP140.dll
 0000:ffd9b000       .debug$S                   0000000140000000     msvcprt:MSVCP140.dll
 0000:ffd9b000       .debug$S                   0000000140000000     msvcprt:MSVCP140.dll
 0000:ffd9b000       .debug$S                   0000000140000000     msvcprt:MSVCP140.dll
 0000:ffd9b000       .debug$S                   0000000140000000     msvcprt:MSVCP140.dll
 0000:ffd9b000       .debug$S                   0000000140000000     msvcprt:MSVCP140.dll
 0000:ffd9b000       .debug$S                   0000000140000000     msvcprt:MSVCP140.dll
 0000:ffd9b000       .debug$S                   0000000140000000     msvcprt:MSVCP140.dll
 0000:ffd9b000       .debug$S                   0000000140000000     msvcprt:MSVCP140.dll
 0000:ffd9b000       .debug$S                   0000000140000000     msvcprt:MSVCP140.dll
 0000:ffd9b000       .debug$S                   0000000140000000     msvcprt:MSVCP140.dll
 0000:ffd9b000       .debug$S                   0000000140000000     msvcprt:MSVCP140.dll
 0000:ffd9b000       .debug$S                   0000000140000000     msvcprt:MSVCP140.dll
 0000:ffd9b000       .debug$S                   0000000140000000     msvcprt:MSVCP140.dll
 0000:ffd9b000       .debug$S                   0000000140000000     msvcprt:MSVCP140.dll
 0000:ffd9b000       .debug$S                   0000000140000000     msvcprt:MSVCP140.dll
 0000:ffd9b000       .debug$S                   0000000140000000     msvcprt:MSVCP140.dll
 0000:ffd9b000       .debug$S                   0000000140000000     msvcprt:MSVCP140.dll
 0000:ffd9b000       .debug$S                   0000000140000000     msvcprt:MSVCP140.dll
 0000:ffd9b000       .debug$S                   0000000140000000     msvcprt:MSVCP140.dll
 0000:ffd9b000       .debug$S                   0000000140000000     msvcprt:MSVCP140.dll
 0000:ffd9b000       .debug$S                   0000000140000000     msvcprt:MSVCP140.dll
 0000:ffd9b000       .debug$S                   0000000140000000     msvcprt:MSVCP140.dll
 0000:ffd9b000       .debug$S                   0000000140000000     msvcprt:MSVCP140.dll
 0000:ffd9b000       .debug$S                   0000000140000000     msvcprt:MSVCP140.dll
 0000:ffd9b000       .debug$S                   0000000140000000     msvcprt:MSVCP140.dll
 0000:ffd9b000       .debug$S                   0000000140000000     msvcprt:MSVCP140.dll
 0000:ffd9b000       .debug$S                   0000000140000000     msvcprt:MSVCP140.dll
 0000:ffd9b000       .debug$S                   0000000140000000     msvcprt:MSVCP140.dll
 0000:ffd9b000       .debug$S                   0000000140000000     msvcprt:MSVCP140.dll
 0000:ffd9b000       .debug$S                   0000000140000000     msvcprt:MSVCP140.dll
 0000:ffd9b000       .debug$S                   0000000140000000     msvcprt:MSVCP140.dll
 0000:ffd9b000       .debug$S                   0000000140000000     msvcprt:MSVCP140.dll
 0000:ffd9b000       .debug$S                   0000000140000000     msvcprt:MSVCP140.dll
 0000:ffd9b000       .debug$S                   0000000140000000     msvcprt:MSVCP140.dll
 0000:ffd9b000       .debug$S                   0000000140000000     msvcprt:MSVCP140.dll
 0000:ffd9b000       .debug$S                   0000000140000000     kernel32:KERNEL32.dll
 0000:ffd9b000       .debug$S                   0000000140000000     mfc140:mfc140.dll
 0000:ffd9b000       .debug$S                   0000000140000000     ucrt:api-ms-win-crt-string-l1-1-0.dll
 0000:ffd9b000       .debug$S                   0000000140000000     mfc140:mfc140.dll
 0000:ffd9b000       .debug$S                   0000000140000000     mfc140:mfc140.dll
 0000:ffd9b000       .debug$S                   0000000140000000     ucrt:api-ms-win-crt-stdio-l1-1-0.dll
 0000:ffd9b000       .debug$S                   0000000140000000     mfc140:mfc140.dll
 0000:ffd9b000       .debug$S                   0000000140000000     mfc140:mfc140.dll
 0000:ffd9b000       .debug$S                   0000000140000000     mfc140:mfc140.dll
 0000:ffd9b000       .debug$S                   0000000140000000     ucrt:api-ms-win-crt-string-l1-1-0.dll
 0000:ffd9b000       .debug$S                   0000000140000000     mfc140:mfc140.dll
 0000:ffd9b000       .debug$S                   0000000140000000     mfc140:mfc140.dll
 0000:ffd9b000       .debug$S                   0000000140000000     ucrt:api-ms-win-crt-heap-l1-1-0.dll
 0000:ffd9b000       .debug$S                   0000000140000000     mfc140:mfc140.dll
 0000:ffd9b000       .debug$S                   0000000140000000     mfc140:mfc140.dll
 0000:ffd9b000       .debug$S                   0000000140000000     mfc140:mfc140.dll
 0000:ffd9b000       .debug$S                   0000000140000000     ucrt:api-ms-win-crt-runtime-l1-1-0.dll
 0000:ffd9b000       .debug$S                   0000000140000000     mfc140:mfc140.dll
 0000:ffd9b000       .debug$S                   0000000140000000     mfc140:mfc140.dll
 0000:ffd9b000       .debug$S                   0000000140000000     ucrt:api-ms-win-crt-stdio-l1-1-0.dll
 0000:ffd9b000       .debug$S                   0000000140000000     mfc140:mfc140.dll
 0000:ffd9b000       .debug$S                   0000000140000000     mfc140:mfc140.dll
 0000:ffd9b000       .debug$S                   0000000140000000     mfc140:mfc140.dll
 0000:ffd9b000       .debug$S                   0000000140000000     mfc140:mfc140.dll
 0000:ffd9b000       .debug$S                   0000000140000000     mfc140:mfc140.dll
 0000:ffd9b000       .debug$S                   0000000140000000     mfc140:mfc140.dll
 0000:ffd9b000       .debug$S                   0000000140000000     mfc140:mfc140.dll
 0000:ffd9b000       .debug$S                   0000000140000000     ucrt:api-ms-win-crt-heap-l1-1-0.dll
 0000:ffd9b000       .debug$S                   0000000140000000     mfc140:mfc140.dll
 0000:ffd9b000       .debug$S                   0000000140000000     mfc140:mfc140.dll
 0000:ffd9b000       .debug$S                   0000000140000000     ucrt:api-ms-win-crt-locale-l1-1-0.dll
 0000:ffd9b000       .debug$S                   0000000140000000     mfc140:mfc140.dll
 0000:ffd9b000       .debug$S                   0000000140000000     mfc140:mfc140.dll
 0000:ffd9b000       .debug$S                   0000000140000000     mfc140:mfc140.dll
 0000:ffd9b000       .debug$S                   0000000140000000     mfc140:mfc140.dll
 0000:ffd9b000       .debug$S                   0000000140000000     mfc140:mfc140.dll
 0000:ffd9b000       .debug$S                   0000000140000000     mfc140:mfc140.dll
 0000:ffd9b000       .debug$S                   0000000140000000     mfc140:mfc140.dll
 0000:ffd9b000       .debug$S                   0000000140000000     mfc140:mfc140.dll
 0000:ffd9b000       .debug$S                   0000000140000000     mfc140:mfc140.dll
 0000:ffd9b000       .debug$S                   0000000140000000     mfc140:mfc140.dll
 0000:ffd9b000       .debug$S                   0000000140000000     mfc140:mfc140.dll
 0000:ffd9b000       .debug$S                   0000000140000000     mfc140:mfc140.dll
 0000:ffd9b000       .debug$S                   0000000140000000     mfc140:mfc140.dll
 0000:ffd9b000       .debug$S                   0000000140000000     mfc140:mfc140.dll
 0000:ffd9b000       .debug$S                   0000000140000000     mfc140:mfc140.dll
 0000:ffd9b000       .debug$S                   0000000140000000     mfc140:mfc140.dll
 0000:ffd9b000       .debug$S                   0000000140000000     ucrt:api-ms-win-crt-runtime-l1-1-0.dll
 0000:ffd9b000       .debug$S                   0000000140000000     mfc140:mfc140.dll
 0000:ffd9b000       .debug$S                   0000000140000000     mfc140:mfc140.dll
 0000:ffd9b000       .debug$S                   0000000140000000     mfc140:mfc140.dll
 0000:ffd9b000       .debug$S                   0000000140000000     ucrt:api-ms-win-crt-runtime-l1-1-0.dll
 0000:ffd9b000       .debug$S                   0000000140000000     mfc140:mfc140.dll
 0000:ffd9b000       .debug$S                   0000000140000000     mfc140:mfc140.dll
 0000:ffd9b000       .debug$S                   0000000140000000     mfc140:mfc140.dll
 0000:ffd9b000       .debug$S                   0000000140000000     mfc140:mfc140.dll
 0000:ffd9b000       .debug$S                   0000000140000000     mfc140:mfc140.dll
 0000:ffd9b000       .debug$S                   0000000140000000     mfc140:mfc140.dll
 0000:ffd9b000       .debug$S                   0000000140000000     mfc140:mfc140.dll
 0000:ffd9b000       .debug$S                   0000000140000000     mfc140:mfc140.dll
 0000:ffd9b000       .debug$S                   0000000140000000     ucrt:api-ms-win-crt-stdio-l1-1-0.dll
 0000:ffd9b000       .debug$S                   0000000140000000     mfc140:mfc140.dll
 0000:ffd9b000       .debug$S                   0000000140000000     mfc140:mfc140.dll
 0000:ffd9b000       .debug$S                   0000000140000000     mfc140:mfc140.dll
 0000:ffd9b000       .debug$S                   0000000140000000     mfc140:mfc140.dll
 0000:ffd9b000       .debug$S                   0000000140000000     ucrt:api-ms-win-crt-runtime-l1-1-0.dll
 0000:ffd9b000       .debug$S                   0000000140000000     ucrt:api-ms-win-crt-runtime-l1-1-0.dll
 0000:ffd9b000       .debug$S                   0000000140000000     ucrt:api-ms-win-crt-runtime-l1-1-0.dll
 0000:ffd9b000       .debug$S                   0000000140000000     ucrt:api-ms-win-crt-runtime-l1-1-0.dll
 0000:ffd9b000       .debug$S                   0000000140000000     ucrt:api-ms-win-crt-runtime-l1-1-0.dll
 0000:ffd9b000       .debug$S                   0000000140000000     ucrt:api-ms-win-crt-math-l1-1-0.dll
 0000:ffd9b000       .debug$S                   0000000140000000     ucrt:api-ms-win-crt-runtime-l1-1-0.dll
 0000:ffd9b000       .debug$S                   0000000140000000     ucrt:api-ms-win-crt-runtime-l1-1-0.dll
 0000:ffd9b000       .debug$S                   0000000140000000     ucrt:api-ms-win-crt-runtime-l1-1-0.dll
 0000:ffd9b000       .debug$S                   0000000140000000     ucrt:api-ms-win-crt-runtime-l1-1-0.dll
 0000:ffd9b000       .debug$S                   0000000140000000     ucrt:api-ms-win-crt-runtime-l1-1-0.dll
 0000:ffd9b000       .debug$S                   0000000140000000     ucrt:api-ms-win-crt-runtime-l1-1-0.dll
 0000:ffd9b000       .debug$S                   0000000140000000     ucrt:api-ms-win-crt-runtime-l1-1-0.dll
 0000:ffd9b000       .debug$S                   0000000140000000     ucrt:api-ms-win-crt-runtime-l1-1-0.dll
 0000:ffd9b000       .debug$S                   0000000140000000     ucrt:api-ms-win-crt-runtime-l1-1-0.dll
 0000:ffd9b000       .debug$S                   0000000140000000     ucrt:api-ms-win-crt-runtime-l1-1-0.dll
 0000:ffd9b000       .debug$S                   0000000140000000     ucrt:api-ms-win-crt-runtime-l1-1-0.dll
 0000:ffd9b000       .debug$S                   0000000140000000     ucrt:api-ms-win-crt-heap-l1-1-0.dll
 0000:ffd9b000       .debug$S                   0000000140000000     mfc140:mfc140.dll
 0000:ffd9b000       .debug$S                   0000000140000000     mfc140:mfc140.dll
 0000:ffd9b000       .debug$S                   0000000140000000     mfc140:mfc140.dll
 0000:ffd9b000       .debug$S                   0000000140000000     mfc140:mfc140.dll
 0000:ffd9b000       .debug$S                   0000000140000000     mfc140:mfc140.dll
 0000:ffd9b000       .debug$S                   0000000140000000     mfc140:mfc140.dll
 0000:ffd9b000       .debug$S                   0000000140000000     mfc140:mfc140.dll
 0000:ffd9b000       .debug$S                   0000000140000000     mfc140:mfc140.dll
 0000:ffd9b000       .debug$S                   0000000140000000     mfc140:mfc140.dll
 0000:ffd9b000       .debug$S                   0000000140000000     mfc140:mfc140.dll
 0000:ffd9b000       .debug$S                   0000000140000000     mfc140:mfc140.dll
 0000:ffd9b000       .debug$S                   0000000140000000     mfc140:mfc140.dll
 0000:ffd9b000       .debug$S                   0000000140000000     mfc140:mfc140.dll
 0000:ffd9b000       .debug$S                   0000000140000000     mfc140:mfc140.dll
 0000:ffd9b000       .debug$S                   0000000140000000     mfc140:mfc140.dll
 0000:ffd9b000       .debug$S                   0000000140000000     mfc140:mfc140.dll
 0000:ffd9b000       .debug$S                   0000000140000000     mfc140:mfc140.dll
 0000:ffd9b000       .debug$S                   0000000140000000     mfc140:mfc140.dll
 0000:ffd9b000       .debug$S                   0000000140000000     mfc140:mfc140.dll
 0000:ffd9b000       .debug$S                   0000000140000000     mfc140:mfc140.dll
 0000:ffd9b000       .debug$S                   0000000140000000     mfc140:mfc140.dll
 0000:ffd9b000       .debug$S                   0000000140000000     mfc140:mfc140.dll
 0000:ffd9b000       .debug$S                   0000000140000000     mfc140:mfc140.dll
 0000:ffd9b000       .debug$S                   0000000140000000     mfc140:mfc140.dll
 0000:ffd9b000       .debug$S                   0000000140000000     mfc140:mfc140.dll
 0000:ffd9b000       .debug$S                   0000000140000000     mfc140:mfc140.dll
 0000:ffd9b000       .debug$S                   0000000140000000     mfc140:mfc140.dll
 0000:ffd9b000       .debug$S                   0000000140000000     ucrt:api-ms-win-crt-filesystem-l1-1-0.dll
 0000:ffd9b000       .debug$S                   0000000140000000     mfc140:mfc140.dll
 0000:ffd9b000       .debug$S                   0000000140000000     mfc140:mfc140.dll
 0000:ffd9b000       .debug$S                   0000000140000000     mfc140:mfc140.dll
 0000:ffd9b000       .debug$S                   0000000140000000     mfc140:mfc140.dll
 0000:ffd9b000       .debug$S                   0000000140000000     ucrt:api-ms-win-crt-filesystem-l1-1-0.dll
 0000:ffd9b000       .debug$S                   0000000140000000     mfc140:mfc140.dll
 0000:ffd9b000       .debug$S                   0000000140000000     mfc140:mfc140.dll
 0000:ffd9b000       .debug$S                   0000000140000000     mfc140:mfc140.dll
 0000:ffd9b000       .debug$S                   0000000140000000     mfc140:mfc140.dll
 0000:ffd9b000       .debug$S                   0000000140000000     mfc140:mfc140.dll
 0000:ffd9b000       .debug$S                   0000000140000000     mfc140:mfc140.dll
 0000:ffd9b000       .debug$S                   0000000140000000     mfc140:mfc140.dll
 0000:ffd9b000       .debug$S                   0000000140000000     mfc140:mfc140.dll
 0000:ffd9b000       .debug$S                   0000000140000000     ucrt:api-ms-win-crt-stdio-l1-1-0.dll
 0000:ffd9b000       .debug$S                   0000000140000000     mfc140:mfc140.dll
 0000:ffd9b000       .debug$S                   0000000140000000     mfc140:mfc140.dll
 0000:ffd9b000       .debug$S                   0000000140000000     mfc140:mfc140.dll
 0000:ffd9b000       .debug$S                   0000000140000000     mfc140:mfc140.dll
 0000:ffd9b000       .debug$S                   0000000140000000     mfc140:mfc140.dll
 0000:ffd9b000       .debug$S                   0000000140000000     mfc140:mfc140.dll
 0000:ffd9b000       .debug$S                   0000000140000000     mfc140:mfc140.dll
 0000:ffd9b000       .debug$S                   0000000140000000     mfc140:mfc140.dll
 0000:ffd9b000       .debug$S                   0000000140000000     mfc140:mfc140.dll
 0000:ffd9b000       .debug$S                   0000000140000000     mfc140:mfc140.dll
 0000:ffd9b000       .debug$S                   0000000140000000     mfc140:mfc140.dll
 0000:ffd9b000       .debug$S                   0000000140000000     mfc140:mfc140.dll
 0000:ffd9b000       .debug$S                   0000000140000000     mfc140:mfc140.dll
 0000:ffd9b000       .debug$S                   0000000140000000     mfc140:mfc140.dll
 0000:ffd9b000       .debug$S                   0000000140000000     mfc140:mfc140.dll
 0000:ffd9b000       .debug$S                   0000000140000000     mfc140:mfc140.dll
 0000:ffd9b000       .debug$S                   0000000140000000     mfc140:mfc140.dll
 0000:ffd9b000       .debug$S                   0000000140000000     mfc140:mfc140.dll
 0000:ffd9b000       .debug$S                   0000000140000000     mfc140:mfc140.dll
 0000:ffd9b000       .debug$S                   0000000140000000     mfc140:mfc140.dll
 0000:ffd9b000       .debug$S                   0000000140000000     mfc140:mfc140.dll
 0000:ffd9b000       .debug$S                   0000000140000000     mfc140:mfc140.dll
 0000:ffd9b000       .debug$S                   0000000140000000     ucrt:api-ms-win-crt-runtime-l1-1-0.dll
 0000:ffd9b000       .debug$S                   0000000140000000     ucrt:api-ms-win-crt-runtime-l1-1-0.dll
 0000:ffd9b000       .debug$S                   0000000140000000     ucrt:api-ms-win-crt-convert-l1-1-0.dll
 0000:ffd9b000       .debug$S                   0000000140000000     ucrt:api-ms-win-crt-convert-l1-1-0.dll
 0000:ffd9b000       .debug$S                   0000000140000000     ucrt:api-ms-win-crt-runtime-l1-1-0.dll
 0000:ffd9b000       .debug$S                   0000000140000000     ucrt:api-ms-win-crt-convert-l1-1-0.dll
 0000:ffd9b000       .debug$S                   0000000140000000     ucrt:api-ms-win-crt-runtime-l1-1-0.dll
 0000:ffd9b000       .debug$S                   0000000140000000     ucrt:api-ms-win-crt-time-l1-1-0.dll
 0000:ffd9b000       .debug$S                   0000000140000000     ucrt:api-ms-win-crt-utility-l1-1-0.dll
 0000:ffd9b000       .debug$S                   0000000140000000     ucrt:api-ms-win-crt-runtime-l1-1-0.dll
 0000:ffd9b000       .debug$S                   0000000140000000     ucrt:api-ms-win-crt-runtime-l1-1-0.dll
 0000:ffd9b000       .debug$S                   0000000140000000     ucrt:api-ms-win-crt-stdio-l1-1-0.dll
 0000:ffd9b000       .debug$S                   0000000140000000     ucrt:api-ms-win-crt-stdio-l1-1-0.dll
 0000:ffd9b000       .debug$S                   0000000140000000     mfc140:mfc140.dll
 0000:ffd9b000       .debug$S                   0000000140000000     mfc140:mfc140.dll
 0000:ffd9b000       .debug$S                   0000000140000000     ucrt:api-ms-win-crt-string-l1-1-0.dll
 0000:ffd9b000       .debug$S                   0000000140000000     mfc140:mfc140.dll
 0000:ffd9b000       .debug$S                   0000000140000000     mfc140:mfc140.dll
 0000:ffd9b000       .debug$S                   0000000140000000     mfc140:mfc140.dll
 0000:ffd9b000       .debug$S                   0000000140000000     mfc140:mfc140.dll
 0000:ffd9b000       .debug$S                   0000000140000000     ucrt:api-ms-win-crt-stdio-l1-1-0.dll
 0000:ffd9b000       .debug$S                   0000000140000000     mfc140:mfc140.dll
 0000:ffd9b000       .debug$S                   0000000140000000     mfc140:mfc140.dll
 0000:ffd9b000       .debug$S                   0000000140000000     mfc140:mfc140.dll
 0000:ffd9b000       .debug$S                   0000000140000000     mfc140:mfc140.dll
 0000:ffd9b000       .debug$S                   0000000140000000     mfc140:mfc140.dll
 0000:ffd9b000       .debug$S                   0000000140000000     mfc140:mfc140.dll
 0000:ffd9b000       .debug$S                   0000000140000000     mfc140:mfc140.dll
 0000:ffd9b000       .debug$S                   0000000140000000     mfc140:mfc140.dll
 0000:ffd9b000       .debug$S                   0000000140000000     ucrt:api-ms-win-crt-stdio-l1-1-0.dll
 0000:ffd9b000       .debug$S                   0000000140000000     mfc140:mfc140.dll
 0000:ffd9b000       .debug$S                   0000000140000000     mfc140:mfc140.dll
 0000:ffd9b000       .debug$S                   0000000140000000     mfc140:mfc140.dll
 0000:ffd9b000       .debug$S                   0000000140000000     mfc140:mfc140.dll
 0000:ffd9b000       .debug$S                   0000000140000000     mfc140:mfc140.dll
 0000:ffd9b000       .debug$S                   0000000140000000     mfc140:mfc140.dll
 0000:ffd9b000       .debug$S                   0000000140000000     ucrt:api-ms-win-crt-stdio-l1-1-0.dll
 0000:ffd9b000       .debug$S                   0000000140000000     mfc140:mfc140.dll
 0000:ffd9b000       .debug$S                   0000000140000000     mfc140:mfc140.dll
 0000:ffd9b000       .debug$S                   0000000140000000     mfc140:mfc140.dll
 0000:ffd9b000       .debug$S                   0000000140000000     mfc140:mfc140.dll
 0000:ffd9b000       .debug$S                   0000000140000000     ucrt:api-ms-win-crt-stdio-l1-1-0.dll
 0000:ffd9b000       .debug$S                   0000000140000000     mfc140:mfc140.dll
 0000:ffd9b000       .debug$S                   0000000140000000     mfc140:mfc140.dll
 0000:ffd9b000       .debug$S                   0000000140000000     mfc140:mfc140.dll
 0000:ffd9b000       .debug$S                   0000000140000000     mfc140:mfc140.dll
 0000:ffd9b000       .debug$S                   0000000140000000     mfc140:mfc140.dll
 0000:ffd9b000       .debug$S                   0000000140000000     mfc140:mfc140.dll
 0000:ffd9b000       .debug$S                   0000000140000000     mfc140:mfc140.dll
 0000:ffd9b000       .debug$S                   0000000140000000     mfc140:mfc140.dll
 0000:ffd9b000       .debug$S                   0000000140000000     mfc140:mfc140.dll
 0000:ffd9b000       .debug$S                   0000000140000000     mfc140:mfc140.dll
 0000:ffd9b000       .debug$S                   0000000140000000     mfc140:mfc140.dll
 0000:ffd9b000       .debug$S                   0000000140000000     mfc140:mfc140.dll
 0000:ffd9b000       .debug$S                   0000000140000000     mfc140:mfc140.dll
 0000:ffd9b000       .debug$S                   0000000140000000     mfc140:mfc140.dll
 0000:ffd9b000       .debug$S                   0000000140000000     mfc140:mfc140.dll
 0000:ffd9b000       .debug$S                   0000000140000000     mfc140:mfc140.dll
 0000:ffd9b000       .debug$S                   0000000140000000     mfc140:mfc140.dll
 0000:ffd9b000       .debug$S                   0000000140000000     mfc140:mfc140.dll
 0000:ffd9b000       .debug$S                   0000000140000000     mfc140:mfc140.dll
 0000:ffd9b000       .debug$S                   0000000140000000     mfc140:mfc140.dll
 0000:ffd9b000       .debug$S                   0000000140000000     mfc140:mfc140.dll
 0000:ffd9b000       .debug$S                   0000000140000000     mfc140:mfc140.dll
 0000:ffd9b000       .debug$S                   0000000140000000     mfc140:mfc140.dll
 0000:ffd9b000       .debug$S                   0000000140000000     mfc140:mfc140.dll
 0000:ffd9b000       .debug$S                   0000000140000000     ucrt:api-ms-win-crt-stdio-l1-1-0.dll
 0000:ffd9b000       .debug$S                   0000000140000000     mfc140:mfc140.dll
 0000:ffd9b000       .debug$S                   0000000140000000     mfc140:mfc140.dll
 0000:ffd9b000       .debug$S                   0000000140000000     mfc140:mfc140.dll
 0000:ffd9b000       .debug$S                   0000000140000000     mfc140:mfc140.dll
 0000:ffd9b000       .debug$S                   0000000140000000     ucrt:api-ms-win-crt-stdio-l1-1-0.dll
 0000:ffd9b000       .debug$S                   0000000140000000     mfc140:mfc140.dll
 0000:ffd9b000       .debug$S                   0000000140000000     mfc140:mfc140.dll
 0000:ffd9b000       .debug$S                   0000000140000000     mfc140:mfc140.dll
 0000:ffd9b000       .debug$S                   0000000140000000     mfc140:mfc140.dll
 0000:ffd9b000       .debug$S                   0000000140000000     ucrt:api-ms-win-crt-string-l1-1-0.dll
 0000:ffd9b000       .debug$S                   0000000140000000     mfc140:mfc140.dll
 0000:ffd9b000       .debug$S                   0000000140000000     mfc140:mfc140.dll
 0000:ffd9b000       .debug$S                   0000000140000000     mfc140:mfc140.dll
 0000:ffd9b000       .debug$S                   0000000140000000     ucrt:api-ms-win-crt-convert-l1-1-0.dll
 0000:ffd9b000       .debug$S                   0000000140000000     mfc140:mfc140.dll
 0000:ffd9b000       .debug$S                   0000000140000000     mfc140:mfc140.dll
 0000:ffd9b000       .debug$S                   0000000140000000     ucrt:api-ms-win-crt-stdio-l1-1-0.dll
 0000:ffd9b000       .debug$S                   0000000140000000     mfc140:mfc140.dll
 0000:ffd9b000       .debug$S                   0000000140000000     mfc140:mfc140.dll
 0000:ffd9b000       .debug$S                   0000000140000000     mfc140:mfc140.dll
 0000:ffd9b000       .debug$S                   0000000140000000     mfc140:mfc140.dll
 0000:ffd9b000       .debug$S                   0000000140000000     ucrt:api-ms-win-crt-string-l1-1-0.dll
 0000:ffd9b000       .debug$S                   0000000140000000     mfc140:mfc140.dll
 0000:ffd9b000       .debug$S                   0000000140000000     mfc140:mfc140.dll
 0000:ffd9b000       .debug$S                   0000000140000000     mfc140:mfc140.dll
 0000:ffd9b000       .debug$S                   0000000140000000     mfc140:mfc140.dll
 0000:ffd9b000       .debug$S                   0000000140000000     ucrt:api-ms-win-crt-runtime-l1-1-0.dll
 0000:ffd9b000       .debug$S                   0000000140000000     mfc140:mfc140.dll
 0000:ffd9b000       .debug$S                   0000000140000000     mfc140:mfc140.dll
 0000:ffd9b000       .debug$S                   0000000140000000     mfc140:mfc140.dll
 0000:ffd9b000       .debug$S                   0000000140000000     mfc140:mfc140.dll
 0000:ffd9b000       .debug$S                   0000000140000000     ucrt:api-ms-win-crt-filesystem-l1-1-0.dll
 0000:ffd9b000       .debug$S                   0000000140000000     mfc140:mfc140.dll
 0000:ffd9b000       .debug$S                   0000000140000000     mfc140:mfc140.dll
 0000:ffd9b000       .debug$S                   0000000140000000     mfc140:mfc140.dll
 0000:ffd9b000       .debug$S                   0000000140000000     mfc140:mfc140.dll
 0000:ffd9b000       .debug$S                   0000000140000000     ucrt:api-ms-win-crt-string-l1-1-0.dll
 0000:ffd9b000       .debug$S                   0000000140000000     mfc140:mfc140.dll
 0000:ffd9b000       .debug$S                   0000000140000000     ucrt:api-ms-win-crt-filesystem-l1-1-0.dll
 0000:ffd9b000       .debug$S                   0000000140000000     ucrt:api-ms-win-crt-runtime-l1-1-0.dll
 0000:ffd9b000       .debug$S                   0000000140000000     ucrt:api-ms-win-crt-stdio-l1-1-0.dll
 0000:ffd9b000       .debug$S                   0000000140000000     vcruntime:VCRUNTIME140.dll
 0000:ffd9b000       .debug$S                   0000000140000000     vcruntime:VCRUNTIME140.dll
 0000:ffd9b000       .debug$S                   0000000140000000     vcruntime:VCRUNTIME140.dll
 0000:ffd9b000       .debug$S                   0000000140000000     vcruntime:VCRUNTIME140.dll
 0000:ffd9b000       .debug$S                   0000000140000000     vcruntime:VCRUNTIME140.dll
 0000:ffd9b000       .debug$S                   0000000140000000     vcruntime:VCRUNTIME140.dll
 0000:ffd9b000       .debug$S                   0000000140000000     vcruntime:VCRUNTIME140.dll
 0000:ffd9b000       .debug$S                   0000000140000000     vcruntime:VCRUNTIME140.dll
 0000:ffd9b000       .debug$S                   0000000140000000     vcruntime:VCRUNTIME140.dll
 0000:ffd9b000       .debug$S                   0000000140000000     vcruntime:VCRUNTIME140.dll
 0000:ffd9b000       .debug$S                   0000000140000000     vcruntime:VCRUNTIME140.dll
 0000:ffd9b000       .debug$S                   0000000140000000     ws2_32:WS2_32.dll
 0000:ffd9b000       .debug$S                   0000000140000000     ws2_32:WS2_32.dll
 0000:ffd9b000       .debug$S                   0000000140000000     ws2_32:WS2_32.dll
 0000:ffd9b000       .debug$S                   0000000140000000     winhttp:WINHTTP.dll
 0000:ffd9b000       .debug$S                   0000000140000000     winhttp:WINHTTP.dll
 0000:ffd9b000       .debug$S                   0000000140000000     winhttp:WINHTTP.dll
 0000:ffd9b000       .debug$S                   0000000140000000     winhttp:WINHTTP.dll
 0000:ffd9b000       .debug$S                   0000000140000000     winhttp:WINHTTP.dll
 0000:ffd9b000       .debug$S                   0000000140000000     kernel32:KERNEL32.dll
 0000:ffd9b000       .debug$S                   0000000140000000     winhttp:WINHTTP.dll
 0000:ffd9b000       .debug$S                   0000000140000000     kernel32:KERNEL32.dll
 0000:ffd9b000       .debug$S                   0000000140000000     kernel32:KERNEL32.dll
 0000:ffd9b000       .debug$S                   0000000140000000     kernel32:KERNEL32.dll
 0000:ffd9b000       .debug$S                   0000000140000000     kernel32:KERNEL32.dll
 0000:ffd9b000       .debug$S                   0000000140000000     winhttp:WINHTTP.dll
 0000:ffd9b000       .debug$S                   0000000140000000     kernel32:KERNEL32.dll
 0000:ffd9b000       .debug$S                   0000000140000000     kernel32:KERNEL32.dll
 0000:ffd9b000       .debug$S                   0000000140000000     kernel32:KERNEL32.dll
 0000:ffd9b000       .debug$S                   0000000140000000     kernel32:KERNEL32.dll
 0000:ffd9b000       .debug$S                   0000000140000000     kernel32:KERNEL32.dll
 0000:ffd9b000       .debug$S                   0000000140000000     kernel32:KERNEL32.dll
 0000:ffd9b000       .debug$S                   0000000140000000     winhttp:WINHTTP.dll
 0000:ffd9b000       .debug$S                   0000000140000000     kernel32:KERNEL32.dll
 0000:ffd9b000       .debug$S                   0000000140000000     kernel32:KERNEL32.dll
 0000:ffd9b000       .debug$S                   0000000140000000     kernel32:KERNEL32.dll
 0000:ffd9b000       .debug$S                   0000000140000000     kernel32:KERNEL32.dll
 0000:ffd9b000       .debug$S                   0000000140000000     winhttp:WINHTTP.dll
 0000:ffd9b000       .debug$S                   0000000140000000     kernel32:KERNEL32.dll
 0000:ffd9b000       .debug$S                   0000000140000000     kernel32:KERNEL32.dll
 0000:ffd9b000       .debug$S                   0000000140000000     kernel32:KERNEL32.dll
 0000:ffd9b000       .debug$S                   0000000140000000     kernel32:KERNEL32.dll
 0000:ffd9b000       .debug$S                   0000000140000000     winmm:WINMM.dll
 0000:ffd9b000       .debug$S                   0000000140000000     kernel32:KERNEL32.dll
 0000:ffd9b000       .debug$S                   0000000140000000     kernel32:KERNEL32.dll
 0000:ffd9b000       .debug$S                   0000000140000000     kernel32:KERNEL32.dll
 0000:ffd9b000       .debug$S                   0000000140000000     kernel32:KERNEL32.dll
 0000:ffd9b000       .debug$S                   0000000140000000     kernel32:KERNEL32.dll
 0000:ffd9b000       .debug$S                   0000000140000000     kernel32:KERNEL32.dll
 0000:ffd9b000       .debug$S                   0000000140000000     DbgHelp:dbghelp.dll
 0000:ffd9b000       .debug$S                   0000000140000000     kernel32:KERNEL32.dll
 0000:ffd9b000       .debug$S                   0000000140000000     kernel32:KERNEL32.dll
 0000:ffd9b000       .debug$S                   0000000140000000     kernel32:KERNEL32.dll
 0000:ffd9b000       .debug$S                   0000000140000000     kernel32:KERNEL32.dll
 0000:ffd9b000       .debug$S                   0000000140000000     DbgHelp:dbghelp.dll
 0000:ffd9b000       .debug$S                   0000000140000000     kernel32:KERNEL32.dll
 0000:ffd9b000       .debug$S                   0000000140000000     kernel32:KERNEL32.dll
 0000:ffd9b000       .debug$S                   0000000140000000     kernel32:KERNEL32.dll
 0000:ffd9b000       .debug$S                   0000000140000000     kernel32:KERNEL32.dll
 0000:ffd9b000       .debug$S                   0000000140000000     DbgHelp:dbghelp.dll
 0000:ffd9b000       .debug$S                   0000000140000000     kernel32:KERNEL32.dll
 0000:ffd9b000       .debug$S                   0000000140000000     kernel32:KERNEL32.dll
 0000:ffd9b000       .debug$S                   0000000140000000     kernel32:KERNEL32.dll
 0000:ffd9b000       .debug$S                   0000000140000000     kernel32:KERNEL32.dll
 0000:ffd9b000       .debug$S                   0000000140000000     DbgHelp:dbghelp.dll
 0000:ffd9b000       .debug$S                   0000000140000000     kernel32:KERNEL32.dll
 0000:ffd9b000       .debug$S                   0000000140000000     kernel32:KERNEL32.dll
 0000:ffd9b000       .debug$S                   0000000140000000     kernel32:KERNEL32.dll
 0000:ffd9b000       .debug$S                   0000000140000000     kernel32:KERNEL32.dll
 0000:ffd9b000       .debug$S                   0000000140000000     DbgHelp:dbghelp.dll
 0000:ffd9b000       .debug$S                   0000000140000000     kernel32:KERNEL32.dll
 0000:ffd9b000       .debug$S                   0000000140000000     kernel32:KERNEL32.dll
 0000:ffd9b000       .debug$S                   0000000140000000     kernel32:KERNEL32.dll
 0000:ffd9b000       .debug$S                   0000000140000000     DbgHelp:dbghelp.dll
 0000:ffd9b000       .debug$S                   0000000140000000     kernel32:KERNEL32.dll
 0000:ffd9b000       .debug$S                   0000000140000000     DbgHelp:dbghelp.dll
 0000:ffd9b000       .debug$S                   0000000140000000     kernel32:KERNEL32.dll
 0000:ffd9b000       .debug$S                   0000000140000000     kernel32:KERNEL32.dll
 0000:ffd9b000       .debug$S                   0000000140000000     DbgHelp:dbghelp.dll
 0000:ffd9b000       .debug$S                   0000000140000000     kernel32:KERNEL32.dll
 0000:ffd9b000       .debug$S                   0000000140000000     kernel32:KERNEL32.dll
 0000:ffd9b000       .debug$S                   0000000140000000     kernel32:KERNEL32.dll
 0000:ffd9b000       .debug$S                   0000000140000000     kernel32:KERNEL32.dll
 0000:ffd9b000       .debug$S                   0000000140000000     Wininet:WININET.dll
 0000:ffd9b000       .debug$S                   0000000140000000     kernel32:KERNEL32.dll
 0000:ffd9b000       .debug$S                   0000000140000000     kernel32:KERNEL32.dll
 0000:ffd9b000       .debug$S                   0000000140000000     kernel32:KERNEL32.dll
 0000:ffd9b000       .debug$S                   0000000140000000     Wininet:WININET.dll
 0000:ffd9b000       .debug$S                   0000000140000000     kernel32:KERNEL32.dll
 0000:ffd9b000       .debug$S                   0000000140000000     kernel32:KERNEL32.dll
 0000:ffd9b000       .debug$S                   0000000140000000     Wininet:WININET.dll
 0000:ffd9b000       .debug$S                   0000000140000000     kernel32:KERNEL32.dll
 0000:ffd9b000       .debug$S                   0000000140000000     kernel32:KERNEL32.dll
 0000:ffd9b000       .debug$S                   0000000140000000     kernel32:KERNEL32.dll
 0000:ffd9b000       .debug$S                   0000000140000000     kernel32:KERNEL32.dll
 0000:ffd9b000       .debug$S                   0000000140000000     Wininet:WININET.dll
 0000:ffd9b000       .debug$S                   0000000140000000     kernel32:KERNEL32.dll
 0000:ffd9b000       .debug$S                   0000000140000000     kernel32:KERNEL32.dll
 0000:ffd9b000       .debug$S                   0000000140000000     kernel32:KERNEL32.dll
 0000:ffd9b000       .debug$S                   0000000140000000     Wininet:WININET.dll
 0000:ffd9b000       .debug$S                   0000000140000000     kernel32:KERNEL32.dll
 0000:ffd9b000       .debug$S                   0000000140000000     kernel32:KERNEL32.dll
 0000:ffd9b000       .debug$S                   0000000140000000     kernel32:KERNEL32.dll
 0000:ffd9b000       .debug$S                   0000000140000000     kernel32:KERNEL32.dll
 0000:ffd9b000       .debug$S                   0000000140000000     kernel32:KERNEL32.dll
 0000:ffd9b000       .debug$S                   0000000140000000     Wininet:WININET.dll
 0000:ffd9b000       .debug$S                   0000000140000000     kernel32:KERNEL32.dll
 0000:ffd9b000       .debug$S                   0000000140000000     kernel32:KERNEL32.dll
 0000:ffd9b000       .debug$S                   0000000140000000     Wininet:WININET.dll
 0000:ffd9b000       .debug$S                   0000000140000000     kernel32:KERNEL32.dll
 0000:ffd9b000       .debug$S                   0000000140000000     kernel32:KERNEL32.dll
 0000:ffd9b000       .debug$S                   0000000140000000     kernel32:KERNEL32.dll
 0000:ffd9b000       .debug$S                   0000000140000000     kernel32:KERNEL32.dll
 0000:ffd9b000       .debug$S                   0000000140000000     kernel32:KERNEL32.dll
 0000:ffd9b000       .debug$S                   0000000140000000     kernel32:KERNEL32.dll
 0000:ffd9b000       .debug$S                   0000000140000000     kernel32:KERNEL32.dll
 0000:ffd9b000       .debug$S                   0000000140000000     kernel32:KERNEL32.dll
 0000:ffd9b000       .debug$S                   0000000140000000     kernel32:KERNEL32.dll
 0000:ffd9b000       .debug$S                   0000000140000000     kernel32:KERNEL32.dll
 0000:ffd9b000       .debug$S                   0000000140000000     kernel32:KERNEL32.dll
 0000:ffd9b000       .debug$S                   0000000140000000     user32:USER32.dll
 0000:ffd9b000       .debug$S                   0000000140000000     user32:USER32.dll
 0000:ffd9b000       .debug$S                   0000000140000000     user32:USER32.dll
 0000:ffd9b000       .debug$S                   0000000140000000     user32:USER32.dll
 0000:ffd9b000       .debug$S                   0000000140000000     user32:USER32.dll
 0000:ffd9b000       .debug$S                   0000000140000000     user32:USER32.dll
 0000:ffd9b000       .debug$S                   0000000140000000     user32:USER32.dll
 0000:ffd9b000       .debug$S                   0000000140000000     user32:USER32.dll
 0000:ffd9b000       .debug$S                   0000000140000000     user32:USER32.dll
 0000:ffd9b000       .debug$S                   0000000140000000     shell32:SHELL32.dll
 0000:ffd9b000       .debug$S                   0000000140000000     shlwapi:SHLWAPI.dll
 0000:ffd9b000       .debug$S                   0000000140000000     Wininet:WININET.dll
 0000:ffd9b000       .debug$S                   0000000140000000     msvcprt:MSVCP140.dll
 0000:ffd9b000       .debug$S                   0000000140000000     msvcprt:MSVCP140.dll
 0002:fffe6000       .idata$6                   0000000140000000     oleaut32:OLEAUT32.dll
 0000:ffd9b000       .debug$S                   0000000140000000     oleaut32:OLEAUT32.dll
 0001:00000000       ??__EFloatOne@GlobalVectorConstants@@YAXXZ 0000000140001000 f   ltmodule.obj
 0001:00000010       ??__EFloatZero@GlobalVectorConstants@@YAXXZ 0000000140001010 f   ltmodule.obj
 0001:00000020       ??__EFloatMinusOne@GlobalVectorConstants@@YAXXZ 0000000140001020 f   ltmodule.obj
 0001:00000030       ??__EFloatOneHalf@GlobalVectorConstants@@YAXXZ 0000000140001030 f   ltmodule.obj
 0001:00000040       ??__EXYZMask@GlobalVectorConstants@@YAXXZ 0000000140001040 f   ltmodule.obj
 0001:00000060       ??__ETwoPi@GlobalVectorConstants@@YAXXZ 0000000140001060 f   ltmodule.obj
 0001:00000070       ??__EPiByTwo@GlobalVectorConstants@@YAXXZ 0000000140001070 f   ltmodule.obj
 0001:00000080       ??__EOneOverTwoPi@GlobalVectorConstants@@YAXXZ 0000000140001080 f   ltmodule.obj
 0001:00000090       ??__Ea@VectorSinConstantsSSE@@YAXXZ 0000000140001090 f   ltmodule.obj
 0001:000000c0       ??__Eb@VectorSinConstantsSSE@@YAXXZ 00000001400010c0 f   ltmodule.obj
 0001:000000f0       ??__EA@VectorSinConstantsSSE@@YAXXZ 00000001400010f0 f   ltmodule.obj
 0001:00000110       ??__EB@VectorSinConstantsSSE@@YAXXZ 0000000140001110 f   ltmodule.obj
 0001:00000130       ??__EPI@@YAXXZ             0000000140001130 f   ltmodule.obj
 0001:00000160       ??__E_FILE_SHUTDOWN_var_ltmod_database_@@YAXXZ 0000000140001160 f   ltmodule.obj
 0001:00000170       ??__E?m_strFileFormat@CHLogger@@0V?$basic_string@DU?$char_traits@D@std@@V?$allocator@D@2@@std@@A@@YAXXZ 0000000140001170 f   HostLogger.obj
 0001:00000180       ??__E?m_strBRFileFormat@CHLogger@@0V?$basic_string@DU?$char_traits@D@std@@V?$allocator@D@2@@std@@A@@YAXXZ 0000000140001180 f   HostLogger.obj
 0001:00000190       ??__E?m_strKernelFileFormat@CHLogger@@0V?$basic_string@DU?$char_traits@D@std@@V?$allocator@D@2@@std@@A@@YAXXZ 0000000140001190 f   HostLogger.obj
 0001:000001a0       ??__E?m_strEtcFileFormat@CHLogger@@0V?$basic_string@DU?$char_traits@D@std@@V?$allocator@D@2@@std@@A@@YAXXZ 00000001400011a0 f   HostLogger.obj
 0001:000001b0       ??__E?m_strRWProcessMemoryFileFormat@CHLogger@@0V?$basic_string@DU?$char_traits@D@std@@V?$allocator@D@2@@std@@A@@YAXXZ 00000001400011b0 f   HostLogger.obj
 0001:000001c0       ??__E?m_strIPCMessageFileFormat@CHLogger@@0V?$basic_string@DU?$char_traits@D@std@@V?$allocator@D@2@@std@@A@@YAXXZ 00000001400011c0 f   HostLogger.obj
 0001:000001d0       ??__E?m_strTimeOutFileFormat@CHLogger@@0V?$basic_string@DU?$char_traits@D@std@@V?$allocator@D@2@@std@@A@@YAXXZ 00000001400011d0 f   HostLogger.obj
 0001:000001e0       ??__E?m_strPacketFileFormat@CHLogger@@0V?$basic_string@DU?$char_traits@D@std@@V?$allocator@D@2@@std@@A@@YAXXZ 00000001400011e0 f   HostLogger.obj
 0001:000001f0       ??__E?m_strHostName@CHLogger@@0V?$basic_string@DU?$char_traits@D@std@@V?$allocator@D@2@@std@@A@@YAXXZ 00000001400011f0 f   HostLogger.obj
 0001:00000200       ??__E?m_strServerName@CHLogger@@0V?$basic_string@DU?$char_traits@D@std@@V?$allocator@D@2@@std@@A@@YAXXZ 0000000140001200 f   HostLogger.obj
 0001:00000210       ??__E?m_strLogFolder@CHLogger@@0V?$basic_string@DU?$char_traits@D@std@@V?$allocator@D@2@@std@@A@@YAXXZ 0000000140001210 f   HostLogger.obj
 0001:00000220       ??__E?m_strModeUserCountFormat@CHLogger@@0V?$basic_string@DU?$char_traits@D@std@@V?$allocator@D@2@@std@@A@@YAXXZ 0000000140001220 f   HostLogger.obj
 0001:00000230       ??__E?m_strServerAppUseCountFormat@CHLogger@@0V?$basic_string@DU?$char_traits@D@std@@V?$allocator@D@2@@std@@A@@YAXXZ 0000000140001230 f   HostLogger.obj
 0001:00000240       ??__E?m_LogLock@CHLogger@@0VCMustSyncObjectLog@@A@@YAXXZ 0000000140001240 f   HostLogger.obj
 0001:00000270       ??__E?m_LogPacketLock@CHLogger@@0VCMustSyncObjectLog@@A@@YAXXZ 0000000140001270 f   HostLogger.obj
 0001:000002a0       ??__E?m_vectSharedMapHandles@CLogMsgManager@@0V?$vector@PEAXV?$allocator@PEAX@std@@@std@@A@@YAXXZ 00000001400012a0 f   LogMsgManager.obj
 0001:000002b0       ??__EtheApp@@YAXXZ         00000001400012b0 f   ServerApp.obj
 0001:000002f0       ??__Eg_cServerLog@@YAXXZ   00000001400012f0 f   ServerAppDlg.obj
 0001:00000440       ??__E__api_holder_ILTCommon_Server_g_pLTSCommon__@@YAXXZ 0000000140001440 f   ServerAppDlg.obj
 0001:00000530       ??__Eg_sGameInfos@@YAXXZ   0000000140001530 f   ServerAppDlg.obj
 0001:000005c0       ??__Eg_sUserInfos@@YAXXZ   00000001400015c0 f   ServerAppDlg.obj
 0001:00000600       ??__EFloatOne@GlobalVectorConstants@@YAXXZ 0000000140001600 f   StdAfx.obj
 0001:00000610       ??__EFloatZero@GlobalVectorConstants@@YAXXZ 0000000140001610 f   StdAfx.obj
 0001:00000620       ??__EFloatMinusOne@GlobalVectorConstants@@YAXXZ 0000000140001620 f   StdAfx.obj
 0001:00000630       ??__EFloatOneHalf@GlobalVectorConstants@@YAXXZ 0000000140001630 f   StdAfx.obj
 0001:00000640       ??__EXYZMask@GlobalVectorConstants@@YAXXZ 0000000140001640 f   StdAfx.obj
 0001:00000660       ??__ETwoPi@GlobalVectorConstants@@YAXXZ 0000000140001660 f   StdAfx.obj
 0001:00000670       ??__EPiByTwo@GlobalVectorConstants@@YAXXZ 0000000140001670 f   StdAfx.obj
 0001:00000680       ??__EOneOverTwoPi@GlobalVectorConstants@@YAXXZ 0000000140001680 f   StdAfx.obj
 0001:00000690       ??__Ea@VectorSinConstantsSSE@@YAXXZ 0000000140001690 f   StdAfx.obj
 0001:000006c0       ??__Eb@VectorSinConstantsSSE@@YAXXZ 00000001400016c0 f   StdAfx.obj
 0001:000006f0       ??__EA@VectorSinConstantsSSE@@YAXXZ 00000001400016f0 f   StdAfx.obj
 0001:00000710       ??__EB@VectorSinConstantsSSE@@YAXXZ 0000000140001710 f   StdAfx.obj
 0001:00000730       ??__EPI@@YAXXZ             0000000140001730 f   StdAfx.obj
 0001:0000075c       ??__E_AtlBaseModule@ATL@@YAXXZ 000000014000175c f   atls:atlbase.obj
 0001:0000077c       ??__E_afxInitAppState@@YAXXZ 000000014000177c f   mfcs140:appmodul.obj
 0001:000007a0       ?CRSUploader@@YAAEAVUploader@crs@@XZ 00000001400017a0 f   BugReporter.obj
 0001:00002800       ?EnumModuleDetail@ModuleInfo@?1??makeExceptionLog@Uploader@crs@@QEAAXPEAU_EXCEPTION_POINTERS@@AEAVLogBuffer@4@@Z@SAHPEBD_KKPEAX@Z 0000000140003800 f   crs_uploader.obj
 0001:00004a90       ?LTStrCpyCreate@?A0xaa4cf837@@YAPEADPEBD@Z 0000000140005a90 f   ltmodule.obj
 0001:00004b00       ?check_delete_pointers@@YAXXZ 0000000140005b00 f   ltmodule.obj
 0001:0000a688       $LN153                     000000014000b688     ServerAppDlg.obj
 0001:0000d878       $LN1487                    000000014000e878     ServerAppDlg.obj
 0001:0000ffcc       $LN329                     0000000140010fcc     ServerAppDlg.obj
 0001:00010000       $LN328                     0000000140011000     ServerAppDlg.obj
 0001:00014380       ?USNtoStr@EXPAND_USN@@YA?AV?$basic_string@DU?$char_traits@D@std@@V?$allocator@D@2@@std@@_J@Z 0000000140015380 f   ServerAppDlg.obj
 0001:00015e70       $$000000                   0000000140016e70     msvcrt:amdsecgs.obj
 0001:00015eac       ?__scrt_initialize_thread_safe_statics@@YAHXZ 0000000140016eac f   msvcrt:thread_safe_statics.obj
 0001:0001600c       ?__scrt_uninitialize_thread_safe_statics@@YAXXZ 000000014001700c f   msvcrt:thread_safe_statics.obj
 0001:000165dc       capture_previous_context   00000001400175dc f   msvcrt:gs_report.obj
 0001:00016650       ?pre_c_initialization@@YAHXZ 0000000140017650 f   msvcrt:exe_winmain.obj
 0001:00016708       ?post_pgo_initialization@@YAHXZ 0000000140017708 f   msvcrt:exe_winmain.obj
 0001:00016718       ?pre_cpp_initialization@@YAXXZ 0000000140017718 f   msvcrt:exe_winmain.obj
 0001:00016734       ?__scrt_common_main_seh@@YAHXZ 0000000140017734 f   msvcrt:exe_winmain.obj
 0001:00017100       $$000000                   0000000140018100     msvcrt:chkstk.obj
 0001:000171a0       $$000000                   00000001400181a0     msvcrt:guard_dispatch.obj
 0001:000171c0       ?dtor$0@?0??CRSUploader@@YAAEAVUploader@crs@@XZ@4HA 00000001400181c0 f   BugReporter.obj
 0001:000171cc       ?dtor$1@?0??CRSUploader@@YAAEAVUploader@crs@@XZ@4HA 00000001400181cc f   BugReporter.obj
 0001:000171e9       ?dtor$8@?0??CRSUploader@@YAAEAVUploader@crs@@XZ@4HA 00000001400181e9 f   BugReporter.obj
 0001:00017200       ?dtor$0@?0??threadCreateDumpFile@@YAKPEAX@Z@4HA 0000000140018200 f   BugReporter.obj
 0001:00017210       ?dtor$0@?0??readURL@Uploader@crs@@AEAAXAEAV?$basic_string@_WU?$char_traits@_W@std@@V?$allocator@_W@2@@std@@@Z@4HA 0000000140018210 f   crs_uploader.obj
 0001:0001721c       ?dtor$1@?0??readURL@Uploader@crs@@AEAAXAEAV?$basic_string@_WU?$char_traits@_W@std@@V?$allocator@_W@2@@std@@@Z@4HA 000000014001821c f   crs_uploader.obj
 0001:00017230       ?dtor$0@?0??init@Uploader@crs@@QEAA_N_NPEAD1@Z@4HA 0000000140018230 f   crs_uploader.obj
 0001:00017240       ?dtor$0@?0???0CInterfaceDatabase@@QEAA@XZ@4HA 0000000140018240 f   ltmodule.obj
 0001:00017250       ?dtor$1@?0???0CInterfaceDatabase@@QEAA@XZ@4HA 0000000140018250 f   ltmodule.obj
 0001:00017270       ?dtor$0@?0??AddHolder@CInterfaceDatabase@@SAXPEAVCAPIHolderBase@@@Z@4HA 0000000140018270 f   ltmodule.obj
 0001:00017290       ?dtor$0@?0??Add@CInterfaceDatabase@@EEAAXPEAVCInterfaceChooser@@@Z@4HA 0000000140018290 f   ltmodule.obj
 0001:00017290       ?dtor$0@?0??Add@CInterfaceDatabase@@EEAAXPEAVCAPIHolderBase@@@Z@4HA 0000000140018290 f   ltmodule.obj
 0001:00017290       ?dtor$0@?0??Add@CInterfaceDatabase@@EEAAXPEAVIBase@@PEBDH@Z@4HA 0000000140018290 f   ltmodule.obj
 0001:000172b0       ?dtor$0@?0??TransferFrom@CInterfaceDatabase@@UEAAXPEAV1@@Z@4HA 00000001400182b0 f   ltmodule.obj
 0001:000172d0       ?dtor$0@?0???0CInterfaceNameMgr@@QEAA@PEBDH@Z@4HA 00000001400182d0 f   ltmodule.obj
 0001:000172ed       ?dtor$1@?0???0CInterfaceNameMgr@@QEAA@PEBDH@Z@4HA 00000001400182ed f   ltmodule.obj
 0001:0001730a       ?dtor$2@?0???0CInterfaceNameMgr@@QEAA@PEBDH@Z@4HA 000000014001830a f   ltmodule.obj
 0001:00017330       ?dtor$0@?0??TransferFrom@CInterfaceNameMgr@@QEAAXPEAV1@@Z@4HA 0000000140018330 f   ltmodule.obj
 0001:0001734d       ?dtor$1@?0??TransferFrom@CInterfaceNameMgr@@QEAAXPEAV1@@Z@4HA 000000014001834d f   ltmodule.obj
 0001:0001736a       ?dtor$2@?0??TransferFrom@CInterfaceNameMgr@@QEAAXPEAV1@@Z@4HA 000000014001836a f   ltmodule.obj
 0001:00017390       ?dtor$0@?0??LogPacket@CHLogger@@SAXPEBDZZ@4HA 0000000140018390 f   HostLogger.obj
 0001:000173a0       ?dtor$0@?0??_BuildDirectory@CHLogger@@CAXAEBU_SYSTEMTIME@@@Z@4HA 00000001400183a0 f   HostLogger.obj
 0001:000173ac       ?dtor$1@?0??_BuildDirectory@CHLogger@@CAXAEBU_SYSTEMTIME@@@Z@4HA 00000001400183ac f   HostLogger.obj
 0001:000173b8       ?dtor$2@?0??_BuildDirectory@CHLogger@@CAXAEBU_SYSTEMTIME@@@Z@4HA 00000001400183b8 f   HostLogger.obj
 0001:000173d0       ?dtor$0@?0??_DoLogWithLevel@CHLogger@@CAXPEBDW4ELOG_LEVEL@1@0PEAD@Z@4HA 00000001400183d0 f   HostLogger.obj
 0001:000173e0       ?dtor$0@?0??Init@CLogMsgManager@@SA_NW4ESHARED_MEM_USAGE_TYPE@1@@Z@4HA 00000001400183e0 f   LogMsgManager.obj
 0001:000173fd       ?dtor$1@?0??Init@CLogMsgManager@@SA_NW4ESHARED_MEM_USAGE_TYPE@1@@Z@4HA 00000001400183fd f   LogMsgManager.obj
 0001:00017420       ?dtor$0@?0??RECV_MSG_USER_DISCONNECTED@CServerAppDlg@@AEAAX_J@Z@4HA 0000000140018420 f   ServerAppDlg.obj
 0001:00017420       ?dtor$0@?0??_WriteXlsDataToSharedMemory@CLogMsgManager@@CA_NXZ@4HA 0000000140018420 f   LogMsgManager.obj
 0001:00017420       ?dtor$0@?0??OnTimer@CServerAppDlg@@QEAAX_K@Z@4HA 0000000140018420 f   ServerAppDlg.obj
 0001:00017430       ?dtor$0@?0??LoadWMszFile@FindXlsMsg@@QEAA_NPEAD@Z@4HA 0000000140018430 f   LoadXlsMsg.obj
 0001:00017440       ?catch$0@?0???$_Insert_hint@AEAU?$pair@$$CB_JV?$basic_string@DU?$char_traits@D@std@@V?$allocator@D@2@@std@@@std@@PEAU?$_Tree_node@U?$pair@$$CB_JV?$basic_string@DU?$char_traits@D@std@@V?$allocator@D@2@@std@@@std@@PEAX@2@@?$_Tree@V?$_Tmap_traits@_JV?$basic_string@DU?$char_traits@D@std@@V?$allocator@D@2@@std@@U?$less@_J@2@V?$allocator@U?$pair@$$CB_JV?$basic_string@DU?$char_traits@D@std@@V?$allocator@D@2@@std@@@std@@@2@$0A@@std@@@std@@IEAA?AV?$_Tree_iterator@V?$_Tree_val@U?$_Tree_simple_types@U?$pair@$$CB_JV?$basic_string@DU?$char_traits@D@std@@V?$allocator@D@2@@std@@@std@@@std@@@std@@@1@V?$_Tree_const_iterator@V?$_Tree_val@U?$_Tree_simple_types@U?$pair@$$CB_JV?$basic_string@DU?$char_traits@D@std@@V?$allocator@D@2@@std@@@std@@@std@@@std@@@1@AEAU?$pair@$$CB_JV?$basic_string@DU?$char_traits@D@std@@V?$allocator@D@2@@std@@@1@PEAU?$_Tree_node@U?$pair@$$CB_JV?$basic_string@DU?$char_traits@D@std@@V?$allocator@D@2@@std@@@std@@PEAX@1@@Z@4HA 0000000140018440 f   LoadXlsMsg.obj
 0001:0001744d       __catch$??$_Insert_hint@AEAU?$pair@$$CB_JV?$basic_string@DU?$char_traits@D@std@@V?$allocator@D@2@@std@@@std@@PEAU?$_Tree_node@U?$pair@$$CB_JV?$basic_string@DU?$char_traits@D@std@@V?$allocator@D@2@@std@@@std@@PEAX@2@@?$_Tree@V?$_Tmap_traits@_JV?$basic_string@DU?$char_traits@D@std@@V?$allocator@D@2@@std@@U?$less@_J@2@V?$allocator@U?$pair@$$CB_JV?$basic_string@DU?$char_traits@D@std@@V?$allocator@D@2@@std@@@std@@@2@$0A@@std@@@std@@IEAA?AV?$_Tree_iterator@V?$_Tree_val@U?$_Tree_simple_types@U?$pair@$$CB_JV?$basic_string@DU?$char_traits@D@std@@V?$allocator@D@2@@std@@@std@@@std@@@std@@@1@V?$_Tree_const_iterator@V?$_Tree_val@U?$_Tree_simple_types@U?$pair@$$CB_JV?$basic_string@DU?$char_traits@D@std@@V?$allocator@D@2@@std@@@std@@@std@@@std@@@1@AEAU?$pair@$$CB_JV?$basic_string@DU?$char_traits@D@std@@V?$allocator@D@2@@std@@@1@PEAU?$_Tree_node@U?$pair@$$CB_JV?$basic_string@DU?$char_traits@D@std@@V?$allocator@D@2@@std@@@std@@PEAX@1@@Z$0 000000014001844d f   LoadXlsMsg.obj
 0001:00017470       ?catch$0@?0???$_Insert_nohint@AEAU?$pair@$$CB_JV?$basic_string@DU?$char_traits@D@std@@V?$allocator@D@2@@std@@@std@@PEAU?$_Tree_node@U?$pair@$$CB_JV?$basic_string@DU?$char_traits@D@std@@V?$allocator@D@2@@std@@@std@@PEAX@2@@?$_Tree@V?$_Tmap_traits@_JV?$basic_string@DU?$char_traits@D@std@@V?$allocator@D@2@@std@@U?$less@_J@2@V?$allocator@U?$pair@$$CB_JV?$basic_string@DU?$char_traits@D@std@@V?$allocator@D@2@@std@@@std@@@2@$0A@@std@@@std@@IEAA?AU?$pair@V?$_Tree_iterator@V?$_Tree_val@U?$_Tree_simple_types@U?$pair@$$CB_JV?$basic_string@DU?$char_traits@D@std@@V?$allocator@D@2@@std@@@std@@@std@@@std@@@std@@_N@1@_NAEAU?$pair@$$CB_JV?$basic_string@DU?$char_traits@D@std@@V?$allocator@D@2@@std@@@1@PEAU?$_Tree_node@U?$pair@$$CB_JV?$basic_string@DU?$char_traits@D@std@@V?$allocator@D@2@@std@@@std@@PEAX@1@@Z@4HA 0000000140018470 f   LoadXlsMsg.obj
 0001:0001747d       __catch$??$_Insert_nohint@AEAU?$pair@$$CB_JV?$basic_string@DU?$char_traits@D@std@@V?$allocator@D@2@@std@@@std@@PEAU?$_Tree_node@U?$pair@$$CB_JV?$basic_string@DU?$char_traits@D@std@@V?$allocator@D@2@@std@@@std@@PEAX@2@@?$_Tree@V?$_Tmap_traits@_JV?$basic_string@DU?$char_traits@D@std@@V?$allocator@D@2@@std@@U?$less@_J@2@V?$allocator@U?$pair@$$CB_JV?$basic_string@DU?$char_traits@D@std@@V?$allocator@D@2@@std@@@std@@@2@$0A@@std@@@std@@IEAA?AU?$pair@V?$_Tree_iterator@V?$_Tree_val@U?$_Tree_simple_types@U?$pair@$$CB_JV?$basic_string@DU?$char_traits@D@std@@V?$allocator@D@2@@std@@@std@@@std@@@std@@@std@@_N@1@_NAEAU?$pair@$$CB_JV?$basic_string@DU?$char_traits@D@std@@V?$allocator@D@2@@std@@@1@PEAU?$_Tree_node@U?$pair@$$CB_JV?$basic_string@DU?$char_traits@D@std@@V?$allocator@D@2@@std@@@std@@PEAX@1@@Z$0 000000014001847d f   LoadXlsMsg.obj
 0001:00017490       ?dtor$0@?0??Run@CServerAppApp@@UEAAHXZ@4HA 0000000140018490 f   ServerApp.obj
 0001:000174a0       ?dtor$0@?0???__E__api_holder_ILTCommon_Server_g_pLTSCommon__@@YAXXZ@4HA 00000001400184a0 f   ServerAppDlg.obj
 0001:000174b0       ?dtor$0@?0??OutOfMemory@CGameServerAppHandler@@UEAAIXZ@4HA 00000001400184b0 f   ServerAppDlg.obj
 0001:000174b0       ?dtor$0@?0??ServerUpdate@CServerAppDlg@@QEAAXXZ@4HA 00000001400184b0 f   ServerAppDlg.obj
 0001:000174b0       ?dtor$0@?0??ConsoleOutputFn@CGameServerAppHandler@@UEAAIHHPEBD@Z@4HA 00000001400184b0 f   ServerAppDlg.obj
 0001:000174b0       ?dtor$0@?0??StopServer@CServerAppDlg@@QEAA_NXZ@4HA 00000001400184b0 f   ServerAppDlg.obj
 0001:000174c0       ?dtor$0@?0???0CServerAppDlg@@QEAA@PEAVCWnd@@@Z@4HA 00000001400184c0 f   ServerAppDlg.obj
 0001:000174ce       ?dtor$1@?0???0CServerAppDlg@@QEAA@PEAVCWnd@@@Z@4HA 00000001400184ce f   ServerAppDlg.obj
 0001:000174e3       ?dtor$2@?0???0CServerAppDlg@@QEAA@PEAVCWnd@@@Z@4HA 00000001400184e3 f   ServerAppDlg.obj
 0001:000174f8       ?dtor$3@?0???0CServerAppDlg@@QEAA@PEAVCWnd@@@Z@4HA 00000001400184f8 f   ServerAppDlg.obj
 0001:0001750d       ?dtor$4@?0???0CServerAppDlg@@QEAA@PEAVCWnd@@@Z@4HA 000000014001850d f   ServerAppDlg.obj
 0001:00017520       ?dtor$5@?0???0CServerAppDlg@@QEAA@PEAVCWnd@@@Z@4HA 0000000140018520 f   ServerAppDlg.obj
 0001:00017540       ?dtor$0@?0??OnInitDialog@CServerAppDlg@@MEAAHXZ@4HA 0000000140018540 f   ServerAppDlg.obj
 0001:0001754c       ?dtor$1@?0??OnInitDialog@CServerAppDlg@@MEAAHXZ@4HA 000000014001854c f   ServerAppDlg.obj
 0001:0001755a       ?dtor$2@?0??OnInitDialog@CServerAppDlg@@MEAAHXZ@4HA 000000014001855a f   ServerAppDlg.obj
 0001:00017566       ?dtor$3@?0??OnInitDialog@CServerAppDlg@@MEAAHXZ@4HA 0000000140018566 f   ServerAppDlg.obj
 0001:00017574       ?dtor$4@?0??OnInitDialog@CServerAppDlg@@MEAAHXZ@4HA 0000000140018574 f   ServerAppDlg.obj
 0001:00017580       ?dtor$5@?0??OnInitDialog@CServerAppDlg@@MEAAHXZ@4HA 0000000140018580 f   ServerAppDlg.obj
 0001:0001758c       ?dtor$34@?0??OnInitDialog@CServerAppDlg@@MEAAHXZ@4HA 000000014001858c f   ServerAppDlg.obj
 0001:00017598       ?dtor$35@?0??OnInitDialog@CServerAppDlg@@MEAAHXZ@4HA 0000000140018598 f   ServerAppDlg.obj
 0001:000175b0       ?dtor$0@?0??OnShellMessage@CServerAppDlg@@QEAAXAEAVILTMessage_Read@@@Z@4HA 00000001400185b0 f   ServerAppDlg.obj
 0001:000175bc       ?dtor$1@?0??OnShellMessage@CServerAppDlg@@QEAAXAEAVILTMessage_Read@@@Z@4HA 00000001400185bc f   ServerAppDlg.obj
 0001:000175c8       ?dtor$12@?0??OnShellMessage@CServerAppDlg@@QEAAXAEAVILTMessage_Read@@@Z@4HA 00000001400185c8 f   ServerAppDlg.obj
 0001:000175d4       ?dtor$3@?0??OnShellMessage@CServerAppDlg@@QEAAXAEAVILTMessage_Read@@@Z@4HA 00000001400185d4 f   ServerAppDlg.obj
 0001:000175e0       ?dtor$4@?0??OnShellMessage@CServerAppDlg@@QEAAXAEAVILTMessage_Read@@@Z@4HA 00000001400185e0 f   ServerAppDlg.obj
 0001:000175ec       ?dtor$5@?0??OnShellMessage@CServerAppDlg@@QEAAXAEAVILTMessage_Read@@@Z@4HA 00000001400185ec f   ServerAppDlg.obj
 0001:000175f8       ?dtor$6@?0??OnShellMessage@CServerAppDlg@@QEAAXAEAVILTMessage_Read@@@Z@4HA 00000001400185f8 f   ServerAppDlg.obj
 0001:00017604       ?dtor$7@?0??OnShellMessage@CServerAppDlg@@QEAAXAEAVILTMessage_Read@@@Z@4HA 0000000140018604 f   ServerAppDlg.obj
 0001:00017610       ?dtor$1@?0??SendToServerShellAutoMatchStartingUserInfo@CServerAppDlg@@AEAAXPEAUtagCOPYDATASTRUCT@@@Z@4HA 0000000140018610 f   ServerAppDlg.obj
 0001:00017610       ?dtor$0@?0??AddServerMsg@CServerAppDlg@@QEAAXPEBDH@Z@4HA 0000000140018610 f   ServerAppDlg.obj
 0001:00017610       ?dtor$1@?0??RECV_MSG_AIITEM_GROUP_RATE_RESULT@CServerAppDlg@@AEAAX_J@Z@4HA 0000000140018610 f   ServerAppDlg.obj
 0001:00017620       ?dtor$0@?0??LoadServer@CServerAppDlg@@QEAA_NXZ@4HA 0000000140018620 f   ServerAppDlg.obj
 0001:0001762c       ?dtor$1@?0??LoadServer@CServerAppDlg@@QEAA_NXZ@4HA 000000014001862c f   ServerAppDlg.obj
 0001:0001763a       ?dtor$2@?0??LoadServer@CServerAppDlg@@QEAA_NXZ@4HA 000000014001863a f   ServerAppDlg.obj
 0001:00017648       ?dtor$3@?0??LoadServer@CServerAppDlg@@QEAA_NXZ@4HA 0000000140018648 f   ServerAppDlg.obj
 0001:00017656       ?dtor$6@?0??LoadServer@CServerAppDlg@@QEAA_NXZ@4HA 0000000140018656 f   ServerAppDlg.obj
 0001:00017673       ?dtor$4@?0??LoadServer@CServerAppDlg@@QEAA_NXZ@4HA 0000000140018673 f   ServerAppDlg.obj
 0001:0001767f       ?dtor$5@?0??LoadServer@CServerAppDlg@@QEAA_NXZ@4HA 000000014001867f f   ServerAppDlg.obj
 0001:00017690       ?dtor$0@?0??RunServer@CServerAppDlg@@QEAA_NXZ@4HA 0000000140018690 f   ServerAppDlg.obj
 0001:0001769c       ?dtor$1@?0??RunServer@CServerAppDlg@@QEAA_NXZ@4HA 000000014001869c f   ServerAppDlg.obj
 0001:000176a8       ?dtor$8@?0??RunServer@CServerAppDlg@@QEAA_NXZ@4HA 00000001400186a8 f   ServerAppDlg.obj
 0001:000176b4       ?dtor$2@?0??RunServer@CServerAppDlg@@QEAA_NXZ@4HA 00000001400186b4 f   ServerAppDlg.obj
 0001:000176c0       ?dtor$3@?0??RunServer@CServerAppDlg@@QEAA_NXZ@4HA 00000001400186c0 f   ServerAppDlg.obj
 0001:000176d0       ?dtor$0@?0??Thread_SendGameInfo@@YAXPEAVCServerAppDlg@@AEAUPROTO_START_HOST_tag@@@Z@4HA 00000001400186d0 f   ServerAppDlg.obj
 0001:000176dc       ?dtor$1@?0??Thread_SendGameInfo@@YAXPEAVCServerAppDlg@@AEAUPROTO_START_HOST_tag@@@Z@4HA 00000001400186dc f   ServerAppDlg.obj
 0001:000176e8       ?dtor$2@?0??Thread_SendGameInfo@@YAXPEAVCServerAppDlg@@AEAUPROTO_START_HOST_tag@@@Z@4HA 00000001400186e8 f   ServerAppDlg.obj
 0001:000176f4       ?dtor$3@?0??Thread_SendGameInfo@@YAXPEAVCServerAppDlg@@AEAUPROTO_START_HOST_tag@@@Z@4HA 00000001400186f4 f   ServerAppDlg.obj
 0001:00017700       ?dtor$4@?0??Thread_SendGameInfo@@YAXPEAVCServerAppDlg@@AEAUPROTO_START_HOST_tag@@@Z@4HA 0000000140018700 f   ServerAppDlg.obj
 0001:00017710       ?dtor$0@?0??Thread_SendUserInfo@@YAXPEAVCServerAppDlg@@AEAUPROTO_GAME_USER_INFO_tag@@@Z@4HA 0000000140018710 f   ServerAppDlg.obj
 0001:0001771c       ?dtor$1@?0??Thread_SendUserInfo@@YAXPEAVCServerAppDlg@@AEAUPROTO_GAME_USER_INFO_tag@@@Z@4HA 000000014001871c f   ServerAppDlg.obj
 0001:00017730       ?dtor$0@?0??ThreadUpdate@CServerAppDlg@@SAXPEAX@Z@4HA 0000000140018730 f   ServerAppDlg.obj
 0001:0001773c       ?dtor$1@?0??ThreadUpdate@CServerAppDlg@@SAXPEAX@Z@4HA 000000014001873c f   ServerAppDlg.obj
 0001:00017750       ?dtor$0@?0??AddResources@CServerAppDlg@@QEAA_NXZ@4HA 0000000140018750 f   ServerAppDlg.obj
 0001:0001775c       ?dtor$1@?0??AddResources@CServerAppDlg@@QEAA_NXZ@4HA 000000014001875c f   ServerAppDlg.obj
 0001:0001776a       ?dtor$2@?0??AddResources@CServerAppDlg@@QEAA_NXZ@4HA 000000014001876a f   ServerAppDlg.obj
 0001:00017778       ?dtor$3@?0??AddResources@CServerAppDlg@@QEAA_NXZ@4HA 0000000140018778 f   ServerAppDlg.obj
 0001:00017786       ?dtor$4@?0??AddResources@CServerAppDlg@@QEAA_NXZ@4HA 0000000140018786 f   ServerAppDlg.obj
 0001:00017794       ?dtor$5@?0??AddResources@CServerAppDlg@@QEAA_NXZ@4HA 0000000140018794 f   ServerAppDlg.obj
 0001:000177a2       ?dtor$6@?0??AddResources@CServerAppDlg@@QEAA_NXZ@4HA 00000001400187a2 f   ServerAppDlg.obj
 0001:000177b0       ?dtor$7@?0??AddResources@CServerAppDlg@@QEAA_NXZ@4HA 00000001400187b0 f   ServerAppDlg.obj
 0001:000177c0       ?dtor$0@?0??OnGameServerMsg@CServerAppDlg@@IEAA_J_K_J@Z@4HA 00000001400187c0 f   ServerAppDlg.obj
 0001:000177cc       ?dtor$1@?0??OnGameServerMsg@CServerAppDlg@@IEAA_J_K_J@Z@4HA 00000001400187cc f   ServerAppDlg.obj
 0001:000177d8       ?dtor$2@?0??OnGameServerMsg@CServerAppDlg@@IEAA_J_K_J@Z@4HA 00000001400187d8 f   ServerAppDlg.obj
 0001:000177f0       ?dtor$0@?0??OnCopyData@CServerAppDlg@@IEAAHPEAVCWnd@@PEAUtagCOPYDATASTRUCT@@@Z@4HA 00000001400187f0 f   ServerAppDlg.obj
 0001:000177fc       ?dtor$1@?0??OnCopyData@CServerAppDlg@@IEAAHPEAVCWnd@@PEAUtagCOPYDATASTRUCT@@@Z@4HA 00000001400187fc f   ServerAppDlg.obj
 0001:00017808       ?dtor$2@?0??OnCopyData@CServerAppDlg@@IEAAHPEAVCWnd@@PEAUtagCOPYDATASTRUCT@@@Z@4HA 0000000140018808 f   ServerAppDlg.obj
 0001:00017814       ?dtor$3@?0??OnCopyData@CServerAppDlg@@IEAAHPEAVCWnd@@PEAUtagCOPYDATASTRUCT@@@Z@4HA 0000000140018814 f   ServerAppDlg.obj
 0001:00017820       ?dtor$4@?0??OnCopyData@CServerAppDlg@@IEAAHPEAVCWnd@@PEAUtagCOPYDATASTRUCT@@@Z@4HA 0000000140018820 f   ServerAppDlg.obj
 0001:0001782e       ?dtor$5@?0??OnCopyData@CServerAppDlg@@IEAAHPEAVCWnd@@PEAUtagCOPYDATASTRUCT@@@Z@4HA 000000014001882e f   ServerAppDlg.obj
 0001:0001783a       ?dtor$6@?0??OnCopyData@CServerAppDlg@@IEAAHPEAVCWnd@@PEAUtagCOPYDATASTRUCT@@@Z@4HA 000000014001883a f   ServerAppDlg.obj
 0001:00017846       ?dtor$7@?0??OnCopyData@CServerAppDlg@@IEAAHPEAVCWnd@@PEAUtagCOPYDATASTRUCT@@@Z@4HA 0000000140018846 f   ServerAppDlg.obj
 0001:00017860       ?dtor$0@?0??SaveHostGameInfo@CServerAppDlg@@IEAAXXZ@4HA 0000000140018860 f   ServerAppDlg.obj
 0001:0001786c       ?dtor$1@?0??SaveHostGameInfo@CServerAppDlg@@IEAAXXZ@4HA 000000014001886c f   ServerAppDlg.obj
 0001:00017878       ?dtor$2@?0??SaveHostGameInfo@CServerAppDlg@@IEAAXXZ@4HA 0000000140018878 f   ServerAppDlg.obj
 0001:00017890       ?dtor$0@?0??LoadHostGameInfo@CServerAppDlg@@IEAAXXZ@4HA 0000000140018890 f   ServerAppDlg.obj
 0001:0001789c       ?dtor$1@?0??LoadHostGameInfo@CServerAppDlg@@IEAAXXZ@4HA 000000014001889c f   ServerAppDlg.obj
 0001:000178a8       ?dtor$2@?0??LoadHostGameInfo@CServerAppDlg@@IEAAXXZ@4HA 00000001400188a8 f   ServerAppDlg.obj
 0001:000178c0       ?dtor$0@?0??GetOptionValueString@CServerAppDlg@@IEAA?AV?$basic_string@DU?$char_traits@D@std@@V?$allocator@D@2@@std@@V23@00@Z@4HA 00000001400188c0 f   ServerAppDlg.obj
 0001:000178cc       ?dtor$1@?0??GetOptionValueString@CServerAppDlg@@IEAA?AV?$basic_string@DU?$char_traits@D@std@@V?$allocator@D@2@@std@@V23@00@Z@4HA 00000001400188cc f   ServerAppDlg.obj
 0001:000178d8       ?dtor$2@?0??GetOptionValueString@CServerAppDlg@@IEAA?AV?$basic_string@DU?$char_traits@D@std@@V?$allocator@D@2@@std@@V23@00@Z@4HA 00000001400188d8 f   ServerAppDlg.obj
 0001:000178e4       ?dtor$3@?0??GetOptionValueString@CServerAppDlg@@IEAA?AV?$basic_string@DU?$char_traits@D@std@@V?$allocator@D@2@@std@@V23@00@Z@4HA 00000001400188e4 f   ServerAppDlg.obj
 0001:000178f0       ?dtor$1@?0??RECV_MSG_INSERTCHARACTER@CServerAppDlg@@AEAAX_J@Z@4HA 00000001400188f0 f   ServerAppDlg.obj
 0001:000178fc       ?dtor$2@?0??RECV_MSG_INSERTCHARACTER@CServerAppDlg@@AEAAX_J@Z@4HA 00000001400188fc f   ServerAppDlg.obj
 0001:00017910       ?dtor$1@?0??RECV_MSG_AIITEM_DEC@CServerAppDlg@@AEAAX_J@Z@4HA 0000000140018910 f   ServerAppDlg.obj
 0001:00017920       ?dtor$0@?0??SendServerAppInit@CServerAppDlg@@AEAAXXZ@4HA 0000000140018920 f   ServerAppDlg.obj
 0001:00017930       ?dtor$0@?0??DownloadUCCMapFile_HTTP@CServerAppDlg@@AEAA?AW4UCCMAPDOWNLOADREAULT@@V?$basic_string@DU?$char_traits@D@std@@V?$allocator@D@2@@std@@@Z@4HA 0000000140018930 f   ServerAppDlg.obj
 0001:0001793c       ?dtor$1@?0??DownloadUCCMapFile_HTTP@CServerAppDlg@@AEAA?AW4UCCMAPDOWNLOADREAULT@@V?$basic_string@DU?$char_traits@D@std@@V?$allocator@D@2@@std@@@Z@4HA 000000014001893c f   ServerAppDlg.obj
 0001:00017948       ?dtor$2@?0??DownloadUCCMapFile_HTTP@CServerAppDlg@@AEAA?AW4UCCMAPDOWNLOADREAULT@@V?$basic_string@DU?$char_traits@D@std@@V?$allocator@D@2@@std@@@Z@4HA 0000000140018948 f   ServerAppDlg.obj
 0001:00017954       ?dtor$22@?0??DownloadUCCMapFile_HTTP@CServerAppDlg@@AEAA?AW4UCCMAPDOWNLOADREAULT@@V?$basic_string@DU?$char_traits@D@std@@V?$allocator@D@2@@std@@@Z@4HA 0000000140018954 f   ServerAppDlg.obj
 0001:0001797d       ?dtor$4@?0??DownloadUCCMapFile_HTTP@CServerAppDlg@@AEAA?AW4UCCMAPDOWNLOADREAULT@@V?$basic_string@DU?$char_traits@D@std@@V?$allocator@D@2@@std@@@Z@4HA 000000014001897d f   ServerAppDlg.obj
 0001:00017989       ?dtor$40@?0??DownloadUCCMapFile_HTTP@CServerAppDlg@@AEAA?AW4UCCMAPDOWNLOADREAULT@@V?$basic_string@DU?$char_traits@D@std@@V?$allocator@D@2@@std@@@Z@4HA 0000000140018989 f   ServerAppDlg.obj
 0001:000179b2       ?dtor$6@?0??DownloadUCCMapFile_HTTP@CServerAppDlg@@AEAA?AW4UCCMAPDOWNLOADREAULT@@V?$basic_string@DU?$char_traits@D@std@@V?$allocator@D@2@@std@@@Z@4HA 00000001400189b2 f   ServerAppDlg.obj
 0001:000179be       ?dtor$7@?0??DownloadUCCMapFile_HTTP@CServerAppDlg@@AEAA?AW4UCCMAPDOWNLOADREAULT@@V?$basic_string@DU?$char_traits@D@std@@V?$allocator@D@2@@std@@@Z@4HA 00000001400189be f   ServerAppDlg.obj
 0001:000179ca       ?dtor$8@?0??DownloadUCCMapFile_HTTP@CServerAppDlg@@AEAA?AW4UCCMAPDOWNLOADREAULT@@V?$basic_string@DU?$char_traits@D@std@@V?$allocator@D@2@@std@@@Z@4HA 00000001400189ca f   ServerAppDlg.obj
 0001:000179e0       ?dtor$0@?0??SendServerAppInitFail@CServerAppDlg@@AEAAXHH@Z@4HA 00000001400189e0 f   ServerAppDlg.obj
 0001:000179ee       ?dtor$1@?0??SendServerAppInitFail@CServerAppDlg@@AEAAXHH@Z@4HA 00000001400189ee f   ServerAppDlg.obj
 0001:00017a00       ?dtor$0@?0??GetDownloadPath@CServerAppDlg@@AEAA?AV?$basic_string@DU?$char_traits@D@std@@V?$allocator@D@2@@std@@XZ@4HA 0000000140018a00 f   ServerAppDlg.obj
 0001:00017a30       ?dtor$0@?0???$?HDU?$char_traits@D@std@@V?$allocator@D@1@@std@@YA?AV?$basic_string@DU?$char_traits@D@std@@V?$allocator@D@2@@0@AEBV10@0@Z@4HA 0000000140018a30 f   ServerAppDlg.obj
 0001:00017a60       ?catch$1@?0???1CWaitCursor@@QEAA@XZ@4HA 0000000140018a60 f   ServerAppDlg.obj
 0001:00017a6e       __catch$??1CWaitCursor@@QEAA@XZ$0 0000000140018a6e f   ServerAppDlg.obj
 0001:00017b16       ?dtor$0@?0???1CWaitCursor@@QEAA@XZ@4HA 0000000140018b16 f   ServerAppDlg.obj
 0001:00017b30       ?dtor$0@?0??sprintf_s@internal@cf@@YAHPEAD_KPEBDAEAPEAD@Z@4HA 0000000140018b30 f   safe_string_x64:safe_string.obj
 0001:00017b3c       ?dtor$1@?0??sprintf_s@internal@cf@@YAHPEAD_KPEBDAEAPEAD@Z@4HA 0000000140018b3c f   safe_string_x64:safe_string.obj
 0001:00017b48       ?dtor$4@?0??sprintf_s@internal@cf@@YAHPEAD_KPEBDAEAPEAD@Z@4HA 0000000140018b48 f   safe_string_x64:safe_string.obj
 0001:00017b71       ?dtor$2@?0??sprintf_s@internal@cf@@YAHPEAD_KPEBDAEAPEAD@Z@4HA 0000000140018b71 f   safe_string_x64:safe_string.obj
 0001:00017b80       ?dtor$0@?0??strcpy_s@cf@@YAHPEAD_KPEBD@Z@4HA 0000000140018b80 f   safe_string_x64:safe_string.obj
 0001:00017b80       ?dtor$0@?0??strncpy_s@cf@@YAHPEAD_KPEBD1@Z@4HA 0000000140018b80 f   safe_string_x64:safe_string.obj
 0001:00017b8c       ?dtor$1@?0??strcpy_s@cf@@YAHPEAD_KPEBD@Z@4HA 0000000140018b8c f   safe_string_x64:safe_string.obj
 0001:00017b8c       ?dtor$1@?0??strncpy_s@cf@@YAHPEAD_KPEBD1@Z@4HA 0000000140018b8c f   safe_string_x64:safe_string.obj
 0001:00017b98       ?dtor$4@?0??strncpy_s@cf@@YAHPEAD_KPEBD1@Z@4HA 0000000140018b98 f   safe_string_x64:safe_string.obj
 0001:00017b98       ?dtor$4@?0??strcpy_s@cf@@YAHPEAD_KPEBD@Z@4HA 0000000140018b98 f   safe_string_x64:safe_string.obj
 0001:00017bc1       ?dtor$2@?0??strncpy_s@cf@@YAHPEAD_KPEBD1@Z@4HA 0000000140018bc1 f   safe_string_x64:safe_string.obj
 0001:00017bc1       ?dtor$2@?0??strcpy_s@cf@@YAHPEAD_KPEBD@Z@4HA 0000000140018bc1 f   safe_string_x64:safe_string.obj
 0001:00017bd0       ?dtor$0@?0???0?$basic_stringstream@DU?$char_traits@D@std@@V?$allocator@D@2@@std@@QEAA@H@Z@4HA 0000000140018bd0 f   safe_string_x64:safe_string.obj
 0001:00017bfe       ?dtor$1@?0???0?$basic_stringstream@DU?$char_traits@D@std@@V?$allocator@D@2@@std@@QEAA@H@Z@4HA 0000000140018bfe f   safe_string_x64:safe_string.obj
 0001:00017c10       ?dtor$1@?0???$?6U?$char_traits@D@std@@@std@@YAAEAV?$basic_ostream@DU?$char_traits@D@std@@@0@AEAV10@PEBD@Z@4HA 0000000140018c10 f   safe_string_x64:safe_string.obj
 0001:00017c1c       ?dtor$0@?0???$?6U?$char_traits@D@std@@@std@@YAAEAV?$basic_ostream@DU?$char_traits@D@std@@@0@AEAV10@PEBD@Z@4HA 0000000140018c1c f   safe_string_x64:safe_string.obj
 0001:00017c28       ?catch$4@?0???$?6U?$char_traits@D@std@@@std@@YAAEAV?$basic_ostream@DU?$char_traits@D@std@@@0@AEAV10@PEBD@Z@4HA 0000000140018c28 f   safe_string_x64:safe_string.obj
 0001:00017c35       __catch$??$?6U?$char_traits@D@std@@@std@@YAAEAV?$basic_ostream@DU?$char_traits@D@std@@@0@AEAV10@PEBD@Z$0 0000000140018c35 f   safe_string_x64:safe_string.obj
 0001:00017c60       __scrt_is_nonwritable_in_current_image$filt$0 0000000140018c60 f   msvcrt:utility.obj
 0001:00017c78       ?filt$0@?0??__scrt_common_main_seh@@YAHXZ@4HA 0000000140018c78 f   msvcrt:exe_winmain.obj
 0001:00017ca0       ??__Fcrs_uploader@?1??CRSUploader@@YAAEAVUploader@crs@@XZ@YAXXZ 0000000140018ca0 f   BugReporter.obj
 0001:00017cb0       ??__F_FILE_SHUTDOWN_var_ltmod_database_@@YAXXZ 0000000140018cb0 f   ltmodule.obj
 0001:00017cc0       ??__F?m_strEtcFileFormat@CHLogger@@0V?$basic_string@DU?$char_traits@D@std@@V?$allocator@D@2@@std@@A@@YAXXZ 0000000140018cc0 f   HostLogger.obj
 0001:00017d30       ??__F?m_strKernelFileFormat@CHLogger@@0V?$basic_string@DU?$char_traits@D@std@@V?$allocator@D@2@@std@@A@@YAXXZ 0000000140018d30 f   HostLogger.obj
 0001:00017da0       ??__F?m_strBRFileFormat@CHLogger@@0V?$basic_string@DU?$char_traits@D@std@@V?$allocator@D@2@@std@@A@@YAXXZ 0000000140018da0 f   HostLogger.obj
 0001:00017e10       ??__F?m_strFileFormat@CHLogger@@0V?$basic_string@DU?$char_traits@D@std@@V?$allocator@D@2@@std@@A@@YAXXZ 0000000140018e10 f   HostLogger.obj
 0001:00017e80       ??__F?m_strRWProcessMemoryFileFormat@CHLogger@@0V?$basic_string@DU?$char_traits@D@std@@V?$allocator@D@2@@std@@A@@YAXXZ 0000000140018e80 f   HostLogger.obj
 0001:00017ef0       ??__F?m_strIPCMessageFileFormat@CHLogger@@0V?$basic_string@DU?$char_traits@D@std@@V?$allocator@D@2@@std@@A@@YAXXZ 0000000140018ef0 f   HostLogger.obj
 0001:00017f60       ??__F?m_strPacketFileFormat@CHLogger@@0V?$basic_string@DU?$char_traits@D@std@@V?$allocator@D@2@@std@@A@@YAXXZ 0000000140018f60 f   HostLogger.obj
 0001:00017fd0       ??__F?m_strTimeOutFileFormat@CHLogger@@0V?$basic_string@DU?$char_traits@D@std@@V?$allocator@D@2@@std@@A@@YAXXZ 0000000140018fd0 f   HostLogger.obj
 0001:00018040       ??__F?m_strHostName@CHLogger@@0V?$basic_string@DU?$char_traits@D@std@@V?$allocator@D@2@@std@@A@@YAXXZ 0000000140019040 f   HostLogger.obj
 0001:000180b0       ??__F?m_strServerName@CHLogger@@0V?$basic_string@DU?$char_traits@D@std@@V?$allocator@D@2@@std@@A@@YAXXZ 00000001400190b0 f   HostLogger.obj
 0001:00018120       ??__F?m_strLogFolder@CHLogger@@0V?$basic_string@DU?$char_traits@D@std@@V?$allocator@D@2@@std@@A@@YAXXZ 0000000140019120 f   HostLogger.obj
 0001:00018190       ??__F?m_strModeUserCountFormat@CHLogger@@0V?$basic_string@DU?$char_traits@D@std@@V?$allocator@D@2@@std@@A@@YAXXZ 0000000140019190 f   HostLogger.obj
 0001:00018200       ??__F?m_strServerAppUseCountFormat@CHLogger@@0V?$basic_string@DU?$char_traits@D@std@@V?$allocator@D@2@@std@@A@@YAXXZ 0000000140019200 f   HostLogger.obj
 0001:00018270       ??__F?m_LogLock@CHLogger@@0VCMustSyncObjectLog@@A@@YAXXZ 0000000140019270 f   HostLogger.obj
 0001:00018290       ??__F?m_LogPacketLock@CHLogger@@0VCMustSyncObjectLog@@A@@YAXXZ 0000000140019290 f   HostLogger.obj
 0001:000182b0       ??__F?m_vectSharedMapHandles@CLogMsgManager@@0V?$vector@PEAXV?$allocator@PEAX@std@@@std@@A@@YAXXZ 00000001400192b0 f   LogMsgManager.obj
 0001:00018320       ??__FtheApp@@YAXXZ         0000000140019320 f   ServerApp.obj
 0001:00018340       ??__Fg_cServerLog@@YAXXZ   0000000140019340 f   ServerAppDlg.obj
 0001:00018350       ??__F__api_holder_ILTCommon_Server_g_pLTSCommon__@@YAXXZ 0000000140019350 f   ServerAppDlg.obj
 0001:0001835c       ??__F_AtlBaseModule@ATL@@YAXXZ 000000014001935c f   atls:atlbase.obj
 0002:00000d30       ?pre_cpp_initializer@@3P6AXXZEA 000000014001ad30     msvcrt:exe_winmain.obj
 0002:00000d38       ?_AtlBaseModule$initializer$@ATL@@3P6AXXZEA 000000014001ad38     atls:atlbase.obj
 0002:00000d40       ?_afxInitAppState$initializer$@@3P6AXXZEA 000000014001ad40     mfcs140:appmodul.obj
 0002:00000d48       ?FloatOne$initializer$@GlobalVectorConstants@@3P6AXXZEA 000000014001ad48     ltmodule.obj
 0002:00000d50       ?FloatZero$initializer$@GlobalVectorConstants@@3P6AXXZEA 000000014001ad50     ltmodule.obj
 0002:00000d58       ?FloatMinusOne$initializer$@GlobalVectorConstants@@3P6AXXZEA 000000014001ad58     ltmodule.obj
 0002:00000d60       ?FloatOneHalf$initializer$@GlobalVectorConstants@@3P6AXXZEA 000000014001ad60     ltmodule.obj
 0002:00000d68       ?XYZMask$initializer$@GlobalVectorConstants@@3P6AXXZEA 000000014001ad68     ltmodule.obj
 0002:00000d70       ?TwoPi$initializer$@GlobalVectorConstants@@3P6AXXZEA 000000014001ad70     ltmodule.obj
 0002:00000d78       ?PiByTwo$initializer$@GlobalVectorConstants@@3P6AXXZEA 000000014001ad78     ltmodule.obj
 0002:00000d80       ?OneOverTwoPi$initializer$@GlobalVectorConstants@@3P6AXXZEA 000000014001ad80     ltmodule.obj
 0002:00000d88       ?a$initializer$@VectorSinConstantsSSE@@3P6AXXZEA 000000014001ad88     ltmodule.obj
 0002:00000d90       ?b$initializer$@VectorSinConstantsSSE@@3P6AXXZEA 000000014001ad90     ltmodule.obj
 0002:00000d98       ?A$initializer$@VectorSinConstantsSSE@@3P6AXXZEA 000000014001ad98     ltmodule.obj
 0002:00000da0       ?B$initializer$@VectorSinConstantsSSE@@3P6AXXZEA 000000014001ada0     ltmodule.obj
 0002:00000da8       ?PI$initializer$@@3P6AXXZEA 000000014001ada8     ltmodule.obj
 0002:00000db0       ?_FILE_SHUTDOWN_var_ltmod_database_$initializer$@@3P6AXXZEA 000000014001adb0     ltmodule.obj
 0002:00000db8       ??m_strFileFormat$initializer$@CHLogger@@0P6AXXZEA@@3P6AXXZEA 000000014001adb8     HostLogger.obj
 0002:00000dc0       ??m_strBRFileFormat$initializer$@CHLogger@@0P6AXXZEA@@3P6AXXZEA 000000014001adc0     HostLogger.obj
 0002:00000dc8       ??m_strKernelFileFormat$initializer$@CHLogger@@0P6AXXZEA@@3P6AXXZEA 000000014001adc8     HostLogger.obj
 0002:00000dd0       ??m_strEtcFileFormat$initializer$@CHLogger@@0P6AXXZEA@@3P6AXXZEA 000000014001add0     HostLogger.obj
 0002:00000dd8       ??m_strRWProcessMemoryFileFormat$initializer$@CHLogger@@0P6AXXZEA@@3P6AXXZEA 000000014001add8     HostLogger.obj
 0002:00000de0       ??m_strIPCMessageFileFormat$initializer$@CHLogger@@0P6AXXZEA@@3P6AXXZEA 000000014001ade0     HostLogger.obj
 0002:00000de8       ??m_strTimeOutFileFormat$initializer$@CHLogger@@0P6AXXZEA@@3P6AXXZEA 000000014001ade8     HostLogger.obj
 0002:00000df0       ??m_strPacketFileFormat$initializer$@CHLogger@@0P6AXXZEA@@3P6AXXZEA 000000014001adf0     HostLogger.obj
 0002:00000df8       ??m_strHostName$initializer$@CHLogger@@0P6AXXZEA@@3P6AXXZEA 000000014001adf8     HostLogger.obj
 0002:00000e00       ??m_strServerName$initializer$@CHLogger@@0P6AXXZEA@@3P6AXXZEA 000000014001ae00     HostLogger.obj
 0002:00000e08       ??m_strLogFolder$initializer$@CHLogger@@0P6AXXZEA@@3P6AXXZEA 000000014001ae08     HostLogger.obj
 0002:00000e10       ??m_strModeUserCountFormat$initializer$@CHLogger@@0P6AXXZEA@@3P6AXXZEA 000000014001ae10     HostLogger.obj
 0002:00000e18       ??m_strServerAppUseCountFormat$initializer$@CHLogger@@0P6AXXZEA@@3P6AXXZEA 000000014001ae18     HostLogger.obj
 0002:00000e20       ??m_LogLock$initializer$@CHLogger@@0P6AXXZEA@@3P6AXXZEA 000000014001ae20     HostLogger.obj
 0002:00000e28       ??m_LogPacketLock$initializer$@CHLogger@@0P6AXXZEA@@3P6AXXZEA 000000014001ae28     HostLogger.obj
 0002:00000e30       ??m_vectSharedMapHandles$initializer$@CLogMsgManager@@0P6AXXZEA@@3P6AXXZEA 000000014001ae30     LogMsgManager.obj
 0002:00000e38       ?theApp$initializer$@@3P6AXXZEA 000000014001ae38     ServerApp.obj
 0002:00000e40       ?g_cServerLog$initializer$@@3P6AXXZEA 000000014001ae40     ServerAppDlg.obj
 0002:00000e48       ?__api_holder_ILTCommon_Server_g_pLTSCommon__$initializer$@@3P6AXXZEA 000000014001ae48     ServerAppDlg.obj
 0002:00000e50       ?g_sGameInfos$initializer$@@3P6AXXZEA 000000014001ae50     ServerAppDlg.obj
 0002:00000e58       ?g_sUserInfos$initializer$@@3P6AXXZEA 000000014001ae58     ServerAppDlg.obj
 0002:00000e60       ?FloatOne$initializer$@GlobalVectorConstants@@3P6AXXZEA 000000014001ae60     StdAfx.obj
 0002:00000e68       ?FloatZero$initializer$@GlobalVectorConstants@@3P6AXXZEA 000000014001ae68     StdAfx.obj
 0002:00000e70       ?FloatMinusOne$initializer$@GlobalVectorConstants@@3P6AXXZEA 000000014001ae70     StdAfx.obj
 0002:00000e78       ?FloatOneHalf$initializer$@GlobalVectorConstants@@3P6AXXZEA 000000014001ae78     StdAfx.obj
 0002:00000e80       ?XYZMask$initializer$@GlobalVectorConstants@@3P6AXXZEA 000000014001ae80     StdAfx.obj
 0002:00000e88       ?TwoPi$initializer$@GlobalVectorConstants@@3P6AXXZEA 000000014001ae88     StdAfx.obj
 0002:00000e90       ?PiByTwo$initializer$@GlobalVectorConstants@@3P6AXXZEA 000000014001ae90     StdAfx.obj
 0002:00000e98       ?OneOverTwoPi$initializer$@GlobalVectorConstants@@3P6AXXZEA 000000014001ae98     StdAfx.obj
 0002:00000ea0       ?a$initializer$@VectorSinConstantsSSE@@3P6AXXZEA 000000014001aea0     StdAfx.obj
 0002:00000ea8       ?b$initializer$@VectorSinConstantsSSE@@3P6AXXZEA 000000014001aea8     StdAfx.obj
 0002:00000eb0       ?A$initializer$@VectorSinConstantsSSE@@3P6AXXZEA 000000014001aeb0     StdAfx.obj
 0002:00000eb8       ?B$initializer$@VectorSinConstantsSSE@@3P6AXXZEA 000000014001aeb8     StdAfx.obj
 0002:00000ec0       ?PI$initializer$@@3P6AXXZEA 000000014001aec0     StdAfx.obj
 0002:00000ed8       ?pre_c_initializer@@3P6AHXZEA 000000014001aed8     msvcrt:exe_winmain.obj
 0002:00000ee0       ?post_pgo_initializer@@3P6AHXZEA 000000014001aee0     msvcrt:exe_winmain.obj
 0002:00000ee8       ?__scrt_initialize_tss_var@@3P6AHXZEA 000000014001aee8     msvcrt:thread_safe_statics.obj
 0002:00000f30       $cppxdata$?__scrt_initialize_thread_safe_statics@@YAHXZ 000000014001af30     msvcrt:thread_safe_statics.obj
 0002:00001038       GS_ExceptionPointers       000000014001b038     msvcrt:gs_report.obj
 0002:00001220       ?g_szDmp_FileName_Format@@3PEADEA 000000014001b220     BugReporter.obj
 0002:00001228       ?szDmp_ErrorFile@@3PEADEA  000000014001b228     BugReporter.obj
 0002:00001230       ?szDmp_Folder@@3PEADEA     000000014001b230     BugReporter.obj
 0002:00001238       ?AlmostTwoBits@GlobalVectorConstants@@3IB 000000014001b238     ltmodule.obj
 0002:0000123c       ?piecewise_construct@std@@3Upiecewise_construct_t@1@B 000000014001b23c     LoadXlsMsg.obj
 0002:00001240       ?AlmostTwoBits@GlobalVectorConstants@@3IB 000000014001b240     StdAfx.obj
 0002:00001250       ?g_szCommonAnimNames@@3QAY0IA@$$CBDA 000000014001b250     StdAfx.obj
 0002:00005250       ?WORLD_FORWARD@@3V?$LTVector3@M@@B 000000014001f250     ltmodule.obj
 0002:00005260       ?WORLD_RIGHT@@3V?$LTVector3@M@@B 000000014001f260     ltmodule.obj
 0002:00005270       ?WORLD_UP@@3V?$LTVector3@M@@B 000000014001f270     ltmodule.obj
 0002:00005280       ?WORLD_FORWARD@@3V?$LTVector3@M@@B 000000014001f280     StdAfx.obj
 0002:00005290       ?WORLD_RIGHT@@3V?$LTVector3@M@@B 000000014001f290     StdAfx.obj
 0002:000052a0       ?WORLD_UP@@3V?$LTVector3@M@@B 000000014001f2a0     StdAfx.obj
 0002:00005db8       ?messageMap@?1??GetThisMessageMap@CServerAppApp@@KAPEBUAFX_MSGMAP@@XZ@4U3@B 000000014001fdb8     ServerApp.obj
 0002:00005dd0       ?_messageEntries@?1??GetThisMessageMap@CServerAppApp@@KAPEBUAFX_MSGMAP@@XZ@4QBUAFX_MSGMAP_ENTRY@@B 000000014001fdd0     ServerApp.obj
 0002:000074e8       ?messageMap@?1??GetThisMessageMap@CServerAppDlg@@KAPEBUAFX_MSGMAP@@XZ@4U3@B 00000001400214e8     ServerAppDlg.obj
 0002:00007500       ?_messageEntries@?1??GetThisMessageMap@CServerAppDlg@@KAPEBUAFX_MSGMAP@@XZ@4QBUAFX_MSGMAP_ENTRY@@B 0000000140021500     ServerAppDlg.obj
 0002:00008078       $cppxdata$?threadCreateDumpFile@@YAKPEAX@Z 0000000140022078     BugReporter.obj
 0002:000080a0       $cppxdata$?CRSUploader@@YAAEAVUploader@crs@@XZ 00000001400220a0     BugReporter.obj
 0002:00008190       $cppxdata$?readURL@Uploader@crs@@AEAAXAEAV?$basic_string@_WU?$char_traits@_W@std@@V?$allocator@_W@2@@std@@@Z 0000000140022190     crs_uploader.obj
 0002:000081b8       $cppxdata$?init@Uploader@crs@@QEAA_N_NPEAD1@Z 00000001400221b8     crs_uploader.obj
 0002:000081e0       $cppxdata$?TransferFrom@CInterfaceNameMgr@@QEAAXPEAV1@@Z 00000001400221e0     ltmodule.obj
 0002:00008208       $cppxdata$??0CInterfaceNameMgr@@QEAA@PEBDH@Z 0000000140022208     ltmodule.obj
 0002:00008230       $cppxdata$?TransferFrom@CInterfaceDatabase@@UEAAXPEAV1@@Z 0000000140022230     ltmodule.obj
 0002:00008258       $cppxdata$?Add@CInterfaceDatabase@@EEAAXPEAVCInterfaceChooser@@@Z 0000000140022258     ltmodule.obj
 0002:00008280       $cppxdata$?Add@CInterfaceDatabase@@EEAAXPEAVCAPIHolderBase@@@Z 0000000140022280     ltmodule.obj
 0002:000082a8       $cppxdata$?Add@CInterfaceDatabase@@EEAAXPEAVIBase@@PEBDH@Z 00000001400222a8     ltmodule.obj
 0002:000082d0       $cppxdata$?AddHolder@CInterfaceDatabase@@SAXPEAVCAPIHolderBase@@@Z 00000001400222d0     ltmodule.obj
 0002:000082f8       $cppxdata$??0CInterfaceDatabase@@QEAA@XZ 00000001400222f8     ltmodule.obj
 0002:00008320       $cppxdata$?_DoLogWithLevel@CHLogger@@CAXPEBDW4ELOG_LEVEL@1@0PEAD@Z 0000000140022320     HostLogger.obj
 0002:00008348       $cppxdata$?_BuildDirectory@CHLogger@@CAXAEBU_SYSTEMTIME@@@Z 0000000140022348     HostLogger.obj
 0002:00008370       $cppxdata$?LogPacket@CHLogger@@SAXPEBDZZ 0000000140022370     HostLogger.obj
 0002:00008398       $cppxdata$?_WriteXlsDataToSharedMemory@CLogMsgManager@@CA_NXZ 0000000140022398     LogMsgManager.obj
 0002:000083c0       $cppxdata$?Init@CLogMsgManager@@SA_NW4ESHARED_MEM_USAGE_TYPE@1@@Z 00000001400223c0     LogMsgManager.obj
 0002:000083e8       $cppxdata$??$_Insert_nohint@AEAU?$pair@$$CB_JV?$basic_string@DU?$char_traits@D@std@@V?$allocator@D@2@@std@@@std@@PEAU?$_Tree_node@U?$pair@$$CB_JV?$basic_string@DU?$char_traits@D@std@@V?$allocator@D@2@@std@@@std@@PEAX@2@@?$_Tree@V?$_Tmap_traits@_JV?$basic_string@DU?$char_traits@D@std@@V?$allocator@D@2@@std@@U?$less@_J@2@V?$allocator@U?$pair@$$CB_JV?$basic_string@DU?$char_traits@D@std@@V?$allocator@D@2@@std@@@std@@@2@$0A@@std@@@std@@IEAA?AU?$pair@V?$_Tree_iterator@V?$_Tree_val@U?$_Tree_simple_types@U?$pair@$$CB_JV?$basic_string@DU?$char_traits@D@std@@V?$allocator@D@2@@std@@@std@@@std@@@std@@@std@@_N@1@_NAEAU?$pair@$$CB_JV?$basic_string@DU?$char_traits@D@std@@V?$allocator@D@2@@std@@@1@PEAU?$_Tree_node@U?$pair@$$CB_JV?$basic_string@DU?$char_traits@D@std@@V?$allocator@D@2@@std@@@std@@PEAX@1@@Z 00000001400223e8     LoadXlsMsg.obj
 0002:00008410       $cppxdata$??$_Insert_hint@AEAU?$pair@$$CB_JV?$basic_string@DU?$char_traits@D@std@@V?$allocator@D@2@@std@@@std@@PEAU?$_Tree_node@U?$pair@$$CB_JV?$basic_string@DU?$char_traits@D@std@@V?$allocator@D@2@@std@@@std@@PEAX@2@@?$_Tree@V?$_Tmap_traits@_JV?$basic_string@DU?$char_traits@D@std@@V?$allocator@D@2@@std@@U?$less@_J@2@V?$allocator@U?$pair@$$CB_JV?$basic_string@DU?$char_traits@D@std@@V?$allocator@D@2@@std@@@std@@@2@$0A@@std@@@std@@IEAA?AV?$_Tree_iterator@V?$_Tree_val@U?$_Tree_simple_types@U?$pair@$$CB_JV?$basic_string@DU?$char_traits@D@std@@V?$allocator@D@2@@std@@@std@@@std@@@std@@@1@V?$_Tree_const_iterator@V?$_Tree_val@U?$_Tree_simple_types@U?$pair@$$CB_JV?$basic_string@DU?$char_traits@D@std@@V?$allocator@D@2@@std@@@std@@@std@@@std@@@1@AEAU?$pair@$$CB_JV?$basic_string@DU?$char_traits@D@std@@V?$allocator@D@2@@std@@@1@PEAU?$_Tree_node@U?$pair@$$CB_JV?$basic_string@DU?$char_traits@D@std@@V?$allocator@D@2@@std@@@std@@PEAX@1@@Z 0000000140022410     LoadXlsMsg.obj
 0002:00008438       $cppxdata$?erase@?$_Tree@V?$_Tmap_traits@_JV?$basic_string@DU?$char_traits@D@std@@V?$allocator@D@2@@std@@U?$less@_J@2@V?$allocator@U?$pair@$$CB_JV?$basic_string@DU?$char_traits@D@std@@V?$allocator@D@2@@std@@@std@@@2@$0A@@std@@@std@@QEAA?AV?$_Tree_iterator@V?$_Tree_val@U?$_Tree_simple_types@U?$pair@$$CB_JV?$basic_string@DU?$char_traits@D@std@@V?$allocator@D@2@@std@@@std@@@std@@@std@@@2@V?$_Tree_const_iterator@V?$_Tree_val@U?$_Tree_simple_types@U?$pair@$$CB_JV?$basic_string@DU?$char_traits@D@std@@V?$allocator@D@2@@std@@@std@@@std@@@std@@@2@0@Z 0000000140022438     LoadXlsMsg.obj
 0002:00008460       $cppxdata$??_GFindXlsMsg@@UEAAPEAXI@Z 0000000140022460     LoadXlsMsg.obj
 0002:00008488       $cppxdata$?LoadWMszFile@FindXlsMsg@@QEAA_NPEAD@Z 0000000140022488     LoadXlsMsg.obj
 0002:000084b0       $cppxdata$?Run@CServerAppApp@@UEAAHXZ 00000001400224b0     ServerApp.obj
 0002:000084d8       $cppxdata$??1CWaitCursor@@QEAA@XZ 00000001400224d8     ServerAppDlg.obj
 0002:00008500       $cppxdata$??$?HDU?$char_traits@D@std@@V?$allocator@D@1@@std@@YA?AV?$basic_string@DU?$char_traits@D@std@@V?$allocator@D@2@@0@AEBV10@0@Z 0000000140022500     ServerAppDlg.obj
 0002:00008528       $cppxdata$??1?$CAPIHolder@VILTCommon@@@@UEAA@XZ 0000000140022528     ServerAppDlg.obj
 0002:00008550       $cppxdata$?SendToServerShellAutoMatchStartingUserInfo@CServerAppDlg@@AEAAXPEAUtagCOPYDATASTRUCT@@@Z 0000000140022550     ServerAppDlg.obj
 0002:00008578       $cppxdata$?GetDownloadPath@CServerAppDlg@@AEAA?AV?$basic_string@DU?$char_traits@D@std@@V?$allocator@D@2@@std@@XZ 0000000140022578     ServerAppDlg.obj
 0002:000085a0       $cppxdata$?SendServerAppInitFail@CServerAppDlg@@AEAAXHH@Z 00000001400225a0     ServerAppDlg.obj
 0002:000085c8       $cppxdata$?DownloadUCCMapFile_HTTP@CServerAppDlg@@AEAA?AW4UCCMAPDOWNLOADREAULT@@V?$basic_string@DU?$char_traits@D@std@@V?$allocator@D@2@@std@@@Z 00000001400225c8     ServerAppDlg.obj
 0002:000085f0       $cppxdata$?SendServerAppInit@CServerAppDlg@@AEAAXXZ 00000001400225f0     ServerAppDlg.obj
 0002:00008618       $cppxdata$?RECV_MSG_USER_DISCONNECTED@CServerAppDlg@@AEAAX_J@Z 0000000140022618     ServerAppDlg.obj
 0002:00008640       $cppxdata$?RECV_MSG_AIITEM_GROUP_RATE_RESULT@CServerAppDlg@@AEAAX_J@Z 0000000140022640     ServerAppDlg.obj
 0002:00008668       $cppxdata$?RECV_MSG_AIITEM_DEC@CServerAppDlg@@AEAAX_J@Z 0000000140022668     ServerAppDlg.obj
 0002:00008690       $cppxdata$?RECV_MSG_INSERTCHARACTER@CServerAppDlg@@AEAAX_J@Z 0000000140022690     ServerAppDlg.obj
 0002:000086b8       $cppxdata$?GetOptionValueString@CServerAppDlg@@IEAA?AV?$basic_string@DU?$char_traits@D@std@@V?$allocator@D@2@@std@@V23@00@Z 00000001400226b8     ServerAppDlg.obj
 0002:000086e0       $cppxdata$?LoadHostGameInfo@CServerAppDlg@@IEAAXXZ 00000001400226e0     ServerAppDlg.obj
 0002:00008708       $cppxdata$?SaveHostGameInfo@CServerAppDlg@@IEAAXXZ 0000000140022708     ServerAppDlg.obj
 0002:00008730       $cppxdata$?OnTimer@CServerAppDlg@@QEAAX_K@Z 0000000140022730     ServerAppDlg.obj
 0002:00008758       $cppxdata$?OnCopyData@CServerAppDlg@@IEAAHPEAVCWnd@@PEAUtagCOPYDATASTRUCT@@@Z 0000000140022758     ServerAppDlg.obj
 0002:00008780       $cppxdata$?OnGameServerMsg@CServerAppDlg@@IEAA_J_K_J@Z 0000000140022780     ServerAppDlg.obj
 0002:000087a8       $cppxdata$?AddResources@CServerAppDlg@@QEAA_NXZ 00000001400227a8     ServerAppDlg.obj
 0002:000087d0       $cppxdata$?ServerUpdate@CServerAppDlg@@QEAAXXZ 00000001400227d0     ServerAppDlg.obj
 0002:000087f8       $cppxdata$?ThreadUpdate@CServerAppDlg@@SAXPEAX@Z 00000001400227f8     ServerAppDlg.obj
 0002:00008820       $cppxdata$?Thread_SendUserInfo@@YAXPEAVCServerAppDlg@@AEAUPROTO_GAME_USER_INFO_tag@@@Z 0000000140022820     ServerAppDlg.obj
 0002:00008848       $cppxdata$?Thread_SendGameInfo@@YAXPEAVCServerAppDlg@@AEAUPROTO_START_HOST_tag@@@Z 0000000140022848     ServerAppDlg.obj
 0002:00008870       $cppxdata$?StopServer@CServerAppDlg@@QEAA_NXZ 0000000140022870     ServerAppDlg.obj
 0002:00008898       $cppxdata$?RunServer@CServerAppDlg@@QEAA_NXZ 0000000140022898     ServerAppDlg.obj
 0002:000088c0       $cppxdata$?LoadServer@CServerAppDlg@@QEAA_NXZ 00000001400228c0     ServerAppDlg.obj
 0002:000088e8       $cppxdata$?AddServerMsg@CServerAppDlg@@QEAAXPEBDH@Z 00000001400228e8     ServerAppDlg.obj
 0002:00008910       $cppxdata$?OnShellMessage@CServerAppDlg@@QEAAXAEAVILTMessage_Read@@@Z 0000000140022910     ServerAppDlg.obj
 0002:00008938       $cppxdata$?OnInitDialog@CServerAppDlg@@MEAAHXZ 0000000140022938     ServerAppDlg.obj
 0002:00008960       $cppxdata$?OutOfMemory@CGameServerAppHandler@@UEAAIXZ 0000000140022960     ServerAppDlg.obj
 0002:00008988       $cppxdata$?ConsoleOutputFn@CGameServerAppHandler@@UEAAIHHPEBD@Z 0000000140022988     ServerAppDlg.obj
 0002:000089b0       $cppxdata$??__E__api_holder_ILTCommon_Server_g_pLTSCommon__@@YAXXZ 00000001400229b0     ServerAppDlg.obj
 0002:000089d8       $cppxdata$??0CServerAppDlg@@QEAA@PEAVCWnd@@@Z 00000001400229d8     ServerAppDlg.obj
 0002:00008a00       $cppxdata$??1CServerAppDlg@@UEAA@XZ 0000000140022a00     ServerAppDlg.obj
 0002:00008a28       $cppxdata$??$?6U?$char_traits@D@std@@@std@@YAAEAV?$basic_ostream@DU?$char_traits@D@std@@@0@AEAV10@PEBD@Z 0000000140022a28     safe_string_x64:safe_string.obj
 0002:00008a50       $cppxdata$??1_Sentry_base@?$basic_ostream@DU?$char_traits@D@std@@@std@@QEAA@XZ 0000000140022a50     safe_string_x64:safe_string.obj
 0002:00008a78       $cppxdata$??1sentry@?$basic_ostream@DU?$char_traits@D@std@@@std@@QEAA@XZ 0000000140022a78     safe_string_x64:safe_string.obj
 0002:00008aa0       $cppxdata$??0?$basic_stringstream@DU?$char_traits@D@std@@V?$allocator@D@2@@std@@QEAA@H@Z 0000000140022aa0     safe_string_x64:safe_string.obj
 0002:00008ac8       $cppxdata$?strncpy_s@cf@@YAHPEAD_KPEBD1@Z 0000000140022ac8     safe_string_x64:safe_string.obj
 0002:00008af0       $cppxdata$?sprintf_s@internal@cf@@YAHPEAD_KPEBDAEAPEAD@Z 0000000140022af0     safe_string_x64:safe_string.obj
 0002:00008b18       $cppxdata$?strcpy_s@cf@@YAHPEAD_KPEBD@Z 0000000140022b18     safe_string_x64:safe_string.obj
 0002:0000a120       $unwind$?CRSUploader@@YAAEAVUploader@crs@@XZ 0000000140024120     BugReporter.obj
 0002:0000a134       $stateUnwindMap$?CRSUploader@@YAAEAVUploader@crs@@XZ 0000000140024134     BugReporter.obj
 0002:0000a150       $ip2state$?CRSUploader@@YAAEAVUploader@crs@@XZ 0000000140024150     BugReporter.obj
 0002:0000a160       $unwind$?filt$0@?0??__scrt_common_main_seh@@YAHXZ@4HA 0000000140024160     msvcrt:exe_winmain.obj
 0002:0000a160       $unwind$?dtor$1@?0??TransferFrom@CInterfaceNameMgr@@QEAAXPEAV1@@Z@4HA 0000000140024160     ltmodule.obj
 0002:0000a160       $unwind$?dtor$0@?0??TransferFrom@CInterfaceNameMgr@@QEAAXPEAV1@@Z@4HA 0000000140024160     ltmodule.obj
 0002:0000a160       $unwind$?dtor$6@?0??LoadServer@CServerAppDlg@@QEAA_NXZ@4HA 0000000140024160     ServerAppDlg.obj
 0002:0000a160       $unwind$?dtor$2@?0??TransferFrom@CInterfaceNameMgr@@QEAAXPEAV1@@Z@4HA 0000000140024160     ltmodule.obj
 0002:0000a160       $unwind$?dtor$0@?0???0CInterfaceNameMgr@@QEAA@PEBDH@Z@4HA 0000000140024160     ltmodule.obj
 0002:0000a160       $unwind$?dtor$2@?0???0CInterfaceNameMgr@@QEAA@PEBDH@Z@4HA 0000000140024160     ltmodule.obj
 0002:0000a160       $unwind$?dtor$0@?0??Add@CInterfaceDatabase@@EEAAXPEAVCInterfaceChooser@@@Z@4HA 0000000140024160     ltmodule.obj
 0002:0000a160       $unwind$?dtor$0@?0??Add@CInterfaceDatabase@@EEAAXPEAVCAPIHolderBase@@@Z@4HA 0000000140024160     ltmodule.obj
 0002:0000a160       $unwind$?dtor$0@?0???0?$basic_stringstream@DU?$char_traits@D@std@@V?$allocator@D@2@@std@@QEAA@H@Z@4HA 0000000140024160     safe_string_x64:safe_string.obj
 0002:0000a160       $unwind$?dtor$1@?0??Init@CLogMsgManager@@SA_NW4ESHARED_MEM_USAGE_TYPE@1@@Z@4HA 0000000140024160     LogMsgManager.obj
 0002:0000a160       $unwind$?dtor$0@?0??Add@CInterfaceDatabase@@EEAAXPEAVIBase@@PEBDH@Z@4HA 0000000140024160     ltmodule.obj
 0002:0000a160       $unwind$?dtor$40@?0??DownloadUCCMapFile_HTTP@CServerAppDlg@@AEAA?AW4UCCMAPDOWNLOADREAULT@@V?$basic_string@DU?$char_traits@D@std@@V?$allocator@D@2@@std@@@Z@4HA 0000000140024160     ServerAppDlg.obj
 0002:0000a160       $unwind$?dtor$22@?0??DownloadUCCMapFile_HTTP@CServerAppDlg@@AEAA?AW4UCCMAPDOWNLOADREAULT@@V?$basic_string@DU?$char_traits@D@std@@V?$allocator@D@2@@std@@@Z@4HA 0000000140024160     ServerAppDlg.obj
 0002:0000a160       $unwind$?dtor$0@?0??Init@CLogMsgManager@@SA_NW4ESHARED_MEM_USAGE_TYPE@1@@Z@4HA 0000000140024160     LogMsgManager.obj
 0002:0000a160       $unwind$?dtor$4@?0??strncpy_s@cf@@YAHPEAD_KPEBD1@Z@4HA 0000000140024160     safe_string_x64:safe_string.obj
 0002:0000a160       $unwind$?dtor$0@?0??GetDownloadPath@CServerAppDlg@@AEAA?AV?$basic_string@DU?$char_traits@D@std@@V?$allocator@D@2@@std@@XZ@4HA 0000000140024160     ServerAppDlg.obj
 0002:0000a160       $unwind$?dtor$0@?0??AddHolder@CInterfaceDatabase@@SAXPEAVCAPIHolderBase@@@Z@4HA 0000000140024160     ltmodule.obj
 0002:0000a160       $unwind$?dtor$4@?0??sprintf_s@internal@cf@@YAHPEAD_KPEBDAEAPEAD@Z@4HA 0000000140024160     safe_string_x64:safe_string.obj
 0002:0000a160       $unwind$?dtor$1@?0???0CInterfaceDatabase@@QEAA@XZ@4HA 0000000140024160     ltmodule.obj
 0002:0000a160       $unwind$?dtor$0@?0???$?HDU?$char_traits@D@std@@V?$allocator@D@1@@std@@YA?AV?$basic_string@DU?$char_traits@D@std@@V?$allocator@D@2@@0@AEBV10@0@Z@4HA 0000000140024160     ServerAppDlg.obj
 0002:0000a160       $unwind$?dtor$4@?0??strcpy_s@cf@@YAHPEAD_KPEBD@Z@4HA 0000000140024160     safe_string_x64:safe_string.obj
 0002:0000a160       $unwind$?dtor$1@?0???0CInterfaceNameMgr@@QEAA@PEBDH@Z@4HA 0000000140024160     ltmodule.obj
 0002:0000a160       $unwind$?dtor$0@?0??TransferFrom@CInterfaceDatabase@@UEAAXPEAV1@@Z@4HA 0000000140024160     ltmodule.obj
 0002:0000a160       $unwind$?dtor$1@?0??CRSUploader@@YAAEAVUploader@crs@@XZ@4HA 0000000140024160     BugReporter.obj
 0002:0000a168       $unwind$?threadCreateDumpFile@@YAKPEAX@Z 0000000140024168     BugReporter.obj
 0002:0000a190       $stateUnwindMap$?threadCreateDumpFile@@YAKPEAX@Z 0000000140024190     BugReporter.obj
 0002:0000a198       $ip2state$?threadCreateDumpFile@@YAKPEAX@Z 0000000140024198     BugReporter.obj
 0002:0000a1b0       $unwind$?CrashExceptionDump@@YAJPEAU_EXCEPTION_POINTERS@@@Z 00000001400241b0     BugReporter.obj
 0002:0000a1b8       $chain$0$?CrashExceptionDump@@YAJPEAU_EXCEPTION_POINTERS@@@Z 00000001400241b8     BugReporter.obj
 0002:0000a1cc       $chain$1$?CrashExceptionDump@@YAJPEAU_EXCEPTION_POINTERS@@@Z 00000001400241cc     BugReporter.obj
 0002:0000a1dc       $unwind$?InitBugReporter@@YAXPEAD0000@Z 00000001400241dc     BugReporter.obj
 0002:0000a1fc       $unwind$??$sprintf_s@$0CA@@cf@@YAHAEAY0CA@DPEBDZZ 00000001400241fc     LogMsgManager.obj
 0002:0000a1fc       $unwind$??$sprintf_s@$0EA@@cf@@YAHAEAY0EA@DPEBDZZ 00000001400241fc     RWPMLog.obj
 0002:0000a1fc       $unwind$??$sprintf_s@$0BAA@@cf@@YAHAEAY0BAA@DPEBDZZ 00000001400241fc     BugReporter.obj
 0002:0000a1fc       $unwind$??$sprintf_s@$0BAE@@cf@@YAHAEAY0BAE@DPEBDZZ 00000001400241fc     BugReporter.obj
 0002:0000a1fc       $unwind$??$sprintf_s@$0DOJ@@cf@@YAHAEAY0DOJ@DPEBDZZ 00000001400241fc     BugReporter.obj
 0002:0000a1fc       $unwind$??$sprintf_s@$0BJB@@cf@@YAHAEAY0BJB@DPEBDZZ 00000001400241fc     BugReporter.obj
 0002:0000a1fc       $unwind$??$sprintf_s@$0IA@@cf@@YAHAEAY0IA@DPEBDZZ 00000001400241fc     ServerAppDlg.obj
 0002:0000a1fc       $unwind$??$sprintf_s@$0BE@@cf@@YAHAEAY0BE@DPEBDZZ 00000001400241fc     BugReporter.obj
 0002:0000a204       $unwind$__scrt_uninitialize_crt 0000000140024204     msvcrt:utility.obj
 0002:0000a204       $unwind$??_Gtype_info@@UEAAPEAXI@Z 0000000140024204     msvcrt:std_type_info_static.obj
 0002:0000a204       $unwind$?Run@CInterfaceDatabase@@EEAA?AW4EChooserRun@@PEAVCInterfaceChooser@@@Z 0000000140024204     ltmodule.obj
 0002:0000a204       $unwind$__raise_securityfailure 0000000140024204     msvcrt:gs_report.obj
 0002:0000a204       $unwind$_Init_thread_header 0000000140024204     msvcrt:thread_safe_statics.obj
 0002:0000a204       $unwind$__scrt_initialize_crt 0000000140024204     msvcrt:utility.obj
 0002:0000a204       $unwind$??1?$auto_ptr@VUrl@crs@@@std@@QEAA@XZ 0000000140024204     crs_uploader.obj
 0002:0000a204       $unwind$??1?$basic_stringbuf@DU?$char_traits@D@std@@V?$allocator@D@2@@std@@UEAA@XZ 0000000140024204     safe_string_x64:safe_string.obj
 0002:0000a204       $unwind$??$_Buynode@AEBUpiecewise_construct_t@std@@V?$tuple@AEB_J@2@V?$tuple@$$V@2@@?$_Tree_comp_alloc@V?$_Tmap_traits@_JV?$basic_string@DU?$char_traits@D@std@@V?$allocator@D@2@@std@@U?$less@_J@2@V?$allocator@U?$pair@$$CB_JV?$basic_string@DU?$char_traits@D@std@@V?$allocator@D@2@@std@@@std@@@2@$0A@@std@@@std@@QEAAPEAU?$_Tree_node@U?$pair@$$CB_JV?$basic_string@DU?$char_traits@D@std@@V?$allocator@D@2@@std@@@std@@PEAX@1@AEBUpiecewise_construct_t@1@$$QEAV?$tuple@AEB_J@1@$$QEAV?$tuple@$$V@1@@Z 0000000140024204     LoadXlsMsg.obj
 0002:0000a204       $unwind$??1tUCCGamePlayInfo@CServerAppDlg@@QEAA@XZ 0000000140024204     ServerAppDlg.obj
 0002:0000a204       $unwind$?_Tidy_deallocate@?$basic_string@_WU?$char_traits@_W@std@@V?$allocator@_W@2@@std@@QEAAXXZ 0000000140024204     crs_uploader.obj
 0002:0000a204       $unwind$??1CAtlBaseModule@ATL@@QEAA@XZ 0000000140024204     atls:atlbase.obj
 0002:0000a204       $unwind$??1?$basic_string@_WU?$char_traits@_W@std@@V?$allocator@_W@2@@std@@QEAA@XZ 0000000140024204     crs_uploader.obj
 0002:0000a204       $unwind$??$endl@DU?$char_traits@D@std@@@std@@YAAEAV?$basic_ostream@DU?$char_traits@D@std@@@0@AEAV10@@Z 0000000140024204     safe_string_x64:safe_string.obj
 0002:0000a204       $unwind$?_Destroy_if_node@?$_Tree@V?$_Tmap_traits@_JV?$basic_string@DU?$char_traits@D@std@@V?$allocator@D@2@@std@@U?$less@_J@2@V?$allocator@U?$pair@$$CB_JV?$basic_string@DU?$char_traits@D@std@@V?$allocator@D@2@@std@@@std@@@2@$0A@@std@@@std@@IEAAXPEAU?$_Tree_node@U?$pair@$$CB_JV?$basic_string@DU?$char_traits@D@std@@V?$allocator@D@2@@std@@@std@@PEAX@2@@Z 0000000140024204     LoadXlsMsg.obj
 0002:0000a204       $unwind$??1Uploader@crs@@QEAA@XZ 0000000140024204     crs_uploader.obj
 0002:0000a204       $unwind$__scrt_release_startup_lock 0000000140024204     msvcrt:utility.obj
 0002:0000a204       $unwind$??1CServerLog@@UEAA@XZ 0000000140024204     LogMgmt.obj
 0002:0000a204       $unwind$_onexit            0000000140024204     msvcrt:utility.obj
 0002:0000a204       $unwind$??0exception@std@@QEAA@AEBV01@@Z 0000000140024204     ServerAppDlg.obj
 0002:0000a204       $unwind$??_D?$basic_stringstream@DU?$char_traits@D@std@@V?$allocator@D@2@@std@@QEAAXXZ 0000000140024204     safe_string_x64:safe_string.obj
 0002:0000a204       $unwind$_Init_thread_wait  0000000140024204     msvcrt:thread_safe_statics.obj
 0002:0000a204       $unwind$??1?$basic_string@DU?$char_traits@D@std@@V?$allocator@D@2@@std@@QEAA@XZ 0000000140024204     BugReporter.obj
 0002:0000a204       $unwind$_Init_thread_footer 0000000140024204     msvcrt:thread_safe_statics.obj
 0002:0000a204       $unwind$_Init_thread_abort 0000000140024204     msvcrt:thread_safe_statics.obj
 0002:0000a204       $unwind$?_Buynode0@?$_Tree_comp_alloc@V?$_Tmap_traits@_JV?$basic_string@DU?$char_traits@D@std@@V?$allocator@D@2@@std@@U?$less@_J@2@V?$allocator@U?$pair@$$CB_JV?$basic_string@DU?$char_traits@D@std@@V?$allocator@D@2@@std@@@std@@@2@$0A@@std@@@std@@QEAAPEAU?$_Tree_node@U?$pair@$$CB_JV?$basic_string@DU?$char_traits@D@std@@V?$allocator@D@2@@std@@@std@@PEAX@2@XZ 0000000140024204     LoadXlsMsg.obj
 0002:0000a204       $unwind$?pre_c_initialization@@YAHXZ 0000000140024204     msvcrt:exe_winmain.obj
 0002:0000a20c       $unwind$??__F?m_strPacketFileFormat@CHLogger@@0V?$basic_string@DU?$char_traits@D@std@@V?$allocator@D@2@@std@@A@@YAXXZ 000000014002420c     HostLogger.obj
 0002:0000a20c       $unwind$??__F?m_strTimeOutFileFormat@CHLogger@@0V?$basic_string@DU?$char_traits@D@std@@V?$allocator@D@2@@std@@A@@YAXXZ 000000014002420c     HostLogger.obj
 0002:0000a20c       $unwind$?_Xlen@?$basic_string@DU?$char_traits@D@std@@V?$allocator@D@2@@std@@SAXXZ 000000014002420c     BugReporter.obj
 0002:0000a20c       $unwind$??__F?m_strServerAppUseCountFormat@CHLogger@@0V?$basic_string@DU?$char_traits@D@std@@V?$allocator@D@2@@std@@A@@YAXXZ 000000014002420c     HostLogger.obj
 0002:0000a20c       $unwind$??__F?m_strIPCMessageFileFormat@CHLogger@@0V?$basic_string@DU?$char_traits@D@std@@V?$allocator@D@2@@std@@A@@YAXXZ 000000014002420c     HostLogger.obj
 0002:0000a20c       $unwind$??__E?m_LogPacketLock@CHLogger@@0VCMustSyncObjectLog@@A@@YAXXZ 000000014002420c     HostLogger.obj
 0002:0000a20c       $unwind$??__E_afxInitAppState@@YAXXZ 000000014002420c     mfcs140:appmodul.obj
 0002:0000a20c       $unwind$??__EPI@@YAXXZ     000000014002420c     StdAfx.obj
 0002:0000a20c       $unwind$??__Eb@VectorSinConstantsSSE@@YAXXZ 000000014002420c     StdAfx.obj
 0002:0000a20c       $unwind$??__F?m_strKernelFileFormat@CHLogger@@0V?$basic_string@DU?$char_traits@D@std@@V?$allocator@D@2@@std@@A@@YAXXZ 000000014002420c     HostLogger.obj
 0002:0000a20c       $unwind$??__F?m_strEtcFileFormat@CHLogger@@0V?$basic_string@DU?$char_traits@D@std@@V?$allocator@D@2@@std@@A@@YAXXZ 000000014002420c     HostLogger.obj
 0002:0000a20c       $unwind$?ShellMessageFn@CGameServerAppHandler@@UEAAIAEAVILTMessage_Read@@@Z 000000014002420c     ServerAppDlg.obj
 0002:0000a20c       $unwind$__GSHandlerCheck   000000014002420c     msvcrt:gshandler.obj
 0002:0000a20c       $unwind$_Init_thread_notify 000000014002420c     msvcrt:thread_safe_statics.obj
 0002:0000a20c       $unwind$?__scrt_uninitialize_thread_safe_statics@@YAXXZ 000000014002420c     msvcrt:thread_safe_statics.obj
 0002:0000a20c       $unwind$?_Xlen@?$basic_string@_WU?$char_traits@_W@std@@V?$allocator@_W@2@@std@@SAXXZ 000000014002420c     crs_uploader.obj
 0002:0000a20c       $unwind$??__F?m_strHostName@CHLogger@@0V?$basic_string@DU?$char_traits@D@std@@V?$allocator@D@2@@std@@A@@YAXXZ 000000014002420c     HostLogger.obj
 0002:0000a20c       $unwind$??__EtheApp@@YAXXZ 000000014002420c     ServerApp.obj
 0002:0000a20c       $unwind$??__Ea@VectorSinConstantsSSE@@YAXXZ 000000014002420c     ltmodule.obj
 0002:0000a20c       $unwind$__scrt_initialize_default_local_stdio_options 000000014002420c     msvcrt:default_local_stdio_options.obj
 0002:0000a20c       $unwind$??__Eb@VectorSinConstantsSSE@@YAXXZ 000000014002420c     ltmodule.obj
 0002:0000a20c       $unwind$??__F?m_strRWProcessMemoryFileFormat@CHLogger@@0V?$basic_string@DU?$char_traits@D@std@@V?$allocator@D@2@@std@@A@@YAXXZ 000000014002420c     HostLogger.obj
 0002:0000a20c       $unwind$??__EPI@@YAXXZ     000000014002420c     ltmodule.obj
 0002:0000a20c       $unwind$??__Ea@VectorSinConstantsSSE@@YAXXZ 000000014002420c     StdAfx.obj
 0002:0000a20c       $unwind$??__F?m_strServerName@CHLogger@@0V?$basic_string@DU?$char_traits@D@std@@V?$allocator@D@2@@std@@A@@YAXXZ 000000014002420c     HostLogger.obj
 0002:0000a20c       $unwind$?_Buyheadnode@?$_Tree_comp_alloc@V?$_Tmap_traits@_JV?$basic_string@DU?$char_traits@D@std@@V?$allocator@D@2@@std@@U?$less@_J@2@V?$allocator@U?$pair@$$CB_JV?$basic_string@DU?$char_traits@D@std@@V?$allocator@D@2@@std@@@std@@@2@$0A@@std@@@std@@QEAAPEAU?$_Tree_node@U?$pair@$$CB_JV?$basic_string@DU?$char_traits@D@std@@V?$allocator@D@2@@std@@@std@@PEAX@2@XZ 000000014002420c     LoadXlsMsg.obj
 0002:0000a20c       $unwind$atexit             000000014002420c     msvcrt:utility.obj
 0002:0000a20c       $unwind$??__F?m_strFileFormat@CHLogger@@0V?$basic_string@DU?$char_traits@D@std@@V?$allocator@D@2@@std@@A@@YAXXZ 000000014002420c     HostLogger.obj
 0002:0000a20c       $unwind$??__F?m_strModeUserCountFormat@CHLogger@@0V?$basic_string@DU?$char_traits@D@std@@V?$allocator@D@2@@std@@A@@YAXXZ 000000014002420c     HostLogger.obj
 0002:0000a20c       $unwind$?post_pgo_initialization@@YAHXZ 000000014002420c     msvcrt:exe_winmain.obj
 0002:0000a20c       $unwind$?check_delete_pointers@@YAXXZ 000000014002420c     ltmodule.obj
 0002:0000a20c       $unwind$__scrt_unhandled_exception_filter 000000014002420c     msvcrt:utility_desktop.obj
 0002:0000a20c       $unwind$?NetworkDelayCount@CGameServerAppHandler@@UEAAIXZ 000000014002420c     ServerAppDlg.obj
 0002:0000a20c       $unwind$?_Xlength@?$vector@PEAXV?$allocator@PEAX@std@@@std@@CAXXZ 000000014002420c     LogMsgManager.obj
 0002:0000a20c       $unwind$?pre_cpp_initialization@@YAXXZ 000000014002420c     msvcrt:exe_winmain.obj
 0002:0000a20c       $unwind$?_Xran@?$_String_val@U?$_Simple_types@D@std@@@std@@SAXXZ 000000014002420c     HostLogger.obj
 0002:0000a20c       $unwind$__scrt_is_managed_app 000000014002420c     msvcrt:utility_desktop.obj
 0002:0000a20c       $unwind$??__E_AtlBaseModule@ATL@@YAXXZ 000000014002420c     atls:atlbase.obj
 0002:0000a20c       $unwind$__scrt_acquire_startup_lock 000000014002420c     msvcrt:utility.obj
 0002:0000a20c       $unwind$??__F?m_strBRFileFormat@CHLogger@@0V?$basic_string@DU?$char_traits@D@std@@V?$allocator@D@2@@std@@A@@YAXXZ 000000014002420c     HostLogger.obj
 0002:0000a20c       $unwind$??__F?m_vectSharedMapHandles@CLogMsgManager@@0V?$vector@PEAXV?$allocator@PEAX@std@@@std@@A@@YAXXZ 000000014002420c     LogMsgManager.obj
 0002:0000a20c       $unwind$??__F?m_strLogFolder@CHLogger@@0V?$basic_string@DU?$char_traits@D@std@@V?$allocator@D@2@@std@@A@@YAXXZ 000000014002420c     HostLogger.obj
 0002:0000a20c       $unwind$WinMainCRTStartup  000000014002420c     msvcrt:exe_winmain.obj
 0002:0000a20c       $unwind$??__E?m_LogLock@CHLogger@@0VCMustSyncObjectLog@@A@@YAXXZ 000000014002420c     HostLogger.obj
 0002:0000a214       $unwind$?assign@?$basic_string@DU?$char_traits@D@std@@V?$allocator@D@2@@std@@QEAAAEAV12@QEBD_K@Z 0000000140024214     BugReporter.obj
 0002:0000a228       $chain$0$?assign@?$basic_string@DU?$char_traits@D@std@@V?$allocator@D@2@@std@@QEAAAEAV12@QEBD_K@Z 0000000140024228     BugReporter.obj
 0002:0000a23c       $chain$3$?assign@?$basic_string@DU?$char_traits@D@std@@V?$allocator@D@2@@std@@QEAAAEAV12@QEBD_K@Z 000000014002423c     BugReporter.obj
 0002:0000a23c       $chain$1$?assign@?$basic_string@DU?$char_traits@D@std@@V?$allocator@D@2@@std@@QEAAAEAV12@QEBD_K@Z 000000014002423c     BugReporter.obj
 0002:0000a24c       $chain$2$?assign@?$basic_string@DU?$char_traits@D@std@@V?$allocator@D@2@@std@@QEAAAEAV12@QEBD_K@Z 000000014002424c     BugReporter.obj
 0002:0000a260       $unwind$_snprintf_s        0000000140024260     BugReporter.obj
 0002:0000a260       $unwind$_snwprintf_s       0000000140024260     crs_uploader.obj
 0002:0000a270       $unwind$?recordExceptionLog@Uploader@crs@@QEAAXAEAVLogBuffer@2@PEBDZZ 0000000140024270     crs_uploader.obj
 0002:0000a284       $chain$0$?recordExceptionLog@Uploader@crs@@QEAAXAEAVLogBuffer@2@PEBDZZ 0000000140024284     crs_uploader.obj
 0002:0000a298       $chain$1$?recordExceptionLog@Uploader@crs@@QEAAXAEAVLogBuffer@2@PEBDZZ 0000000140024298     crs_uploader.obj
 0002:0000a2a8       $unwind$?readURL@Uploader@crs@@AEAAXAEAV?$basic_string@_WU?$char_traits@_W@std@@V?$allocator@_W@2@@std@@@Z 00000001400242a8     crs_uploader.obj
 0002:0000a2c4       $stateUnwindMap$?readURL@Uploader@crs@@AEAAXAEAV?$basic_string@_WU?$char_traits@_W@std@@V?$allocator@_W@2@@std@@@Z 00000001400242c4     crs_uploader.obj
 0002:0000a2e0       $ip2state$?readURL@Uploader@crs@@AEAAXAEAV?$basic_string@_WU?$char_traits@_W@std@@V?$allocator@_W@2@@std@@@Z 00000001400242e0     crs_uploader.obj
 0002:0000a300       $unwind$?iniPath@Uploader@crs@@AEAA?AV?$basic_string@_WU?$char_traits@_W@std@@V?$allocator@_W@2@@std@@AEBV34@@Z 0000000140024300     crs_uploader.obj
 0002:0000a31c       $chain$1$?iniPath@Uploader@crs@@AEAA?AV?$basic_string@_WU?$char_traits@_W@std@@V?$allocator@_W@2@@std@@AEBV34@@Z 000000014002431c     crs_uploader.obj
 0002:0000a330       $chain$2$?iniPath@Uploader@crs@@AEAA?AV?$basic_string@_WU?$char_traits@_W@std@@V?$allocator@_W@2@@std@@AEBV34@@Z 0000000140024330     crs_uploader.obj
 0002:0000a340       $unwind$?makeBaseInfo@Uploader@crs@@AEAAXPEAD0@Z 0000000140024340     crs_uploader.obj
 0002:0000a35c       $unwind$?error@Uploader@crs@@AEAA_NPEBDZZ 000000014002435c     crs_uploader.obj
 0002:0000a368       $unwind$?init@Uploader@crs@@QEAA_N_NPEAD1@Z 0000000140024368     crs_uploader.obj
 0002:0000a38c       $stateUnwindMap$?init@Uploader@crs@@QEAA_N_NPEAD1@Z 000000014002438c     crs_uploader.obj
 0002:0000a398       $ip2state$?init@Uploader@crs@@QEAA_N_NPEAD1@Z 0000000140024398     crs_uploader.obj
 0002:0000a3a8       $unwind$?upload@Uploader@crs@@QEAA_N_NAEBV?$basic_string@DU?$char_traits@D@std@@V?$allocator@D@2@@std@@AEAVLogBuffer@2@@Z 00000001400243a8     crs_uploader.obj
 0002:0000a3c4       $unwind$?makeExceptionLog@Uploader@crs@@QEAAXPEAU_EXCEPTION_POINTERS@@AEAVLogBuffer@2@@Z 00000001400243c4     crs_uploader.obj
 0002:0000a3dc       $chain$3$?makeExceptionLog@Uploader@crs@@QEAAXPEAU_EXCEPTION_POINTERS@@AEAVLogBuffer@2@@Z 00000001400243dc     crs_uploader.obj
 0002:0000a3fc       $chain$4$?makeExceptionLog@Uploader@crs@@QEAAXPEAU_EXCEPTION_POINTERS@@AEAVLogBuffer@2@@Z 00000001400243fc     crs_uploader.obj
 0002:0000a40c       $unwind$?EnumModuleDetail@ModuleInfo@?1??makeExceptionLog@Uploader@crs@@QEAAXPEAU_EXCEPTION_POINTERS@@AEAVLogBuffer@4@@Z@SAHPEBD_KKPEAX@Z 000000014002440c     crs_uploader.obj
 0002:0000a420       $chain$0$?EnumModuleDetail@ModuleInfo@?1??makeExceptionLog@Uploader@crs@@QEAAXPEAU_EXCEPTION_POINTERS@@AEAVLogBuffer@4@@Z@SAHPEBD_KKPEAX@Z 0000000140024420     crs_uploader.obj
 0002:0000a434       $chain$1$?EnumModuleDetail@ModuleInfo@?1??makeExceptionLog@Uploader@crs@@QEAAXPEAU_EXCEPTION_POINTERS@@AEAVLogBuffer@4@@Z@SAHPEBD_KKPEAX@Z 0000000140024434     crs_uploader.obj
 0002:0000a444       $unwind$?prepare@Uploader@crs@@AEAA_NAEAVHttpHandles@2@@Z 0000000140024444     crs_uploader.obj
 0002:0000a458       $unwind$?uploadHTTP@Uploader@crs@@AEAA_NAEAVHttpHandle@2@PEBDPEB_W2@Z 0000000140024458     crs_uploader.obj
 0002:0000a474       $unwind$?uploadLOG@Uploader@crs@@AEAA_NAEAVHttpHandle@2@AEAU_SYSTEMTIME@@AEAVLogBuffer@2@@Z 0000000140024474     crs_uploader.obj
 0002:0000a490       $chain$0$?uploadLOG@Uploader@crs@@AEAA_NAEAVHttpHandle@2@AEAU_SYSTEMTIME@@AEAVLogBuffer@2@@Z 0000000140024490     crs_uploader.obj
 0002:0000a4a4       $chain$1$?uploadLOG@Uploader@crs@@AEAA_NAEAVHttpHandle@2@AEAU_SYSTEMTIME@@AEAVLogBuffer@2@@Z 00000001400244a4     crs_uploader.obj
 0002:0000a4b8       $chain$2$?uploadLOG@Uploader@crs@@AEAA_NAEAVHttpHandle@2@AEAU_SYSTEMTIME@@AEAVLogBuffer@2@@Z 00000001400244b8     crs_uploader.obj
 0002:0000a4c8       $chain$3$?uploadLOG@Uploader@crs@@AEAA_NAEAVHttpHandle@2@AEAU_SYSTEMTIME@@AEAVLogBuffer@2@@Z 00000001400244c8     crs_uploader.obj
 0002:0000a4d8       $unwind$?success@Uploader@crs@@AEAA_NPEBDAEAVHttpHandle@2@@Z 00000001400244d8     crs_uploader.obj
 0002:0000a4e8       $chain$0$??1?$auto_ptr@VUrl@crs@@@std@@QEAA@XZ 00000001400244e8     crs_uploader.obj
 0002:0000a4fc       $chain$1$??1?$auto_ptr@VUrl@crs@@@std@@QEAA@XZ 00000001400244fc     crs_uploader.obj
 0002:0000a50c       $chain$2$??1?$auto_ptr@VUrl@crs@@@std@@QEAA@XZ 000000014002450c     crs_uploader.obj
 0002:0000a520       $unwind$??$_snprintf_s@$0IA@@@YAHAEAY0IA@D_KPEBDZZ 0000000140024520     crs_uploader.obj
 0002:0000a530       $unwind$??$_Reallocate_grow_by@V<lambda_65e615be2a453ca0576c979606f46740>@@PEBD_K@?$basic_string@DU?$char_traits@D@std@@V?$allocator@D@2@@std@@QEAAAEAV01@_KV<lambda_65e615be2a453ca0576c979606f46740>@@PEBD_K@Z 0000000140024530     HostLogger.obj
 0002:0000a530       $unwind$??$_Reallocate_grow_by@V<lambda_1dfe18491bcca09701d8ccb01d0b0af4>@@PEB_W_K@?$basic_string@_WU?$char_traits@_W@std@@V?$allocator@_W@2@@std@@QEAAAEAV01@_KV<lambda_1dfe18491bcca09701d8ccb01d0b0af4>@@PEB_W_K@Z 0000000140024530     crs_uploader.obj
 0002:0000a540       $chain$3$??$_Reallocate_grow_by@V<lambda_1dfe18491bcca09701d8ccb01d0b0af4>@@PEB_W_K@?$basic_string@_WU?$char_traits@_W@std@@V?$allocator@_W@2@@std@@QEAAAEAV01@_KV<lambda_1dfe18491bcca09701d8ccb01d0b0af4>@@PEB_W_K@Z 0000000140024540     crs_uploader.obj
 0002:0000a560       $chain$4$??$_Reallocate_grow_by@V<lambda_1dfe18491bcca09701d8ccb01d0b0af4>@@PEB_W_K@?$basic_string@_WU?$char_traits@_W@std@@V?$allocator@_W@2@@std@@QEAAAEAV01@_KV<lambda_1dfe18491bcca09701d8ccb01d0b0af4>@@PEB_W_K@Z 0000000140024560     crs_uploader.obj
 0002:0000a570       $unwind$??0exception@std@@QEAA@QEBD@Z 0000000140024570     ServerAppDlg.obj
 0002:0000a570       $unwind$?append@?$basic_string@_WU?$char_traits@_W@std@@V?$allocator@_W@2@@std@@QEAAAEAV12@QEB_W_K@Z 0000000140024570     crs_uploader.obj
 0002:0000a578       $chain$1$?append@?$basic_string@_WU?$char_traits@_W@std@@V?$allocator@_W@2@@std@@QEAAAEAV12@QEB_W_K@Z 0000000140024578     crs_uploader.obj
 0002:0000a590       $chain$2$?append@?$basic_string@_WU?$char_traits@_W@std@@V?$allocator@_W@2@@std@@QEAAAEAV12@QEB_W_K@Z 0000000140024590     crs_uploader.obj
 0002:0000a5a0       $unwind$?assign@?$basic_string@_WU?$char_traits@_W@std@@V?$allocator@_W@2@@std@@QEAAAEAV12@QEB_W_K@Z 00000001400245a0     crs_uploader.obj
 0002:0000a5a0       $unwind$?overflow@?$basic_stringbuf@DU?$char_traits@D@std@@V?$allocator@D@2@@std@@MEAAHH@Z 00000001400245a0     safe_string_x64:safe_string.obj
 0002:0000a5bc       $unwind$_RTC_Terminate     00000001400245bc     msvcrt:initsect.obj
 0002:0000a5bc       $unwind$_RTC_Initialize    00000001400245bc     msvcrt:initsect.obj
 0002:0000a5bc       $unwind$??_GCServerAppApp@@UEAAPEAXI@Z 00000001400245bc     ServerApp.obj
 0002:0000a5bc       $unwind$??_GCMustSyncObjectLog@@UEAAPEAXI@Z 00000001400245bc     HostLogger.obj
 0002:0000a5bc       $unwind$?DoDataExchange@CServerAppDlg@@MEAAXPEAVCDataExchange@@@Z 00000001400245bc     ServerAppDlg.obj
 0002:0000a5bc       $unwind$??_G?$CAPIHolder@VILTCommon@@@@UEAAPEAXI@Z 00000001400245bc     ServerAppDlg.obj
 0002:0000a5bc       $unwind$??_GCAPIHolderBase@@UEAAPEAXI@Z 00000001400245bc     ltmodule.obj
 0002:0000a5bc       $unwind$??_GCEdit@@UEAAPEAXI@Z 00000001400245bc     ServerAppDlg.obj
 0002:0000a5bc       $unwind$??_G?$basic_stringbuf@DU?$char_traits@D@std@@V?$allocator@D@2@@std@@UEAAPEAXI@Z 00000001400245bc     safe_string_x64:safe_string.obj
 0002:0000a5bc       $unwind$??_Gexception@std@@UEAAPEAXI@Z 00000001400245bc     ServerAppDlg.obj
 0002:0000a5bc       $unwind$??0CAtlBaseModule@ATL@@QEAA@XZ 00000001400245bc     atls:atlbase.obj
 0002:0000a5bc       $unwind$??_GCListBox@@UEAAPEAXI@Z 00000001400245bc     ServerAppDlg.obj
 0002:0000a5bc       $unwind$??4?$basic_string@DU?$char_traits@D@std@@V?$allocator@D@2@@std@@QEAAAEAV01@$$QEAV01@@Z 00000001400245bc     LoadXlsMsg.obj
 0002:0000a5bc       $unwind$??_GCServerAppDlg@@UEAAPEAXI@Z 00000001400245bc     ServerAppDlg.obj
 0002:0000a5bc       $unwind$?PostWriteData@GAMEPROTO_SC_COMMON@@UEAA_NPEAVILTMessage_Write@@@Z 00000001400245bc     ServerAppDlg.obj
 0002:0000a5bc       $unwind$?AfxInitialize@@YAHHK@Z 00000001400245bc     mfcs140:appmodul.obj
 0002:0000a5bc       $unwind$??_GCServerLog@@UEAAPEAXI@Z 00000001400245bc     LogMgmt.obj
 0002:0000a5bc       $unwind$??__Eg_sUserInfos@@YAXXZ 00000001400245bc     ServerAppDlg.obj
 0002:0000a5c8       $unwind$?Log@rwpmlog@@YAXPEBDFPEBUPROTO_START_HOST_tag@@@Z 00000001400245c8     RWPMLog.obj
 0002:0000a5e4       $unwind$?Log@rwpmlog@@YAXPEBDFPEBUPROTO_GAME_USER_INFO_tag@@@Z 00000001400245e4     RWPMLog.obj
 0002:0000a604       $unwind$?Log@rwpmlog@@YAXPEBDFPEBUPROTO_GAMEGT_INGAME_AIGACHA_GROUP_RATE_RESULT@@@Z 0000000140024604     RWPMLog.obj
 0002:0000a604       $unwind$?Log@rwpmlog@@YAXPEBDFPEBUPROTO_GAMEGT_INGAME_AIGACHA_ITEM_INSERT_RESULT@@@Z 0000000140024604     RWPMLog.obj
 0002:0000a620       $unwind$?LTStrCpyCreate@?A0xaa4cf837@@YAPEADPEBD@Z 0000000140024620     ltmodule.obj
 0002:0000a630       $chain$0$?check_delete_pointers@@YAXXZ 0000000140024630     ltmodule.obj
 0002:0000a644       $chain$1$?check_delete_pointers@@YAXXZ 0000000140024644     ltmodule.obj
 0002:0000a654       $unwind$??0CInterfaceDatabase@@QEAA@XZ 0000000140024654     ltmodule.obj
 0002:0000a668       $stateUnwindMap$??0CInterfaceDatabase@@QEAA@XZ 0000000140024668     ltmodule.obj
 0002:0000a678       $ip2state$??0CInterfaceDatabase@@QEAA@XZ 0000000140024678     ltmodule.obj
 0002:0000a688       $unwind$?AddHolder@CInterfaceDatabase@@SAXPEAVCAPIHolderBase@@@Z 0000000140024688     ltmodule.obj
 0002:0000a698       $stateUnwindMap$?AddHolder@CInterfaceDatabase@@SAXPEAVCAPIHolderBase@@@Z 0000000140024698     ltmodule.obj
 0002:0000a6a0       $ip2state$?AddHolder@CInterfaceDatabase@@SAXPEAVCAPIHolderBase@@@Z 00000001400246a0     ltmodule.obj
 0002:0000a6b8       $unwind$?Add@CInterfaceDatabase@@EEAAXPEAVIBase@@PEBDH@Z 00000001400246b8     ltmodule.obj
 0002:0000a6d4       $stateUnwindMap$?Add@CInterfaceDatabase@@EEAAXPEAVIBase@@PEBDH@Z 00000001400246d4     ltmodule.obj
 0002:0000a6d4       $stateUnwindMap$?Add@CInterfaceDatabase@@EEAAXPEAVCInterfaceChooser@@@Z 00000001400246d4     ltmodule.obj
 0002:0000a6d4       $stateUnwindMap$?Add@CInterfaceDatabase@@EEAAXPEAVCAPIHolderBase@@@Z 00000001400246d4     ltmodule.obj
 0002:0000a6e0       $ip2state$?Add@CInterfaceDatabase@@EEAAXPEAVIBase@@PEBDH@Z 00000001400246e0     ltmodule.obj
 0002:0000a6f8       $unwind$?Remove@CInterfaceDatabase@@EEAAXPEAVIBase@@PEBD@Z 00000001400246f8     ltmodule.obj
 0002:0000a704       $chain$0$?Remove@CInterfaceDatabase@@EEAAXPEAVIBase@@PEBD@Z 0000000140024704     ltmodule.obj
 0002:0000a718       $chain$1$?Remove@CInterfaceDatabase@@EEAAXPEAVIBase@@PEBD@Z 0000000140024718     ltmodule.obj
 0002:0000a72c       $chain$2$?Remove@CInterfaceDatabase@@EEAAXPEAVIBase@@PEBD@Z 000000014002472c     ltmodule.obj
 0002:0000a73c       $chain$3$?Remove@CInterfaceDatabase@@EEAAXPEAVIBase@@PEBD@Z 000000014002473c     ltmodule.obj
 0002:0000a74c       $unwind$?Add@CInterfaceDatabase@@EEAAXPEAVCAPIHolderBase@@@Z 000000014002474c     ltmodule.obj
 0002:0000a768       $ip2state$?Add@CInterfaceDatabase@@EEAAXPEAVCAPIHolderBase@@@Z 0000000140024768     ltmodule.obj
 0002:0000a780       $unwind$?Remove@CInterfaceDatabase@@EEAAXPEAVCAPIHolderBase@@@Z 0000000140024780     ltmodule.obj
 0002:0000a780       $unwind$?Remove@CInterfaceDatabase@@EEAAXPEAVCInterfaceChooser@@@Z 0000000140024780     ltmodule.obj
 0002:0000a78c       $chain$0$?Remove@CInterfaceDatabase@@EEAAXPEAVCAPIHolderBase@@@Z 000000014002478c     ltmodule.obj
 0002:0000a7a0       $chain$1$?Remove@CInterfaceDatabase@@EEAAXPEAVCAPIHolderBase@@@Z 00000001400247a0     ltmodule.obj
 0002:0000a7b0       $unwind$?Add@CInterfaceDatabase@@EEAAXPEAVCInterfaceChooser@@@Z 00000001400247b0     ltmodule.obj
 0002:0000a7d0       $ip2state$?Add@CInterfaceDatabase@@EEAAXPEAVCInterfaceChooser@@@Z 00000001400247d0     ltmodule.obj
 0002:0000a7e8       $chain$0$?Remove@CInterfaceDatabase@@EEAAXPEAVCInterfaceChooser@@@Z 00000001400247e8     ltmodule.obj
 0002:0000a7fc       $chain$1$?Remove@CInterfaceDatabase@@EEAAXPEAVCInterfaceChooser@@@Z 00000001400247fc     ltmodule.obj
 0002:0000a80c       $unwind$?TransferFrom@CInterfaceDatabase@@UEAAXPEAV1@@Z 000000014002480c     ltmodule.obj
 0002:0000a82c       $stateUnwindMap$?TransferFrom@CInterfaceDatabase@@UEAAXPEAV1@@Z 000000014002482c     ltmodule.obj
 0002:0000a838       $ip2state$?TransferFrom@CInterfaceDatabase@@UEAAXPEAV1@@Z 0000000140024838     ltmodule.obj
 0002:0000a850       $unwind$?Destroy@CInterfaceDatabase@@UEAAXXZ 0000000140024850     ltmodule.obj
 0002:0000a858       $chain$1$?Destroy@CInterfaceDatabase@@UEAAXXZ 0000000140024858     ltmodule.obj
 0002:0000a870       $chain$2$?Destroy@CInterfaceDatabase@@UEAAXXZ 0000000140024870     ltmodule.obj
 0002:0000a884       $chain$3$?Destroy@CInterfaceDatabase@@UEAAXXZ 0000000140024884     ltmodule.obj
 0002:0000a898       $chain$4$?Destroy@CInterfaceDatabase@@UEAAXXZ 0000000140024898     ltmodule.obj
 0002:0000a8a8       $chain$5$?Destroy@CInterfaceDatabase@@UEAAXXZ 00000001400248a8     ltmodule.obj
 0002:0000a8b8       $chain$6$?Destroy@CInterfaceDatabase@@UEAAXXZ 00000001400248b8     ltmodule.obj
 0002:0000a8cc       $chain$7$?Destroy@CInterfaceDatabase@@UEAAXXZ 00000001400248cc     ltmodule.obj
 0002:0000a8dc       $unwind$??0CInterfaceNameMgr@@QEAA@PEBDH@Z 00000001400248dc     ltmodule.obj
 0002:0000a8f4       $stateUnwindMap$??0CInterfaceNameMgr@@QEAA@PEBDH@Z 00000001400248f4     ltmodule.obj
 0002:0000a910       $ip2state$??0CInterfaceNameMgr@@QEAA@PEBDH@Z 0000000140024910     ltmodule.obj
 0002:0000a948       $unwind$??_GCInterfaceNameMgr@@UEAAPEAXI@Z 0000000140024948     ltmodule.obj
 0002:0000a950       $chain$2$??_GCInterfaceNameMgr@@UEAAPEAXI@Z 0000000140024950     ltmodule.obj
 0002:0000a96c       $chain$3$??_GCInterfaceNameMgr@@UEAAPEAXI@Z 000000014002496c     ltmodule.obj
 0002:0000a980       $chain$4$??_GCInterfaceNameMgr@@UEAAPEAXI@Z 0000000140024980     ltmodule.obj
 0002:0000a994       $chain$5$??_GCInterfaceNameMgr@@UEAAPEAXI@Z 0000000140024994     ltmodule.obj
 0002:0000a9a4       $chain$6$??_GCInterfaceNameMgr@@UEAAPEAXI@Z 00000001400249a4     ltmodule.obj
 0002:0000a9b4       $chain$7$??_GCInterfaceNameMgr@@UEAAPEAXI@Z 00000001400249b4     ltmodule.obj
 0002:0000a9c4       $unwind$?Add@CInterfaceNameMgr@@QEAAXPEAVIBase@@@Z 00000001400249c4     ltmodule.obj
 0002:0000a9d0       $chain$5$?Add@CInterfaceNameMgr@@QEAAXPEAVIBase@@@Z 00000001400249d0     ltmodule.obj
 0002:0000a9f8       $chain$6$?Add@CInterfaceNameMgr@@QEAAXPEAVIBase@@@Z 00000001400249f8     ltmodule.obj
 0002:0000a9f8       $chain$8$?Add@CInterfaceNameMgr@@QEAAXPEAVIBase@@@Z 00000001400249f8     ltmodule.obj
 0002:0000aa0c       $chain$9$?Add@CInterfaceNameMgr@@QEAAXPEAVIBase@@@Z 0000000140024a0c     ltmodule.obj
 0002:0000aa1c       $unwind$?ConnectHolders@CInterfaceNameMgr@@IEAAXPEAVIBase@@@Z 0000000140024a1c     ltmodule.obj
 0002:0000aa24       $chain$1$?ConnectHolders@CInterfaceNameMgr@@IEAAXPEAVIBase@@@Z 0000000140024a24     ltmodule.obj
 0002:0000aa3c       $chain$2$?ConnectHolders@CInterfaceNameMgr@@IEAAXPEAVIBase@@@Z 0000000140024a3c     ltmodule.obj
 0002:0000aa4c       $unwind$?TransferFrom@CInterfaceNameMgr@@QEAAXPEAV1@@Z 0000000140024a4c     ltmodule.obj
 0002:0000aa68       $stateUnwindMap$?TransferFrom@CInterfaceNameMgr@@QEAAXPEAV1@@Z 0000000140024a68     ltmodule.obj
 0002:0000aa80       $ip2state$?TransferFrom@CInterfaceNameMgr@@QEAAXPEAV1@@Z 0000000140024a80     ltmodule.obj
 0002:0000aab8       $unwind$SetMasterDatabase  0000000140024ab8     ltmodule.obj
 0002:0000aac0       $chain$0$SetMasterDatabase 0000000140024ac0     ltmodule.obj
 0002:0000aad4       $chain$1$SetMasterDatabase 0000000140024ad4     ltmodule.obj
 0002:0000aae4       $unwind$?add@?$database_array@VCInterfaceNameMgr@@PEBD@@QEAAXPEAVCInterfaceNameMgr@@P6A?AW4RELATION@@00@Z@Z 0000000140024ae4     ltmodule.obj
 0002:0000aaf0       $chain$1$?add@?$database_array@VCInterfaceNameMgr@@PEBD@@QEAAXPEAVCInterfaceNameMgr@@P6A?AW4RELATION@@00@Z@Z 0000000140024af0     ltmodule.obj
 0002:0000ab08       $chain$2$?add@?$database_array@VCInterfaceNameMgr@@PEBD@@QEAAXPEAVCInterfaceNameMgr@@P6A?AW4RELATION@@00@Z@Z 0000000140024b08     ltmodule.obj
 0002:0000ab18       $chain$3$?add@?$database_array@VCInterfaceNameMgr@@PEBD@@QEAAXPEAVCInterfaceNameMgr@@P6A?AW4RELATION@@00@Z@Z 0000000140024b18     ltmodule.obj
 0002:0000ab30       $unwind$?get@?$database_array@VCInterfaceNameMgr@@PEBD@@QEAAPEAVCInterfaceNameMgr@@PEBDP6A?AW4RELATION@@0PEAV2@@Z@Z 0000000140024b30     ltmodule.obj
 0002:0000ab30       $unwind$??__Eg_sGameInfos@@YAXXZ 0000000140024b30     ServerAppDlg.obj
 0002:0000ab48       $unwind$?insert@?$database_array@VCInterfaceNameMgr@@PEBD@@IEAAXPEAVCInterfaceNameMgr@@I@Z 0000000140024b48     ltmodule.obj
 0002:0000ab48       $unwind$?insert@?$database_array@VIBase@@PEBD@@IEAAXPEAVIBase@@I@Z 0000000140024b48     ltmodule.obj
 0002:0000ab58       $chain$0$?insert@?$database_array@VIBase@@PEBD@@IEAAXPEAVIBase@@I@Z 0000000140024b58     ltmodule.obj
 0002:0000ab58       $chain$0$?insert@?$database_array@VCInterfaceNameMgr@@PEBD@@IEAAXPEAVCInterfaceNameMgr@@I@Z 0000000140024b58     ltmodule.obj
 0002:0000ab6c       $chain$1$?insert@?$database_array@VCInterfaceNameMgr@@PEBD@@IEAAXPEAVCInterfaceNameMgr@@I@Z 0000000140024b6c     ltmodule.obj
 0002:0000ab6c       $chain$1$?insert@?$database_array@VIBase@@PEBD@@IEAAXPEAVIBase@@I@Z 0000000140024b6c     ltmodule.obj
 0002:0000ab7c       $unwind$?_InitPathNameInfo@CHLogger@@CAXPEBD000@Z 0000000140024b7c     HostLogger.obj
 0002:0000aba0       $unwind$?Log@CHLogger@@SAXW4ELOG_LEVEL@1@PEBDZZ 0000000140024ba0     HostLogger.obj
 0002:0000aba0       $unwind$?LogKernel@CHLogger@@SAXW4ELOG_LEVEL@1@PEBDZZ 0000000140024ba0     HostLogger.obj
 0002:0000aba8       $unwind$?LogTimeOut@CHLogger@@SAXPEBDZZ 0000000140024ba8     HostLogger.obj
 0002:0000aba8       $unwind$?LogEtc@CHLogger@@SAXPEBDZZ 0000000140024ba8     HostLogger.obj
 0002:0000abbc       $chain$0$?LogTimeOut@CHLogger@@SAXPEBDZZ 0000000140024bbc     HostLogger.obj
 0002:0000abd0       $chain$3$?LogTimeOut@CHLogger@@SAXPEBDZZ 0000000140024bd0     HostLogger.obj
 0002:0000abec       $chain$4$?LogTimeOut@CHLogger@@SAXPEBDZZ 0000000140024bec     HostLogger.obj
 0002:0000abfc       $chain$5$?LogTimeOut@CHLogger@@SAXPEBDZZ 0000000140024bfc     HostLogger.obj
 0002:0000ac0c       $chain$0$?LogEtc@CHLogger@@SAXPEBDZZ 0000000140024c0c     HostLogger.obj
 0002:0000ac20       $chain$3$?LogEtc@CHLogger@@SAXPEBDZZ 0000000140024c20     HostLogger.obj
 0002:0000ac3c       $chain$4$?LogEtc@CHLogger@@SAXPEBDZZ 0000000140024c3c     HostLogger.obj
 0002:0000ac4c       $chain$5$?LogEtc@CHLogger@@SAXPEBDZZ 0000000140024c4c     HostLogger.obj
 0002:0000ac5c       $unwind$?LogPacket@CHLogger@@SAXPEBDZZ 0000000140024c5c     HostLogger.obj
 0002:0000ac7c       $stateUnwindMap$?LogPacket@CHLogger@@SAXPEBDZZ 0000000140024c7c     HostLogger.obj
 0002:0000ac88       $ip2state$?LogPacket@CHLogger@@SAXPEBDZZ 0000000140024c88     HostLogger.obj
 0002:0000ac98       $unwind$?LogRWProcessMemory@CHLogger@@SAXPEBDZZ 0000000140024c98     HostLogger.obj
 0002:0000ac98       $unwind$?LogIPCMessage@CHLogger@@SAXPEBDZZ 0000000140024c98     HostLogger.obj
 0002:0000acac       $chain$0$?LogRWProcessMemory@CHLogger@@SAXPEBDZZ 0000000140024cac     HostLogger.obj
 0002:0000acc0       $chain$1$?LogRWProcessMemory@CHLogger@@SAXPEBDZZ 0000000140024cc0     HostLogger.obj
 0002:0000acd4       $chain$2$?LogRWProcessMemory@CHLogger@@SAXPEBDZZ 0000000140024cd4     HostLogger.obj
 0002:0000ace4       $chain$3$?LogRWProcessMemory@CHLogger@@SAXPEBDZZ 0000000140024ce4     HostLogger.obj
 0002:0000acf4       $chain$0$?LogIPCMessage@CHLogger@@SAXPEBDZZ 0000000140024cf4     HostLogger.obj
 0002:0000ad08       $chain$1$?LogIPCMessage@CHLogger@@SAXPEBDZZ 0000000140024d08     HostLogger.obj
 0002:0000ad1c       $chain$2$?LogIPCMessage@CHLogger@@SAXPEBDZZ 0000000140024d1c     HostLogger.obj
 0002:0000ad2c       $chain$3$?LogIPCMessage@CHLogger@@SAXPEBDZZ 0000000140024d2c     HostLogger.obj
 0002:0000ad3c       $unwind$?_BuildDirectory@CHLogger@@CAXAEBU_SYSTEMTIME@@@Z 0000000140024d3c     HostLogger.obj
 0002:0000ad68       $stateUnwindMap$?_BuildDirectory@CHLogger@@CAXAEBU_SYSTEMTIME@@@Z 0000000140024d68     HostLogger.obj
 0002:0000ad80       $ip2state$?_BuildDirectory@CHLogger@@CAXAEBU_SYSTEMTIME@@@Z 0000000140024d80     HostLogger.obj
 0002:0000adb0       $unwind$?_DoLogWithLevel@CHLogger@@CAXPEBDW4ELOG_LEVEL@1@0PEAD@Z 0000000140024db0     HostLogger.obj
 0002:0000add0       $stateUnwindMap$?_DoLogWithLevel@CHLogger@@CAXPEBDW4ELOG_LEVEL@1@0PEAD@Z 0000000140024dd0     HostLogger.obj
 0002:0000add8       $ip2state$?_DoLogWithLevel@CHLogger@@CAXPEBDW4ELOG_LEVEL@1@0PEAD@Z 0000000140024dd8     HostLogger.obj
 0002:0000ade8       $unwind$??$_Traits_find@U?$char_traits@D@std@@@std@@YA_KQEBD_K101@Z 0000000140024de8     HostLogger.obj
 0002:0000ae00       $chain$3$??$_Reallocate_grow_by@V<lambda_65e615be2a453ca0576c979606f46740>@@PEBD_K@?$basic_string@DU?$char_traits@D@std@@V?$allocator@D@2@@std@@QEAAAEAV01@_KV<lambda_65e615be2a453ca0576c979606f46740>@@PEBD_K@Z 0000000140024e00     HostLogger.obj
 0002:0000ae20       $chain$4$??$_Reallocate_grow_by@V<lambda_65e615be2a453ca0576c979606f46740>@@PEBD_K@?$basic_string@DU?$char_traits@D@std@@V?$allocator@D@2@@std@@QEAAAEAV01@_KV<lambda_65e615be2a453ca0576c979606f46740>@@PEBD_K@Z 0000000140024e20     HostLogger.obj
 0002:0000ae30       $unwind$?append@?$basic_string@DU?$char_traits@D@std@@V?$allocator@D@2@@std@@QEAAAEAV12@QEBD_K@Z 0000000140024e30     HostLogger.obj
 0002:0000ae3c       $chain$0$?append@?$basic_string@DU?$char_traits@D@std@@V?$allocator@D@2@@std@@QEAAAEAV12@QEBD_K@Z 0000000140024e3c     HostLogger.obj
 0002:0000ae50       $chain$1$?append@?$basic_string@DU?$char_traits@D@std@@V?$allocator@D@2@@std@@QEAAAEAV12@QEBD_K@Z 0000000140024e50     HostLogger.obj
 0002:0000ae60       $unwind$?Init@CLogMsgManager@@SA_NW4ESHARED_MEM_USAGE_TYPE@1@@Z 0000000140024e60     LogMsgManager.obj
 0002:0000ae78       $stateUnwindMap$?Init@CLogMsgManager@@SA_NW4ESHARED_MEM_USAGE_TYPE@1@@Z 0000000140024e78     LogMsgManager.obj
 0002:0000ae88       $ip2state$?Init@CLogMsgManager@@SA_NW4ESHARED_MEM_USAGE_TYPE@1@@Z 0000000140024e88     LogMsgManager.obj
 0002:0000aeb0       $unwind$?GetString@CLogMsgManager@@SA?BV?$basic_string@DU?$char_traits@D@std@@V?$allocator@D@2@@std@@I@Z 0000000140024eb0     LogMsgManager.obj
 0002:0000aec0       $chain$0$?GetString@CLogMsgManager@@SA?BV?$basic_string@DU?$char_traits@D@std@@V?$allocator@D@2@@std@@I@Z 0000000140024ec0     LogMsgManager.obj
 0002:0000aed4       $chain$1$?GetString@CLogMsgManager@@SA?BV?$basic_string@DU?$char_traits@D@std@@V?$allocator@D@2@@std@@I@Z 0000000140024ed4     LogMsgManager.obj
 0002:0000aed4       $chain$3$?GetString@CLogMsgManager@@SA?BV?$basic_string@DU?$char_traits@D@std@@V?$allocator@D@2@@std@@I@Z 0000000140024ed4     LogMsgManager.obj
 0002:0000aee4       $chain$2$?GetString@CLogMsgManager@@SA?BV?$basic_string@DU?$char_traits@D@std@@V?$allocator@D@2@@std@@I@Z 0000000140024ee4     LogMsgManager.obj
 0002:0000aef8       $unwind$?_WriteXlsDataToSharedMemory@CLogMsgManager@@CA_NXZ 0000000140024ef8     LogMsgManager.obj
 0002:0000af20       $stateUnwindMap$?OnTimer@CServerAppDlg@@QEAAX_K@Z 0000000140024f20     ServerAppDlg.obj
 0002:0000af20       $stateUnwindMap$?_WriteXlsDataToSharedMemory@CLogMsgManager@@CA_NXZ 0000000140024f20     LogMsgManager.obj
 0002:0000af20       $stateUnwindMap$?RECV_MSG_USER_DISCONNECTED@CServerAppDlg@@AEAAX_J@Z 0000000140024f20     ServerAppDlg.obj
 0002:0000af28       $ip2state$?_WriteXlsDataToSharedMemory@CLogMsgManager@@CA_NXZ 0000000140024f28     LogMsgManager.obj
 0002:0000af48       $unwind$??$_Emplace_reallocate@AEBQEAX@?$vector@PEAXV?$allocator@PEAX@std@@@std@@QEAAPEAPEAXQEAPEAXAEBQEAX@Z 0000000140024f48     LogMsgManager.obj
 0002:0000af54       $chain$2$??$_Emplace_reallocate@AEBQEAX@?$vector@PEAXV?$allocator@PEAX@std@@@std@@QEAAPEAPEAXQEAPEAXAEBQEAX@Z 0000000140024f54     LogMsgManager.obj
 0002:0000af70       $chain$4$??$_Emplace_reallocate@AEBQEAX@?$vector@PEAXV?$allocator@PEAX@std@@@std@@QEAAPEAPEAXQEAPEAXAEBQEAX@Z 0000000140024f70     LogMsgManager.obj
 0002:0000af8c       $chain$5$??$_Emplace_reallocate@AEBQEAX@?$vector@PEAXV?$allocator@PEAX@std@@@std@@QEAAPEAPEAXQEAPEAXAEBQEAX@Z 0000000140024f8c     LogMsgManager.obj
 0002:0000af9c       $unwind$??0FindXlsMsg@@QEAA@XZ 0000000140024f9c     LoadXlsMsg.obj
 0002:0000afa8       $unwind$??_GFindXlsMsg@@UEAAPEAXI@Z 0000000140024fa8     LoadXlsMsg.obj
 0002:0000afc4       $stateUnwindMap$?__scrt_initialize_thread_safe_statics@@YAHXZ 0000000140024fc4     msvcrt:thread_safe_statics.obj
 0002:0000afc4       $stateUnwindMap$??_GFindXlsMsg@@UEAAPEAXI@Z 0000000140024fc4     LoadXlsMsg.obj
 0002:0000afc4       $stateUnwindMap$?erase@?$_Tree@V?$_Tmap_traits@_JV?$basic_string@DU?$char_traits@D@std@@V?$allocator@D@2@@std@@U?$less@_J@2@V?$allocator@U?$pair@$$CB_JV?$basic_string@DU?$char_traits@D@std@@V?$allocator@D@2@@std@@@std@@@2@$0A@@std@@@std@@QEAA?AV?$_Tree_iterator@V?$_Tree_val@U?$_Tree_simple_types@U?$pair@$$CB_JV?$basic_string@DU?$char_traits@D@std@@V?$allocator@D@2@@std@@@std@@@std@@@std@@@2@V?$_Tree_const_iterator@V?$_Tree_val@U?$_Tree_simple_types@U?$pair@$$CB_JV?$basic_string@DU?$char_traits@D@std@@V?$allocator@D@2@@std@@@std@@@std@@@std@@@2@0@Z 0000000140024fc4     LoadXlsMsg.obj
 0002:0000afc4       $stateUnwindMap$??1sentry@?$basic_ostream@DU?$char_traits@D@std@@@std@@QEAA@XZ 0000000140024fc4     safe_string_x64:safe_string.obj
 0002:0000afd0       $ip2state$??_GFindXlsMsg@@UEAAPEAXI@Z 0000000140024fd0     LoadXlsMsg.obj
 0002:0000afd8       $unwind$?GetMessageByIndex@FindXlsMsg@@QEAAPEBD_JPEAD@Z 0000000140024fd8     LoadXlsMsg.obj
 0002:0000afe4       $unwind$?LoadWMszFile@FindXlsMsg@@QEAA_NPEAD@Z 0000000140024fe4     LoadXlsMsg.obj
 0002:0000b010       $stateUnwindMap$?LoadWMszFile@FindXlsMsg@@QEAA_NPEAD@Z 0000000140025010     LoadXlsMsg.obj
 0002:0000b018       $ip2state$?LoadWMszFile@FindXlsMsg@@QEAA_NPEAD@Z 0000000140025018     LoadXlsMsg.obj
 0002:0000b030       $unwind$??A?$map@_JV?$basic_string@DU?$char_traits@D@std@@V?$allocator@D@2@@std@@U?$less@_J@2@V?$allocator@U?$pair@$$CB_JV?$basic_string@DU?$char_traits@D@std@@V?$allocator@D@2@@std@@@std@@@2@@std@@QEAAAEAV?$basic_string@DU?$char_traits@D@std@@V?$allocator@D@2@@1@AEB_J@Z 0000000140025030     LoadXlsMsg.obj
 0002:0000b03c       $unwind$?_Erase@?$_Tree@V?$_Tmap_traits@_JV?$basic_string@DU?$char_traits@D@std@@V?$allocator@D@2@@std@@U?$less@_J@2@V?$allocator@U?$pair@$$CB_JV?$basic_string@DU?$char_traits@D@std@@V?$allocator@D@2@@std@@@std@@@2@$0A@@std@@@std@@IEAAXPEAU?$_Tree_node@U?$pair@$$CB_JV?$basic_string@DU?$char_traits@D@std@@V?$allocator@D@2@@std@@@std@@PEAX@2@@Z 000000014002503c     LoadXlsMsg.obj
 0002:0000b04c       $chain$0$?_Erase@?$_Tree@V?$_Tmap_traits@_JV?$basic_string@DU?$char_traits@D@std@@V?$allocator@D@2@@std@@U?$less@_J@2@V?$allocator@U?$pair@$$CB_JV?$basic_string@DU?$char_traits@D@std@@V?$allocator@D@2@@std@@@std@@@2@$0A@@std@@@std@@IEAAXPEAU?$_Tree_node@U?$pair@$$CB_JV?$basic_string@DU?$char_traits@D@std@@V?$allocator@D@2@@std@@@std@@PEAX@2@@Z 000000014002504c     LoadXlsMsg.obj
 0002:0000b060       $chain$1$?_Erase@?$_Tree@V?$_Tmap_traits@_JV?$basic_string@DU?$char_traits@D@std@@V?$allocator@D@2@@std@@U?$less@_J@2@V?$allocator@U?$pair@$$CB_JV?$basic_string@DU?$char_traits@D@std@@V?$allocator@D@2@@std@@@std@@@2@$0A@@std@@@std@@IEAAXPEAU?$_Tree_node@U?$pair@$$CB_JV?$basic_string@DU?$char_traits@D@std@@V?$allocator@D@2@@std@@@std@@PEAX@2@@Z 0000000140025060     LoadXlsMsg.obj
 0002:0000b070       $chain$2$?_Erase@?$_Tree@V?$_Tmap_traits@_JV?$basic_string@DU?$char_traits@D@std@@V?$allocator@D@2@@std@@U?$less@_J@2@V?$allocator@U?$pair@$$CB_JV?$basic_string@DU?$char_traits@D@std@@V?$allocator@D@2@@std@@@std@@@2@$0A@@std@@@std@@IEAAXPEAU?$_Tree_node@U?$pair@$$CB_JV?$basic_string@DU?$char_traits@D@std@@V?$allocator@D@2@@std@@@std@@PEAX@2@@Z 0000000140025070     LoadXlsMsg.obj
 0002:0000b084       $unwind$?erase@?$_Tree@V?$_Tmap_traits@_JV?$basic_string@DU?$char_traits@D@std@@V?$allocator@D@2@@std@@U?$less@_J@2@V?$allocator@U?$pair@$$CB_JV?$basic_string@DU?$char_traits@D@std@@V?$allocator@D@2@@std@@@std@@@2@$0A@@std@@@std@@QEAA?AV?$_Tree_iterator@V?$_Tree_val@U?$_Tree_simple_types@U?$pair@$$CB_JV?$basic_string@DU?$char_traits@D@std@@V?$allocator@D@2@@std@@@std@@@std@@@std@@@2@V?$_Tree_const_iterator@V?$_Tree_val@U?$_Tree_simple_types@U?$pair@$$CB_JV?$basic_string@DU?$char_traits@D@std@@V?$allocator@D@2@@std@@@std@@@std@@@std@@@2@0@Z 0000000140025084     LoadXlsMsg.obj
 0002:0000b0a8       $ip2state$?erase@?$_Tree@V?$_Tmap_traits@_JV?$basic_string@DU?$char_traits@D@std@@V?$allocator@D@2@@std@@U?$less@_J@2@V?$allocator@U?$pair@$$CB_JV?$basic_string@DU?$char_traits@D@std@@V?$allocator@D@2@@std@@@std@@@2@$0A@@std@@@std@@QEAA?AV?$_Tree_iterator@V?$_Tree_val@U?$_Tree_simple_types@U?$pair@$$CB_JV?$basic_string@DU?$char_traits@D@std@@V?$allocator@D@2@@std@@@std@@@std@@@std@@@2@V?$_Tree_const_iterator@V?$_Tree_val@U?$_Tree_simple_types@U?$pair@$$CB_JV?$basic_string@DU?$char_traits@D@std@@V?$allocator@D@2@@std@@@std@@@std@@@std@@@2@0@Z 00000001400250a8     LoadXlsMsg.obj
 0002:0000b0b0       $unwind$?_Extract@?$_Tree_val@U?$_Tree_simple_types@U?$pair@$$CB_JV?$basic_string@DU?$char_traits@D@std@@V?$allocator@D@2@@std@@@std@@@std@@@std@@QEAAPEAU?$_Tree_node@U?$pair@$$CB_JV?$basic_string@DU?$char_traits@D@std@@V?$allocator@D@2@@std@@@std@@PEAX@2@V?$_Tree_const_iterator@V?$_Tree_val@U?$_Tree_simple_types@U?$pair@$$CB_JV?$basic_string@DU?$char_traits@D@std@@V?$allocator@D@2@@std@@@std@@@std@@@std@@@2@@Z 00000001400250b0     LoadXlsMsg.obj
 0002:0000b0b8       $unwind$??$_Insert_hint@AEAU?$pair@$$CB_JV?$basic_string@DU?$char_traits@D@std@@V?$allocator@D@2@@std@@@std@@PEAU?$_Tree_node@U?$pair@$$CB_JV?$basic_string@DU?$char_traits@D@std@@V?$allocator@D@2@@std@@@std@@PEAX@2@@?$_Tree@V?$_Tmap_traits@_JV?$basic_string@DU?$char_traits@D@std@@V?$allocator@D@2@@std@@U?$less@_J@2@V?$allocator@U?$pair@$$CB_JV?$basic_string@DU?$char_traits@D@std@@V?$allocator@D@2@@std@@@std@@@2@$0A@@std@@@std@@IEAA?AV?$_Tree_iterator@V?$_Tree_val@U?$_Tree_simple_types@U?$pair@$$CB_JV?$basic_string@DU?$char_traits@D@std@@V?$allocator@D@2@@std@@@std@@@std@@@std@@@1@V?$_Tree_const_iterator@V?$_Tree_val@U?$_Tree_simple_types@U?$pair@$$CB_JV?$basic_string@DU?$char_traits@D@std@@V?$allocator@D@2@@std@@@std@@@std@@@std@@@1@AEAU?$pair@$$CB_JV?$basic_string@DU?$char_traits@D@std@@V?$allocator@D@2@@std@@@1@PEAU?$_Tree_node@U?$pair@$$CB_JV?$basic_string@DU?$char_traits@D@std@@V?$allocator@D@2@@std@@@std@@PEAX@1@@Z 00000001400250b8     LoadXlsMsg.obj
 0002:0000b0d0       $stateUnwindMap$??$_Insert_nohint@AEAU?$pair@$$CB_JV?$basic_string@DU?$char_traits@D@std@@V?$allocator@D@2@@std@@@std@@PEAU?$_Tree_node@U?$pair@$$CB_JV?$basic_string@DU?$char_traits@D@std@@V?$allocator@D@2@@std@@@std@@PEAX@2@@?$_Tree@V?$_Tmap_traits@_JV?$basic_string@DU?$char_traits@D@std@@V?$allocator@D@2@@std@@U?$less@_J@2@V?$allocator@U?$pair@$$CB_JV?$basic_string@DU?$char_traits@D@std@@V?$allocator@D@2@@std@@@std@@@2@$0A@@std@@@std@@IEAA?AU?$pair@V?$_Tree_iterator@V?$_Tree_val@U?$_Tree_simple_types@U?$pair@$$CB_JV?$basic_string@DU?$char_traits@D@std@@V?$allocator@D@2@@std@@@std@@@std@@@std@@@std@@_N@1@_NAEAU?$pair@$$CB_JV?$basic_string@DU?$char_traits@D@std@@V?$allocator@D@2@@std@@@1@PEAU?$_Tree_node@U?$pair@$$CB_JV?$basic_string@DU?$char_traits@D@std@@V?$allocator@D@2@@std@@@std@@PEAX@1@@Z 00000001400250d0     LoadXlsMsg.obj
 0002:0000b0d0       $stateUnwindMap$??$_Insert_hint@AEAU?$pair@$$CB_JV?$basic_string@DU?$char_traits@D@std@@V?$allocator@D@2@@std@@@std@@PEAU?$_Tree_node@U?$pair@$$CB_JV?$basic_string@DU?$char_traits@D@std@@V?$allocator@D@2@@std@@@std@@PEAX@2@@?$_Tree@V?$_Tmap_traits@_JV?$basic_string@DU?$char_traits@D@std@@V?$allocator@D@2@@std@@U?$less@_J@2@V?$allocator@U?$pair@$$CB_JV?$basic_string@DU?$char_traits@D@std@@V?$allocator@D@2@@std@@@std@@@2@$0A@@std@@@std@@IEAA?AV?$_Tree_iterator@V?$_Tree_val@U?$_Tree_simple_types@U?$pair@$$CB_JV?$basic_string@DU?$char_traits@D@std@@V?$allocator@D@2@@std@@@std@@@std@@@std@@@1@V?$_Tree_const_iterator@V?$_Tree_val@U?$_Tree_simple_types@U?$pair@$$CB_JV?$basic_string@DU?$char_traits@D@std@@V?$allocator@D@2@@std@@@std@@@std@@@std@@@1@AEAU?$pair@$$CB_JV?$basic_string@DU?$char_traits@D@std@@V?$allocator@D@2@@std@@@1@PEAU?$_Tree_node@U?$pair@$$CB_JV?$basic_string@DU?$char_traits@D@std@@V?$allocator@D@2@@std@@@std@@PEAX@1@@Z 00000001400250d0     LoadXlsMsg.obj
 0002:0000b0e0       $tryMap$??$_Insert_hint@AEAU?$pair@$$CB_JV?$basic_string@DU?$char_traits@D@std@@V?$allocator@D@2@@std@@@std@@PEAU?$_Tree_node@U?$pair@$$CB_JV?$basic_string@DU?$char_traits@D@std@@V?$allocator@D@2@@std@@@std@@PEAX@2@@?$_Tree@V?$_Tmap_traits@_JV?$basic_string@DU?$char_traits@D@std@@V?$allocator@D@2@@std@@U?$less@_J@2@V?$allocator@U?$pair@$$CB_JV?$basic_string@DU?$char_traits@D@std@@V?$allocator@D@2@@std@@@std@@@2@$0A@@std@@@std@@IEAA?AV?$_Tree_iterator@V?$_Tree_val@U?$_Tree_simple_types@U?$pair@$$CB_JV?$basic_string@DU?$char_traits@D@std@@V?$allocator@D@2@@std@@@std@@@std@@@std@@@1@V?$_Tree_const_iterator@V?$_Tree_val@U?$_Tree_simple_types@U?$pair@$$CB_JV?$basic_string@DU?$char_traits@D@std@@V?$allocator@D@2@@std@@@std@@@std@@@std@@@1@AEAU?$pair@$$CB_JV?$basic_string@DU?$char_traits@D@std@@V?$allocator@D@2@@std@@@1@PEAU?$_Tree_node@U?$pair@$$CB_JV?$basic_string@DU?$char_traits@D@std@@V?$allocator@D@2@@std@@@std@@PEAX@1@@Z 00000001400250e0     LoadXlsMsg.obj
 0002:0000b0f4       $handlerMap$0$??$_Insert_hint@AEAU?$pair@$$CB_JV?$basic_string@DU?$char_traits@D@std@@V?$allocator@D@2@@std@@@std@@PEAU?$_Tree_node@U?$pair@$$CB_JV?$basic_string@DU?$char_traits@D@std@@V?$allocator@D@2@@std@@@std@@PEAX@2@@?$_Tree@V?$_Tmap_traits@_JV?$basic_string@DU?$char_traits@D@std@@V?$allocator@D@2@@std@@U?$less@_J@2@V?$allocator@U?$pair@$$CB_JV?$basic_string@DU?$char_traits@D@std@@V?$allocator@D@2@@std@@@std@@@2@$0A@@std@@@std@@IEAA?AV?$_Tree_iterator@V?$_Tree_val@U?$_Tree_simple_types@U?$pair@$$CB_JV?$basic_string@DU?$char_traits@D@std@@V?$allocator@D@2@@std@@@std@@@std@@@std@@@1@V?$_Tree_const_iterator@V?$_Tree_val@U?$_Tree_simple_types@U?$pair@$$CB_JV?$basic_string@DU?$char_traits@D@std@@V?$allocator@D@2@@std@@@std@@@std@@@std@@@1@AEAU?$pair@$$CB_JV?$basic_string@DU?$char_traits@D@std@@V?$allocator@D@2@@std@@@1@PEAU?$_Tree_node@U?$pair@$$CB_JV?$basic_string@DU?$char_traits@D@std@@V?$allocator@D@2@@std@@@std@@PEAX@1@@Z 00000001400250f4     LoadXlsMsg.obj
 0002:0000b108       $ip2state$??$_Insert_hint@AEAU?$pair@$$CB_JV?$basic_string@DU?$char_traits@D@std@@V?$allocator@D@2@@std@@@std@@PEAU?$_Tree_node@U?$pair@$$CB_JV?$basic_string@DU?$char_traits@D@std@@V?$allocator@D@2@@std@@@std@@PEAX@2@@?$_Tree@V?$_Tmap_traits@_JV?$basic_string@DU?$char_traits@D@std@@V?$allocator@D@2@@std@@U?$less@_J@2@V?$allocator@U?$pair@$$CB_JV?$basic_string@DU?$char_traits@D@std@@V?$allocator@D@2@@std@@@std@@@2@$0A@@std@@@std@@IEAA?AV?$_Tree_iterator@V?$_Tree_val@U?$_Tree_simple_types@U?$pair@$$CB_JV?$basic_string@DU?$char_traits@D@std@@V?$allocator@D@2@@std@@@std@@@std@@@std@@@1@V?$_Tree_const_iterator@V?$_Tree_val@U?$_Tree_simple_types@U?$pair@$$CB_JV?$basic_string@DU?$char_traits@D@std@@V?$allocator@D@2@@std@@@std@@@std@@@std@@@1@AEAU?$pair@$$CB_JV?$basic_string@DU?$char_traits@D@std@@V?$allocator@D@2@@std@@@1@PEAU?$_Tree_node@U?$pair@$$CB_JV?$basic_string@DU?$char_traits@D@std@@V?$allocator@D@2@@std@@@std@@PEAX@1@@Z 0000000140025108     LoadXlsMsg.obj
 0002:0000b128       $unwind$?catch$0@?0???$_Insert_hint@AEAU?$pair@$$CB_JV?$basic_string@DU?$char_traits@D@std@@V?$allocator@D@2@@std@@@std@@PEAU?$_Tree_node@U?$pair@$$CB_JV?$basic_string@DU?$char_traits@D@std@@V?$allocator@D@2@@std@@@std@@PEAX@2@@?$_Tree@V?$_Tmap_traits@_JV?$basic_string@DU?$char_traits@D@std@@V?$allocator@D@2@@std@@U?$less@_J@2@V?$allocator@U?$pair@$$CB_JV?$basic_string@DU?$char_traits@D@std@@V?$allocator@D@2@@std@@@std@@@2@$0A@@std@@@std@@IEAA?AV?$_Tree_iterator@V?$_Tree_val@U?$_Tree_simple_types@U?$pair@$$CB_JV?$basic_string@DU?$char_traits@D@std@@V?$allocator@D@2@@std@@@std@@@std@@@std@@@1@V?$_Tree_const_iterator@V?$_Tree_val@U?$_Tree_simple_types@U?$pair@$$CB_JV?$basic_string@DU?$char_traits@D@std@@V?$allocator@D@2@@std@@@std@@@std@@@std@@@1@AEAU?$pair@$$CB_JV?$basic_string@DU?$char_traits@D@std@@V?$allocator@D@2@@std@@@1@PEAU?$_Tree_node@U?$pair@$$CB_JV?$basic_string@DU?$char_traits@D@std@@V?$allocator@D@2@@std@@@std@@PEAX@1@@Z@4HA 0000000140025128     LoadXlsMsg.obj
 0002:0000b138       $unwind$??$_Insert_at@AEAU?$pair@$$CB_JV?$basic_string@DU?$char_traits@D@std@@V?$allocator@D@2@@std@@@std@@PEAU?$_Tree_node@U?$pair@$$CB_JV?$basic_string@DU?$char_traits@D@std@@V?$allocator@D@2@@std@@@std@@PEAX@2@@?$_Tree@V?$_Tmap_traits@_JV?$basic_string@DU?$char_traits@D@std@@V?$allocator@D@2@@std@@U?$less@_J@2@V?$allocator@U?$pair@$$CB_JV?$basic_string@DU?$char_traits@D@std@@V?$allocator@D@2@@std@@@std@@@2@$0A@@std@@@std@@IEAA?AV?$_Tree_iterator@V?$_Tree_val@U?$_Tree_simple_types@U?$pair@$$CB_JV?$basic_string@DU?$char_traits@D@std@@V?$allocator@D@2@@std@@@std@@@std@@@std@@@1@_NPEAU?$_Tree_node@U?$pair@$$CB_JV?$basic_string@DU?$char_traits@D@std@@V?$allocator@D@2@@std@@@std@@PEAX@1@AEAU?$pair@$$CB_JV?$basic_string@DU?$char_traits@D@std@@V?$allocator@D@2@@std@@@1@1@Z 0000000140025138     LoadXlsMsg.obj
 0002:0000b144       $unwind$??$_Insert_nohint@AEAU?$pair@$$CB_JV?$basic_string@DU?$char_traits@D@std@@V?$allocator@D@2@@std@@@std@@PEAU?$_Tree_node@U?$pair@$$CB_JV?$basic_string@DU?$char_traits@D@std@@V?$allocator@D@2@@std@@@std@@PEAX@2@@?$_Tree@V?$_Tmap_traits@_JV?$basic_string@DU?$char_traits@D@std@@V?$allocator@D@2@@std@@U?$less@_J@2@V?$allocator@U?$pair@$$CB_JV?$basic_string@DU?$char_traits@D@std@@V?$allocator@D@2@@std@@@std@@@2@$0A@@std@@@std@@IEAA?AU?$pair@V?$_Tree_iterator@V?$_Tree_val@U?$_Tree_simple_types@U?$pair@$$CB_JV?$basic_string@DU?$char_traits@D@std@@V?$allocator@D@2@@std@@@std@@@std@@@std@@@std@@_N@1@_NAEAU?$pair@$$CB_JV?$basic_string@DU?$char_traits@D@std@@V?$allocator@D@2@@std@@@1@PEAU?$_Tree_node@U?$pair@$$CB_JV?$basic_string@DU?$char_traits@D@std@@V?$allocator@D@2@@std@@@std@@PEAX@1@@Z 0000000140025144     LoadXlsMsg.obj
 0002:0000b160       $tryMap$??$_Insert_nohint@AEAU?$pair@$$CB_JV?$basic_string@DU?$char_traits@D@std@@V?$allocator@D@2@@std@@@std@@PEAU?$_Tree_node@U?$pair@$$CB_JV?$basic_string@DU?$char_traits@D@std@@V?$allocator@D@2@@std@@@std@@PEAX@2@@?$_Tree@V?$_Tmap_traits@_JV?$basic_string@DU?$char_traits@D@std@@V?$allocator@D@2@@std@@U?$less@_J@2@V?$allocator@U?$pair@$$CB_JV?$basic_string@DU?$char_traits@D@std@@V?$allocator@D@2@@std@@@std@@@2@$0A@@std@@@std@@IEAA?AU?$pair@V?$_Tree_iterator@V?$_Tree_val@U?$_Tree_simple_types@U?$pair@$$CB_JV?$basic_string@DU?$char_traits@D@std@@V?$allocator@D@2@@std@@@std@@@std@@@std@@@std@@_N@1@_NAEAU?$pair@$$CB_JV?$basic_string@DU?$char_traits@D@std@@V?$allocator@D@2@@std@@@1@PEAU?$_Tree_node@U?$pair@$$CB_JV?$basic_string@DU?$char_traits@D@std@@V?$allocator@D@2@@std@@@std@@PEAX@1@@Z 0000000140025160     LoadXlsMsg.obj
 0002:0000b174       $handlerMap$0$??$_Insert_nohint@AEAU?$pair@$$CB_JV?$basic_string@DU?$char_traits@D@std@@V?$allocator@D@2@@std@@@std@@PEAU?$_Tree_node@U?$pair@$$CB_JV?$basic_string@DU?$char_traits@D@std@@V?$allocator@D@2@@std@@@std@@PEAX@2@@?$_Tree@V?$_Tmap_traits@_JV?$basic_string@DU?$char_traits@D@std@@V?$allocator@D@2@@std@@U?$less@_J@2@V?$allocator@U?$pair@$$CB_JV?$basic_string@DU?$char_traits@D@std@@V?$allocator@D@2@@std@@@std@@@2@$0A@@std@@@std@@IEAA?AU?$pair@V?$_Tree_iterator@V?$_Tree_val@U?$_Tree_simple_types@U?$pair@$$CB_JV?$basic_string@DU?$char_traits@D@std@@V?$allocator@D@2@@std@@@std@@@std@@@std@@@std@@_N@1@_NAEAU?$pair@$$CB_JV?$basic_string@DU?$char_traits@D@std@@V?$allocator@D@2@@std@@@1@PEAU?$_Tree_node@U?$pair@$$CB_JV?$basic_string@DU?$char_traits@D@std@@V?$allocator@D@2@@std@@@std@@PEAX@1@@Z 0000000140025174     LoadXlsMsg.obj
 0002:0000b188       $ip2state$??$_Insert_nohint@AEAU?$pair@$$CB_JV?$basic_string@DU?$char_traits@D@std@@V?$allocator@D@2@@std@@@std@@PEAU?$_Tree_node@U?$pair@$$CB_JV?$basic_string@DU?$char_traits@D@std@@V?$allocator@D@2@@std@@@std@@PEAX@2@@?$_Tree@V?$_Tmap_traits@_JV?$basic_string@DU?$char_traits@D@std@@V?$allocator@D@2@@std@@U?$less@_J@2@V?$allocator@U?$pair@$$CB_JV?$basic_string@DU?$char_traits@D@std@@V?$allocator@D@2@@std@@@std@@@2@$0A@@std@@@std@@IEAA?AU?$pair@V?$_Tree_iterator@V?$_Tree_val@U?$_Tree_simple_types@U?$pair@$$CB_JV?$basic_string@DU?$char_traits@D@std@@V?$allocator@D@2@@std@@@std@@@std@@@std@@@std@@_N@1@_NAEAU?$pair@$$CB_JV?$basic_string@DU?$char_traits@D@std@@V?$allocator@D@2@@std@@@1@PEAU?$_Tree_node@U?$pair@$$CB_JV?$basic_string@DU?$char_traits@D@std@@V?$allocator@D@2@@std@@@std@@PEAX@1@@Z 0000000140025188     LoadXlsMsg.obj
 0002:0000b198       $unwind$?catch$0@?0???$_Insert_nohint@AEAU?$pair@$$CB_JV?$basic_string@DU?$char_traits@D@std@@V?$allocator@D@2@@std@@@std@@PEAU?$_Tree_node@U?$pair@$$CB_JV?$basic_string@DU?$char_traits@D@std@@V?$allocator@D@2@@std@@@std@@PEAX@2@@?$_Tree@V?$_Tmap_traits@_JV?$basic_string@DU?$char_traits@D@std@@V?$allocator@D@2@@std@@U?$less@_J@2@V?$allocator@U?$pair@$$CB_JV?$basic_string@DU?$char_traits@D@std@@V?$allocator@D@2@@std@@@std@@@2@$0A@@std@@@std@@IEAA?AU?$pair@V?$_Tree_iterator@V?$_Tree_val@U?$_Tree_simple_types@U?$pair@$$CB_JV?$basic_string@DU?$char_traits@D@std@@V?$allocator@D@2@@std@@@std@@@std@@@std@@@std@@_N@1@_NAEAU?$pair@$$CB_JV?$basic_string@DU?$char_traits@D@std@@V?$allocator@D@2@@std@@@1@PEAU?$_Tree_node@U?$pair@$$CB_JV?$basic_string@DU?$char_traits@D@std@@V?$allocator@D@2@@std@@@std@@PEAX@1@@Z@4HA 0000000140025198     LoadXlsMsg.obj
 0002:0000b1a8       $unwind$?Run@CServerAppApp@@UEAAHXZ 00000001400251a8     ServerApp.obj
 0002:0000b1c0       $stateUnwindMap$?Run@CServerAppApp@@UEAAHXZ 00000001400251c0     ServerApp.obj
 0002:0000b1c8       $ip2state$?Run@CServerAppApp@@UEAAHXZ 00000001400251c8     ServerApp.obj
 0002:0000b1e0       $unwind$??0PROTO_GAME_USER_INFO_tag@@QEAA@XZ 00000001400251e0     ServerAppDlg.obj
 0002:0000b1f4       $unwind$??__Eg_cServerLog@@YAXXZ 00000001400251f4     ServerAppDlg.obj
 0002:0000b204       $unwind$??__E__api_holder_ILTCommon_Server_g_pLTSCommon__@@YAXXZ 0000000140025204     ServerAppDlg.obj
 0002:0000b214       $stateUnwindMap$??__E__api_holder_ILTCommon_Server_g_pLTSCommon__@@YAXXZ 0000000140025214     ServerAppDlg.obj
 0002:0000b220       $ip2state$??__E__api_holder_ILTCommon_Server_g_pLTSCommon__@@YAXXZ 0000000140025220     ServerAppDlg.obj
 0002:0000b238       $unwind$?ConsoleOutputFn@CGameServerAppHandler@@UEAAIHHPEBD@Z 0000000140025238     ServerAppDlg.obj
 0002:0000b25c       $stateUnwindMap$?StopServer@CServerAppDlg@@QEAA_NXZ 000000014002525c     ServerAppDlg.obj
 0002:0000b25c       $stateUnwindMap$?ServerUpdate@CServerAppDlg@@QEAAXXZ 000000014002525c     ServerAppDlg.obj
 0002:0000b25c       $stateUnwindMap$?ConsoleOutputFn@CGameServerAppHandler@@UEAAIHHPEBD@Z 000000014002525c     ServerAppDlg.obj
 0002:0000b25c       $stateUnwindMap$?OutOfMemory@CGameServerAppHandler@@UEAAIXZ 000000014002525c     ServerAppDlg.obj
 0002:0000b268       $ip2state$?ConsoleOutputFn@CGameServerAppHandler@@UEAAIHHPEBD@Z 0000000140025268     ServerAppDlg.obj
 0002:0000b288       $unwind$?OutOfMemory@CGameServerAppHandler@@UEAAIXZ 0000000140025288     ServerAppDlg.obj
 0002:0000b2a0       $ip2state$?OutOfMemory@CGameServerAppHandler@@UEAAIXZ 00000001400252a0     ServerAppDlg.obj
 0002:0000b2b8       $unwind$?GetProcessMemoryUsage@CGameServerAppHandler@@UEAAKXZ 00000001400252b8     ServerAppDlg.obj
 0002:0000b2c8       $chain$0$?GetProcessMemoryUsage@CGameServerAppHandler@@UEAAKXZ 00000001400252c8     ServerAppDlg.obj
 0002:0000b2dc       $chain$1$?GetProcessMemoryUsage@CGameServerAppHandler@@UEAAKXZ 00000001400252dc     ServerAppDlg.obj
 0002:0000b2ec       $unwind$?WriteData@PROTO_SERVERAPPMSG_INIT@@UEAA_NPEAVILTMessage_Write@@@Z 00000001400252ec     ServerAppDlg.obj
 0002:0000b2ec       $unwind$??0PROTO_START_HOST_tag@@QEAA@XZ 00000001400252ec     ServerAppDlg.obj
 0002:0000b2ec       $unwind$??_G?$basic_stringstream@DU?$char_traits@D@std@@V?$allocator@D@2@@std@@UEAAPEAXI@Z 00000001400252ec     safe_string_x64:safe_string.obj
 0002:0000b2fc       $unwind$??0CServerAppDlg@@QEAA@PEAVCWnd@@@Z 00000001400252fc     ServerAppDlg.obj
 0002:0000b314       $stateUnwindMap$??0CServerAppDlg@@QEAA@PEAVCWnd@@@Z 0000000140025314     ServerAppDlg.obj
 0002:0000b348       $ip2state$??0CServerAppDlg@@QEAA@PEAVCWnd@@@Z 0000000140025348     ServerAppDlg.obj
 0002:0000b370       $unwind$??1CServerAppDlg@@UEAA@XZ 0000000140025370     ServerAppDlg.obj
 0002:0000b388       $ip2state$??1CServerAppDlg@@UEAA@XZ 0000000140025388     ServerAppDlg.obj
 0002:0000b390       $unwind$?OnInitDialog@CServerAppDlg@@MEAAHXZ 0000000140025390     ServerAppDlg.obj
 0002:0000b3b4       $stateUnwindMap$?OnInitDialog@CServerAppDlg@@MEAAHXZ 00000001400253b4     ServerAppDlg.obj
 0002:0000b400       $ip2state$?OnInitDialog@CServerAppDlg@@MEAAHXZ 0000000140025400     ServerAppDlg.obj
 0002:0000b480       $unwind$?OnShellMessage@CServerAppDlg@@QEAAXAEAVILTMessage_Read@@@Z 0000000140025480     ServerAppDlg.obj
 0002:0000b4a8       $stateUnwindMap$?OnShellMessage@CServerAppDlg@@QEAAXAEAVILTMessage_Read@@@Z 00000001400254a8     ServerAppDlg.obj
 0002:0000b4f0       $ip2state$?OnShellMessage@CServerAppDlg@@QEAAXAEAVILTMessage_Read@@@Z 00000001400254f0     ServerAppDlg.obj
 0002:0000b590       $unwind$?AddServerMsg@CServerAppDlg@@QEAAXPEBDH@Z 0000000140025590     ServerAppDlg.obj
 0002:0000b5ac       $stateUnwindMap$?AddServerMsg@CServerAppDlg@@QEAAXPEBDH@Z 00000001400255ac     ServerAppDlg.obj
 0002:0000b5ac       $stateUnwindMap$?RECV_MSG_AIITEM_GROUP_RATE_RESULT@CServerAppDlg@@AEAAX_J@Z 00000001400255ac     ServerAppDlg.obj
 0002:0000b5ac       $stateUnwindMap$?SendToServerShellAutoMatchStartingUserInfo@CServerAppDlg@@AEAAXPEAUtagCOPYDATASTRUCT@@@Z 00000001400255ac     ServerAppDlg.obj
 0002:0000b5b8       $ip2state$?AddServerMsg@CServerAppDlg@@QEAAXPEBDH@Z 00000001400255b8     ServerAppDlg.obj
 0002:0000b5d0       $unwind$?LoadServer@CServerAppDlg@@QEAA_NXZ 00000001400255d0     ServerAppDlg.obj
 0002:0000b5f0       $stateUnwindMap$?LoadServer@CServerAppDlg@@QEAA_NXZ 00000001400255f0     ServerAppDlg.obj
 0002:0000b630       $ip2state$?LoadServer@CServerAppDlg@@QEAA_NXZ 0000000140025630     ServerAppDlg.obj
 0002:0000b688       $unwind$?RunServer@CServerAppDlg@@QEAA_NXZ 0000000140025688     ServerAppDlg.obj
 0002:0000b6a4       $stateUnwindMap$?RunServer@CServerAppDlg@@QEAA_NXZ 00000001400256a4     ServerAppDlg.obj
 0002:0000b6d0       $ip2state$?RunServer@CServerAppDlg@@QEAA_NXZ 00000001400256d0     ServerAppDlg.obj
 0002:0000b728       $unwind$?StopServer@CServerAppDlg@@QEAA_NXZ 0000000140025728     ServerAppDlg.obj
 0002:0000b740       $ip2state$?StopServer@CServerAppDlg@@QEAA_NXZ 0000000140025740     ServerAppDlg.obj
 0002:0000b758       $unwind$?Thread_SendGameInfo@@YAXPEAVCServerAppDlg@@AEAUPROTO_START_HOST_tag@@@Z 0000000140025758     ServerAppDlg.obj
 0002:0000b77c       $stateUnwindMap$?Thread_SendGameInfo@@YAXPEAVCServerAppDlg@@AEAUPROTO_START_HOST_tag@@@Z 000000014002577c     ServerAppDlg.obj
 0002:0000b7b0       $ip2state$?Thread_SendGameInfo@@YAXPEAVCServerAppDlg@@AEAUPROTO_START_HOST_tag@@@Z 00000001400257b0     ServerAppDlg.obj
 0002:0000b808       $unwind$?Thread_SendUserInfo@@YAXPEAVCServerAppDlg@@AEAUPROTO_GAME_USER_INFO_tag@@@Z 0000000140025808     ServerAppDlg.obj
 0002:0000b828       $stateUnwindMap$?Thread_SendUserInfo@@YAXPEAVCServerAppDlg@@AEAUPROTO_GAME_USER_INFO_tag@@@Z 0000000140025828     ServerAppDlg.obj
 0002:0000b838       $ip2state$?Thread_SendUserInfo@@YAXPEAVCServerAppDlg@@AEAUPROTO_GAME_USER_INFO_tag@@@Z 0000000140025838     ServerAppDlg.obj
 0002:0000b860       $unwind$?ThreadUpdate@CServerAppDlg@@SAXPEAX@Z 0000000140025860     ServerAppDlg.obj
 0002:0000b88c       $stateUnwindMap$?ThreadUpdate@CServerAppDlg@@SAXPEAX@Z 000000014002588c     ServerAppDlg.obj
 0002:0000b8a0       $ip2state$?ThreadUpdate@CServerAppDlg@@SAXPEAX@Z 00000001400258a0     ServerAppDlg.obj
 0002:0000b8c8       $unwind$?ServerUpdate@CServerAppDlg@@QEAAXXZ 00000001400258c8     ServerAppDlg.obj
 0002:0000b8f0       $ip2state$?ServerUpdate@CServerAppDlg@@QEAAXXZ 00000001400258f0     ServerAppDlg.obj
 0002:0000b908       $unwind$?AddResources@CServerAppDlg@@QEAA_NXZ 0000000140025908     ServerAppDlg.obj
 0002:0000b928       $stateUnwindMap$?AddResources@CServerAppDlg@@QEAA_NXZ 0000000140025928     ServerAppDlg.obj
 0002:0000b970       $ip2state$?AddResources@CServerAppDlg@@QEAA_NXZ 0000000140025970     ServerAppDlg.obj
 0002:0000b9d8       $unwind$?OnGameServerMsg@CServerAppDlg@@IEAA_J_K_J@Z 00000001400259d8     ServerAppDlg.obj
 0002:0000b9fc       $stateUnwindMap$?OnGameServerMsg@CServerAppDlg@@IEAA_J_K_J@Z 00000001400259fc     ServerAppDlg.obj
 0002:0000ba20       $ip2state$?OnGameServerMsg@CServerAppDlg@@IEAA_J_K_J@Z 0000000140025a20     ServerAppDlg.obj
 0002:0000ba60       $unwind$?OnCopyData@CServerAppDlg@@IEAAHPEAVCWnd@@PEAUtagCOPYDATASTRUCT@@@Z 0000000140025a60     ServerAppDlg.obj
 0002:0000ba88       $stateUnwindMap$?OnCopyData@CServerAppDlg@@IEAAHPEAVCWnd@@PEAUtagCOPYDATASTRUCT@@@Z 0000000140025a88     ServerAppDlg.obj
 0002:0000bad0       $ip2state$?OnCopyData@CServerAppDlg@@IEAAHPEAVCWnd@@PEAUtagCOPYDATASTRUCT@@@Z 0000000140025ad0     ServerAppDlg.obj
 0002:0000bb58       $unwind$?OnTimer@CServerAppDlg@@QEAAX_K@Z 0000000140025b58     ServerAppDlg.obj
 0002:0000bb70       $ip2state$?OnTimer@CServerAppDlg@@QEAAX_K@Z 0000000140025b70     ServerAppDlg.obj
 0002:0000bb88       $unwind$?OnBnClickedButtonGo@CServerAppDlg@@QEAAXXZ 0000000140025b88     ServerAppDlg.obj
 0002:0000bb9c       $unwind$?SaveHostGameInfo@CServerAppDlg@@IEAAXXZ 0000000140025b9c     ServerAppDlg.obj
 0002:0000bbc8       $stateUnwindMap$?SaveHostGameInfo@CServerAppDlg@@IEAAXXZ 0000000140025bc8     ServerAppDlg.obj
 0002:0000bbe0       $ip2state$?SaveHostGameInfo@CServerAppDlg@@IEAAXXZ 0000000140025be0     ServerAppDlg.obj
 0002:0000bc10       $unwind$?LoadHostGameInfo@CServerAppDlg@@IEAAXXZ 0000000140025c10     ServerAppDlg.obj
 0002:0000bc3c       $stateUnwindMap$?LoadHostGameInfo@CServerAppDlg@@IEAAXXZ 0000000140025c3c     ServerAppDlg.obj
 0002:0000bc58       $ip2state$?LoadHostGameInfo@CServerAppDlg@@IEAAXXZ 0000000140025c58     ServerAppDlg.obj
 0002:0000bc88       $unwind$?GetOptionValueString@CServerAppDlg@@IEAA?AV?$basic_string@DU?$char_traits@D@std@@V?$allocator@D@2@@std@@V23@00@Z 0000000140025c88     ServerAppDlg.obj
 0002:0000bcb0       $stateUnwindMap$?GetOptionValueString@CServerAppDlg@@IEAA?AV?$basic_string@DU?$char_traits@D@std@@V?$allocator@D@2@@std@@V23@00@Z 0000000140025cb0     ServerAppDlg.obj
 0002:0000bcd0       $ip2state$?GetOptionValueString@CServerAppDlg@@IEAA?AV?$basic_string@DU?$char_traits@D@std@@V?$allocator@D@2@@std@@V23@00@Z 0000000140025cd0     ServerAppDlg.obj
 0002:0000bcf0       $unwind$?ReadGSMMemory@CServerAppDlg@@QEAA_NPEAX0_K@Z 0000000140025cf0     ServerAppDlg.obj
 0002:0000bd04       $unwind$?RECV_MSG_INSERTCHARACTER@CServerAppDlg@@AEAAX_J@Z 0000000140025d04     ServerAppDlg.obj
 0002:0000bd20       $stateUnwindMap$?RECV_MSG_INSERTCHARACTER@CServerAppDlg@@AEAAX_J@Z 0000000140025d20     ServerAppDlg.obj
 0002:0000bd30       $ip2state$?RECV_MSG_INSERTCHARACTER@CServerAppDlg@@AEAAX_J@Z 0000000140025d30     ServerAppDlg.obj
 0002:0000bd58       $unwind$?RECV_MSG_AIITEM_DEC@CServerAppDlg@@AEAAX_J@Z 0000000140025d58     ServerAppDlg.obj
 0002:0000bd74       $stateUnwindMap$?RECV_MSG_AIITEM_DEC@CServerAppDlg@@AEAAX_J@Z 0000000140025d74     ServerAppDlg.obj
 0002:0000bd80       $ip2state$?RECV_MSG_AIITEM_DEC@CServerAppDlg@@AEAAX_J@Z 0000000140025d80     ServerAppDlg.obj
 0002:0000bd98       $unwind$?RECV_MSG_AIITEM_GROUP_RATE_RESULT@CServerAppDlg@@AEAAX_J@Z 0000000140025d98     ServerAppDlg.obj
 0002:0000bdb8       $ip2state$?RECV_MSG_AIITEM_GROUP_RATE_RESULT@CServerAppDlg@@AEAAX_J@Z 0000000140025db8     ServerAppDlg.obj
 0002:0000bdd0       $unwind$?RECV_MSG_USER_DISCONNECTED@CServerAppDlg@@AEAAX_J@Z 0000000140025dd0     ServerAppDlg.obj
 0002:0000bdf0       $ip2state$?RECV_MSG_USER_DISCONNECTED@CServerAppDlg@@AEAAX_J@Z 0000000140025df0     ServerAppDlg.obj
 0002:0000be08       $unwind$?SendServerAppInit@CServerAppDlg@@AEAAXXZ 0000000140025e08     ServerAppDlg.obj
 0002:0000be20       $stateUnwindMap$?SendServerAppInit@CServerAppDlg@@AEAAXXZ 0000000140025e20     ServerAppDlg.obj
 0002:0000be28       $ip2state$?SendServerAppInit@CServerAppDlg@@AEAAXXZ 0000000140025e28     ServerAppDlg.obj
 0002:0000be40       $unwind$?DownloadUCCMapFile_HTTP@CServerAppDlg@@AEAA?AW4UCCMAPDOWNLOADREAULT@@V?$basic_string@DU?$char_traits@D@std@@V?$allocator@D@2@@std@@@Z 0000000140025e40     ServerAppDlg.obj
 0002:0000be6c       $stateUnwindMap$?DownloadUCCMapFile_HTTP@CServerAppDlg@@AEAA?AW4UCCMAPDOWNLOADREAULT@@V?$basic_string@DU?$char_traits@D@std@@V?$allocator@D@2@@std@@@Z 0000000140025e6c     ServerAppDlg.obj
 0002:0000bed0       $ip2state$?DownloadUCCMapFile_HTTP@CServerAppDlg@@AEAA?AW4UCCMAPDOWNLOADREAULT@@V?$basic_string@DU?$char_traits@D@std@@V?$allocator@D@2@@std@@@Z 0000000140025ed0     ServerAppDlg.obj
 0002:0000bf38       $unwind$?SendServerAppInitFail@CServerAppDlg@@AEAAXHH@Z 0000000140025f38     ServerAppDlg.obj
 0002:0000bf50       $stateUnwindMap$?SendServerAppInitFail@CServerAppDlg@@AEAAXHH@Z 0000000140025f50     ServerAppDlg.obj
 0002:0000bf60       $ip2state$?SendServerAppInitFail@CServerAppDlg@@AEAAXHH@Z 0000000140025f60     ServerAppDlg.obj
 0002:0000bf80       $unwind$?GetDownloadPath@CServerAppDlg@@AEAA?AV?$basic_string@DU?$char_traits@D@std@@V?$allocator@D@2@@std@@XZ 0000000140025f80     ServerAppDlg.obj
 0002:0000bf98       $stateUnwindMap$?GetDownloadPath@CServerAppDlg@@AEAA?AV?$basic_string@DU?$char_traits@D@std@@V?$allocator@D@2@@std@@XZ 0000000140025f98     ServerAppDlg.obj
 0002:0000bfa0       $ip2state$?GetDownloadPath@CServerAppDlg@@AEAA?AV?$basic_string@DU?$char_traits@D@std@@V?$allocator@D@2@@std@@XZ 0000000140025fa0     ServerAppDlg.obj
 0002:0000bfa8       $unwind$?SendToServerShellAutoMatchStartingUserInfo@CServerAppDlg@@AEAAXPEAUtagCOPYDATASTRUCT@@@Z 0000000140025fa8     ServerAppDlg.obj
 0002:0000bfc8       $ip2state$?SendToServerShellAutoMatchStartingUserInfo@CServerAppDlg@@AEAAXPEAUtagCOPYDATASTRUCT@@@Z 0000000140025fc8     ServerAppDlg.obj
 0002:0000bfe0       $unwind$??1?$CAPIHolder@VILTCommon@@@@UEAA@XZ 0000000140025fe0     ServerAppDlg.obj
 0002:0000bff8       $ip2state$??1?$CAPIHolder@VILTCommon@@@@UEAA@XZ 0000000140025ff8     ServerAppDlg.obj
 0002:0000c000       $unwind$??$?HDU?$char_traits@D@std@@V?$allocator@D@1@@std@@YA?AV?$basic_string@DU?$char_traits@D@std@@V?$allocator@D@2@@0@AEBV10@0@Z 0000000140026000     ServerAppDlg.obj
 0002:0000c01c       $stateUnwindMap$??$?HDU?$char_traits@D@std@@V?$allocator@D@1@@std@@YA?AV?$basic_string@DU?$char_traits@D@std@@V?$allocator@D@2@@0@AEBV10@0@Z 000000014002601c     ServerAppDlg.obj
 0002:0000c028       $ip2state$??$?HDU?$char_traits@D@std@@V?$allocator@D@1@@std@@YA?AV?$basic_string@DU?$char_traits@D@std@@V?$allocator@D@2@@0@AEBV10@0@Z 0000000140026028     ServerAppDlg.obj
 0002:0000c030       $unwind$?reserve@?$basic_string@DU?$char_traits@D@std@@V?$allocator@D@2@@std@@QEAAX_K@Z 0000000140026030     ServerAppDlg.obj
 0002:0000c03c       $chain$0$?reserve@?$basic_string@DU?$char_traits@D@std@@V?$allocator@D@2@@std@@QEAAX_K@Z 000000014002603c     ServerAppDlg.obj
 0002:0000c050       $chain$2$?reserve@?$basic_string@DU?$char_traits@D@std@@V?$allocator@D@2@@std@@QEAAX_K@Z 0000000140026050     ServerAppDlg.obj
 0002:0000c068       $chain$3$?reserve@?$basic_string@DU?$char_traits@D@std@@V?$allocator@D@2@@std@@QEAAX_K@Z 0000000140026068     ServerAppDlg.obj
 0002:0000c078       $chain$4$?reserve@?$basic_string@DU?$char_traits@D@std@@V?$allocator@D@2@@std@@QEAAX_K@Z 0000000140026078     ServerAppDlg.obj
 0002:0000c088       $chain$5$?reserve@?$basic_string@DU?$char_traits@D@std@@V?$allocator@D@2@@std@@QEAAX_K@Z 0000000140026088     ServerAppDlg.obj
 0002:0000c0a4       $unwind$fscanf_s           00000001400260a4     ServerAppDlg.obj
 0002:0000c0b0       $unwind$??1CWaitCursor@@QEAA@XZ 00000001400260b0     ServerAppDlg.obj
 0002:0000c0c4       $stateUnwindMap$??1CWaitCursor@@QEAA@XZ 00000001400260c4     ServerAppDlg.obj
 0002:0000c0dc       $tryMap$??1CWaitCursor@@QEAA@XZ 00000001400260dc     ServerAppDlg.obj
 0002:0000c0f0       $handlerMap$0$??1CWaitCursor@@QEAA@XZ 00000001400260f0     ServerAppDlg.obj
 0002:0000c108       $ip2state$??1CWaitCursor@@QEAA@XZ 0000000140026108     ServerAppDlg.obj
 0002:0000c130       $unwind$?catch$1@?0???1CWaitCursor@@QEAA@XZ@4HA 0000000140026130     ServerAppDlg.obj
 0002:0000c144       $unwind$?Readint32@ILTMessage_Read@@QEAAHXZ 0000000140026144     ServerAppDlg.obj
 0002:0000c144       $unwind$?Readuint32@ILTMessage_Read@@QEAAIXZ 0000000140026144     ServerAppDlg.obj
 0002:0000c14c       $unwind$?USNtoStr@EXPAND_USN@@YA?AV?$basic_string@DU?$char_traits@D@std@@V?$allocator@D@2@@std@@_J@Z 000000014002614c     ServerAppDlg.obj
 0002:0000c15c       $unwind$?PostReadData@GAMEPROTO_SC_COMMON@@UEAA_NPEAVILTMessage_Read@@@Z 000000014002615c     ServerAppDlg.obj
 0002:0000c15c       $unwind$?ReadData@PROTO_SERVERAPPMSG_INIT@@UEAA_NPEAVILTMessage_Read@@@Z 000000014002615c     ServerAppDlg.obj
 0002:0000c168       $chain$0$?PostReadData@GAMEPROTO_SC_COMMON@@UEAA_NPEAVILTMessage_Read@@@Z 0000000140026168     ServerAppDlg.obj
 0002:0000c17c       $chain$1$?PostReadData@GAMEPROTO_SC_COMMON@@UEAA_NPEAVILTMessage_Read@@@Z 000000014002617c     ServerAppDlg.obj
 0002:0000c18c       $chain$0$?ReadData@PROTO_SERVERAPPMSG_INIT@@UEAA_NPEAVILTMessage_Read@@@Z 000000014002618c     ServerAppDlg.obj
 0002:0000c1a0       $chain$1$?ReadData@PROTO_SERVERAPPMSG_INIT@@UEAA_NPEAVILTMessage_Read@@@Z 00000001400261a0     ServerAppDlg.obj
 0002:0000c1b0       $unwind$?sprintf_s@internal@cf@@YAHPEAD_KPEBDAEAPEAD@Z 00000001400261b0     safe_string_x64:safe_string.obj
 0002:0000c1d4       $stateUnwindMap$?sprintf_s@internal@cf@@YAHPEAD_KPEBDAEAPEAD@Z 00000001400261d4     safe_string_x64:safe_string.obj
 0002:0000c1f8       $ip2state$?sprintf_s@internal@cf@@YAHPEAD_KPEBDAEAPEAD@Z 00000001400261f8     safe_string_x64:safe_string.obj
 0002:0000c228       $unwind$?strcpy_s@cf@@YAHPEAD_KPEBD@Z 0000000140026228     safe_string_x64:safe_string.obj
 0002:0000c248       $stateUnwindMap$?strncpy_s@cf@@YAHPEAD_KPEBD1@Z 0000000140026248     safe_string_x64:safe_string.obj
 0002:0000c248       $stateUnwindMap$?strcpy_s@cf@@YAHPEAD_KPEBD@Z 0000000140026248     safe_string_x64:safe_string.obj
 0002:0000c268       $ip2state$?strcpy_s@cf@@YAHPEAD_KPEBD@Z 0000000140026268     safe_string_x64:safe_string.obj
 0002:0000c298       $unwind$?strncpy_s@cf@@YAHPEAD_KPEBD1@Z 0000000140026298     safe_string_x64:safe_string.obj
 0002:0000c2b8       $ip2state$?strncpy_s@cf@@YAHPEAD_KPEBD1@Z 00000001400262b8     safe_string_x64:safe_string.obj
 0002:0000c2e8       $unwind$?sprintf_s@cf@@YAHPEAD_KPEBDZZ 00000001400262e8     safe_string_x64:safe_string.obj
 0002:0000c2f0       $unwind$??0?$basic_stringstream@DU?$char_traits@D@std@@V?$allocator@D@2@@std@@QEAA@H@Z 00000001400262f0     safe_string_x64:safe_string.obj
 0002:0000c304       $stateUnwindMap$??0?$basic_stringstream@DU?$char_traits@D@std@@V?$allocator@D@2@@std@@QEAA@H@Z 0000000140026304     safe_string_x64:safe_string.obj
 0002:0000c318       $ip2state$??0?$basic_stringstream@DU?$char_traits@D@std@@V?$allocator@D@2@@std@@QEAA@H@Z 0000000140026318     safe_string_x64:safe_string.obj
 0002:0000c330       $unwind$?seekpos@?$basic_stringbuf@DU?$char_traits@D@std@@V?$allocator@D@2@@std@@MEAA?AV?$fpos@U_Mbstatet@@@2@V32@H@Z 0000000140026330     safe_string_x64:safe_string.obj
 0002:0000c344       $unwind$?seekoff@?$basic_stringbuf@DU?$char_traits@D@std@@V?$allocator@D@2@@std@@MEAA?AV?$fpos@U_Mbstatet@@@2@_JHH@Z 0000000140026344     safe_string_x64:safe_string.obj
 0002:0000c35c       $unwind$??1sentry@?$basic_ostream@DU?$char_traits@D@std@@@std@@QEAA@XZ 000000014002635c     safe_string_x64:safe_string.obj
 0002:0000c370       $ip2state$??1sentry@?$basic_ostream@DU?$char_traits@D@std@@@std@@QEAA@XZ 0000000140026370     safe_string_x64:safe_string.obj
 0002:0000c380       $unwind$??1_Sentry_base@?$basic_ostream@DU?$char_traits@D@std@@@std@@QEAA@XZ 0000000140026380     safe_string_x64:safe_string.obj
 0002:0000c390       $ip2state$??1_Sentry_base@?$basic_ostream@DU?$char_traits@D@std@@@std@@QEAA@XZ 0000000140026390     safe_string_x64:safe_string.obj
 0002:0000c398       $unwind$??$?6U?$char_traits@D@std@@@std@@YAAEAV?$basic_ostream@DU?$char_traits@D@std@@@0@AEAV10@PEBD@Z 0000000140026398     safe_string_x64:safe_string.obj
 0002:0000c3b4       $stateUnwindMap$??$?6U?$char_traits@D@std@@@std@@YAAEAV?$basic_ostream@DU?$char_traits@D@std@@@0@AEAV10@PEBD@Z 00000001400263b4     safe_string_x64:safe_string.obj
 0002:0000c3e4       $tryMap$??$?6U?$char_traits@D@std@@@std@@YAAEAV?$basic_ostream@DU?$char_traits@D@std@@@0@AEAV10@PEBD@Z 00000001400263e4     safe_string_x64:safe_string.obj
 0002:0000c3f8       $handlerMap$0$??$?6U?$char_traits@D@std@@@std@@YAAEAV?$basic_ostream@DU?$char_traits@D@std@@@0@AEAV10@PEBD@Z 00000001400263f8     safe_string_x64:safe_string.obj
 0002:0000c410       $ip2state$??$?6U?$char_traits@D@std@@@std@@YAAEAV?$basic_ostream@DU?$char_traits@D@std@@@0@AEAV10@PEBD@Z 0000000140026410     safe_string_x64:safe_string.obj
 0002:0000c450       $unwind$?catch$4@?0???$?6U?$char_traits@D@std@@@std@@YAAEAV?$basic_ostream@DU?$char_traits@D@std@@@0@AEAV10@PEBD@Z@4HA 0000000140026450     safe_string_x64:safe_string.obj
 0002:0000c460       $xdatasym                  0000000140026460     msvcrt:amdsecgs.obj
 0002:0000c464       $unwind$?__scrt_initialize_thread_safe_statics@@YAHXZ 0000000140026464     msvcrt:thread_safe_statics.obj
 0002:0000c480       $ip2state$?__scrt_initialize_thread_safe_statics@@YAHXZ 0000000140026480     msvcrt:thread_safe_statics.obj
 0002:0000c488       $unwind$__scrt_is_nonwritable_in_current_image 0000000140026488     msvcrt:utility.obj
 0002:0000c4a8       $unwind$__scrt_is_nonwritable_in_current_image$filt$0 00000001400264a8     msvcrt:utility.obj
 0002:0000c4b0       $unwind$__scrt_initialize_onexit_tables 00000001400264b0     msvcrt:utility.obj
 0002:0000c4b8       $unwind$__report_gsfailure 00000001400264b8     msvcrt:gs_report.obj
 0002:0000c4c0       $unwind$capture_previous_context 00000001400264c0     msvcrt:gs_report.obj
 0002:0000c4cc       $unwind$?__scrt_common_main_seh@@YAHXZ 00000001400264cc     msvcrt:exe_winmain.obj
 0002:0000c500       $unwind$__scrt_get_show_window_mode 0000000140026500     msvcrt:utility_desktop.obj
 0002:0000c508       $unwind$__scrt_fastfail    0000000140026508     msvcrt:utility_desktop.obj
 0002:0000c518       $unwind$__isa_available_init 0000000140026518     msvcrt:cpu_disp.obj
 0002:0000c528       $unwind$__security_init_cookie 0000000140026528     msvcrt:gs_support.obj
 0002:0000c534       $unwind$__GSHandlerCheckCommon 0000000140026534     msvcrt:gshandler.obj
 0002:0000c540       $xdatasym                  0000000140026540     msvcrt:guard_dispatch.obj
 0002:0000c544       $unwind$__GSHandlerCheck_EH 0000000140026544     msvcrt:gshandlereh.obj
 0002:0000c560       $xdatasym                  0000000140026560     msvcrt:chkstk.obj
 0002:0000c5c0       .edata                     00000001400265c0     ServerApp_x64.exp
 0002:0000c5e8       rgpv                       00000001400265e8     ServerApp_x64.exp
 0002:0000c5f0       rgszName                   00000001400265f0     ServerApp_x64.exp
 0002:0000c5f8       rgwOrd                     00000001400265f8     ServerApp_x64.exp
 0002:0000c5fc       szName                     00000001400265fc     ServerApp_x64.exp
 0002:0000c60e       $N00001                    000000014002660e     ServerApp_x64.exp
 0002:0000c61a       $N00002                    000000014002661a     ServerApp_x64.exp
 0002:0000d540       .idata$6                   0000000140027540     Psapi:PSAPI.DLL
 0002:0000d54a       .idata$6                   000000014002754a     mfc140:mfc140.dll
 0002:0000d9fa       .idata$6                   00000001400279fa     kernel32:KERNEL32.dll
 0002:0000da84       .idata$6                   0000000140027a84     user32:USER32.dll
 0002:0000daa8       .idata$6                   0000000140027aa8     shell32:SHELL32.dll
 0002:0000dac6       .idata$6                   0000000140027ac6     shlwapi:SHLWAPI.dll
 0002:0000db16       .idata$6                   0000000140027b16     msvcprt:MSVCP140.dll
 0002:0000db72       .idata$6                   0000000140027b72     Wininet:WININET.dll
 0002:0000dc1c       .idata$6                   0000000140027c1c     DbgHelp:dbghelp.dll
 0002:0000dc36       .idata$6                   0000000140027c36     winmm:WINMM.dll
 0002:0000dcf8       .idata$6                   0000000140027cf8     winhttp:WINHTTP.dll
 0002:0000dd04       .idata$6                   0000000140027d04     ws2_32:WS2_32.dll
 0002:0000ddb6       .idata$6                   0000000140027db6     vcruntime:VCRUNTIME140.dll
 0002:0000e18e       .idata$6                   000000014002818e     ucrt:api-ms-win-crt-stdio-l1-1-0.dll
 0002:0000e1ae       .idata$6                   00000001400281ae     ucrt:api-ms-win-crt-runtime-l1-1-0.dll
 0002:0000e1d0       .idata$6                   00000001400281d0     ucrt:api-ms-win-crt-filesystem-l1-1-0.dll
 0002:0000e1f6       .idata$6                   00000001400281f6     ucrt:api-ms-win-crt-string-l1-1-0.dll
 0002:0000e218       .idata$6                   0000000140028218     ucrt:api-ms-win-crt-convert-l1-1-0.dll
 0002:0000e23a       .idata$6                   000000014002823a     ucrt:api-ms-win-crt-utility-l1-1-0.dll
 0002:0000e25c       .idata$6                   000000014002825c     ucrt:api-ms-win-crt-time-l1-1-0.dll
 0002:0000e27c       .idata$6                   000000014002827c     ucrt:api-ms-win-crt-heap-l1-1-0.dll
 0002:0000e29c       .idata$6                   000000014002829c     ucrt:api-ms-win-crt-math-l1-1-0.dll
 0002:0000e2bc       .idata$6                   00000001400282bc     ucrt:api-ms-win-crt-locale-l1-1-0.dll
 0003:00000034       ?prefix@?1??uploadLOG@Uploader@crs@@AEAA_NAEAVHttpHandle@3@AEAU_SYSTEMTIME@@AEAVLogBuffer@3@@Z@4PADA 0000000140029034     crs_uploader.obj
 0003:000005a0       ?__api_holder_ILTCommon_Server_g_pLTSCommon__@@3V?$CAPIHolder@VILTCommon@@@@A 00000001400295a0     ServerAppDlg.obj
 0003:00000c68       ?_Tss_mutex@@3U_RTL_CRITICAL_SECTION@@A 0000000140029c68     msvcrt:thread_safe_statics.obj
 0003:00000c90       ?_Tss_cv@@3U_RTL_CONDITION_VARIABLE@@A 0000000140029c90     msvcrt:thread_safe_statics.obj
 0003:00000c98       ?_Tss_event@@3PEAXEA       0000000140029c98     msvcrt:thread_safe_statics.obj
 0003:00000ca0       ?encoded_sleep_condition_variable_cs@@3P6AHPEAU_RTL_CONDITION_VARIABLE@@PEAU_RTL_CRITICAL_SECTION@@K@ZEA 0000000140029ca0     msvcrt:thread_safe_statics.obj
 0003:00000ca8       ?encoded_wake_all_condition_variable@@3P6AXPEAU_RTL_CONDITION_VARIABLE@@@ZEA 0000000140029ca8     msvcrt:thread_safe_statics.obj
 0003:00000cc0       ?is_initialized_as_dll@@3_NA 0000000140029cc0     msvcrt:utility.obj
 0003:00000cc1       ?module_local_atexit_table_initialized@@3_NA 0000000140029cc1     msvcrt:utility.obj
 0003:00000cc8       ?module_local_atexit_table@@3U_onexit_table_t@@A 0000000140029cc8     msvcrt:utility.obj
 0003:00000ce0       ?module_local_at_quick_exit_table@@3U_onexit_table_t@@A 0000000140029ce0     msvcrt:utility.obj
 0003:00000d00       GS_ExceptionRecord         0000000140029d00     msvcrt:gs_report.obj
 0003:00000da0       GS_ContextRecord           0000000140029da0     msvcrt:gs_report.obj
 0003:000068d0       ?a@VectorSinConstantsSSE@@3MB 000000014002f8d0     ltmodule.obj
 0003:000068d4       ?RADIANS_PER_DEGREE@@3MB   000000014002f8d4     ltmodule.obj
 0003:000068d8       ?b@VectorSinConstantsSSE@@3MB 000000014002f8d8     ltmodule.obj
 0003:000068dc       ?PI_3@@3MB                 000000014002f8dc     ltmodule.obj
 0003:000068e0       ?PiByTwo@GlobalVectorConstants@@3T__m128@@B 000000014002f8e0     ltmodule.obj
 0003:000068f0       ?FloatMinusOneHalf@GlobalVectorConstants@@3T__m128@@B 000000014002f8f0     ltmodule.obj
 0003:00006900       ?IntAllMask@GlobalVectorConstants@@3T__m128i@@B 000000014002f900     ltmodule.obj
 0003:00006910       ?TwoPi@GlobalVectorConstants@@3T__m128@@B 000000014002f910     ltmodule.obj
 0003:00006920       ?SmallLengthThreshold@GlobalVectorConstants@@3T__m128@@B 000000014002f920     ltmodule.obj
 0003:00006930       ?OneOverPi@GlobalVectorConstants@@3T__m128@@B 000000014002f930     ltmodule.obj
 0003:00006940       ?AllMask@GlobalVectorConstants@@3T__m128@@B 000000014002f940     ltmodule.obj
 0003:00006950       ?ThreshQuatNormalized@GlobalVectorConstants@@3T__m128@@B 000000014002f950     ltmodule.obj
 0003:00006960       ?SignBit@GlobalVectorConstants@@3T__m128@@B 000000014002f960     ltmodule.obj
 0003:00006970       ?Float360@GlobalVectorConstants@@3T__m128@@B 000000014002f970     ltmodule.obj
 0003:00006980       ?QMULTI_SIGN_MASK0@GlobalVectorConstants@@3T__m128@@B 000000014002f980     ltmodule.obj
 0003:00006990       ?OneOverTwoPi@GlobalVectorConstants@@3T__m128@@B 000000014002f990     ltmodule.obj
 0003:000069a0       ?DEG_TO_RAD@GlobalVectorConstants@@3T__m128@@B 000000014002f9a0     ltmodule.obj
 0003:000069b0       ?BigNumber@GlobalVectorConstants@@3T__m128@@B 000000014002f9b0     ltmodule.obj
 0003:000069c0       ?FloatOneHundredth@GlobalVectorConstants@@3T__m128@@B 000000014002f9c0     ltmodule.obj
 0003:000069d0       ?FloatTwo@GlobalVectorConstants@@3T__m128@@B 000000014002f9d0     ltmodule.obj
 0003:000069e0       ?Float0001@GlobalVectorConstants@@3T__m128@@B 000000014002f9e0     ltmodule.obj
 0003:000069f0       ?FloatAlmostTwo@GlobalVectorConstants@@3T__m128@@B 000000014002f9f0     ltmodule.obj
 0003:00006a00       ?QMULTI_SIGN_MASK2@GlobalVectorConstants@@3T__m128@@B 000000014002fa00     ltmodule.obj
 0003:00006a10       ?SignMask@GlobalVectorConstants@@3T__m128@@B 000000014002fa10     ltmodule.obj
 0003:00006a20       ?FloatMinus1_111@GlobalVectorConstants@@3T__m128@@B 000000014002fa20     ltmodule.obj
 0003:00006a30       ?QMULTI_SIGN_MASK1@GlobalVectorConstants@@3T__m128@@B 000000014002fa30     ltmodule.obj
 0003:00006a40       ?IntMinusOne@GlobalVectorConstants@@3T__m128i@@B 000000014002fa40     ltmodule.obj
 0003:00006a50       ?FloatOneHalf@GlobalVectorConstants@@3T__m128@@B 000000014002fa50     ltmodule.obj
 0003:00006a60       ?FloatZero@GlobalVectorConstants@@3T__m128@@B 000000014002fa60     ltmodule.obj
 0003:00006a70       ?B@VectorSinConstantsSSE@@3T__m128@@B 000000014002fa70     ltmodule.obj
 0003:00006a80       ?Float255@GlobalVectorConstants@@3T__m128@@B 000000014002fa80     ltmodule.obj
 0003:00006a90       ?Float127@GlobalVectorConstants@@3T__m128@@B 000000014002fa90     ltmodule.obj
 0003:00006aa0       ?QINV_SIGN_MASK@GlobalVectorConstants@@3T__m128@@B 000000014002faa0     ltmodule.obj
 0003:00006ab0       ?DEG_TO_RAD_HALF@GlobalVectorConstants@@3T__m128@@B 000000014002fab0     ltmodule.obj
 0003:00006ac0       ?FloatOne@GlobalVectorConstants@@3T__m128@@B 000000014002fac0     ltmodule.obj
 0003:00006ad0       ?A@VectorSinConstantsSSE@@3T__m128@@B 000000014002fad0     ltmodule.obj
 0003:00006ae0       ?IntSignBit@GlobalVectorConstants@@3T__m128i@@B 000000014002fae0     ltmodule.obj
 0003:00006af0       ?FloatMinusOne@GlobalVectorConstants@@3T__m128@@B 000000014002faf0     ltmodule.obj
 0003:00006b00       ?FloatNeg127@GlobalVectorConstants@@3T__m128@@B 000000014002fb00     ltmodule.obj
 0003:00006b10       ?Float111_Minus1@GlobalVectorConstants@@3T__m128@@B 000000014002fb10     ltmodule.obj
 0003:00006b20       ?XYZMask@GlobalVectorConstants@@3T__m128@@B 000000014002fb20     ltmodule.obj
 0003:00006b30       ?KindaSmallNumber@GlobalVectorConstants@@3T__m128@@B 000000014002fb30     ltmodule.obj
 0003:00006b40       ?IntOne@GlobalVectorConstants@@3T__m128i@@B 000000014002fb40     ltmodule.obj
 0003:00006b50       ?SmallNumber@GlobalVectorConstants@@3T__m128@@B 000000014002fb50     ltmodule.obj
 0003:00006b60       ?PiByFour@GlobalVectorConstants@@3T__m128@@B 000000014002fb60     ltmodule.obj
 0003:00006b80       ?Pi@GlobalVectorConstants@@3T__m128@@B 000000014002fb80     ltmodule.obj
 0003:00006b90       ?DEGREES_PER_RADIAN@@3MB   000000014002fb90     ltmodule.obj
 0003:00006b94       ?PI@@3MB                   000000014002fb94     ltmodule.obj
 0003:00006b98       ?PI_4@@3MB                 000000014002fb98     ltmodule.obj
 0003:00006ba0       ?FloatInfinity@GlobalVectorConstants@@3T__m128@@B 000000014002fba0     ltmodule.obj
 0003:00006bb0       ?IntZero@GlobalVectorConstants@@3T__m128i@@B 000000014002fbb0     ltmodule.obj
 0003:00006bc0       ?IntSignMask@GlobalVectorConstants@@3T__m128i@@B 000000014002fbc0     ltmodule.obj
 0003:00006bd0       ?RAD_TO_DEG@GlobalVectorConstants@@3T__m128@@B 000000014002fbd0     ltmodule.obj
 0003:00006be0       ?PI_2@@3MB                 000000014002fbe0     ltmodule.obj
 0003:00006be4       ?a@VectorSinConstantsSSE@@3MB 000000014002fbe4     StdAfx.obj
 0003:00006c00       ?Float180@GlobalVectorConstants@@3T__m128@@B 000000014002fc00     ltmodule.obj
 0003:00006d88       ?RADIANS_PER_DEGREE@@3MB   000000014002fd88     StdAfx.obj
 0003:00235504       ?b@VectorSinConstantsSSE@@3MB 000000014025e504     StdAfx.obj
 0003:00235508       ?PI_3@@3MB                 000000014025e508     StdAfx.obj
 0003:00235510       ?PiByTwo@GlobalVectorConstants@@3T__m128@@B 000000014025e510     StdAfx.obj
 0003:00235520       ?FloatMinusOneHalf@GlobalVectorConstants@@3T__m128@@B 000000014025e520     StdAfx.obj
 0003:00235530       ?IntAllMask@GlobalVectorConstants@@3T__m128i@@B 000000014025e530     StdAfx.obj
 0003:00235540       ?TwoPi@GlobalVectorConstants@@3T__m128@@B 000000014025e540     StdAfx.obj
 0003:00235550       ?SmallLengthThreshold@GlobalVectorConstants@@3T__m128@@B 000000014025e550     StdAfx.obj
 0003:00235560       ?OneOverPi@GlobalVectorConstants@@3T__m128@@B 000000014025e560     StdAfx.obj
 0003:00235570       ?AllMask@GlobalVectorConstants@@3T__m128@@B 000000014025e570     StdAfx.obj
 0003:00235580       ?ThreshQuatNormalized@GlobalVectorConstants@@3T__m128@@B 000000014025e580     StdAfx.obj
 0003:00235590       ?SignBit@GlobalVectorConstants@@3T__m128@@B 000000014025e590     StdAfx.obj
 0003:002355a0       ?Float360@GlobalVectorConstants@@3T__m128@@B 000000014025e5a0     StdAfx.obj
 0003:002355b0       ?QMULTI_SIGN_MASK0@GlobalVectorConstants@@3T__m128@@B 000000014025e5b0     StdAfx.obj
 0003:002355c0       ?OneOverTwoPi@GlobalVectorConstants@@3T__m128@@B 000000014025e5c0     StdAfx.obj
 0003:002355d0       ?DEG_TO_RAD@GlobalVectorConstants@@3T__m128@@B 000000014025e5d0     StdAfx.obj
 0003:002355e0       ?BigNumber@GlobalVectorConstants@@3T__m128@@B 000000014025e5e0     StdAfx.obj
 0003:002355f0       ?FloatOneHundredth@GlobalVectorConstants@@3T__m128@@B 000000014025e5f0     StdAfx.obj
 0003:00235600       ?FloatTwo@GlobalVectorConstants@@3T__m128@@B 000000014025e600     StdAfx.obj
 0003:00235610       ?Float0001@GlobalVectorConstants@@3T__m128@@B 000000014025e610     StdAfx.obj
 0003:00235620       ?FloatAlmostTwo@GlobalVectorConstants@@3T__m128@@B 000000014025e620     StdAfx.obj
 0003:00235630       ?QMULTI_SIGN_MASK2@GlobalVectorConstants@@3T__m128@@B 000000014025e630     StdAfx.obj
 0003:00235640       ?SignMask@GlobalVectorConstants@@3T__m128@@B 000000014025e640     StdAfx.obj
 0003:00235650       ?FloatMinus1_111@GlobalVectorConstants@@3T__m128@@B 000000014025e650     StdAfx.obj
 0003:00235660       ?QMULTI_SIGN_MASK1@GlobalVectorConstants@@3T__m128@@B 000000014025e660     StdAfx.obj
 0003:00235670       ?IntMinusOne@GlobalVectorConstants@@3T__m128i@@B 000000014025e670     StdAfx.obj
 0003:00235680       ?FloatOneHalf@GlobalVectorConstants@@3T__m128@@B 000000014025e680     StdAfx.obj
 0003:00235690       ?FloatZero@GlobalVectorConstants@@3T__m128@@B 000000014025e690     StdAfx.obj
 0003:002356a0       ?B@VectorSinConstantsSSE@@3T__m128@@B 000000014025e6a0     StdAfx.obj
 0003:002356b0       ?Float255@GlobalVectorConstants@@3T__m128@@B 000000014025e6b0     StdAfx.obj
 0003:002356c0       ?Float127@GlobalVectorConstants@@3T__m128@@B 000000014025e6c0     StdAfx.obj
 0003:002356d0       ?QINV_SIGN_MASK@GlobalVectorConstants@@3T__m128@@B 000000014025e6d0     StdAfx.obj
 0003:002356e0       ?DEG_TO_RAD_HALF@GlobalVectorConstants@@3T__m128@@B 000000014025e6e0     StdAfx.obj
 0003:002356f0       ?FloatOne@GlobalVectorConstants@@3T__m128@@B 000000014025e6f0     StdAfx.obj
 0003:00235700       ?A@VectorSinConstantsSSE@@3T__m128@@B 000000014025e700     StdAfx.obj
 0003:00235710       ?IntSignBit@GlobalVectorConstants@@3T__m128i@@B 000000014025e710     StdAfx.obj
 0003:00235720       ?FloatMinusOne@GlobalVectorConstants@@3T__m128@@B 000000014025e720     StdAfx.obj
 0003:00235730       ?FloatNeg127@GlobalVectorConstants@@3T__m128@@B 000000014025e730     StdAfx.obj
 0003:00235740       ?Float111_Minus1@GlobalVectorConstants@@3T__m128@@B 000000014025e740     StdAfx.obj
 0003:00235750       ?XYZMask@GlobalVectorConstants@@3T__m128@@B 000000014025e750     StdAfx.obj
 0003:00235760       ?KindaSmallNumber@GlobalVectorConstants@@3T__m128@@B 000000014025e760     StdAfx.obj
 0003:00235770       ?IntOne@GlobalVectorConstants@@3T__m128i@@B 000000014025e770     StdAfx.obj
 0003:00235780       ?SmallNumber@GlobalVectorConstants@@3T__m128@@B 000000014025e780     StdAfx.obj
 0003:00235790       ?PiByFour@GlobalVectorConstants@@3T__m128@@B 000000014025e790     StdAfx.obj
 0003:002357a0       ?Pi@GlobalVectorConstants@@3T__m128@@B 000000014025e7a0     StdAfx.obj
 0003:002357b0       ?DEGREES_PER_RADIAN@@3MB   000000014025e7b0     StdAfx.obj
 0003:002357b4       ?PI@@3MB                   000000014025e7b4     StdAfx.obj
 0003:002357b8       ?PI_4@@3MB                 000000014025e7b8     StdAfx.obj
 0003:002357c0       ?FloatInfinity@GlobalVectorConstants@@3T__m128@@B 000000014025e7c0     StdAfx.obj
 0003:002357d0       ?IntZero@GlobalVectorConstants@@3T__m128i@@B 000000014025e7d0     StdAfx.obj
 0003:002357e0       ?IntSignMask@GlobalVectorConstants@@3T__m128i@@B 000000014025e7e0     StdAfx.obj
 0003:002357f0       ?RAD_TO_DEG@GlobalVectorConstants@@3T__m128@@B 000000014025e7f0     StdAfx.obj
 0003:00235800       ?PI_2@@3MB                 000000014025e800     StdAfx.obj
 0003:00235804       ?database_item_count@@3HA  000000014025e804     ltmodule.obj
 0003:00235808       ?ptrs@@3PEAVCDatabasePtrs@@EA 000000014025e808     ltmodule.obj
 0003:00235810       ?Float180@GlobalVectorConstants@@3T__m128@@B 000000014025e810     StdAfx.obj
 0003:00235820       ?g_szHostName@@3PADA       000000014025e820     BugReporter.obj
 0003:00235890       ?g_szServerName@@3PADA     000000014025e890     BugReporter.obj
 0003:00235900       ?g_szDmpFolder@@3PADA      000000014025e900     BugReporter.obj
 0003:00235aa0       ?g_szDmpFileName@@3PADA    000000014025eaa0     BugReporter.obj
 0003:00235e90       ?g_szSubDir@@3PADA         000000014025ee90     BugReporter.obj
 0003:00235f08       ?$TSS0@?1??CRSUploader@@YAAEAVUploader@crs@@XZ@4HA 000000014025ef08     BugReporter.obj
 0003:00235f10       ?crs_uploader@?1??CRSUploader@@YAAEAVUploader@crs@@XZ@4V23@A 000000014025ef10     BugReporter.obj
 0004:00000000       $pdata$??__Ea@VectorSinConstantsSSE@@YAXXZ 0000000140260000     ltmodule.obj
 0004:0000000c       $pdata$??__Eb@VectorSinConstantsSSE@@YAXXZ 000000014026000c     ltmodule.obj
 0004:00000018       $pdata$??__EPI@@YAXXZ      0000000140260018     ltmodule.obj
 0004:00000024       $pdata$??__E?m_LogLock@CHLogger@@0VCMustSyncObjectLog@@A@@YAXXZ 0000000140260024     HostLogger.obj
 0004:00000030       $pdata$??__E?m_LogPacketLock@CHLogger@@0VCMustSyncObjectLog@@A@@YAXXZ 0000000140260030     HostLogger.obj
 0004:0000003c       $pdata$??__EtheApp@@YAXXZ  000000014026003c     ServerApp.obj
 0004:00000048       $pdata$??__Eg_cServerLog@@YAXXZ 0000000140260048     ServerAppDlg.obj
 0004:00000054       $pdata$??__E__api_holder_ILTCommon_Server_g_pLTSCommon__@@YAXXZ 0000000140260054     ServerAppDlg.obj
 0004:00000060       $pdata$??__Eg_sGameInfos@@YAXXZ 0000000140260060     ServerAppDlg.obj
 0004:0000006c       $pdata$??__Eg_sUserInfos@@YAXXZ 000000014026006c     ServerAppDlg.obj
 0004:00000078       $pdata$??__Ea@VectorSinConstantsSSE@@YAXXZ 0000000140260078     StdAfx.obj
 0004:00000084       $pdata$??__Eb@VectorSinConstantsSSE@@YAXXZ 0000000140260084     StdAfx.obj
 0004:00000090       $pdata$??__EPI@@YAXXZ      0000000140260090     StdAfx.obj
 0004:0000009c       $pdata$??__E_AtlBaseModule@ATL@@YAXXZ 000000014026009c     atls:atlbase.obj
 0004:000000a8       $pdata$??__E_afxInitAppState@@YAXXZ 00000001402600a8     mfcs140:appmodul.obj
 0004:000000b4       $pdata$?CRSUploader@@YAAEAVUploader@crs@@XZ 00000001402600b4     BugReporter.obj
 0004:000000c0       $pdata$?threadCreateDumpFile@@YAKPEAX@Z 00000001402600c0     BugReporter.obj
 0004:000000cc       $pdata$?CrashExceptionDump@@YAJPEAU_EXCEPTION_POINTERS@@@Z 00000001402600cc     BugReporter.obj
 0004:000000d8       $pdata$0$?CrashExceptionDump@@YAJPEAU_EXCEPTION_POINTERS@@@Z 00000001402600d8     BugReporter.obj
 0004:000000e4       $pdata$1$?CrashExceptionDump@@YAJPEAU_EXCEPTION_POINTERS@@@Z 00000001402600e4     BugReporter.obj
 0004:000000f0       $pdata$?InitBugReporter@@YAXPEAD0000@Z 00000001402600f0     BugReporter.obj
 0004:000000fc       $pdata$??$sprintf_s@$0BAA@@cf@@YAHAEAY0BAA@DPEBDZZ 00000001402600fc     BugReporter.obj
 0004:00000108       $pdata$??$sprintf_s@$0BJB@@cf@@YAHAEAY0BJB@DPEBDZZ 0000000140260108     BugReporter.obj
 0004:00000114       $pdata$??$sprintf_s@$0BE@@cf@@YAHAEAY0BE@DPEBDZZ 0000000140260114     BugReporter.obj
 0004:00000120       $pdata$??$sprintf_s@$0DOJ@@cf@@YAHAEAY0DOJ@DPEBDZZ 0000000140260120     BugReporter.obj
 0004:0000012c       $pdata$??$sprintf_s@$0BAE@@cf@@YAHAEAY0BAE@DPEBDZZ 000000014026012c     BugReporter.obj
 0004:00000138       $pdata$??1?$basic_string@DU?$char_traits@D@std@@V?$allocator@D@2@@std@@QEAA@XZ 0000000140260138     BugReporter.obj
 0004:00000144       $pdata$?_Xlen@?$basic_string@DU?$char_traits@D@std@@V?$allocator@D@2@@std@@SAXXZ 0000000140260144     BugReporter.obj
 0004:00000144       $pdata$?_Xlen@?$basic_string@_WU?$char_traits@_W@std@@V?$allocator@_W@2@@std@@SAXXZ 0000000140260144     crs_uploader.obj
 0004:00000150       $pdata$?assign@?$basic_string@DU?$char_traits@D@std@@V?$allocator@D@2@@std@@QEAAAEAV12@QEBD_K@Z 0000000140260150     BugReporter.obj
 0004:0000015c       $pdata$0$?assign@?$basic_string@DU?$char_traits@D@std@@V?$allocator@D@2@@std@@QEAAAEAV12@QEBD_K@Z 000000014026015c     BugReporter.obj
 0004:00000168       $pdata$1$?assign@?$basic_string@DU?$char_traits@D@std@@V?$allocator@D@2@@std@@QEAAAEAV12@QEBD_K@Z 0000000140260168     BugReporter.obj
 0004:00000174       $pdata$2$?assign@?$basic_string@DU?$char_traits@D@std@@V?$allocator@D@2@@std@@QEAAAEAV12@QEBD_K@Z 0000000140260174     BugReporter.obj
 0004:00000180       $pdata$3$?assign@?$basic_string@DU?$char_traits@D@std@@V?$allocator@D@2@@std@@QEAAAEAV12@QEBD_K@Z 0000000140260180     BugReporter.obj
 0004:0000018c       $pdata$_snprintf_s         000000014026018c     BugReporter.obj
 0004:00000198       $pdata$?recordExceptionLog@Uploader@crs@@QEAAXAEAVLogBuffer@2@PEBDZZ 0000000140260198     crs_uploader.obj
 0004:000001a4       $pdata$0$?recordExceptionLog@Uploader@crs@@QEAAXAEAVLogBuffer@2@PEBDZZ 00000001402601a4     crs_uploader.obj
 0004:000001b0       $pdata$1$?recordExceptionLog@Uploader@crs@@QEAAXAEAVLogBuffer@2@PEBDZZ 00000001402601b0     crs_uploader.obj
 0004:000001bc       $pdata$?readURL@Uploader@crs@@AEAAXAEAV?$basic_string@_WU?$char_traits@_W@std@@V?$allocator@_W@2@@std@@@Z 00000001402601bc     crs_uploader.obj
 0004:000001c8       $pdata$?iniPath@Uploader@crs@@AEAA?AV?$basic_string@_WU?$char_traits@_W@std@@V?$allocator@_W@2@@std@@AEBV34@@Z 00000001402601c8     crs_uploader.obj
 0004:000001d4       $pdata$1$?iniPath@Uploader@crs@@AEAA?AV?$basic_string@_WU?$char_traits@_W@std@@V?$allocator@_W@2@@std@@AEBV34@@Z 00000001402601d4     crs_uploader.obj
 0004:000001e0       $pdata$2$?iniPath@Uploader@crs@@AEAA?AV?$basic_string@_WU?$char_traits@_W@std@@V?$allocator@_W@2@@std@@AEBV34@@Z 00000001402601e0     crs_uploader.obj
 0004:000001ec       $pdata$?makeBaseInfo@Uploader@crs@@AEAAXPEAD0@Z 00000001402601ec     crs_uploader.obj
 0004:000001f8       $pdata$?error@Uploader@crs@@AEAA_NPEBDZZ 00000001402601f8     crs_uploader.obj
 0004:00000204       $pdata$??1Uploader@crs@@QEAA@XZ 0000000140260204     crs_uploader.obj
 0004:00000210       $pdata$?init@Uploader@crs@@QEAA_N_NPEAD1@Z 0000000140260210     crs_uploader.obj
 0004:0000021c       $pdata$?upload@Uploader@crs@@QEAA_N_NAEBV?$basic_string@DU?$char_traits@D@std@@V?$allocator@D@2@@std@@AEAVLogBuffer@2@@Z 000000014026021c     crs_uploader.obj
 0004:00000228       $pdata$?makeExceptionLog@Uploader@crs@@QEAAXPEAU_EXCEPTION_POINTERS@@AEAVLogBuffer@2@@Z 0000000140260228     crs_uploader.obj
 0004:00000234       $pdata$3$?makeExceptionLog@Uploader@crs@@QEAAXPEAU_EXCEPTION_POINTERS@@AEAVLogBuffer@2@@Z 0000000140260234     crs_uploader.obj
 0004:00000240       $pdata$4$?makeExceptionLog@Uploader@crs@@QEAAXPEAU_EXCEPTION_POINTERS@@AEAVLogBuffer@2@@Z 0000000140260240     crs_uploader.obj
 0004:0000024c       $pdata$?EnumModuleDetail@ModuleInfo@?1??makeExceptionLog@Uploader@crs@@QEAAXPEAU_EXCEPTION_POINTERS@@AEAVLogBuffer@4@@Z@SAHPEBD_KKPEAX@Z 000000014026024c     crs_uploader.obj
 0004:00000258       $pdata$0$?EnumModuleDetail@ModuleInfo@?1??makeExceptionLog@Uploader@crs@@QEAAXPEAU_EXCEPTION_POINTERS@@AEAVLogBuffer@4@@Z@SAHPEBD_KKPEAX@Z 0000000140260258     crs_uploader.obj
 0004:00000264       $pdata$1$?EnumModuleDetail@ModuleInfo@?1??makeExceptionLog@Uploader@crs@@QEAAXPEAU_EXCEPTION_POINTERS@@AEAVLogBuffer@4@@Z@SAHPEBD_KKPEAX@Z 0000000140260264     crs_uploader.obj
 0004:00000270       $pdata$?prepare@Uploader@crs@@AEAA_NAEAVHttpHandles@2@@Z 0000000140260270     crs_uploader.obj
 0004:0000027c       $pdata$?uploadHTTP@Uploader@crs@@AEAA_NAEAVHttpHandle@2@PEBDPEB_W2@Z 000000014026027c     crs_uploader.obj
 0004:00000288       $pdata$?uploadLOG@Uploader@crs@@AEAA_NAEAVHttpHandle@2@AEAU_SYSTEMTIME@@AEAVLogBuffer@2@@Z 0000000140260288     crs_uploader.obj
 0004:00000294       $pdata$0$?uploadLOG@Uploader@crs@@AEAA_NAEAVHttpHandle@2@AEAU_SYSTEMTIME@@AEAVLogBuffer@2@@Z 0000000140260294     crs_uploader.obj
 0004:000002a0       $pdata$1$?uploadLOG@Uploader@crs@@AEAA_NAEAVHttpHandle@2@AEAU_SYSTEMTIME@@AEAVLogBuffer@2@@Z 00000001402602a0     crs_uploader.obj
 0004:000002ac       $pdata$2$?uploadLOG@Uploader@crs@@AEAA_NAEAVHttpHandle@2@AEAU_SYSTEMTIME@@AEAVLogBuffer@2@@Z 00000001402602ac     crs_uploader.obj
 0004:000002b8       $pdata$3$?uploadLOG@Uploader@crs@@AEAA_NAEAVHttpHandle@2@AEAU_SYSTEMTIME@@AEAVLogBuffer@2@@Z 00000001402602b8     crs_uploader.obj
 0004:000002c4       $pdata$?success@Uploader@crs@@AEAA_NPEBDAEAVHttpHandle@2@@Z 00000001402602c4     crs_uploader.obj
 0004:000002d0       $pdata$??1?$auto_ptr@VUrl@crs@@@std@@QEAA@XZ 00000001402602d0     crs_uploader.obj
 0004:000002dc       $pdata$0$??1?$auto_ptr@VUrl@crs@@@std@@QEAA@XZ 00000001402602dc     crs_uploader.obj
 0004:000002e8       $pdata$1$??1?$auto_ptr@VUrl@crs@@@std@@QEAA@XZ 00000001402602e8     crs_uploader.obj
 0004:000002f4       $pdata$2$??1?$auto_ptr@VUrl@crs@@@std@@QEAA@XZ 00000001402602f4     crs_uploader.obj
 0004:00000300       $pdata$??$_snprintf_s@$0IA@@@YAHAEAY0IA@D_KPEBDZZ 0000000140260300     crs_uploader.obj
 0004:0000030c       $pdata$??$_Reallocate_grow_by@V<lambda_1dfe18491bcca09701d8ccb01d0b0af4>@@PEB_W_K@?$basic_string@_WU?$char_traits@_W@std@@V?$allocator@_W@2@@std@@QEAAAEAV01@_KV<lambda_1dfe18491bcca09701d8ccb01d0b0af4>@@PEB_W_K@Z 000000014026030c     crs_uploader.obj
 0004:00000318       $pdata$3$??$_Reallocate_grow_by@V<lambda_1dfe18491bcca09701d8ccb01d0b0af4>@@PEB_W_K@?$basic_string@_WU?$char_traits@_W@std@@V?$allocator@_W@2@@std@@QEAAAEAV01@_KV<lambda_1dfe18491bcca09701d8ccb01d0b0af4>@@PEB_W_K@Z 0000000140260318     crs_uploader.obj
 0004:00000324       $pdata$4$??$_Reallocate_grow_by@V<lambda_1dfe18491bcca09701d8ccb01d0b0af4>@@PEB_W_K@?$basic_string@_WU?$char_traits@_W@std@@V?$allocator@_W@2@@std@@QEAAAEAV01@_KV<lambda_1dfe18491bcca09701d8ccb01d0b0af4>@@PEB_W_K@Z 0000000140260324     crs_uploader.obj
 0004:00000330       $pdata$?append@?$basic_string@_WU?$char_traits@_W@std@@V?$allocator@_W@2@@std@@QEAAAEAV12@QEB_W_K@Z 0000000140260330     crs_uploader.obj
 0004:0000033c       $pdata$1$?append@?$basic_string@_WU?$char_traits@_W@std@@V?$allocator@_W@2@@std@@QEAAAEAV12@QEB_W_K@Z 000000014026033c     crs_uploader.obj
 0004:00000348       $pdata$2$?append@?$basic_string@_WU?$char_traits@_W@std@@V?$allocator@_W@2@@std@@QEAAAEAV12@QEB_W_K@Z 0000000140260348     crs_uploader.obj
 0004:00000354       $pdata$_snwprintf_s        0000000140260354     crs_uploader.obj
 0004:00000360       $pdata$?_Tidy_deallocate@?$basic_string@_WU?$char_traits@_W@std@@V?$allocator@_W@2@@std@@QEAAXXZ 0000000140260360     crs_uploader.obj
 0004:00000360       $pdata$??1?$basic_string@_WU?$char_traits@_W@std@@V?$allocator@_W@2@@std@@QEAA@XZ 0000000140260360     crs_uploader.obj
 0004:0000036c       $pdata$?assign@?$basic_string@_WU?$char_traits@_W@std@@V?$allocator@_W@2@@std@@QEAAAEAV12@QEB_W_K@Z 000000014026036c     crs_uploader.obj
 0004:00000378       $pdata$??_GCServerLog@@UEAAPEAXI@Z 0000000140260378     LogMgmt.obj
 0004:00000384       $pdata$??1CServerLog@@UEAA@XZ 0000000140260384     LogMgmt.obj
 0004:00000390       $pdata$?Log@rwpmlog@@YAXPEBDFPEBUPROTO_START_HOST_tag@@@Z 0000000140260390     RWPMLog.obj
 0004:0000039c       $pdata$?Log@rwpmlog@@YAXPEBDFPEBUPROTO_GAME_USER_INFO_tag@@@Z 000000014026039c     RWPMLog.obj
 0004:000003a8       $pdata$?Log@rwpmlog@@YAXPEBDFPEBUPROTO_GAMEGT_INGAME_AIGACHA_ITEM_INSERT_RESULT@@@Z 00000001402603a8     RWPMLog.obj
 0004:000003b4       $pdata$?Log@rwpmlog@@YAXPEBDFPEBUPROTO_GAMEGT_INGAME_AIGACHA_GROUP_RATE_RESULT@@@Z 00000001402603b4     RWPMLog.obj
 0004:000003c0       $pdata$??$sprintf_s@$0EA@@cf@@YAHAEAY0EA@DPEBDZZ 00000001402603c0     RWPMLog.obj
 0004:000003cc       $pdata$?LTStrCpyCreate@?A0xaa4cf837@@YAPEADPEBD@Z 00000001402603cc     ltmodule.obj
 0004:000003d8       $pdata$?check_delete_pointers@@YAXXZ 00000001402603d8     ltmodule.obj
 0004:000003e4       $pdata$0$?check_delete_pointers@@YAXXZ 00000001402603e4     ltmodule.obj
 0004:000003f0       $pdata$1$?check_delete_pointers@@YAXXZ 00000001402603f0     ltmodule.obj
 0004:000003fc       $pdata$??0CInterfaceDatabase@@QEAA@XZ 00000001402603fc     ltmodule.obj
 0004:00000408       $pdata$?AddHolder@CInterfaceDatabase@@SAXPEAVCAPIHolderBase@@@Z 0000000140260408     ltmodule.obj
 0004:00000414       $pdata$?Add@CInterfaceDatabase@@EEAAXPEAVIBase@@PEBDH@Z 0000000140260414     ltmodule.obj
 0004:00000420       $pdata$?Remove@CInterfaceDatabase@@EEAAXPEAVIBase@@PEBD@Z 0000000140260420     ltmodule.obj
 0004:0000042c       $pdata$0$?Remove@CInterfaceDatabase@@EEAAXPEAVIBase@@PEBD@Z 000000014026042c     ltmodule.obj
 0004:00000438       $pdata$1$?Remove@CInterfaceDatabase@@EEAAXPEAVIBase@@PEBD@Z 0000000140260438     ltmodule.obj
 0004:00000444       $pdata$2$?Remove@CInterfaceDatabase@@EEAAXPEAVIBase@@PEBD@Z 0000000140260444     ltmodule.obj
 0004:00000450       $pdata$3$?Remove@CInterfaceDatabase@@EEAAXPEAVIBase@@PEBD@Z 0000000140260450     ltmodule.obj
 0004:0000045c       $pdata$?Add@CInterfaceDatabase@@EEAAXPEAVCAPIHolderBase@@@Z 000000014026045c     ltmodule.obj
 0004:00000468       $pdata$?Remove@CInterfaceDatabase@@EEAAXPEAVCAPIHolderBase@@@Z 0000000140260468     ltmodule.obj
 0004:00000474       $pdata$0$?Remove@CInterfaceDatabase@@EEAAXPEAVCAPIHolderBase@@@Z 0000000140260474     ltmodule.obj
 0004:00000480       $pdata$1$?Remove@CInterfaceDatabase@@EEAAXPEAVCAPIHolderBase@@@Z 0000000140260480     ltmodule.obj
 0004:0000048c       $pdata$?Add@CInterfaceDatabase@@EEAAXPEAVCInterfaceChooser@@@Z 000000014026048c     ltmodule.obj
 0004:00000498       $pdata$?Remove@CInterfaceDatabase@@EEAAXPEAVCInterfaceChooser@@@Z 0000000140260498     ltmodule.obj
 0004:000004a4       $pdata$0$?Remove@CInterfaceDatabase@@EEAAXPEAVCInterfaceChooser@@@Z 00000001402604a4     ltmodule.obj
 0004:000004b0       $pdata$1$?Remove@CInterfaceDatabase@@EEAAXPEAVCInterfaceChooser@@@Z 00000001402604b0     ltmodule.obj
 0004:000004bc       $pdata$?Run@CInterfaceDatabase@@EEAA?AW4EChooserRun@@PEAVCInterfaceChooser@@@Z 00000001402604bc     ltmodule.obj
 0004:000004c8       $pdata$?TransferFrom@CInterfaceDatabase@@UEAAXPEAV1@@Z 00000001402604c8     ltmodule.obj
 0004:000004d4       $pdata$?Destroy@CInterfaceDatabase@@UEAAXXZ 00000001402604d4     ltmodule.obj
 0004:000004e0       $pdata$1$?Destroy@CInterfaceDatabase@@UEAAXXZ 00000001402604e0     ltmodule.obj
 0004:000004ec       $pdata$2$?Destroy@CInterfaceDatabase@@UEAAXXZ 00000001402604ec     ltmodule.obj
 0004:000004f8       $pdata$3$?Destroy@CInterfaceDatabase@@UEAAXXZ 00000001402604f8     ltmodule.obj
 0004:00000504       $pdata$4$?Destroy@CInterfaceDatabase@@UEAAXXZ 0000000140260504     ltmodule.obj
 0004:00000510       $pdata$5$?Destroy@CInterfaceDatabase@@UEAAXXZ 0000000140260510     ltmodule.obj
 0004:0000051c       $pdata$6$?Destroy@CInterfaceDatabase@@UEAAXXZ 000000014026051c     ltmodule.obj
 0004:00000528       $pdata$7$?Destroy@CInterfaceDatabase@@UEAAXXZ 0000000140260528     ltmodule.obj
 0004:00000534       $pdata$??0CInterfaceNameMgr@@QEAA@PEBDH@Z 0000000140260534     ltmodule.obj
 0004:00000540       $pdata$??_GCInterfaceNameMgr@@UEAAPEAXI@Z 0000000140260540     ltmodule.obj
 0004:0000054c       $pdata$2$??_GCInterfaceNameMgr@@UEAAPEAXI@Z 000000014026054c     ltmodule.obj
 0004:00000558       $pdata$3$??_GCInterfaceNameMgr@@UEAAPEAXI@Z 0000000140260558     ltmodule.obj
 0004:00000564       $pdata$4$??_GCInterfaceNameMgr@@UEAAPEAXI@Z 0000000140260564     ltmodule.obj
 0004:00000570       $pdata$5$??_GCInterfaceNameMgr@@UEAAPEAXI@Z 0000000140260570     ltmodule.obj
 0004:0000057c       $pdata$6$??_GCInterfaceNameMgr@@UEAAPEAXI@Z 000000014026057c     ltmodule.obj
 0004:00000588       $pdata$7$??_GCInterfaceNameMgr@@UEAAPEAXI@Z 0000000140260588     ltmodule.obj
 0004:00000594       $pdata$?Add@CInterfaceNameMgr@@QEAAXPEAVIBase@@@Z 0000000140260594     ltmodule.obj
 0004:000005a0       $pdata$5$?Add@CInterfaceNameMgr@@QEAAXPEAVIBase@@@Z 00000001402605a0     ltmodule.obj
 0004:000005ac       $pdata$6$?Add@CInterfaceNameMgr@@QEAAXPEAVIBase@@@Z 00000001402605ac     ltmodule.obj
 0004:000005b8       $pdata$8$?Add@CInterfaceNameMgr@@QEAAXPEAVIBase@@@Z 00000001402605b8     ltmodule.obj
 0004:000005c4       $pdata$9$?Add@CInterfaceNameMgr@@QEAAXPEAVIBase@@@Z 00000001402605c4     ltmodule.obj
 0004:000005d0       $pdata$?ConnectHolders@CInterfaceNameMgr@@IEAAXPEAVIBase@@@Z 00000001402605d0     ltmodule.obj
 0004:000005dc       $pdata$1$?ConnectHolders@CInterfaceNameMgr@@IEAAXPEAVIBase@@@Z 00000001402605dc     ltmodule.obj
 0004:000005e8       $pdata$2$?ConnectHolders@CInterfaceNameMgr@@IEAAXPEAVIBase@@@Z 00000001402605e8     ltmodule.obj
 0004:000005f4       $pdata$?TransferFrom@CInterfaceNameMgr@@QEAAXPEAV1@@Z 00000001402605f4     ltmodule.obj
 0004:00000600       $pdata$??_GCAPIHolderBase@@UEAAPEAXI@Z 0000000140260600     ltmodule.obj
 0004:0000060c       $pdata$SetMasterDatabase   000000014026060c     ltmodule.obj
 0004:00000618       $pdata$0$SetMasterDatabase 0000000140260618     ltmodule.obj
 0004:00000624       $pdata$1$SetMasterDatabase 0000000140260624     ltmodule.obj
 0004:00000630       $pdata$?add@?$database_array@VCInterfaceNameMgr@@PEBD@@QEAAXPEAVCInterfaceNameMgr@@P6A?AW4RELATION@@00@Z@Z 0000000140260630     ltmodule.obj
 0004:0000063c       $pdata$1$?add@?$database_array@VCInterfaceNameMgr@@PEBD@@QEAAXPEAVCInterfaceNameMgr@@P6A?AW4RELATION@@00@Z@Z 000000014026063c     ltmodule.obj
 0004:00000648       $pdata$2$?add@?$database_array@VCInterfaceNameMgr@@PEBD@@QEAAXPEAVCInterfaceNameMgr@@P6A?AW4RELATION@@00@Z@Z 0000000140260648     ltmodule.obj
 0004:00000654       $pdata$3$?add@?$database_array@VCInterfaceNameMgr@@PEBD@@QEAAXPEAVCInterfaceNameMgr@@P6A?AW4RELATION@@00@Z@Z 0000000140260654     ltmodule.obj
 0004:00000660       $pdata$?get@?$database_array@VCInterfaceNameMgr@@PEBD@@QEAAPEAVCInterfaceNameMgr@@PEBDP6A?AW4RELATION@@0PEAV2@@Z@Z 0000000140260660     ltmodule.obj
 0004:0000066c       $pdata$?insert@?$database_array@VCInterfaceNameMgr@@PEBD@@IEAAXPEAVCInterfaceNameMgr@@I@Z 000000014026066c     ltmodule.obj
 0004:0000066c       $pdata$?insert@?$database_array@VIBase@@PEBD@@IEAAXPEAVIBase@@I@Z 000000014026066c     ltmodule.obj
 0004:00000678       $pdata$0$?insert@?$database_array@VIBase@@PEBD@@IEAAXPEAVIBase@@I@Z 0000000140260678     ltmodule.obj
 0004:00000678       $pdata$0$?insert@?$database_array@VCInterfaceNameMgr@@PEBD@@IEAAXPEAVCInterfaceNameMgr@@I@Z 0000000140260678     ltmodule.obj
 0004:00000684       $pdata$1$?insert@?$database_array@VCInterfaceNameMgr@@PEBD@@IEAAXPEAVCInterfaceNameMgr@@I@Z 0000000140260684     ltmodule.obj
 0004:00000684       $pdata$1$?insert@?$database_array@VIBase@@PEBD@@IEAAXPEAVIBase@@I@Z 0000000140260684     ltmodule.obj
 0004:00000690       $pdata$?_InitPathNameInfo@CHLogger@@CAXPEBD000@Z 0000000140260690     HostLogger.obj
 0004:0000069c       $pdata$?Log@CHLogger@@SAXW4ELOG_LEVEL@1@PEBDZZ 000000014026069c     HostLogger.obj
 0004:000006a8       $pdata$?LogKernel@CHLogger@@SAXW4ELOG_LEVEL@1@PEBDZZ 00000001402606a8     HostLogger.obj
 0004:000006b4       $pdata$?LogTimeOut@CHLogger@@SAXPEBDZZ 00000001402606b4     HostLogger.obj
 0004:000006c0       $pdata$0$?LogTimeOut@CHLogger@@SAXPEBDZZ 00000001402606c0     HostLogger.obj
 0004:000006cc       $pdata$3$?LogTimeOut@CHLogger@@SAXPEBDZZ 00000001402606cc     HostLogger.obj
 0004:000006d8       $pdata$4$?LogTimeOut@CHLogger@@SAXPEBDZZ 00000001402606d8     HostLogger.obj
 0004:000006e4       $pdata$5$?LogTimeOut@CHLogger@@SAXPEBDZZ 00000001402606e4     HostLogger.obj
 0004:000006f0       $pdata$?LogEtc@CHLogger@@SAXPEBDZZ 00000001402606f0     HostLogger.obj
 0004:000006fc       $pdata$0$?LogEtc@CHLogger@@SAXPEBDZZ 00000001402606fc     HostLogger.obj
 0004:00000708       $pdata$3$?LogEtc@CHLogger@@SAXPEBDZZ 0000000140260708     HostLogger.obj
 0004:00000714       $pdata$4$?LogEtc@CHLogger@@SAXPEBDZZ 0000000140260714     HostLogger.obj
 0004:00000720       $pdata$5$?LogEtc@CHLogger@@SAXPEBDZZ 0000000140260720     HostLogger.obj
 0004:0000072c       $pdata$?LogPacket@CHLogger@@SAXPEBDZZ 000000014026072c     HostLogger.obj
 0004:00000738       $pdata$?LogRWProcessMemory@CHLogger@@SAXPEBDZZ 0000000140260738     HostLogger.obj
 0004:00000744       $pdata$0$?LogRWProcessMemory@CHLogger@@SAXPEBDZZ 0000000140260744     HostLogger.obj
 0004:00000750       $pdata$1$?LogRWProcessMemory@CHLogger@@SAXPEBDZZ 0000000140260750     HostLogger.obj
 0004:0000075c       $pdata$2$?LogRWProcessMemory@CHLogger@@SAXPEBDZZ 000000014026075c     HostLogger.obj
 0004:00000768       $pdata$3$?LogRWProcessMemory@CHLogger@@SAXPEBDZZ 0000000140260768     HostLogger.obj
 0004:00000774       $pdata$?LogIPCMessage@CHLogger@@SAXPEBDZZ 0000000140260774     HostLogger.obj
 0004:00000780       $pdata$0$?LogIPCMessage@CHLogger@@SAXPEBDZZ 0000000140260780     HostLogger.obj
 0004:0000078c       $pdata$1$?LogIPCMessage@CHLogger@@SAXPEBDZZ 000000014026078c     HostLogger.obj
 0004:00000798       $pdata$2$?LogIPCMessage@CHLogger@@SAXPEBDZZ 0000000140260798     HostLogger.obj
 0004:000007a4       $pdata$3$?LogIPCMessage@CHLogger@@SAXPEBDZZ 00000001402607a4     HostLogger.obj
 0004:000007b0       $pdata$?_BuildDirectory@CHLogger@@CAXAEBU_SYSTEMTIME@@@Z 00000001402607b0     HostLogger.obj
 0004:000007bc       $pdata$?_DoLogWithLevel@CHLogger@@CAXPEBDW4ELOG_LEVEL@1@0PEAD@Z 00000001402607bc     HostLogger.obj
 0004:000007c8       $pdata$??$_Traits_find@U?$char_traits@D@std@@@std@@YA_KQEBD_K101@Z 00000001402607c8     HostLogger.obj
 0004:000007d4       $pdata$?_Xran@?$_String_val@U?$_Simple_types@D@std@@@std@@SAXXZ 00000001402607d4     HostLogger.obj
 0004:000007e0       $pdata$??$_Reallocate_grow_by@V<lambda_65e615be2a453ca0576c979606f46740>@@PEBD_K@?$basic_string@DU?$char_traits@D@std@@V?$allocator@D@2@@std@@QEAAAEAV01@_KV<lambda_65e615be2a453ca0576c979606f46740>@@PEBD_K@Z 00000001402607e0     HostLogger.obj
 0004:000007ec       $pdata$3$??$_Reallocate_grow_by@V<lambda_65e615be2a453ca0576c979606f46740>@@PEBD_K@?$basic_string@DU?$char_traits@D@std@@V?$allocator@D@2@@std@@QEAAAEAV01@_KV<lambda_65e615be2a453ca0576c979606f46740>@@PEBD_K@Z 00000001402607ec     HostLogger.obj
 0004:000007f8       $pdata$4$??$_Reallocate_grow_by@V<lambda_65e615be2a453ca0576c979606f46740>@@PEBD_K@?$basic_string@DU?$char_traits@D@std@@V?$allocator@D@2@@std@@QEAAAEAV01@_KV<lambda_65e615be2a453ca0576c979606f46740>@@PEBD_K@Z 00000001402607f8     HostLogger.obj
 0004:00000804       $pdata$?append@?$basic_string@DU?$char_traits@D@std@@V?$allocator@D@2@@std@@QEAAAEAV12@QEBD_K@Z 0000000140260804     HostLogger.obj
 0004:00000810       $pdata$0$?append@?$basic_string@DU?$char_traits@D@std@@V?$allocator@D@2@@std@@QEAAAEAV12@QEBD_K@Z 0000000140260810     HostLogger.obj
 0004:0000081c       $pdata$1$?append@?$basic_string@DU?$char_traits@D@std@@V?$allocator@D@2@@std@@QEAAAEAV12@QEBD_K@Z 000000014026081c     HostLogger.obj
 0004:00000828       $pdata$??_GCMustSyncObjectLog@@UEAAPEAXI@Z 0000000140260828     HostLogger.obj
 0004:00000834       $pdata$?Init@CLogMsgManager@@SA_NW4ESHARED_MEM_USAGE_TYPE@1@@Z 0000000140260834     LogMsgManager.obj
 0004:00000840       $pdata$?GetString@CLogMsgManager@@SA?BV?$basic_string@DU?$char_traits@D@std@@V?$allocator@D@2@@std@@I@Z 0000000140260840     LogMsgManager.obj
 0004:0000084c       $pdata$0$?GetString@CLogMsgManager@@SA?BV?$basic_string@DU?$char_traits@D@std@@V?$allocator@D@2@@std@@I@Z 000000014026084c     LogMsgManager.obj
 0004:00000858       $pdata$1$?GetString@CLogMsgManager@@SA?BV?$basic_string@DU?$char_traits@D@std@@V?$allocator@D@2@@std@@I@Z 0000000140260858     LogMsgManager.obj
 0004:00000864       $pdata$2$?GetString@CLogMsgManager@@SA?BV?$basic_string@DU?$char_traits@D@std@@V?$allocator@D@2@@std@@I@Z 0000000140260864     LogMsgManager.obj
 0004:00000870       $pdata$3$?GetString@CLogMsgManager@@SA?BV?$basic_string@DU?$char_traits@D@std@@V?$allocator@D@2@@std@@I@Z 0000000140260870     LogMsgManager.obj
 0004:0000087c       $pdata$?_WriteXlsDataToSharedMemory@CLogMsgManager@@CA_NXZ 000000014026087c     LogMsgManager.obj
 0004:00000888       $pdata$??$sprintf_s@$0CA@@cf@@YAHAEAY0CA@DPEBDZZ 0000000140260888     LogMsgManager.obj
 0004:00000894       $pdata$??$_Emplace_reallocate@AEBQEAX@?$vector@PEAXV?$allocator@PEAX@std@@@std@@QEAAPEAPEAXQEAPEAXAEBQEAX@Z 0000000140260894     LogMsgManager.obj
 0004:000008a0       $pdata$2$??$_Emplace_reallocate@AEBQEAX@?$vector@PEAXV?$allocator@PEAX@std@@@std@@QEAAPEAPEAXQEAPEAXAEBQEAX@Z 00000001402608a0     LogMsgManager.obj
 0004:000008ac       $pdata$4$??$_Emplace_reallocate@AEBQEAX@?$vector@PEAXV?$allocator@PEAX@std@@@std@@QEAAPEAPEAXQEAPEAXAEBQEAX@Z 00000001402608ac     LogMsgManager.obj
 0004:000008b8       $pdata$5$??$_Emplace_reallocate@AEBQEAX@?$vector@PEAXV?$allocator@PEAX@std@@@std@@QEAAPEAPEAXQEAPEAXAEBQEAX@Z 00000001402608b8     LogMsgManager.obj
 0004:000008c4       $pdata$?_Xlength@?$vector@PEAXV?$allocator@PEAX@std@@@std@@CAXXZ 00000001402608c4     LogMsgManager.obj
 0004:000008d0       $pdata$??0FindXlsMsg@@QEAA@XZ 00000001402608d0     LoadXlsMsg.obj
 0004:000008dc       $pdata$??_GFindXlsMsg@@UEAAPEAXI@Z 00000001402608dc     LoadXlsMsg.obj
 0004:000008e8       $pdata$?GetMessageByIndex@FindXlsMsg@@QEAAPEBD_JPEAD@Z 00000001402608e8     LoadXlsMsg.obj
 0004:000008f4       $pdata$?LoadWMszFile@FindXlsMsg@@QEAA_NPEAD@Z 00000001402608f4     LoadXlsMsg.obj
 0004:00000900       $pdata$??A?$map@_JV?$basic_string@DU?$char_traits@D@std@@V?$allocator@D@2@@std@@U?$less@_J@2@V?$allocator@U?$pair@$$CB_JV?$basic_string@DU?$char_traits@D@std@@V?$allocator@D@2@@std@@@std@@@2@@std@@QEAAAEAV?$basic_string@DU?$char_traits@D@std@@V?$allocator@D@2@@1@AEB_J@Z 0000000140260900     LoadXlsMsg.obj
 0004:0000090c       $pdata$?_Erase@?$_Tree@V?$_Tmap_traits@_JV?$basic_string@DU?$char_traits@D@std@@V?$allocator@D@2@@std@@U?$less@_J@2@V?$allocator@U?$pair@$$CB_JV?$basic_string@DU?$char_traits@D@std@@V?$allocator@D@2@@std@@@std@@@2@$0A@@std@@@std@@IEAAXPEAU?$_Tree_node@U?$pair@$$CB_JV?$basic_string@DU?$char_traits@D@std@@V?$allocator@D@2@@std@@@std@@PEAX@2@@Z 000000014026090c     LoadXlsMsg.obj
 0004:00000918       $pdata$0$?_Erase@?$_Tree@V?$_Tmap_traits@_JV?$basic_string@DU?$char_traits@D@std@@V?$allocator@D@2@@std@@U?$less@_J@2@V?$allocator@U?$pair@$$CB_JV?$basic_string@DU?$char_traits@D@std@@V?$allocator@D@2@@std@@@std@@@2@$0A@@std@@@std@@IEAAXPEAU?$_Tree_node@U?$pair@$$CB_JV?$basic_string@DU?$char_traits@D@std@@V?$allocator@D@2@@std@@@std@@PEAX@2@@Z 0000000140260918     LoadXlsMsg.obj
 0004:00000924       $pdata$1$?_Erase@?$_Tree@V?$_Tmap_traits@_JV?$basic_string@DU?$char_traits@D@std@@V?$allocator@D@2@@std@@U?$less@_J@2@V?$allocator@U?$pair@$$CB_JV?$basic_string@DU?$char_traits@D@std@@V?$allocator@D@2@@std@@@std@@@2@$0A@@std@@@std@@IEAAXPEAU?$_Tree_node@U?$pair@$$CB_JV?$basic_string@DU?$char_traits@D@std@@V?$allocator@D@2@@std@@@std@@PEAX@2@@Z 0000000140260924     LoadXlsMsg.obj
 0004:00000930       $pdata$2$?_Erase@?$_Tree@V?$_Tmap_traits@_JV?$basic_string@DU?$char_traits@D@std@@V?$allocator@D@2@@std@@U?$less@_J@2@V?$allocator@U?$pair@$$CB_JV?$basic_string@DU?$char_traits@D@std@@V?$allocator@D@2@@std@@@std@@@2@$0A@@std@@@std@@IEAAXPEAU?$_Tree_node@U?$pair@$$CB_JV?$basic_string@DU?$char_traits@D@std@@V?$allocator@D@2@@std@@@std@@PEAX@2@@Z 0000000140260930     LoadXlsMsg.obj
 0004:0000093c       $pdata$?erase@?$_Tree@V?$_Tmap_traits@_JV?$basic_string@DU?$char_traits@D@std@@V?$allocator@D@2@@std@@U?$less@_J@2@V?$allocator@U?$pair@$$CB_JV?$basic_string@DU?$char_traits@D@std@@V?$allocator@D@2@@std@@@std@@@2@$0A@@std@@@std@@QEAA?AV?$_Tree_iterator@V?$_Tree_val@U?$_Tree_simple_types@U?$pair@$$CB_JV?$basic_string@DU?$char_traits@D@std@@V?$allocator@D@2@@std@@@std@@@std@@@std@@@2@V?$_Tree_const_iterator@V?$_Tree_val@U?$_Tree_simple_types@U?$pair@$$CB_JV?$basic_string@DU?$char_traits@D@std@@V?$allocator@D@2@@std@@@std@@@std@@@std@@@2@0@Z 000000014026093c     LoadXlsMsg.obj
 0004:00000948       $pdata$?_Extract@?$_Tree_val@U?$_Tree_simple_types@U?$pair@$$CB_JV?$basic_string@DU?$char_traits@D@std@@V?$allocator@D@2@@std@@@std@@@std@@@std@@QEAAPEAU?$_Tree_node@U?$pair@$$CB_JV?$basic_string@DU?$char_traits@D@std@@V?$allocator@D@2@@std@@@std@@PEAX@2@V?$_Tree_const_iterator@V?$_Tree_val@U?$_Tree_simple_types@U?$pair@$$CB_JV?$basic_string@DU?$char_traits@D@std@@V?$allocator@D@2@@std@@@std@@@std@@@std@@@2@@Z 0000000140260948     LoadXlsMsg.obj
 0004:00000954       $pdata$?_Buyheadnode@?$_Tree_comp_alloc@V?$_Tmap_traits@_JV?$basic_string@DU?$char_traits@D@std@@V?$allocator@D@2@@std@@U?$less@_J@2@V?$allocator@U?$pair@$$CB_JV?$basic_string@DU?$char_traits@D@std@@V?$allocator@D@2@@std@@@std@@@2@$0A@@std@@@std@@QEAAPEAU?$_Tree_node@U?$pair@$$CB_JV?$basic_string@DU?$char_traits@D@std@@V?$allocator@D@2@@std@@@std@@PEAX@2@XZ 0000000140260954     LoadXlsMsg.obj
 0004:00000960       $pdata$??$_Buynode@AEBUpiecewise_construct_t@std@@V?$tuple@AEB_J@2@V?$tuple@$$V@2@@?$_Tree_comp_alloc@V?$_Tmap_traits@_JV?$basic_string@DU?$char_traits@D@std@@V?$allocator@D@2@@std@@U?$less@_J@2@V?$allocator@U?$pair@$$CB_JV?$basic_string@DU?$char_traits@D@std@@V?$allocator@D@2@@std@@@std@@@2@$0A@@std@@@std@@QEAAPEAU?$_Tree_node@U?$pair@$$CB_JV?$basic_string@DU?$char_traits@D@std@@V?$allocator@D@2@@std@@@std@@PEAX@1@AEBUpiecewise_construct_t@1@$$QEAV?$tuple@AEB_J@1@$$QEAV?$tuple@$$V@1@@Z 0000000140260960     LoadXlsMsg.obj
 0004:0000096c       $pdata$??$_Insert_hint@AEAU?$pair@$$CB_JV?$basic_string@DU?$char_traits@D@std@@V?$allocator@D@2@@std@@@std@@PEAU?$_Tree_node@U?$pair@$$CB_JV?$basic_string@DU?$char_traits@D@std@@V?$allocator@D@2@@std@@@std@@PEAX@2@@?$_Tree@V?$_Tmap_traits@_JV?$basic_string@DU?$char_traits@D@std@@V?$allocator@D@2@@std@@U?$less@_J@2@V?$allocator@U?$pair@$$CB_JV?$basic_string@DU?$char_traits@D@std@@V?$allocator@D@2@@std@@@std@@@2@$0A@@std@@@std@@IEAA?AV?$_Tree_iterator@V?$_Tree_val@U?$_Tree_simple_types@U?$pair@$$CB_JV?$basic_string@DU?$char_traits@D@std@@V?$allocator@D@2@@std@@@std@@@std@@@std@@@1@V?$_Tree_const_iterator@V?$_Tree_val@U?$_Tree_simple_types@U?$pair@$$CB_JV?$basic_string@DU?$char_traits@D@std@@V?$allocator@D@2@@std@@@std@@@std@@@std@@@1@AEAU?$pair@$$CB_JV?$basic_string@DU?$char_traits@D@std@@V?$allocator@D@2@@std@@@1@PEAU?$_Tree_node@U?$pair@$$CB_JV?$basic_string@DU?$char_traits@D@std@@V?$allocator@D@2@@std@@@std@@PEAX@1@@Z 000000014026096c     LoadXlsMsg.obj
 0004:00000978       $pdata$?_Buynode0@?$_Tree_comp_alloc@V?$_Tmap_traits@_JV?$basic_string@DU?$char_traits@D@std@@V?$allocator@D@2@@std@@U?$less@_J@2@V?$allocator@U?$pair@$$CB_JV?$basic_string@DU?$char_traits@D@std@@V?$allocator@D@2@@std@@@std@@@2@$0A@@std@@@std@@QEAAPEAU?$_Tree_node@U?$pair@$$CB_JV?$basic_string@DU?$char_traits@D@std@@V?$allocator@D@2@@std@@@std@@PEAX@2@XZ 0000000140260978     LoadXlsMsg.obj
 0004:00000984       $pdata$?_Destroy_if_node@?$_Tree@V?$_Tmap_traits@_JV?$basic_string@DU?$char_traits@D@std@@V?$allocator@D@2@@std@@U?$less@_J@2@V?$allocator@U?$pair@$$CB_JV?$basic_string@DU?$char_traits@D@std@@V?$allocator@D@2@@std@@@std@@@2@$0A@@std@@@std@@IEAAXPEAU?$_Tree_node@U?$pair@$$CB_JV?$basic_string@DU?$char_traits@D@std@@V?$allocator@D@2@@std@@@std@@PEAX@2@@Z 0000000140260984     LoadXlsMsg.obj
 0004:00000990       $pdata$??$_Insert_at@AEAU?$pair@$$CB_JV?$basic_string@DU?$char_traits@D@std@@V?$allocator@D@2@@std@@@std@@PEAU?$_Tree_node@U?$pair@$$CB_JV?$basic_string@DU?$char_traits@D@std@@V?$allocator@D@2@@std@@@std@@PEAX@2@@?$_Tree@V?$_Tmap_traits@_JV?$basic_string@DU?$char_traits@D@std@@V?$allocator@D@2@@std@@U?$less@_J@2@V?$allocator@U?$pair@$$CB_JV?$basic_string@DU?$char_traits@D@std@@V?$allocator@D@2@@std@@@std@@@2@$0A@@std@@@std@@IEAA?AV?$_Tree_iterator@V?$_Tree_val@U?$_Tree_simple_types@U?$pair@$$CB_JV?$basic_string@DU?$char_traits@D@std@@V?$allocator@D@2@@std@@@std@@@std@@@std@@@1@_NPEAU?$_Tree_node@U?$pair@$$CB_JV?$basic_string@DU?$char_traits@D@std@@V?$allocator@D@2@@std@@@std@@PEAX@1@AEAU?$pair@$$CB_JV?$basic_string@DU?$char_traits@D@std@@V?$allocator@D@2@@std@@@1@1@Z 0000000140260990     LoadXlsMsg.obj
 0004:0000099c       $pdata$??$_Insert_nohint@AEAU?$pair@$$CB_JV?$basic_string@DU?$char_traits@D@std@@V?$allocator@D@2@@std@@@std@@PEAU?$_Tree_node@U?$pair@$$CB_JV?$basic_string@DU?$char_traits@D@std@@V?$allocator@D@2@@std@@@std@@PEAX@2@@?$_Tree@V?$_Tmap_traits@_JV?$basic_string@DU?$char_traits@D@std@@V?$allocator@D@2@@std@@U?$less@_J@2@V?$allocator@U?$pair@$$CB_JV?$basic_string@DU?$char_traits@D@std@@V?$allocator@D@2@@std@@@std@@@2@$0A@@std@@@std@@IEAA?AU?$pair@V?$_Tree_iterator@V?$_Tree_val@U?$_Tree_simple_types@U?$pair@$$CB_JV?$basic_string@DU?$char_traits@D@std@@V?$allocator@D@2@@std@@@std@@@std@@@std@@@std@@_N@1@_NAEAU?$pair@$$CB_JV?$basic_string@DU?$char_traits@D@std@@V?$allocator@D@2@@std@@@1@PEAU?$_Tree_node@U?$pair@$$CB_JV?$basic_string@DU?$char_traits@D@std@@V?$allocator@D@2@@std@@@std@@PEAX@1@@Z 000000014026099c     LoadXlsMsg.obj
 0004:000009a8       $pdata$??4?$basic_string@DU?$char_traits@D@std@@V?$allocator@D@2@@std@@QEAAAEAV01@$$QEAV01@@Z 00000001402609a8     LoadXlsMsg.obj
 0004:000009b4       $pdata$??_GCServerAppApp@@UEAAPEAXI@Z 00000001402609b4     ServerApp.obj
 0004:000009c0       $pdata$?Run@CServerAppApp@@UEAAHXZ 00000001402609c0     ServerApp.obj
 0004:000009cc       $pdata$??0PROTO_GAME_USER_INFO_tag@@QEAA@XZ 00000001402609cc     ServerAppDlg.obj
 0004:000009d8       $pdata$?ShellMessageFn@CGameServerAppHandler@@UEAAIAEAVILTMessage_Read@@@Z 00000001402609d8     ServerAppDlg.obj
 0004:000009e4       $pdata$?ConsoleOutputFn@CGameServerAppHandler@@UEAAIHHPEBD@Z 00000001402609e4     ServerAppDlg.obj
 0004:000009f0       $pdata$?OutOfMemory@CGameServerAppHandler@@UEAAIXZ 00000001402609f0     ServerAppDlg.obj
 0004:000009fc       $pdata$?NetworkDelayCount@CGameServerAppHandler@@UEAAIXZ 00000001402609fc     ServerAppDlg.obj
 0004:00000a08       $pdata$?GetProcessMemoryUsage@CGameServerAppHandler@@UEAAKXZ 0000000140260a08     ServerAppDlg.obj
 0004:00000a14       $pdata$0$?GetProcessMemoryUsage@CGameServerAppHandler@@UEAAKXZ 0000000140260a14     ServerAppDlg.obj
 0004:00000a20       $pdata$1$?GetProcessMemoryUsage@CGameServerAppHandler@@UEAAKXZ 0000000140260a20     ServerAppDlg.obj
 0004:00000a2c       $pdata$??0PROTO_START_HOST_tag@@QEAA@XZ 0000000140260a2c     ServerAppDlg.obj
 0004:00000a38       $pdata$??0CServerAppDlg@@QEAA@PEAVCWnd@@@Z 0000000140260a38     ServerAppDlg.obj
 0004:00000a44       $pdata$??_GCServerAppDlg@@UEAAPEAXI@Z 0000000140260a44     ServerAppDlg.obj
 0004:00000a50       $pdata$??1tUCCGamePlayInfo@CServerAppDlg@@QEAA@XZ 0000000140260a50     ServerAppDlg.obj
 0004:00000a5c       $pdata$??1CServerAppDlg@@UEAA@XZ 0000000140260a5c     ServerAppDlg.obj
 0004:00000a68       $pdata$?DoDataExchange@CServerAppDlg@@MEAAXPEAVCDataExchange@@@Z 0000000140260a68     ServerAppDlg.obj
 0004:00000a74       $pdata$?OnInitDialog@CServerAppDlg@@MEAAHXZ 0000000140260a74     ServerAppDlg.obj
 0004:00000a80       $pdata$?OnShellMessage@CServerAppDlg@@QEAAXAEAVILTMessage_Read@@@Z 0000000140260a80     ServerAppDlg.obj
 0004:00000a8c       $pdata$?AddServerMsg@CServerAppDlg@@QEAAXPEBDH@Z 0000000140260a8c     ServerAppDlg.obj
 0004:00000a98       $pdata$?LoadServer@CServerAppDlg@@QEAA_NXZ 0000000140260a98     ServerAppDlg.obj
 0004:00000aa4       $pdata$?RunServer@CServerAppDlg@@QEAA_NXZ 0000000140260aa4     ServerAppDlg.obj
 0004:00000ab0       $pdata$?StopServer@CServerAppDlg@@QEAA_NXZ 0000000140260ab0     ServerAppDlg.obj
 0004:00000abc       $pdata$?Thread_SendGameInfo@@YAXPEAVCServerAppDlg@@AEAUPROTO_START_HOST_tag@@@Z 0000000140260abc     ServerAppDlg.obj
 0004:00000ac8       $pdata$?Thread_SendUserInfo@@YAXPEAVCServerAppDlg@@AEAUPROTO_GAME_USER_INFO_tag@@@Z 0000000140260ac8     ServerAppDlg.obj
 0004:00000ad4       $pdata$?ThreadUpdate@CServerAppDlg@@SAXPEAX@Z 0000000140260ad4     ServerAppDlg.obj
 0004:00000ae0       $pdata$?ServerUpdate@CServerAppDlg@@QEAAXXZ 0000000140260ae0     ServerAppDlg.obj
 0004:00000aec       $pdata$?AddResources@CServerAppDlg@@QEAA_NXZ 0000000140260aec     ServerAppDlg.obj
 0004:00000af8       $pdata$?OnGameServerMsg@CServerAppDlg@@IEAA_J_K_J@Z 0000000140260af8     ServerAppDlg.obj
 0004:00000b04       $pdata$?OnCopyData@CServerAppDlg@@IEAAHPEAVCWnd@@PEAUtagCOPYDATASTRUCT@@@Z 0000000140260b04     ServerAppDlg.obj
 0004:00000b10       $pdata$?OnTimer@CServerAppDlg@@QEAAX_K@Z 0000000140260b10     ServerAppDlg.obj
 0004:00000b1c       $pdata$?OnBnClickedButtonGo@CServerAppDlg@@QEAAXXZ 0000000140260b1c     ServerAppDlg.obj
 0004:00000b28       $pdata$?SaveHostGameInfo@CServerAppDlg@@IEAAXXZ 0000000140260b28     ServerAppDlg.obj
 0004:00000b34       $pdata$?LoadHostGameInfo@CServerAppDlg@@IEAAXXZ 0000000140260b34     ServerAppDlg.obj
 0004:00000b40       $pdata$?GetOptionValueString@CServerAppDlg@@IEAA?AV?$basic_string@DU?$char_traits@D@std@@V?$allocator@D@2@@std@@V23@00@Z 0000000140260b40     ServerAppDlg.obj
 0004:00000b4c       $pdata$?ReadGSMMemory@CServerAppDlg@@QEAA_NPEAX0_K@Z 0000000140260b4c     ServerAppDlg.obj
 0004:00000b58       $pdata$?RECV_MSG_INSERTCHARACTER@CServerAppDlg@@AEAAX_J@Z 0000000140260b58     ServerAppDlg.obj
 0004:00000b64       $pdata$?RECV_MSG_AIITEM_DEC@CServerAppDlg@@AEAAX_J@Z 0000000140260b64     ServerAppDlg.obj
 0004:00000b70       $pdata$?RECV_MSG_AIITEM_GROUP_RATE_RESULT@CServerAppDlg@@AEAAX_J@Z 0000000140260b70     ServerAppDlg.obj
 0004:00000b7c       $pdata$?RECV_MSG_USER_DISCONNECTED@CServerAppDlg@@AEAAX_J@Z 0000000140260b7c     ServerAppDlg.obj
 0004:00000b88       $pdata$?SendServerAppInit@CServerAppDlg@@AEAAXXZ 0000000140260b88     ServerAppDlg.obj
 0004:00000b94       $pdata$?DownloadUCCMapFile_HTTP@CServerAppDlg@@AEAA?AW4UCCMAPDOWNLOADREAULT@@V?$basic_string@DU?$char_traits@D@std@@V?$allocator@D@2@@std@@@Z 0000000140260b94     ServerAppDlg.obj
 0004:00000ba0       $pdata$?SendServerAppInitFail@CServerAppDlg@@AEAAXHH@Z 0000000140260ba0     ServerAppDlg.obj
 0004:00000bac       $pdata$?GetDownloadPath@CServerAppDlg@@AEAA?AV?$basic_string@DU?$char_traits@D@std@@V?$allocator@D@2@@std@@XZ 0000000140260bac     ServerAppDlg.obj
 0004:00000bb8       $pdata$?SendToServerShellAutoMatchStartingUserInfo@CServerAppDlg@@AEAAXPEAUtagCOPYDATASTRUCT@@@Z 0000000140260bb8     ServerAppDlg.obj
 0004:00000bc4       $pdata$??1?$CAPIHolder@VILTCommon@@@@UEAA@XZ 0000000140260bc4     ServerAppDlg.obj
 0004:00000bd0       $pdata$??$sprintf_s@$0IA@@cf@@YAHAEAY0IA@DPEBDZZ 0000000140260bd0     ServerAppDlg.obj
 0004:00000bdc       $pdata$??$?HDU?$char_traits@D@std@@V?$allocator@D@1@@std@@YA?AV?$basic_string@DU?$char_traits@D@std@@V?$allocator@D@2@@0@AEBV10@0@Z 0000000140260bdc     ServerAppDlg.obj
 0004:00000be8       $pdata$??_G?$CAPIHolder@VILTCommon@@@@UEAAPEAXI@Z 0000000140260be8     ServerAppDlg.obj
 0004:00000bf4       $pdata$?reserve@?$basic_string@DU?$char_traits@D@std@@V?$allocator@D@2@@std@@QEAAX_K@Z 0000000140260bf4     ServerAppDlg.obj
 0004:00000c00       $pdata$0$?reserve@?$basic_string@DU?$char_traits@D@std@@V?$allocator@D@2@@std@@QEAAX_K@Z 0000000140260c00     ServerAppDlg.obj
 0004:00000c0c       $pdata$2$?reserve@?$basic_string@DU?$char_traits@D@std@@V?$allocator@D@2@@std@@QEAAX_K@Z 0000000140260c0c     ServerAppDlg.obj
 0004:00000c18       $pdata$3$?reserve@?$basic_string@DU?$char_traits@D@std@@V?$allocator@D@2@@std@@QEAAX_K@Z 0000000140260c18     ServerAppDlg.obj
 0004:00000c24       $pdata$4$?reserve@?$basic_string@DU?$char_traits@D@std@@V?$allocator@D@2@@std@@QEAAX_K@Z 0000000140260c24     ServerAppDlg.obj
 0004:00000c30       $pdata$5$?reserve@?$basic_string@DU?$char_traits@D@std@@V?$allocator@D@2@@std@@QEAAX_K@Z 0000000140260c30     ServerAppDlg.obj
 0004:00000c3c       $pdata$fscanf_s            0000000140260c3c     ServerAppDlg.obj
 0004:00000c48       $pdata$??1CWaitCursor@@QEAA@XZ 0000000140260c48     ServerAppDlg.obj
 0004:00000c54       $pdata$?Readint32@ILTMessage_Read@@QEAAHXZ 0000000140260c54     ServerAppDlg.obj
 0004:00000c54       $pdata$?Readuint32@ILTMessage_Read@@QEAAIXZ 0000000140260c54     ServerAppDlg.obj
 0004:00000c60       $pdata$??0exception@std@@QEAA@QEBD@Z 0000000140260c60     ServerAppDlg.obj
 0004:00000c6c       $pdata$??_Gexception@std@@UEAAPEAXI@Z 0000000140260c6c     ServerAppDlg.obj
 0004:00000c78       $pdata$??0exception@std@@QEAA@AEBV01@@Z 0000000140260c78     ServerAppDlg.obj
 0004:00000c84       $pdata$?USNtoStr@EXPAND_USN@@YA?AV?$basic_string@DU?$char_traits@D@std@@V?$allocator@D@2@@std@@_J@Z 0000000140260c84     ServerAppDlg.obj
 0004:00000c90       $pdata$?PostReadData@GAMEPROTO_SC_COMMON@@UEAA_NPEAVILTMessage_Read@@@Z 0000000140260c90     ServerAppDlg.obj
 0004:00000c9c       $pdata$0$?PostReadData@GAMEPROTO_SC_COMMON@@UEAA_NPEAVILTMessage_Read@@@Z 0000000140260c9c     ServerAppDlg.obj
 0004:00000ca8       $pdata$1$?PostReadData@GAMEPROTO_SC_COMMON@@UEAA_NPEAVILTMessage_Read@@@Z 0000000140260ca8     ServerAppDlg.obj
 0004:00000cb4       $pdata$?ReadData@PROTO_SERVERAPPMSG_INIT@@UEAA_NPEAVILTMessage_Read@@@Z 0000000140260cb4     ServerAppDlg.obj
 0004:00000cc0       $pdata$0$?ReadData@PROTO_SERVERAPPMSG_INIT@@UEAA_NPEAVILTMessage_Read@@@Z 0000000140260cc0     ServerAppDlg.obj
 0004:00000ccc       $pdata$1$?ReadData@PROTO_SERVERAPPMSG_INIT@@UEAA_NPEAVILTMessage_Read@@@Z 0000000140260ccc     ServerAppDlg.obj
 0004:00000cd8       $pdata$?PostWriteData@GAMEPROTO_SC_COMMON@@UEAA_NPEAVILTMessage_Write@@@Z 0000000140260cd8     ServerAppDlg.obj
 0004:00000ce4       $pdata$?WriteData@PROTO_SERVERAPPMSG_INIT@@UEAA_NPEAVILTMessage_Write@@@Z 0000000140260ce4     ServerAppDlg.obj
 0004:00000cf0       $pdata$??_GCListBox@@UEAAPEAXI@Z 0000000140260cf0     ServerAppDlg.obj
 0004:00000cfc       $pdata$??_GCEdit@@UEAAPEAXI@Z 0000000140260cfc     ServerAppDlg.obj
 0004:00000d08       $pdata$?sprintf_s@internal@cf@@YAHPEAD_KPEBDAEAPEAD@Z 0000000140260d08     safe_string_x64:safe_string.obj
 0004:00000d14       $pdata$??_D?$basic_stringstream@DU?$char_traits@D@std@@V?$allocator@D@2@@std@@QEAAXXZ 0000000140260d14     safe_string_x64:safe_string.obj
 0004:00000d20       $pdata$?strcpy_s@cf@@YAHPEAD_KPEBD@Z 0000000140260d20     safe_string_x64:safe_string.obj
 0004:00000d2c       $pdata$?strncpy_s@cf@@YAHPEAD_KPEBD1@Z 0000000140260d2c     safe_string_x64:safe_string.obj
 0004:00000d38       $pdata$?sprintf_s@cf@@YAHPEAD_KPEBDZZ 0000000140260d38     safe_string_x64:safe_string.obj
 0004:00000d44       $pdata$??0?$basic_stringstream@DU?$char_traits@D@std@@V?$allocator@D@2@@std@@QEAA@H@Z 0000000140260d44     safe_string_x64:safe_string.obj
 0004:00000d50       $pdata$?seekpos@?$basic_stringbuf@DU?$char_traits@D@std@@V?$allocator@D@2@@std@@MEAA?AV?$fpos@U_Mbstatet@@@2@V32@H@Z 0000000140260d50     safe_string_x64:safe_string.obj
 0004:00000d5c       $pdata$?seekoff@?$basic_stringbuf@DU?$char_traits@D@std@@V?$allocator@D@2@@std@@MEAA?AV?$fpos@U_Mbstatet@@@2@_JHH@Z 0000000140260d5c     safe_string_x64:safe_string.obj
 0004:00000d68       $pdata$?overflow@?$basic_stringbuf@DU?$char_traits@D@std@@V?$allocator@D@2@@std@@MEAAHH@Z 0000000140260d68     safe_string_x64:safe_string.obj
 0004:00000d74       $pdata$??1?$basic_stringbuf@DU?$char_traits@D@std@@V?$allocator@D@2@@std@@UEAA@XZ 0000000140260d74     safe_string_x64:safe_string.obj
 0004:00000d80       $pdata$??_G?$basic_stringstream@DU?$char_traits@D@std@@V?$allocator@D@2@@std@@UEAAPEAXI@Z 0000000140260d80     safe_string_x64:safe_string.obj
 0004:00000d8c       $pdata$??_G?$basic_stringbuf@DU?$char_traits@D@std@@V?$allocator@D@2@@std@@UEAAPEAXI@Z 0000000140260d8c     safe_string_x64:safe_string.obj
 0004:00000d98       $pdata$??1sentry@?$basic_ostream@DU?$char_traits@D@std@@@std@@QEAA@XZ 0000000140260d98     safe_string_x64:safe_string.obj
 0004:00000da4       $pdata$??1_Sentry_base@?$basic_ostream@DU?$char_traits@D@std@@@std@@QEAA@XZ 0000000140260da4     safe_string_x64:safe_string.obj
 0004:00000db0       $pdata$??$?6U?$char_traits@D@std@@@std@@YAAEAV?$basic_ostream@DU?$char_traits@D@std@@@0@AEAV10@PEBD@Z 0000000140260db0     safe_string_x64:safe_string.obj
 0004:00000dbc       $pdata$??$endl@DU?$char_traits@D@std@@@std@@YAAEAV?$basic_ostream@DU?$char_traits@D@std@@@0@AEAV10@@Z 0000000140260dbc     safe_string_x64:safe_string.obj
 0004:00000dd4       $pdata$?__scrt_initialize_thread_safe_statics@@YAHXZ 0000000140260dd4     msvcrt:thread_safe_statics.obj
 0004:00000de0       $pdata$?__scrt_uninitialize_thread_safe_statics@@YAXXZ 0000000140260de0     msvcrt:thread_safe_statics.obj
 0004:00000dec       $pdata$_Init_thread_abort  0000000140260dec     msvcrt:thread_safe_statics.obj
 0004:00000df8       $pdata$_Init_thread_footer 0000000140260df8     msvcrt:thread_safe_statics.obj
 0004:00000e04       $pdata$_Init_thread_header 0000000140260e04     msvcrt:thread_safe_statics.obj
 0004:00000e10       $pdata$_Init_thread_notify 0000000140260e10     msvcrt:thread_safe_statics.obj
 0004:00000e1c       $pdata$_Init_thread_wait   0000000140260e1c     msvcrt:thread_safe_statics.obj
 0004:00000e28       $pdata$__scrt_acquire_startup_lock 0000000140260e28     msvcrt:utility.obj
 0004:00000e34       $pdata$__scrt_initialize_crt 0000000140260e34     msvcrt:utility.obj
 0004:00000e40       $pdata$__scrt_initialize_onexit_tables 0000000140260e40     msvcrt:utility.obj
 0004:00000e4c       $pdata$__scrt_is_nonwritable_in_current_image 0000000140260e4c     msvcrt:utility.obj
 0004:00000e58       $pdata$__scrt_release_startup_lock 0000000140260e58     msvcrt:utility.obj
 0004:00000e64       $pdata$__scrt_uninitialize_crt 0000000140260e64     msvcrt:utility.obj
 0004:00000e70       $pdata$_onexit             0000000140260e70     msvcrt:utility.obj
 0004:00000e7c       $pdata$atexit              0000000140260e7c     msvcrt:utility.obj
 0004:00000e88       $pdata$??_Gtype_info@@UEAAPEAXI@Z 0000000140260e88     msvcrt:std_type_info_static.obj
 0004:00000e94       $pdata$__raise_securityfailure 0000000140260e94     msvcrt:gs_report.obj
 0004:00000ea0       $pdata$__report_gsfailure  0000000140260ea0     msvcrt:gs_report.obj
 0004:00000eac       $pdata$capture_previous_context 0000000140260eac     msvcrt:gs_report.obj
 0004:00000eb8       $pdata$?pre_c_initialization@@YAHXZ 0000000140260eb8     msvcrt:exe_winmain.obj
 0004:00000ec4       $pdata$?post_pgo_initialization@@YAHXZ 0000000140260ec4     msvcrt:exe_winmain.obj
 0004:00000ed0       $pdata$?pre_cpp_initialization@@YAXXZ 0000000140260ed0     msvcrt:exe_winmain.obj
 0004:00000edc       $pdata$?__scrt_common_main_seh@@YAHXZ 0000000140260edc     msvcrt:exe_winmain.obj
 0004:00000ee8       $pdata$WinMainCRTStartup   0000000140260ee8     msvcrt:exe_winmain.obj
 0004:00000ef4       $pdata$__scrt_fastfail     0000000140260ef4     msvcrt:utility_desktop.obj
 0004:00000f00       $pdata$__scrt_get_show_window_mode 0000000140260f00     msvcrt:utility_desktop.obj
 0004:00000f0c       $pdata$__scrt_is_managed_app 0000000140260f0c     msvcrt:utility_desktop.obj
 0004:00000f18       $pdata$__scrt_unhandled_exception_filter 0000000140260f18     msvcrt:utility_desktop.obj
 0004:00000f24       $pdata$__isa_available_init 0000000140260f24     msvcrt:cpu_disp.obj
 0004:00000f30       $pdata$__security_init_cookie 0000000140260f30     msvcrt:gs_support.obj
 0004:00000f3c       $pdata$__scrt_initialize_default_local_stdio_options 0000000140260f3c     msvcrt:default_local_stdio_options.obj
 0004:00000f48       $pdata$_RTC_Initialize     0000000140260f48     msvcrt:initsect.obj
 0004:00000f54       $pdata$_RTC_Terminate      0000000140260f54     msvcrt:initsect.obj
 0004:00000f60       $pdata$__GSHandlerCheck    0000000140260f60     msvcrt:gshandler.obj
 0004:00000f6c       $pdata$__GSHandlerCheckCommon 0000000140260f6c     msvcrt:gshandler.obj
 0004:00000f78       $pdata$??0CAtlBaseModule@ATL@@QEAA@XZ 0000000140260f78     atls:atlbase.obj
 0004:00000f84       $pdata$??1CAtlBaseModule@ATL@@QEAA@XZ 0000000140260f84     atls:atlbase.obj
 0004:00000f90       $pdata$?AfxInitialize@@YAHHK@Z 0000000140260f90     mfcs140:appmodul.obj
 0004:00000f9c       $pdata$__GSHandlerCheck_EH 0000000140260f9c     msvcrt:gshandlereh.obj
 0004:00000fc0       $pdata$?dtor$1@?0??CRSUploader@@YAAEAVUploader@crs@@XZ@4HA 0000000140260fc0     BugReporter.obj
 0004:00000fcc       $pdata$?dtor$1@?0???0CInterfaceDatabase@@QEAA@XZ@4HA 0000000140260fcc     ltmodule.obj
 0004:00000fd8       $pdata$?dtor$0@?0??AddHolder@CInterfaceDatabase@@SAXPEAVCAPIHolderBase@@@Z@4HA 0000000140260fd8     ltmodule.obj
 0004:00000fe4       $pdata$?dtor$0@?0??Add@CInterfaceDatabase@@EEAAXPEAVCInterfaceChooser@@@Z@4HA 0000000140260fe4     ltmodule.obj
 0004:00000fe4       $pdata$?dtor$0@?0??Add@CInterfaceDatabase@@EEAAXPEAVCAPIHolderBase@@@Z@4HA 0000000140260fe4     ltmodule.obj
 0004:00000fe4       $pdata$?dtor$0@?0??Add@CInterfaceDatabase@@EEAAXPEAVIBase@@PEBDH@Z@4HA 0000000140260fe4     ltmodule.obj
 0004:00000ff0       $pdata$?dtor$0@?0??TransferFrom@CInterfaceDatabase@@UEAAXPEAV1@@Z@4HA 0000000140260ff0     ltmodule.obj
 0004:00000ffc       $pdata$?dtor$0@?0???0CInterfaceNameMgr@@QEAA@PEBDH@Z@4HA 0000000140260ffc     ltmodule.obj
 0004:00001008       $pdata$?dtor$1@?0???0CInterfaceNameMgr@@QEAA@PEBDH@Z@4HA 0000000140261008     ltmodule.obj
 0004:00001014       $pdata$?dtor$2@?0???0CInterfaceNameMgr@@QEAA@PEBDH@Z@4HA 0000000140261014     ltmodule.obj
 0004:00001020       $pdata$?dtor$0@?0??TransferFrom@CInterfaceNameMgr@@QEAAXPEAV1@@Z@4HA 0000000140261020     ltmodule.obj
 0004:0000102c       $pdata$?dtor$1@?0??TransferFrom@CInterfaceNameMgr@@QEAAXPEAV1@@Z@4HA 000000014026102c     ltmodule.obj
 0004:00001038       $pdata$?dtor$2@?0??TransferFrom@CInterfaceNameMgr@@QEAAXPEAV1@@Z@4HA 0000000140261038     ltmodule.obj
 0004:00001044       $pdata$?dtor$0@?0??Init@CLogMsgManager@@SA_NW4ESHARED_MEM_USAGE_TYPE@1@@Z@4HA 0000000140261044     LogMsgManager.obj
 0004:00001050       $pdata$?dtor$1@?0??Init@CLogMsgManager@@SA_NW4ESHARED_MEM_USAGE_TYPE@1@@Z@4HA 0000000140261050     LogMsgManager.obj
 0004:0000105c       $pdata$?catch$0@?0???$_Insert_hint@AEAU?$pair@$$CB_JV?$basic_string@DU?$char_traits@D@std@@V?$allocator@D@2@@std@@@std@@PEAU?$_Tree_node@U?$pair@$$CB_JV?$basic_string@DU?$char_traits@D@std@@V?$allocator@D@2@@std@@@std@@PEAX@2@@?$_Tree@V?$_Tmap_traits@_JV?$basic_string@DU?$char_traits@D@std@@V?$allocator@D@2@@std@@U?$less@_J@2@V?$allocator@U?$pair@$$CB_JV?$basic_string@DU?$char_traits@D@std@@V?$allocator@D@2@@std@@@std@@@2@$0A@@std@@@std@@IEAA?AV?$_Tree_iterator@V?$_Tree_val@U?$_Tree_simple_types@U?$pair@$$CB_JV?$basic_string@DU?$char_traits@D@std@@V?$allocator@D@2@@std@@@std@@@std@@@std@@@1@V?$_Tree_const_iterator@V?$_Tree_val@U?$_Tree_simple_types@U?$pair@$$CB_JV?$basic_string@DU?$char_traits@D@std@@V?$allocator@D@2@@std@@@std@@@std@@@std@@@1@AEAU?$pair@$$CB_JV?$basic_string@DU?$char_traits@D@std@@V?$allocator@D@2@@std@@@1@PEAU?$_Tree_node@U?$pair@$$CB_JV?$basic_string@DU?$char_traits@D@std@@V?$allocator@D@2@@std@@@std@@PEAX@1@@Z@4HA 000000014026105c     LoadXlsMsg.obj
 0004:00001068       $pdata$?catch$0@?0???$_Insert_nohint@AEAU?$pair@$$CB_JV?$basic_string@DU?$char_traits@D@std@@V?$allocator@D@2@@std@@@std@@PEAU?$_Tree_node@U?$pair@$$CB_JV?$basic_string@DU?$char_traits@D@std@@V?$allocator@D@2@@std@@@std@@PEAX@2@@?$_Tree@V?$_Tmap_traits@_JV?$basic_string@DU?$char_traits@D@std@@V?$allocator@D@2@@std@@U?$less@_J@2@V?$allocator@U?$pair@$$CB_JV?$basic_string@DU?$char_traits@D@std@@V?$allocator@D@2@@std@@@std@@@2@$0A@@std@@@std@@IEAA?AU?$pair@V?$_Tree_iterator@V?$_Tree_val@U?$_Tree_simple_types@U?$pair@$$CB_JV?$basic_string@DU?$char_traits@D@std@@V?$allocator@D@2@@std@@@std@@@std@@@std@@@std@@_N@1@_NAEAU?$pair@$$CB_JV?$basic_string@DU?$char_traits@D@std@@V?$allocator@D@2@@std@@@1@PEAU?$_Tree_node@U?$pair@$$CB_JV?$basic_string@DU?$char_traits@D@std@@V?$allocator@D@2@@std@@@std@@PEAX@1@@Z@4HA 0000000140261068     LoadXlsMsg.obj
 0004:00001074       $pdata$?dtor$6@?0??LoadServer@CServerAppDlg@@QEAA_NXZ@4HA 0000000140261074     ServerAppDlg.obj
 0004:00001080       $pdata$?dtor$22@?0??DownloadUCCMapFile_HTTP@CServerAppDlg@@AEAA?AW4UCCMAPDOWNLOADREAULT@@V?$basic_string@DU?$char_traits@D@std@@V?$allocator@D@2@@std@@@Z@4HA 0000000140261080     ServerAppDlg.obj
 0004:0000108c       $pdata$?dtor$40@?0??DownloadUCCMapFile_HTTP@CServerAppDlg@@AEAA?AW4UCCMAPDOWNLOADREAULT@@V?$basic_string@DU?$char_traits@D@std@@V?$allocator@D@2@@std@@@Z@4HA 000000014026108c     ServerAppDlg.obj
 0004:00001098       $pdata$?dtor$0@?0??GetDownloadPath@CServerAppDlg@@AEAA?AV?$basic_string@DU?$char_traits@D@std@@V?$allocator@D@2@@std@@XZ@4HA 0000000140261098     ServerAppDlg.obj
 0004:000010a4       $pdata$?dtor$0@?0???$?HDU?$char_traits@D@std@@V?$allocator@D@1@@std@@YA?AV?$basic_string@DU?$char_traits@D@std@@V?$allocator@D@2@@0@AEBV10@0@Z@4HA 00000001402610a4     ServerAppDlg.obj
 0004:000010b0       $pdata$?catch$1@?0???1CWaitCursor@@QEAA@XZ@4HA 00000001402610b0     ServerAppDlg.obj
 0004:000010bc       $pdata$?dtor$4@?0??sprintf_s@internal@cf@@YAHPEAD_KPEBDAEAPEAD@Z@4HA 00000001402610bc     safe_string_x64:safe_string.obj
 0004:000010c8       $pdata$?dtor$4@?0??strcpy_s@cf@@YAHPEAD_KPEBD@Z@4HA 00000001402610c8     safe_string_x64:safe_string.obj
 0004:000010c8       $pdata$?dtor$4@?0??strncpy_s@cf@@YAHPEAD_KPEBD1@Z@4HA 00000001402610c8     safe_string_x64:safe_string.obj
 0004:000010d4       $pdata$?dtor$0@?0???0?$basic_stringstream@DU?$char_traits@D@std@@V?$allocator@D@2@@std@@QEAA@H@Z@4HA 00000001402610d4     safe_string_x64:safe_string.obj
 0004:000010e0       $pdata$?catch$4@?0???$?6U?$char_traits@D@std@@@std@@YAAEAV?$basic_ostream@DU?$char_traits@D@std@@@0@AEAV10@PEBD@Z@4HA 00000001402610e0     safe_string_x64:safe_string.obj
 0004:000010ec       $pdata$__scrt_is_nonwritable_in_current_image$filt$0 00000001402610ec     msvcrt:utility.obj
 0004:000010f8       $pdata$?filt$0@?0??__scrt_common_main_seh@@YAHXZ@4HA 00000001402610f8     msvcrt:exe_winmain.obj
 0004:00001104       $pdata$??__F?m_strEtcFileFormat@CHLogger@@0V?$basic_string@DU?$char_traits@D@std@@V?$allocator@D@2@@std@@A@@YAXXZ 0000000140261104     HostLogger.obj
 0004:00001110       $pdata$??__F?m_strKernelFileFormat@CHLogger@@0V?$basic_string@DU?$char_traits@D@std@@V?$allocator@D@2@@std@@A@@YAXXZ 0000000140261110     HostLogger.obj
 0004:0000111c       $pdata$??__F?m_strBRFileFormat@CHLogger@@0V?$basic_string@DU?$char_traits@D@std@@V?$allocator@D@2@@std@@A@@YAXXZ 000000014026111c     HostLogger.obj
 0004:00001128       $pdata$??__F?m_strFileFormat@CHLogger@@0V?$basic_string@DU?$char_traits@D@std@@V?$allocator@D@2@@std@@A@@YAXXZ 0000000140261128     HostLogger.obj
 0004:00001134       $pdata$??__F?m_strRWProcessMemoryFileFormat@CHLogger@@0V?$basic_string@DU?$char_traits@D@std@@V?$allocator@D@2@@std@@A@@YAXXZ 0000000140261134     HostLogger.obj
 0004:00001140       $pdata$??__F?m_strIPCMessageFileFormat@CHLogger@@0V?$basic_string@DU?$char_traits@D@std@@V?$allocator@D@2@@std@@A@@YAXXZ 0000000140261140     HostLogger.obj
 0004:0000114c       $pdata$??__F?m_strPacketFileFormat@CHLogger@@0V?$basic_string@DU?$char_traits@D@std@@V?$allocator@D@2@@std@@A@@YAXXZ 000000014026114c     HostLogger.obj
 0004:00001158       $pdata$??__F?m_strTimeOutFileFormat@CHLogger@@0V?$basic_string@DU?$char_traits@D@std@@V?$allocator@D@2@@std@@A@@YAXXZ 0000000140261158     HostLogger.obj
 0004:00001164       $pdata$??__F?m_strHostName@CHLogger@@0V?$basic_string@DU?$char_traits@D@std@@V?$allocator@D@2@@std@@A@@YAXXZ 0000000140261164     HostLogger.obj
 0004:00001170       $pdata$??__F?m_strServerName@CHLogger@@0V?$basic_string@DU?$char_traits@D@std@@V?$allocator@D@2@@std@@A@@YAXXZ 0000000140261170     HostLogger.obj
 0004:0000117c       $pdata$??__F?m_strLogFolder@CHLogger@@0V?$basic_string@DU?$char_traits@D@std@@V?$allocator@D@2@@std@@A@@YAXXZ 000000014026117c     HostLogger.obj
 0004:00001188       $pdata$??__F?m_strModeUserCountFormat@CHLogger@@0V?$basic_string@DU?$char_traits@D@std@@V?$allocator@D@2@@std@@A@@YAXXZ 0000000140261188     HostLogger.obj
 0004:00001194       $pdata$??__F?m_strServerAppUseCountFormat@CHLogger@@0V?$basic_string@DU?$char_traits@D@std@@V?$allocator@D@2@@std@@A@@YAXXZ 0000000140261194     HostLogger.obj
 0004:000011a0       $pdata$??__F?m_vectSharedMapHandles@CLogMsgManager@@0V?$vector@PEAXV?$allocator@PEAX@std@@@std@@A@@YAXXZ 00000001402611a0     LogMsgManager.obj
 0005:000001b0       $R000000                   00000001402621b0     ServerApp.res
 0005:00000498       $R0002E8                   0000000140262498     ServerApp.res
 0005:000005c0       $R000410                   00000001402625c0     ServerApp.res
 0005:000005e8       $R000438                   00000001402625e8     ServerApp.res
 0005:00000710       $R000560                   0000000140262710     ServerApp.res
 0005:000009c0       $R000810                   00000001402629c0     ServerApp.res

 Exports

  ordinal    name

        1    IsDebugMode
        2    SetMasterDatabase
